 databaseEdit

 Timestamp is 614c7ff4 (Thu Sep 23 13:24:04 2021)

 Preferred load address is 10000000

 Start         Length     Name                   Class
 0001:00000000 000000a5H .text$di                CODE
 0001:000000b0 000089ecH .text$mn                CODE
 0001:00008a9c 0000146dH .text$x                 CODE
 0001:00009f09 00000037H .text$yd                CODE
 0002:00000000 00000e2cH .idata$5                DATA
 0002:00000e2c 00000004H .CRT$XCA                DATA
 0002:00000e30 00000014H .CRT$XCU                DATA
 0002:00000e44 00000004H .CRT$XCZ                DATA
 0002:00000e48 00000004H .CRT$XIA                DATA
 0002:00000e4c 00000004H .CRT$XIAA               DATA
 0002:00000e50 00000004H .CRT$XIC                DATA
 0002:00000e54 00000004H .CRT$XIZ                DATA
 0002:00000e58 00003408H .rdata                  DATA
 0002:00004260 00000f58H .rdata$r                DATA
 0002:000051b8 00000004H .rtc$IAA                DATA
 0002:000051bc 00000004H .rtc$IZZ                DATA
 0002:000051c0 00000004H .rtc$TAA                DATA
 0002:000051c4 00000004H .rtc$TZZ                DATA
 0002:000051c8 0000122cH .xdata$x                DATA
 0002:00006400 00000060H .edata                  DATA
 0002:00006460 00000050H .idata$2                DATA
 0002:000064b0 00000014H .idata$3                DATA
 0002:000064c4 00000e2cH .idata$4                DATA
 0002:000072f0 000093eeH .idata$6                DATA
 0003:00000000 00000074H .data                   DATA
 0003:00000074 000004e8H .data$r                 DATA
 0003:00000560 000003d4H .bss                    DATA
 0004:00000000 000000a0H .rsrc$01                DATA
 0004:000000a0 00000608H .rsrc$02                DATA

  Address         Publics by Value              Rva+Base       Lib:Object

 0000:00000000       ___safe_se_handler_count   00000000     <absolute>
 0000:00000000       ___guard_fids_table        00000000     <absolute>
 0000:00000000       ___safe_se_handler_table   00000000     <absolute>
 0000:00000000       ___guard_flags             00000000     <absolute>
 0000:00000000       ___guard_fids_count        00000000     <absolute>
 0000:00000000       ___ImageBase               10000000     <linker-defined>
 0001:000000b0       ??0?$QGuardedPtr@VQDockWindow@@@@QAE@XZ 100010b0 f i databaseEdit.obj
 0001:000000b0       ??0?$QGuardedPtr@VQPopupMenu@@@@QAE@XZ 100010b0 f i databaseEdit.obj
 0001:000000f1       ??0config_plugin_base@@QAE@ABVQString@@00@Z 100010f1 f i databaseEdit.obj
 0001:0000017e       ??0databaseEdit@@QAE@ABVQString@@00@Z 1000117e f   databaseEdit.obj
 0001:0000067a       ??1?$QDict@VQAction@@@@UAE@XZ 1000167a f i databaseEdit.obj
 0001:000006ad       ??1?$QGuardedPtr@VQDockWindow@@@@QAE@XZ 100016ad f i databaseEdit.obj
 0001:000006ad       ??1?$QGuardedPtr@VQPopupMenu@@@@QAE@XZ 100016ad f i databaseEdit.obj
 0001:000006b2       ??1?$QPtrList@VQPopupMenu@@@@UAE@XZ 100016b2 f i databaseEdit.obj
 0001:000006e5       ??1QDockWindowList@@UAE@XZ 100016e5 f i databaseEdit.obj
 0001:0000072e       ??1QPopupMenuList@@UAE@XZ  1000172e f i databaseEdit.obj
 0001:00000760       ??1config_plugin_base@@UAE@XZ 10001760 f i databaseEdit.obj
 0001:000007ba       ??1databaseEdit@@UAE@XZ    100017ba f   databaseEdit.obj
 0001:0000086a       ??4?$QGuardedPtr@VQDockWindow@@@@QAEAAV0@PAVQDockWindow@@@Z 1000186a f i databaseEdit.obj
 0001:0000086a       ??4?$QGuardedPtr@VQPopupMenu@@@@QAEAAV0@PAVQPopupMenu@@@Z 1000186a f i databaseEdit.obj
 0001:000008c8       ??_EQDockWindow@@WCI@AEPAXI@Z 100018c8 f i databaseEdit.obj
 0001:000008d0       ??_EQPopupMenu@@WCI@AEPAXI@Z 100018d0 f i databaseEdit.obj
 0001:000008d8       ??_EQPopupMenu@@WIM@AEPAXI@Z 100018d8 f i databaseEdit.obj
 0001:000008e3       ??_EQToolBar@@WCI@AEPAXI@Z 100018e3 f i databaseEdit.obj
 0001:000008eb       ??_Econfig_plugin_base@@WCI@AEPAXI@Z 100018eb f i databaseEdit.obj
 0001:000008f3       ??_EdatabaseEdit@@WCI@AEPAXI@Z 100018f3 f i databaseEdit.obj
 0001:000008fb       ??_E?$QDict@VQAction@@@@UAEPAXI@Z 100018fb f i databaseEdit.obj
 0001:000008fb       ??_G?$QDict@VQAction@@@@UAEPAXI@Z 100018fb f i databaseEdit.obj
 0001:0000091a       ??_G?$QPtrList@VQPopupMenu@@@@UAEPAXI@Z 1000191a f i databaseEdit.obj
 0001:0000091a       ??_E?$QPtrList@VQPopupMenu@@@@UAEPAXI@Z 1000191a f i databaseEdit.obj
 0001:00000939       ??_EQAction@@UAEPAXI@Z     10001939 f i databaseEdit.obj
 0001:00000939       ??_GQAction@@UAEPAXI@Z     10001939 f i databaseEdit.obj
 0001:00000959       ??_GQDockWindow@@UAEPAXI@Z 10001959 f i databaseEdit.obj
 0001:00000959       ??_EQDockWindow@@UAEPAXI@Z 10001959 f i databaseEdit.obj
 0001:00000979       ??_GQDockWindowList@@UAEPAXI@Z 10001979 f i databaseEdit.obj
 0001:00000979       ??_EQDockWindowList@@UAEPAXI@Z 10001979 f i databaseEdit.obj
 0001:00000998       ??_GQGuardedPtrPrivate@@UAEPAXI@Z 10001998 f i databaseEdit.obj
 0001:00000998       ??_EQGuardedPtrPrivate@@UAEPAXI@Z 10001998 f i databaseEdit.obj
 0001:000009b8       ??_EQListViewItem@@UAEPAXI@Z 100019b8 f i databaseEdit.obj
 0001:000009b8       ??_GQListViewItem@@UAEPAXI@Z 100019b8 f i databaseEdit.obj
 0001:000009d8       ??_GQPopupMenu@@UAEPAXI@Z  100019d8 f i databaseEdit.obj
 0001:000009d8       ??_EQPopupMenu@@UAEPAXI@Z  100019d8 f i databaseEdit.obj
 0001:000009f8       ??_GQPopupMenuList@@UAEPAXI@Z 100019f8 f i databaseEdit.obj
 0001:000009f8       ??_EQPopupMenuList@@UAEPAXI@Z 100019f8 f i databaseEdit.obj
 0001:00000a17       ??_EQToolBar@@UAEPAXI@Z    10001a17 f i databaseEdit.obj
 0001:00000a17       ??_GQToolBar@@UAEPAXI@Z    10001a17 f i databaseEdit.obj
 0001:00000a37       ??_Econfig_plugin_base@@UAEPAXI@Z 10001a37 f i databaseEdit.obj
 0001:00000a37       ??_Gconfig_plugin_base@@UAEPAXI@Z 10001a37 f i databaseEdit.obj
 0001:00000a56       ??_EdatabaseEdit@@UAEPAXI@Z 10001a56 f i databaseEdit.obj
 0001:00000a56       ??_GdatabaseEdit@@UAEPAXI@Z 10001a56 f i databaseEdit.obj
 0001:00000a75       ?about@config_plugin_base@@UAE?AVQString@@XZ 10001a75 f i databaseEdit.obj
 0001:00000acb       ?about@databaseEdit@@UAE?AVQString@@XZ 10001acb f   databaseEdit.obj
 0001:00000b73       ?reply@config_plugin_base@@UAEXPAVresponse@@@Z 10001b73 f i databaseEdit.obj
 0001:00000b73       ?activate@config_plugin_base@@UAEX_N@Z 10001b73 f i databaseEdit.obj
 0001:00000b76       ?activate@databaseEdit@@UAEX_N@Z 10001b76 f   databaseEdit.obj
 0001:00001078       ?apply@config_plugin_base@@UAEXXZ 10002078 f i databaseEdit.obj
 0001:00001079       ?apply@databaseEdit@@UAEXXZ 10002079 f   databaseEdit.obj
 0001:00001110       ?clear@?$QIntDict@VQTable@@@@UAEXXZ 10002110 f i databaseEditdlgimpl.obj
 0001:00001110       ?clear@?$QDict@VQAction@@@@UAEXXZ 10002110 f i databaseEdit.obj
 0001:00001116       ?clear@?$QPtrList@VQPopupMenu@@@@UAEXXZ 10002116 f i databaseEdit.obj
 0001:0000111c       ?closeEvent@config_plugin_base@@UAEXPAVQCloseEvent@@@Z 1000211c f i databaseEdit.obj
 0001:0000112a       ?closeEvent@databaseEdit@@UAEXPAVQCloseEvent@@@Z 1000212a f   databaseEdit.obj
 0001:000013e7       ?count@?$QPtrList@VQPopupMenu@@@@UBEIXZ 100023e7 f i databaseEdit.obj
 0001:000013eb       ?db@@YAXABVQString@@@Z     100023eb f   databaseEdit.obj
 0001:00001433       ?deleteItem@?$QIntDict@VQTable@@@@EAEXPAX@Z 10002433 f i databaseEditdlgimpl.obj
 0001:00001433       ?deleteItem@?$QPtrList@VQPopupMenu@@@@EAEXPAX@Z 10002433 f i databaseEdit.obj
 0001:00001433       ?deleteItem@?$QDict@VQAction@@@@EAEXPAX@Z 10002433 f i databaseEdit.obj
 0001:0000144e       ?deref@?$QGuardedPtr@VQPopupMenu@@@@AAEXXZ 1000244e f i databaseEdit.obj
 0001:0000144e       ?deref@?$QGuardedPtr@VQDockWindow@@@@AAEXXZ 1000244e f i databaseEdit.obj
 0001:00001463       ?fileSelected@databaseEdit@@AAEXABVQString@@@Z 10002463 f   databaseEdit.obj
 0001:000017ac       ?isDirty@config_plugin_base@@UAE_NXZ 100027ac f i databaseEdit.obj
 0001:000017ac       ?validate@config_plugin_base@@UAE_NXZ 100027ac f i databaseEdit.obj
 0001:000017af       ?isDirty@databaseEdit@@UAE_NXZ 100027af f   databaseEdit.obj
 0001:000017bc       ?menus@config_plugin_base@@UAE?AVQPopupMenuList@@XZ 100027bc f i databaseEdit.obj
 0001:000017df       ?menus@databaseEdit@@UAE?AVQPopupMenuList@@XZ 100027df f   databaseEdit.obj
 0001:00001829       ?metaObject@databaseEdit@@UBEPAVQMetaObject@@XZ 10002829 f i databaseEdit.obj
 0001:0000182e       ?navigate@config_plugin_base@@UAEXABVQString@@0@Z 1000282e f i databaseEdit.obj
 0001:00001831       ?navigate@databaseEdit@@UAEXABVQString@@0@Z 10002831 f   databaseEdit.obj
 0001:000018ae       ?reply@databaseEdit@@UAEXPAVresponse@@@Z 100028ae f   databaseEdit.obj
 0001:0000303d       ?resizeEvent@databaseEdit@@UAEXPAVQResizeEvent@@@Z 1000403d f   databaseEdit.obj
 0001:00003072       ?textStatus@response@@QAE?AVQString@@W4status@1@@Z 10004072 f i databaseEdit.obj
 0001:000030c1       ?toolbars@config_plugin_base@@UAE?AVQDockWindowList@@XZ 100040c1 f i databaseEdit.obj
 0001:000030e4       ?toolbars@databaseEdit@@UAE?AVQDockWindowList@@XZ 100040e4 f   databaseEdit.obj
 0001:0000313c       ??0databaseEditDlg@@QAE@ABVQString@@PAVQWidget@@PBDI@Z 1000413c f   databaseEditdlgimpl.obj
 0001:000032c6       ??1?$QIntDict@VQTable@@@@UAE@XZ 100042c6 f i databaseEditdlgimpl.obj
 0001:000032f9       ??1databaseEditDlg@@UAE@XZ 100042f9 f   databaseEditdlgimpl.obj
 0001:0000335a       ??_EdatabaseEditDlg@@WCI@AEPAXI@Z 1000435a f i databaseEditdlgimpl.obj
 0001:00003362       ??_E?$QIntDict@VQTable@@@@UAEPAXI@Z 10004362 f i databaseEditdlgimpl.obj
 0001:00003362       ??_G?$QIntDict@VQTable@@@@UAEPAXI@Z 10004362 f i databaseEditdlgimpl.obj
 0001:00003381       ??_EdatabaseEditDlg@@UAEPAXI@Z 10004381 f i databaseEditdlgimpl.obj
 0001:00003381       ??_GdatabaseEditDlg@@UAEPAXI@Z 10004381 f i databaseEditdlgimpl.obj
 0001:000033a0       ?count@?$QDict@VQAction@@@@UBEIXZ 100043a0 f i databaseEdit.obj
 0001:000033a0       ?count@?$QIntDict@VQTable@@@@UBEIXZ 100043a0 f i databaseEditdlgimpl.obj
 0001:000033a4       ?inc@?$QMapIterator@VQString@@V1@@@AAEHXZ 100043a4 f i databaseEditdlgimpl.obj
 0001:000033d5       ?load@databaseEditDlg@@QAE_NABVQString@@@Z 100043d5 f   databaseEditdlgimpl.obj
 0001:000033da       ?loadDb@databaseEditDlg@@QAE_NABVQString@@H@Z 100043da f   databaseEditdlgimpl.obj
 0001:0000381e       ?loadIni@databaseEditDlg@@QAE_NABVQString@@@Z 1000481e f   databaseEditdlgimpl.obj
 0001:00003a16       ?metaObject@databaseEditDlg@@UBEPAVQMetaObject@@XZ 10004a16 f i databaseEditdlgimpl.obj
 0001:00003a1b       ?resetDisplays@databaseEditDlg@@QAEXXZ 10004a1b f   databaseEditdlgimpl.obj
 0001:00003b0c       ?save@databaseEditDlg@@QAEXABVQString@@@Z 10004b0c f   databaseEditdlgimpl.obj
 0001:00003b62       ?sortColumn@databaseEditDlg@@QAEXH@Z 10004b62 f   databaseEditdlgimpl.obj
 0001:00003b96       ?textChanged@databaseEditDlg@@QAEXXZ 10004b96 f   databaseEditdlgimpl.obj
 0001:00003bdf       ??_Gconfig_plugin_desc_base@@UAEPAXI@Z 10004bdf f i plugindesc.obj
 0001:00003bdf       ??_Gplugindesc@@UAEPAXI@Z  10004bdf f i plugindesc.obj
 0001:00003bdf       ??_Eplugindesc@@UAEPAXI@Z  10004bdf f i plugindesc.obj
 0001:00003bdf       ??_Econfig_plugin_desc_base@@UAEPAXI@Z 10004bdf f i plugindesc.obj
 0001:00003bff       ?create@plugindesc@@UAEPAVconfig_plugin_base@@ABVQString@@00@Z 10004bff f   plugindesc.obj
 0001:00003c3a       ?keys@plugindesc@@UAE?AVQStringList@@ABVQString@@0@Z 10004c3a f   plugindesc.obj
 0001:00003c95       ?pixmap@plugindesc@@UAE?AVQPixmap@@ABVQString@@@Z 10004c95 f   plugindesc.obj
 0001:00003cb4       _load_bncs_config_plugin_desc 10004cb4 f   plugindesc.obj
 0001:00003cca       ??0toolWindow@@QAE@PAVQWidget@@PBDI@Z 10004cca f   toolwindowimpl.obj
 0001:00003d28       ??1toolWindow@@UAE@XZ      10004d28 f   toolwindowimpl.obj
 0001:00003d3a       ??_EtoolWindow@@WCI@AEPAXI@Z 10004d3a f i toolwindowimpl.obj
 0001:00003d42       ??_EtoolWindow@@UAEPAXI@Z  10004d42 f i toolwindowimpl.obj
 0001:00003d42       ??_GtoolWindow@@UAEPAXI@Z  10004d42 f i toolwindowimpl.obj
 0001:00003d61       ?metaObject@toolWindow@@UBEPAVQMetaObject@@XZ 10004d61 f i toolwindowimpl.obj
 0001:00003d66       ?selectionChanged@toolWindow@@AAEXPAVQListViewItem@@@Z 10004d66 f   toolwindowimpl.obj
 0001:00003daa       ??0databaseEditDlgBase@@QAE@PAVQWidget@@PBDI@Z 10004daa f   databaseEditdlg.obj
 0001:000057d0       ??1databaseEditDlgBase@@UAE@XZ 100067d0 f   databaseEditdlg.obj
 0001:000057e3       ??_EQHBoxLayout@@WCI@AEPAXI@Z 100067e3 f i databaseEditdlg.obj
 0001:000057eb       ??_EQLabel@@WCI@AEPAXI@Z   100067eb f i databaseEditdlg.obj
 0001:000057f3       ??_EQLineEdit@@WCI@AEPAXI@Z 100067f3 f i databaseEditdlg.obj
 0001:000057fb       ??_EQTabWidget@@WCI@AEPAXI@Z 100067fb f i databaseEditdlg.obj
 0001:00005803       ??_EQTable@@WCI@AEPAXI@Z   10006803 f i databaseEditdlg.obj
 0001:0000580b       ??_EQTextEdit@@WCI@AEPAXI@Z 1000680b f i databaseEditdlg.obj
 0001:00005813       ??_EQVBoxLayout@@WCI@AEPAXI@Z 10006813 f i databaseEditdlg.obj
 0001:0000581b       ??_EQWidget@@WCI@AEPAXI@Z  1000681b f i databaseEditdlg.obj
 0001:00005823       ??_EdatabaseEditDlgBase@@WCI@AEPAXI@Z 10006823 f i databaseEditdlg.obj
 0001:0000582b       ??_GQHBoxLayout@@UAEPAXI@Z 1000682b f i databaseEditdlg.obj
 0001:0000582b       ??_EQHBoxLayout@@UAEPAXI@Z 1000682b f i databaseEditdlg.obj
 0001:0000584b       ??_EQLabel@@UAEPAXI@Z      1000684b f i databaseEditdlg.obj
 0001:0000584b       ??_GQLabel@@UAEPAXI@Z      1000684b f i databaseEditdlg.obj
 0001:0000586b       ??_GQLineEdit@@UAEPAXI@Z   1000686b f i databaseEditdlg.obj
 0001:0000586b       ??_EQLineEdit@@UAEPAXI@Z   1000686b f i databaseEditdlg.obj
 0001:0000588b       ??_EQSpacerItem@@UAEPAXI@Z 1000688b f i databaseEditdlg.obj
 0001:0000588b       ??_GQSpacerItem@@UAEPAXI@Z 1000688b f i databaseEditdlg.obj
 0001:000058ab       ??_GQTabWidget@@UAEPAXI@Z  100068ab f i databaseEditdlg.obj
 0001:000058ab       ??_EQTabWidget@@UAEPAXI@Z  100068ab f i databaseEditdlg.obj
 0001:000058cb       ??_GQTable@@UAEPAXI@Z      100068cb f i databaseEditdlg.obj
 0001:000058cb       ??_EQTable@@UAEPAXI@Z      100068cb f i databaseEditdlg.obj
 0001:000058eb       ??_EQTextEdit@@UAEPAXI@Z   100068eb f i databaseEditdlg.obj
 0001:000058eb       ??_GQTextEdit@@UAEPAXI@Z   100068eb f i databaseEditdlg.obj
 0001:0000590b       ??_EQVBoxLayout@@UAEPAXI@Z 1000690b f i databaseEditdlg.obj
 0001:0000590b       ??_GQVBoxLayout@@UAEPAXI@Z 1000690b f i databaseEditdlg.obj
 0001:0000592b       ??_EQWidget@@UAEPAXI@Z     1000692b f i databaseEditdlg.obj
 0001:0000592b       ??_GQWidget@@UAEPAXI@Z     1000692b f i databaseEditdlg.obj
 0001:0000594b       ??_EdatabaseEditDlgBase@@UAEPAXI@Z 1000694b f i databaseEditdlg.obj
 0001:0000594b       ??_GdatabaseEditDlgBase@@UAEPAXI@Z 1000694b f i databaseEditdlg.obj
 0001:0000596a       ?languageChange@databaseEditDlgBase@@MAEXXZ 1000696a f   databaseEditdlg.obj
 0001:000061f1       ?metaObject@databaseEditDlgBase@@UBEPAVQMetaObject@@XZ 100071f1 f i databaseEditdlg.obj
 0001:000061f6       ?className@databaseEdit@@UBEPBDXZ 100071f6 f   moc_databaseEdit.obj
 0001:000061fc       ?command@databaseEdit@@IAEXVQString@@0@Z 100071fc f   moc_databaseEdit.obj
 0001:000062bc       ?qt_cast@databaseEdit@@UAEPAXPBD@Z 100072bc f   moc_databaseEdit.obj
 0001:000062ea       ?qt_emit@databaseEdit@@UAE_NHPAUQUObject@@@Z 100072ea f   moc_databaseEdit.obj
 0001:0000634e       ?qt_invoke@databaseEdit@@UAE_NHPAUQUObject@@@Z 1000734e f   moc_databaseEdit.obj
 0001:00006383       ?staticMetaObject@databaseEdit@@SAPAVQMetaObject@@XZ 10007383 f   moc_databaseEdit.obj
 0001:0000643e       ?className@databaseEditDlgBase@@UBEPBDXZ 1000743e f   moc_databaseEditdlg.obj
 0001:00006444       ?qt_cast@databaseEditDlgBase@@UAEPAXPBD@Z 10007444 f   moc_databaseEditdlg.obj
 0001:00006472       ?qt_emit@toolWindowBase@@UAE_NHPAUQUObject@@@Z 10007472 f   moc_toolwindow.obj
 0001:00006472       ?qt_emit@databaseEditDlgBase@@UAE_NHPAUQUObject@@@Z 10007472 f   moc_databaseEditdlg.obj
 0001:0000647c       ?qt_invoke@databaseEditDlgBase@@UAE_NHPAUQUObject@@@Z 1000747c f   moc_databaseEditdlg.obj
 0001:000064ae       ?staticMetaObject@databaseEditDlgBase@@SAPAVQMetaObject@@XZ 100074ae f   moc_databaseEditdlg.obj
 0001:000064f8       ?tr@databaseEditDlgBase@@SA?AVQString@@PBD0@Z 100074f8 f   moc_databaseEditdlg.obj
 0001:0000653b       ?className@databaseEditDlg@@UBEPBDXZ 1000753b f   moc_databaseEditdlgimpl.obj
 0001:00006541       ?command@databaseEditDlg@@IAEXVQString@@0@Z 10007541 f   moc_databaseEditdlgimpl.obj
 0001:00006601       ?qt_cast@databaseEditDlg@@UAEPAXPBD@Z 10007601 f   moc_databaseEditdlgimpl.obj
 0001:0000662e       ?qt_emit@databaseEditDlg@@UAE_NHPAUQUObject@@@Z 1000762e f   moc_databaseEditdlgimpl.obj
 0001:00006691       ?qt_invoke@databaseEditDlg@@UAE_NHPAUQUObject@@@Z 10007691 f   moc_databaseEditdlgimpl.obj
 0001:000066d2       ?staticMetaObject@databaseEditDlg@@SAPAVQMetaObject@@XZ 100076d2 f   moc_databaseEditdlgimpl.obj
 0001:00006793       ?className@toolWindowBase@@UBEPBDXZ 10007793 f   moc_toolwindow.obj
 0001:00006799       ?qt_cast@toolWindowBase@@UAEPAXPBD@Z 10007799 f   moc_toolwindow.obj
 0001:000067c7       ?qt_invoke@toolWindowBase@@UAE_NHPAUQUObject@@@Z 100077c7 f   moc_toolwindow.obj
 0001:000067f9       ?qt_property@databaseEdit@@UAE_NHHPAVQVariant@@@Z 100077f9 f   moc_databaseEdit.obj
 0001:000067f9       ?qt_property@toolWindowBase@@UAE_NHHPAVQVariant@@@Z 100077f9 f   moc_toolwindow.obj
 0001:000067f9       ?qt_property@databaseEditDlgBase@@UAE_NHHPAVQVariant@@@Z 100077f9 f   moc_databaseEditdlg.obj
 0001:00006803       ?staticMetaObject@toolWindowBase@@SAPAVQMetaObject@@XZ 10007803 f   moc_toolwindow.obj
 0001:0000684d       ?tr@toolWindowBase@@SA?AVQString@@PBD0@Z 1000784d f   moc_toolwindow.obj
 0001:00006890       ?className@toolWindow@@UBEPBDXZ 10007890 f   moc_toolwindowimpl.obj
 0001:00006896       ?fileSelected@toolWindow@@IAEXABVQString@@@Z 10007896 f   moc_toolwindowimpl.obj
 0001:000068d3       ?qt_cast@toolWindow@@UAEPAXPBD@Z 100078d3 f   moc_toolwindowimpl.obj
 0001:00006900       ?qt_emit@toolWindow@@UAE_NHPAUQUObject@@@Z 10007900 f   moc_toolwindowimpl.obj
 0001:00006934       ?qt_invoke@toolWindow@@UAE_NHPAUQUObject@@@Z 10007934 f   moc_toolwindowimpl.obj
 0001:00006968       ?qt_property@databaseEditDlg@@UAE_NHHPAVQVariant@@@Z 10007968 f   moc_databaseEditdlgimpl.obj
 0001:00006968       ?qt_property@toolWindow@@UAE_NHHPAVQVariant@@@Z 10007968 f   moc_toolwindowimpl.obj
 0001:00006971       ?staticMetaObject@toolWindow@@SAPAVQMetaObject@@XZ 10007971 f   moc_toolwindowimpl.obj
 0001:00006a1d       ??0toolWindowBase@@QAE@PAVQWidget@@PBDI@Z 10007a1d f   toolwindow.obj
 0001:00006cc6       ??1toolWindowBase@@UAE@XZ  10007cc6 f   toolwindow.obj
 0001:00006cd9       ??_EQListView@@WCI@AEPAXI@Z 10007cd9 f i toolwindow.obj
 0001:00006ce1       ??_EtoolWindowBase@@WCI@AEPAXI@Z 10007ce1 f i toolwindow.obj
 0001:00006ce9       ??_GQListView@@UAEPAXI@Z   10007ce9 f i toolwindow.obj
 0001:00006ce9       ??_EQListView@@UAEPAXI@Z   10007ce9 f i toolwindow.obj
 0001:00006d09       ??_EtoolWindowBase@@UAEPAXI@Z 10007d09 f i toolwindow.obj
 0001:00006d09       ??_GtoolWindowBase@@UAEPAXI@Z 10007d09 f i toolwindow.obj
 0001:00006d28       ?languageChange@toolWindowBase@@MAEXXZ 10007d28 f   toolwindow.obj
 0001:00006e21       ?metaObject@toolWindowBase@@UBEPAVQMetaObject@@XZ 10007e21 f i toolwindow.obj
 0001:00006e26       ?setName@QWidget@@UAEXPBD@Z 10007e26 f   qt-mt323:qt-mt323.dll
 0001:00006e2c       ?closeEvent@QWidget@@MAEXPAVQCloseEvent@@@Z 10007e2c f   qt-mt323:qt-mt323.dll
 0001:00006e32       ?acceptDrop@QListViewItem@@UBE_NPBVQMimeSource@@@Z 10007e32 f   qt-mt323:qt-mt323.dll
 0001:00006e38       ?activate@QListViewItem@@MAEXXZ 10007e38 f   qt-mt323:qt-mt323.dll
 0001:00006e3e       ?activateItemAt@QPopupMenu@@UAEXH@Z 10007e3e f   qt-mt323:qt-mt323.dll
 0001:00006e44       ?addTo@QAction@@UAE_NPAVQWidget@@@Z 10007e44 f   qt-mt323:qt-mt323.dll
 0001:00006e4a       ?addedTo@QAction@@MAEXHPAVQPopupMenu@@@Z 10007e4a f   qt-mt323:qt-mt323.dll
 0001:00006e50       ?addedTo@QAction@@MAEXPAVQWidget@@0@Z 10007e50 f   qt-mt323:qt-mt323.dll
 0001:00006e56       ?adjustSize@QWidget@@UAEXXZ 10007e56 f   qt-mt323:qt-mt323.dll
 0001:00006e5c       ?cancelRename@QListViewItem@@MAEXH@Z 10007e5c f   qt-mt323:qt-mt323.dll
 0001:00006e62       ?checkConnectArgs@QObject@@MAE_NPBDPBV1@0@Z 10007e62 f   qt-mt323:qt-mt323.dll
 0001:00006e68       ?childEvent@QObject@@MAEXPAVQChildEvent@@@Z 10007e68 f   qt-mt323:qt-mt323.dll
 0001:00006e6e       ?className@QAction@@UBEPBDXZ 10007e6e f   qt-mt323:qt-mt323.dll
 0001:00006e74       ?className@QDockWindow@@UBEPBDXZ 10007e74 f   qt-mt323:qt-mt323.dll
 0001:00006e7a       ?className@QGuardedPtrPrivate@@UBEPBDXZ 10007e7a f   qt-mt323:qt-mt323.dll
 0001:00006e80       ?className@QPopupMenu@@UBEPBDXZ 10007e80 f   qt-mt323:qt-mt323.dll
 0001:00006e86       ?className@QToolBar@@UBEPBDXZ 10007e86 f   qt-mt323:qt-mt323.dll
 0001:00006e8c       ?className@QWidget@@UBEPBDXZ 10007e8c f   qt-mt323:qt-mt323.dll
 0001:00006e92       ?clear@?$QPtrList@VQDockWindow@@@@UAEXXZ 10007e92 f   qt-mt323:qt-mt323.dll
 0001:00006e98       ?clear@QToolBar@@UAEXXZ    10007e98 f   qt-mt323:qt-mt323.dll
 0001:00006e9e       ?close@QWidget@@UAE_N_N@Z  10007e9e f   qt-mt323:qt-mt323.dll
 0001:00006ea4       ?closeEvent@QPopupMenu@@MAEXPAVQCloseEvent@@@Z 10007ea4 f   qt-mt323:qt-mt323.dll
 0001:00006eaa       ?cmd@QPaintDevice@@MAE_NHPAVQPainter@@PATQPDevCmdParam@@@Z 10007eaa f   qt-mt323:qt-mt323.dll
 0001:00006eb0       ?compare@QListViewItem@@UBEHPAV1@H_N@Z 10007eb0 f   qt-mt323:qt-mt323.dll
 0001:00006eb6       ?compareItems@QGList@@MAEHPAX0@Z 10007eb6 f   qt-mt323:qt-mt323.dll
 0001:00006ebc       ?connectNotify@QObject@@MAEXPBD@Z 10007ebc f   qt-mt323:qt-mt323.dll
 0001:00006ec2       ?contextMenuEvent@QDockWindow@@MAEXPAVQContextMenuEvent@@@Z 10007ec2 f   qt-mt323:qt-mt323.dll
 0001:00006ec8       ?contextMenuEvent@QWidget@@MAEXPAVQContextMenuEvent@@@Z 10007ec8 f   qt-mt323:qt-mt323.dll
 0001:00006ece       ?count@?$QPtrList@VQDockWindow@@@@UBEIXZ 10007ece f   qt-mt323:qt-mt323.dll
 0001:00006ed4       ?create@QWidget@@MAEXPAUHWND__@@_N1@Z 10007ed4 f   qt-mt323:qt-mt323.dll
 0001:00006eda       ?customEvent@QObject@@MAEXPAVQCustomEvent@@@Z 10007eda f   qt-mt323:qt-mt323.dll
 0001:00006ee0       ?customWhatsThis@QPopupMenu@@UBE_NXZ 10007ee0 f   qt-mt323:qt-mt323.dll
 0001:00006ee6       ?customWhatsThis@QWidget@@UBE_NXZ 10007ee6 f   qt-mt323:qt-mt323.dll
 0001:00006eec       ?deleteItem@?$QPtrList@VQDockWindow@@@@EAEXPAX@Z 10007eec f   qt-mt323:qt-mt323.dll
 0001:00006ef2       ?destroy@QWidget@@MAEX_N0@Z 10007ef2 f   qt-mt323:qt-mt323.dll
 0001:00006ef8       ?disconnectNotify@QObject@@MAEXPBD@Z 10007ef8 f   qt-mt323:qt-mt323.dll
 0001:00006efe       ?dock@QDockWindow@@UAEXXZ  10007efe f   qt-mt323:qt-mt323.dll
 0001:00006f04       ?dragEnterEvent@QWidget@@MAEXPAVQDragEnterEvent@@@Z 10007f04 f   qt-mt323:qt-mt323.dll
 0001:00006f0a       ?dragEntered@QListViewItem@@MAEXXZ 10007f0a f   qt-mt323:qt-mt323.dll
 0001:00006f10       ?dragLeaveEvent@QWidget@@MAEXPAVQDragLeaveEvent@@@Z 10007f10 f   qt-mt323:qt-mt323.dll
 0001:00006f16       ?dragLeft@QListViewItem@@MAEXXZ 10007f16 f   qt-mt323:qt-mt323.dll
 0001:00006f1c       ?dragMoveEvent@QWidget@@MAEXPAVQDragMoveEvent@@@Z 10007f1c f   qt-mt323:qt-mt323.dll
 0001:00006f22       ?drawContents@QDockWindow@@MAEXPAVQPainter@@@Z 10007f22 f   qt-mt323:qt-mt323.dll
 0001:00006f28       ?drawContents@QPopupMenu@@MAEXPAVQPainter@@@Z 10007f28 f   qt-mt323:qt-mt323.dll
 0001:00006f2e       ?drawFrame@QDockWindow@@MAEXPAVQPainter@@@Z 10007f2e f   qt-mt323:qt-mt323.dll
 0001:00006f34       ?drawFrame@QFrame@@MAEXPAVQPainter@@@Z 10007f34 f   qt-mt323:qt-mt323.dll
 0001:00006f3a       ?dropEvent@QWidget@@MAEXPAVQDropEvent@@@Z 10007f3a f   qt-mt323:qt-mt323.dll
 0001:00006f40       ?dropped@QListViewItem@@MAEXPAVQDropEvent@@@Z 10007f40 f   qt-mt323:qt-mt323.dll
 0001:00006f46       ?enabledChange@QPopupMenu@@MAEX_N@Z 10007f46 f   qt-mt323:qt-mt323.dll
 0001:00006f4c       ?enabledChange@QWidget@@MAEX_N@Z 10007f4c f   qt-mt323:qt-mt323.dll
 0001:00006f52       ?enforceSortOrder@QListViewItem@@MBEXXZ 10007f52 f   qt-mt323:qt-mt323.dll
 0001:00006f58       ?enterEvent@QWidget@@MAEXPAVQEvent@@@Z 10007f58 f   qt-mt323:qt-mt323.dll
 0001:00006f5e       ?event@QDockWindow@@MAE_NPAVQEvent@@@Z 10007f5e f   qt-mt323:qt-mt323.dll
 0001:00006f64       ?event@QObject@@UAE_NPAVQEvent@@@Z 10007f64 f   qt-mt323:qt-mt323.dll
 0001:00006f6a       ?event@QToolBar@@UAE_NPAVQEvent@@@Z 10007f6a f   qt-mt323:qt-mt323.dll
 0001:00006f70       ?event@QWidget@@MAE_NPAVQEvent@@@Z 10007f70 f   qt-mt323:qt-mt323.dll
 0001:00006f76       ?eventFilter@QDockWindow@@UAE_NPAVQObject@@PAVQEvent@@@Z 10007f76 f   qt-mt323:qt-mt323.dll
 0001:00006f7c       ?eventFilter@QObject@@UAE_NPAV1@PAVQEvent@@@Z 10007f7c f   qt-mt323:qt-mt323.dll
 0001:00006f82       ?focusInEvent@QPopupMenu@@MAEXPAVQFocusEvent@@@Z 10007f82 f   qt-mt323:qt-mt323.dll
 0001:00006f88       ?focusInEvent@QWidget@@MAEXPAVQFocusEvent@@@Z 10007f88 f   qt-mt323:qt-mt323.dll
 0001:00006f8e       ?focusNextPrevChild@QPopupMenu@@MAE_N_N@Z 10007f8e f   qt-mt323:qt-mt323.dll
 0001:00006f94       ?focusNextPrevChild@QWidget@@MAE_N_N@Z 10007f94 f   qt-mt323:qt-mt323.dll
 0001:00006f9a       ?focusOutEvent@QPopupMenu@@MAEXPAVQFocusEvent@@@Z 10007f9a f   qt-mt323:qt-mt323.dll
 0001:00006fa0       ?focusOutEvent@QWidget@@MAEXPAVQFocusEvent@@@Z 10007fa0 f   qt-mt323:qt-mt323.dll
 0001:00006fa6       ?fontChange@QWidget@@MAEXABVQFont@@@Z 10007fa6 f   qt-mt323:qt-mt323.dll
 0001:00006fac       ?fontInf@QPaintDevice@@MBEHPAVQFont@@H@Z 10007fac f   qt-mt323:qt-mt323.dll
 0001:00006fb2       ?fontMet@QPaintDevice@@MBEHPAVQFont@@HPBDH@Z 10007fb2 f   qt-mt323:qt-mt323.dll
 0001:00006fb8       ?frameChanged@QFrame@@MAEXXZ 10007fb8 f   qt-mt323:qt-mt323.dll
 0001:00006fbe       ?frameChanged@QPopupMenu@@EAEXXZ 10007fbe f   qt-mt323:qt-mt323.dll
 0001:00006fc4       ?handle@QPaintDevice@@UBEPAUHDC__@@XZ 10007fc4 f   qt-mt323:qt-mt323.dll
 0001:00006fca       ?heightForWidth@QWidget@@UBEHH@Z 10007fca f   qt-mt323:qt-mt323.dll
 0001:00006fd0       ?hide@QPopupMenu@@UAEXXZ   10007fd0 f   qt-mt323:qt-mt323.dll
 0001:00006fd6       ?hide@QToolBar@@UAEXXZ     10007fd6 f   qt-mt323:qt-mt323.dll
 0001:00006fdc       ?hide@QWidget@@UAEXXZ      10007fdc f   qt-mt323:qt-mt323.dll
 0001:00006fe2       ?hideEvent@QDockWindow@@MAEXPAVQHideEvent@@@Z 10007fe2 f   qt-mt323:qt-mt323.dll
 0001:00006fe8       ?hideEvent@QWidget@@MAEXPAVQHideEvent@@@Z 10007fe8 f   qt-mt323:qt-mt323.dll
 0001:00006fee       ?imComposeEvent@QWidget@@MAEXPAVQIMEvent@@@Z 10007fee f   qt-mt323:qt-mt323.dll
 0001:00006ff4       ?imEndEvent@QWidget@@MAEXPAVQIMEvent@@@Z 10007ff4 f   qt-mt323:qt-mt323.dll
 0001:00006ffa       ?imStartEvent@QWidget@@MAEXPAVQIMEvent@@@Z 10007ffa f   qt-mt323:qt-mt323.dll
 0001:00007000       ?insertChild@QObject@@UAEXPAV1@@Z 10008000 f   qt-mt323:qt-mt323.dll
 0001:00007006       ?insertItem@QListViewItem@@UAEXPAV1@@Z 10008006 f   qt-mt323:qt-mt323.dll
 0001:0000700c       ?invalidateHeight@QListViewItem@@UAEXXZ 1000800c f   qt-mt323:qt-mt323.dll
 0001:00007012       ?key@QListViewItem@@UBE?AVQString@@H_N@Z 10008012 f   qt-mt323:qt-mt323.dll
 0001:00007018       ?keyPressEvent@QPopupMenu@@MAEXPAVQKeyEvent@@@Z 10008018 f   qt-mt323:qt-mt323.dll
 0001:0000701e       ?keyPressEvent@QWidget@@MAEXPAVQKeyEvent@@@Z 1000801e f   qt-mt323:qt-mt323.dll
 0001:00007024       ?keyReleaseEvent@QWidget@@MAEXPAVQKeyEvent@@@Z 10008024 f   qt-mt323:qt-mt323.dll
 0001:0000702a       ?leaveEvent@QPopupMenu@@MAEXPAVQEvent@@@Z 1000802a f   qt-mt323:qt-mt323.dll
 0001:00007030       ?leaveEvent@QWidget@@MAEXPAVQEvent@@@Z 10008030 f   qt-mt323:qt-mt323.dll
 0001:00007036       ?menuContentsChanged@QPopupMenu@@EAEXXZ 10008036 f   qt-mt323:qt-mt323.dll
 0001:0000703c       ?menuDelPopup@QPopupMenu@@EAEXPAV1@@Z 1000803c f   qt-mt323:qt-mt323.dll
 0001:00007042       ?menuInsPopup@QPopupMenu@@EAEXPAV1@@Z 10008042 f   qt-mt323:qt-mt323.dll
 0001:00007048       ?menuStateChanged@QPopupMenu@@EAEXXZ 10008048 f   qt-mt323:qt-mt323.dll
 0001:0000704e       ?metaObject@QAction@@UBEPAVQMetaObject@@XZ 1000804e f   qt-mt323:qt-mt323.dll
 0001:00007054       ?metaObject@QDockWindow@@UBEPAVQMetaObject@@XZ 10008054 f   qt-mt323:qt-mt323.dll
 0001:0000705a       ?metaObject@QGuardedPtrPrivate@@UBEPAVQMetaObject@@XZ 1000805a f   qt-mt323:qt-mt323.dll
 0001:00007060       ?metaObject@QPopupMenu@@UBEPAVQMetaObject@@XZ 10008060 f   qt-mt323:qt-mt323.dll
 0001:00007066       ?metaObject@QToolBar@@UBEPAVQMetaObject@@XZ 10008066 f   qt-mt323:qt-mt323.dll
 0001:0000706c       ?metaObject@QWidget@@UBEPAVQMetaObject@@XZ 1000806c f   qt-mt323:qt-mt323.dll
 0001:00007072       ?metric@QWidget@@MBEHH@Z   10008072 f   qt-mt323:qt-mt323.dll
 0001:00007078       ?minimumSizeHint@QDockWindow@@UBE?AVQSize@@XZ 10008078 f   qt-mt323:qt-mt323.dll
 0001:0000707e       ?minimumSizeHint@QToolBar@@UBE?AVQSize@@XZ 1000807e f   qt-mt323:qt-mt323.dll
 0001:00007084       ?minimumSizeHint@QWidget@@UBE?AVQSize@@XZ 10008084 f   qt-mt323:qt-mt323.dll
 0001:0000708a       ?mouseDoubleClickEvent@QWidget@@MAEXPAVQMouseEvent@@@Z 1000808a f   qt-mt323:qt-mt323.dll
 0001:00007090       ?mouseMoveEvent@QPopupMenu@@MAEXPAVQMouseEvent@@@Z 10008090 f   qt-mt323:qt-mt323.dll
 0001:00007096       ?mouseMoveEvent@QWidget@@MAEXPAVQMouseEvent@@@Z 10008096 f   qt-mt323:qt-mt323.dll
 0001:0000709c       ?mousePressEvent@QPopupMenu@@MAEXPAVQMouseEvent@@@Z 1000809c f   qt-mt323:qt-mt323.dll
 0001:000070a2       ?mousePressEvent@QWidget@@MAEXPAVQMouseEvent@@@Z 100080a2 f   qt-mt323:qt-mt323.dll
 0001:000070a8       ?mouseReleaseEvent@QPopupMenu@@MAEXPAVQMouseEvent@@@Z 100080a8 f   qt-mt323:qt-mt323.dll
 0001:000070ae       ?mouseReleaseEvent@QWidget@@MAEXPAVQMouseEvent@@@Z 100080ae f   qt-mt323:qt-mt323.dll
 0001:000070b4       ?move@QWidget@@UAEXHH@Z    100080b4 f   qt-mt323:qt-mt323.dll
 0001:000070ba       ?moveEvent@QWidget@@MAEXPAVQMoveEvent@@@Z 100080ba f   qt-mt323:qt-mt323.dll
 0001:000070c0       ?newItem@QPtrCollection@@MAEPAXPAX@Z 100080c0 f   qt-mt323:qt-mt323.dll
 0001:000070c6       ?okRename@QListViewItem@@MAEXH@Z 100080c6 f   qt-mt323:qt-mt323.dll
 0001:000070cc       ?paintBranches@QListViewItem@@UAEXPAVQPainter@@ABVQColorGroup@@HHH@Z 100080cc f   qt-mt323:qt-mt323.dll
 0001:000070d2       ?paintCell@QListViewItem@@UAEXPAVQPainter@@ABVQColorGroup@@HHH@Z 100080d2 f   qt-mt323:qt-mt323.dll
 0001:000070d8       ?paintEvent@QFrame@@MAEXPAVQPaintEvent@@@Z 100080d8 f   qt-mt323:qt-mt323.dll
 0001:000070de       ?paintEvent@QPopupMenu@@MAEXPAVQPaintEvent@@@Z 100080de f   qt-mt323:qt-mt323.dll
 0001:000070e4       ?paintEvent@QWidget@@MAEXPAVQPaintEvent@@@Z 100080e4 f   qt-mt323:qt-mt323.dll
 0001:000070ea       ?paintFocus@QListViewItem@@UAEXPAVQPainter@@ABVQColorGroup@@ABVQRect@@@Z 100080ea f   qt-mt323:qt-mt323.dll
 0001:000070f0       ?paletteChange@QWidget@@MAEXABVQPalette@@@Z 100080f0 f   qt-mt323:qt-mt323.dll
 0001:000070f6       ?pixmap@QListViewItem@@UBEPBVQPixmap@@H@Z 100080f6 f   qt-mt323:qt-mt323.dll
 0001:000070fc       ?polish@QWidget@@UAEXXZ    100080fc f   qt-mt323:qt-mt323.dll
 0001:00007102       ?property@QObject@@UBE?AVQVariant@@PBD@Z 10008102 f   qt-mt323:qt-mt323.dll
 0001:00007108       ?qt_cast@QAction@@UAEPAXPBD@Z 10008108 f   qt-mt323:qt-mt323.dll
 0001:0000710e       ?qt_cast@QDockWindow@@UAEPAXPBD@Z 1000810e f   qt-mt323:qt-mt323.dll
 0001:00007114       ?qt_cast@QGuardedPtrPrivate@@UAEPAXPBD@Z 10008114 f   qt-mt323:qt-mt323.dll
 0001:0000711a       ?qt_cast@QPopupMenu@@UAEPAXPBD@Z 1000811a f   qt-mt323:qt-mt323.dll
 0001:00007120       ?qt_cast@QToolBar@@UAEPAXPBD@Z 10008120 f   qt-mt323:qt-mt323.dll
 0001:00007126       ?qt_cast@QWidget@@UAEPAXPBD@Z 10008126 f   qt-mt323:qt-mt323.dll
 0001:0000712c       ?qt_emit@QAction@@UAE_NHPAUQUObject@@@Z 1000812c f   qt-mt323:qt-mt323.dll
 0001:00007132       ?qt_emit@QDockWindow@@UAE_NHPAUQUObject@@@Z 10008132 f   qt-mt323:qt-mt323.dll
 0001:00007138       ?qt_emit@QGuardedPtrPrivate@@UAE_NHPAUQUObject@@@Z 10008138 f   qt-mt323:qt-mt323.dll
 0001:0000713e       ?qt_emit@QPopupMenu@@UAE_NHPAUQUObject@@@Z 1000813e f   qt-mt323:qt-mt323.dll
 0001:00007144       ?qt_emit@QToolBar@@UAE_NHPAUQUObject@@@Z 10008144 f   qt-mt323:qt-mt323.dll
 0001:0000714a       ?qt_emit@QWidget@@UAE_NHPAUQUObject@@@Z 1000814a f   qt-mt323:qt-mt323.dll
 0001:00007150       ?qt_invoke@QAction@@UAE_NHPAUQUObject@@@Z 10008150 f   qt-mt323:qt-mt323.dll
 0001:00007156       ?qt_invoke@QDockWindow@@UAE_NHPAUQUObject@@@Z 10008156 f   qt-mt323:qt-mt323.dll
 0001:0000715c       ?qt_invoke@QGuardedPtrPrivate@@UAE_NHPAUQUObject@@@Z 1000815c f   qt-mt323:qt-mt323.dll
 0001:00007162       ?qt_invoke@QPopupMenu@@UAE_NHPAUQUObject@@@Z 10008162 f   qt-mt323:qt-mt323.dll
 0001:00007168       ?qt_invoke@QToolBar@@UAE_NHPAUQUObject@@@Z 10008168 f   qt-mt323:qt-mt323.dll
 0001:0000716e       ?qt_invoke@QWidget@@UAE_NHPAUQUObject@@@Z 1000816e f   qt-mt323:qt-mt323.dll
 0001:00007174       ?qt_property@QAction@@UAE_NHHPAVQVariant@@@Z 10008174 f   qt-mt323:qt-mt323.dll
 0001:0000717a       ?qt_property@QDockWindow@@UAE_NHHPAVQVariant@@@Z 1000817a f   qt-mt323:qt-mt323.dll
 0001:00007180       ?qt_property@QGuardedPtrPrivate@@UAE_NHHPAVQVariant@@@Z 10008180 f   qt-mt323:qt-mt323.dll
 0001:00007186       ?qt_property@QPopupMenu@@UAE_NHHPAVQVariant@@@Z 10008186 f   qt-mt323:qt-mt323.dll
 0001:0000718c       ?qt_property@QToolBar@@UAE_NHHPAVQVariant@@@Z 1000818c f   qt-mt323:qt-mt323.dll
 0001:00007192       ?qt_property@QWidget@@UAE_NHHPAVQVariant@@@Z 10008192 f   qt-mt323:qt-mt323.dll
 0001:00007198       ?read@QGDict@@MAEAAVQDataStream@@AAV2@AAPAX@Z 10008198 f   qt-mt323:qt-mt323.dll
 0001:0000719e       ?read@QGList@@MAEAAVQDataStream@@AAV2@AAPAX@Z 1000819e f   qt-mt323:qt-mt323.dll
 0001:000071a4       ?removeChild@QObject@@UAEXPAV1@@Z 100081a4 f   qt-mt323:qt-mt323.dll
 0001:000071aa       ?removeFrom@QAction@@UAE_NPAVQWidget@@@Z 100081aa f   qt-mt323:qt-mt323.dll
 0001:000071b0       ?removeItem@QListViewItem@@UAEXPAV1@@Z 100081b0 f   qt-mt323:qt-mt323.dll
 0001:000071b6       ?reparent@QWidget@@UAEXPAV1@IABVQPoint@@_N@Z 100081b6 f   qt-mt323:qt-mt323.dll
 0001:000071bc       ?resize@QWidget@@UAEXHH@Z  100081bc f   qt-mt323:qt-mt323.dll
 0001:000071c2       ?resizeEvent@QDockWindow@@MAEXPAVQResizeEvent@@@Z 100081c2 f   qt-mt323:qt-mt323.dll
 0001:000071c8       ?resizeEvent@QFrame@@MAEXPAVQResizeEvent@@@Z 100081c8 f   qt-mt323:qt-mt323.dll
 0001:000071ce       ?resizeEvent@QToolBar@@MAEXPAVQResizeEvent@@@Z 100081ce f   qt-mt323:qt-mt323.dll
 0001:000071d4       ?resizeEvent@QWidget@@MAEXPAVQResizeEvent@@@Z 100081d4 f   qt-mt323:qt-mt323.dll
 0001:000071da       ?resolution@QPaintDevice@@UBEHXZ 100081da f   qt-mt323:qt-mt323.dll
 0001:000071e0       ?rtti@QListViewItem@@UBEHXZ 100081e0 f   qt-mt323:qt-mt323.dll
 0001:000071e6       ?setAccel@QAction@@UAEXABVQKeySequence@@@Z 100081e6 f   qt-mt323:qt-mt323.dll
 0001:000071ec       ?setAcceptDrops@QWidget@@UAEX_N@Z 100081ec f   qt-mt323:qt-mt323.dll
 0001:000071f2       ?setActiveItem@QPopupMenu@@UAEXH@Z 100081f2 f   qt-mt323:qt-mt323.dll
 0001:000071f8       ?setActiveWindow@QWidget@@UAEXXZ 100081f8 f   qt-mt323:qt-mt323.dll
 0001:000071fe       ?setAutoMask@QWidget@@UAEX_N@Z 100081fe f   qt-mt323:qt-mt323.dll
 0001:00007204       ?setBackgroundColor@QWidget@@UAEXABVQColor@@@Z 10008204 f   qt-mt323:qt-mt323.dll
 0001:0000720a       ?setBackgroundMode@QWidget@@UAEXW4BackgroundMode@Qt@@@Z 1000820a f   qt-mt323:qt-mt323.dll
 0001:00007210       ?setBackgroundOrigin@QWidget@@UAEXW4BackgroundOrigin@1@@Z 10008210 f   qt-mt323:qt-mt323.dll
 0001:00007216       ?setBackgroundPixmap@QWidget@@UAEXABVQPixmap@@@Z 10008216 f   qt-mt323:qt-mt323.dll
 0001:0000721c       ?setCaption@QDockWindow@@UAEXABVQString@@@Z 1000821c f   qt-mt323:qt-mt323.dll
 0001:00007222       ?setCaption@QWidget@@UAEXABVQString@@@Z 10008222 f   qt-mt323:qt-mt323.dll
 0001:00007228       ?setCheckable@QPopupMenu@@UAEX_N@Z 10008228 f   qt-mt323:qt-mt323.dll
 0001:0000722e       ?setCloseMode@QDockWindow@@UAEXH@Z 1000822e f   qt-mt323:qt-mt323.dll
 0001:00007234       ?setCursor@QWidget@@UAEXABVQCursor@@@Z 10008234 f   qt-mt323:qt-mt323.dll
 0001:0000723a       ?setDragEnabled@QListViewItem@@UAEX_N@Z 1000823a f   qt-mt323:qt-mt323.dll
 0001:00007240       ?setDropEnabled@QListViewItem@@UAEX_N@Z 10008240 f   qt-mt323:qt-mt323.dll
 0001:00007246       ?setEnabled@QAction@@UAEX_N@Z 10008246 f   qt-mt323:qt-mt323.dll
 0001:0000724c       ?setEnabled@QListViewItem@@UAEX_N@Z 1000824c f   qt-mt323:qt-mt323.dll
 0001:00007252       ?setEnabled@QWidget@@UAEX_N@Z 10008252 f   qt-mt323:qt-mt323.dll
 0001:00007258       ?setEraseColor@QWidget@@UAEXABVQColor@@@Z 10008258 f   qt-mt323:qt-mt323.dll
 0001:0000725e       ?setErasePixmap@QWidget@@UAEXABVQPixmap@@@Z 1000825e f   qt-mt323:qt-mt323.dll
 0001:00007264       ?setExpandable@QListViewItem@@UAEX_N@Z 10008264 f   qt-mt323:qt-mt323.dll
 0001:0000726a       ?setFirstItemActive@QPopupMenu@@EAEXXZ 1000826a f   qt-mt323:qt-mt323.dll
 0001:00007270       ?setFixedExtentHeight@QDockWindow@@UAEXH@Z 10008270 f   qt-mt323:qt-mt323.dll
 0001:00007276       ?setFixedExtentWidth@QDockWindow@@UAEXH@Z 10008276 f   qt-mt323:qt-mt323.dll
 0001:0000727c       ?setFocus@QWidget@@UAEXXZ  1000827c f   qt-mt323:qt-mt323.dll
 0001:00007282       ?setFocusPolicy@QWidget@@UAEXW4FocusPolicy@1@@Z 10008282 f   qt-mt323:qt-mt323.dll
 0001:00007288       ?setFocusProxy@QWidget@@UAEXPAV1@@Z 10008288 f   qt-mt323:qt-mt323.dll
 0001:0000728e       ?setFont@QPopupMenu@@UAEXABVQFont@@@Z 1000828e f   qt-mt323:qt-mt323.dll
 0001:00007294       ?setFont@QWidget@@UAEXABVQFont@@@Z 10008294 f   qt-mt323:qt-mt323.dll
 0001:0000729a       ?setFrameRect@QFrame@@UAEXABVQRect@@@Z 1000829a f   qt-mt323:qt-mt323.dll
 0001:000072a0       ?setFrameStyle@QFrame@@UAEXH@Z 100082a0 f   qt-mt323:qt-mt323.dll
 0001:000072a6       ?setGeometry@QWidget@@UAEXABVQRect@@@Z 100082a6 f   qt-mt323:qt-mt323.dll
 0001:000072ac       ?setGeometry@QWidget@@UAEXHHHH@Z 100082ac f   qt-mt323:qt-mt323.dll
 0001:000072b2       ?setHeight@QListViewItem@@MAEXH@Z 100082b2 f   qt-mt323:qt-mt323.dll
 0001:000072b8       ?setHorizontallyStretchable@QDockWindow@@UAEX_N@Z 100082b8 f   qt-mt323:qt-mt323.dll
 0001:000072be       ?setIcon@QWidget@@UAEXABVQPixmap@@@Z 100082be f   qt-mt323:qt-mt323.dll
 0001:000072c4       ?setIconSet@QAction@@UAEXABVQIconSet@@@Z 100082c4 f   qt-mt323:qt-mt323.dll
 0001:000072ca       ?setIconText@QWidget@@UAEXABVQString@@@Z 100082ca f   qt-mt323:qt-mt323.dll
 0001:000072d0       ?setId@QMenuData@@UAEXHH@Z 100082d0 f   qt-mt323:qt-mt323.dll
 0001:000072d6       ?setKeyCompression@QWidget@@MAEX_N@Z 100082d6 f   qt-mt323:qt-mt323.dll
 0001:000072dc       ?setLabel@QToolBar@@UAEXABVQString@@@Z 100082dc f   qt-mt323:qt-mt323.dll
 0001:000072e2       ?setLineWidth@QFrame@@UAEXH@Z 100082e2 f   qt-mt323:qt-mt323.dll
 0001:000072e8       ?setMargin@QFrame@@UAEXH@Z 100082e8 f   qt-mt323:qt-mt323.dll
 0001:000072ee       ?setMask@QWidget@@UAEXABVQBitmap@@@Z 100082ee f   qt-mt323:qt-mt323.dll
 0001:000072f4       ?setMask@QWidget@@UAEXABVQRegion@@@Z 100082f4 f   qt-mt323:qt-mt323.dll
 0001:000072fa       ?setMaximumSize@QWidget@@UAEXHH@Z 100082fa f   qt-mt323:qt-mt323.dll
 0001:00007300       ?setMenuText@QAction@@UAEXABVQString@@@Z 10008300 f   qt-mt323:qt-mt323.dll
 0001:00007306       ?setMicroFocusHint@QWidget@@MAEXHHHH_NPAVQFont@@@Z 10008306 f   qt-mt323:qt-mt323.dll
 0001:0000730c       ?setMidLineWidth@QFrame@@UAEXH@Z 1000830c f   qt-mt323:qt-mt323.dll
 0001:00007312       ?setMinimumSize@QToolBar@@UAEXHH@Z 10008312 f   qt-mt323:qt-mt323.dll
 0001:00007318       ?setMinimumSize@QWidget@@UAEXHH@Z 10008318 f   qt-mt323:qt-mt323.dll
 0001:0000731e       ?setMouseTracking@QWidget@@UAEX_N@Z 1000831e f   qt-mt323:qt-mt323.dll
 0001:00007324       ?setMovingEnabled@QDockWindow@@UAEX_N@Z 10008324 f   qt-mt323:qt-mt323.dll
 0001:0000732a       ?setMultiLinesEnabled@QListViewItem@@UAEX_N@Z 1000832a f   qt-mt323:qt-mt323.dll
 0001:00007330       ?setName@QObject@@UAEXPBD@Z 10008330 f   qt-mt323:qt-mt323.dll
 0001:00007336       ?setNewLine@QDockWindow@@UAEX_N@Z 10008336 f   qt-mt323:qt-mt323.dll
 0001:0000733c       ?setOffset@QDockWindow@@UAEXH@Z 1000833c f   qt-mt323:qt-mt323.dll
 0001:00007342       ?setOn@QAction@@UAEX_N@Z   10008342 f   qt-mt323:qt-mt323.dll
 0001:00007348       ?setOpaqueMoving@QDockWindow@@UAEX_N@Z 10008348 f   qt-mt323:qt-mt323.dll
 0001:0000734e       ?setOpen@QListViewItem@@UAEX_N@Z 1000834e f   qt-mt323:qt-mt323.dll
 0001:00007354       ?setOrientation@QDockWindow@@UAEXW4Orientation@Qt@@@Z 10008354 f   qt-mt323:qt-mt323.dll
 0001:0000735a       ?setOrientation@QToolBar@@UAEXW4Orientation@Qt@@@Z 1000835a f   qt-mt323:qt-mt323.dll
 0001:00007360       ?setPalette@QWidget@@UAEXABVQPalette@@@Z 10008360 f   qt-mt323:qt-mt323.dll
 0001:00007366       ?setPaletteBackgroundColor@QWidget@@UAEXABVQColor@@@Z 10008366 f   qt-mt323:qt-mt323.dll
 0001:0000736c       ?setPaletteBackgroundPixmap@QWidget@@UAEXABVQPixmap@@@Z 1000836c f   qt-mt323:qt-mt323.dll
 0001:00007372       ?setPixmap@QListViewItem@@UAEXHABVQPixmap@@@Z 10008372 f   qt-mt323:qt-mt323.dll
 0001:00007378       ?setProperty@QObject@@UAE_NPBDABVQVariant@@@Z 10008378 f   qt-mt323:qt-mt323.dll
 0001:0000737e       ?setRenameEnabled@QListViewItem@@UAEXH_N@Z 1000837e f   qt-mt323:qt-mt323.dll
 0001:00007384       ?setResizeEnabled@QDockWindow@@UAEX_N@Z 10008384 f   qt-mt323:qt-mt323.dll
 0001:0000738a       ?setResolution@QPaintDevice@@UAEXH@Z 1000838a f   qt-mt323:qt-mt323.dll
 0001:00007390       ?setSelectable@QListViewItem@@UAEX_N@Z 10008390 f   qt-mt323:qt-mt323.dll
 0001:00007396       ?setSelected@QListViewItem@@UAEX_N@Z 10008396 f   qt-mt323:qt-mt323.dll
 0001:0000739c       ?setSizeIncrement@QWidget@@UAEXHH@Z 1000839c f   qt-mt323:qt-mt323.dll
 0001:000073a2       ?setSizePolicy@QWidget@@UAEXVQSizePolicy@@@Z 100083a2 f   qt-mt323:qt-mt323.dll
 0001:000073a8       ?setStatusTip@QAction@@UAEXABVQString@@@Z 100083a8 f   qt-mt323:qt-mt323.dll
 0001:000073ae       ?setStretchableWidget@QToolBar@@UAEXPAVQWidget@@@Z 100083ae f   qt-mt323:qt-mt323.dll
 0001:000073b4       ?setText@QAction@@UAEXABVQString@@@Z 100083b4 f   qt-mt323:qt-mt323.dll
 0001:000073ba       ?setText@QListViewItem@@UAEXHABVQString@@@Z 100083ba f   qt-mt323:qt-mt323.dll
 0001:000073c0       ?setToggleAction@QAction@@UAEX_N@Z 100083c0 f   qt-mt323:qt-mt323.dll
 0001:000073c6       ?setToolTip@QAction@@UAEXABVQString@@@Z 100083c6 f   qt-mt323:qt-mt323.dll
 0001:000073cc       ?setUpdatesEnabled@QWidget@@UAEX_N@Z 100083cc f   qt-mt323:qt-mt323.dll
 0001:000073d2       ?setVerticallyStretchable@QDockWindow@@UAEX_N@Z 100083d2 f   qt-mt323:qt-mt323.dll
 0001:000073d8       ?setWFlags@QWidget@@MAEXI@Z 100083d8 f   qt-mt323:qt-mt323.dll
 0001:000073de       ?setWState@QWidget@@MAEXI@Z 100083de f   qt-mt323:qt-mt323.dll
 0001:000073e4       ?setWhatsThis@QAction@@UAEXABVQString@@@Z 100083e4 f   qt-mt323:qt-mt323.dll
 0001:000073ea       ?setWidget@QDockWindow@@UAEXPAVQWidget@@@Z 100083ea f   qt-mt323:qt-mt323.dll
 0001:000073f0       ?setup@QListViewItem@@UAEXXZ 100083f0 f   qt-mt323:qt-mt323.dll
 0001:000073f6       ?show@QPopupMenu@@UAEXXZ   100083f6 f   qt-mt323:qt-mt323.dll
 0001:000073fc       ?show@QToolBar@@UAEXXZ     100083fc f   qt-mt323:qt-mt323.dll
 0001:00007402       ?show@QWidget@@UAEXXZ      10008402 f   qt-mt323:qt-mt323.dll
 0001:00007408       ?showEvent@QDockWindow@@MAEXPAVQShowEvent@@@Z 10008408 f   qt-mt323:qt-mt323.dll
 0001:0000740e       ?showEvent@QWidget@@MAEXPAVQShowEvent@@@Z 1000840e f   qt-mt323:qt-mt323.dll
 0001:00007414       ?showMaximized@QWidget@@UAEXXZ 10008414 f   qt-mt323:qt-mt323.dll
 0001:0000741a       ?showMinimized@QWidget@@UAEXXZ 1000841a f   qt-mt323:qt-mt323.dll
 0001:00007420       ?showNormal@QWidget@@UAEXXZ 10008420 f   qt-mt323:qt-mt323.dll
 0001:00007426       ?sizeHint@QDockWindow@@UBE?AVQSize@@XZ 10008426 f   qt-mt323:qt-mt323.dll
 0001:0000742c       ?sizeHint@QPopupMenu@@UBE?AVQSize@@XZ 1000842c f   qt-mt323:qt-mt323.dll
 0001:00007432       ?sizeHint@QWidget@@UBE?AVQSize@@XZ 10008432 f   qt-mt323:qt-mt323.dll
 0001:00007438       ?sizePolicy@QWidget@@UBE?AVQSizePolicy@@XZ 10008438 f   qt-mt323:qt-mt323.dll
 0001:0000743e       ?sort@QListViewItem@@UAEXXZ 1000843e f   qt-mt323:qt-mt323.dll
 0001:00007444       ?sortChildItems@QListViewItem@@UAEXH_N@Z 10008444 f   qt-mt323:qt-mt323.dll
 0001:0000744a       ?startRename@QListViewItem@@UAEXH@Z 1000844a f   qt-mt323:qt-mt323.dll
 0001:00007450       ?styleChange@QFrame@@MAEXAAVQStyle@@@Z 10008450 f   qt-mt323:qt-mt323.dll
 0001:00007456       ?styleChange@QPopupMenu@@MAEXAAVQStyle@@@Z 10008456 f   qt-mt323:qt-mt323.dll
 0001:0000745c       ?styleChange@QToolBar@@MAEXAAVQStyle@@@Z 1000845c f   qt-mt323:qt-mt323.dll
 0001:00007462       ?styleChange@QWidget@@MAEXAAVQStyle@@@Z 10008462 f   qt-mt323:qt-mt323.dll
 0001:00007468       ?tabletEvent@QWidget@@MAEXPAVQTabletEvent@@@Z 10008468 f   qt-mt323:qt-mt323.dll
 0001:0000746e       ?takeItem@QListViewItem@@UAEXPAV1@@Z 1000846e f   qt-mt323:qt-mt323.dll
 0001:00007474       ?text@QListViewItem@@UBE?AVQString@@H@Z 10008474 f   qt-mt323:qt-mt323.dll
 0001:0000747a       ?timerEvent@QObject@@MAEXPAVQTimerEvent@@@Z 1000847a f   qt-mt323:qt-mt323.dll
 0001:00007480       ?timerEvent@QPopupMenu@@MAEXPAVQTimerEvent@@@Z 10008480 f   qt-mt323:qt-mt323.dll
 0001:00007486       ?undock@QDockWindow@@UAEXPAVQWidget@@@Z 10008486 f   qt-mt323:qt-mt323.dll
 0001:0000748c       ?undock@QDockWindow@@UAEXXZ 1000848c f   qt-mt323:qt-mt323.dll
 0001:00007492       ?unsetCursor@QWidget@@UAEXXZ 10008492 f   qt-mt323:qt-mt323.dll
 0001:00007498       ?updateItem@QPopupMenu@@UAEXH@Z 10008498 f   qt-mt323:qt-mt323.dll
 0001:0000749e       ?updateMask@QWidget@@MAEXXZ 1000849e f   qt-mt323:qt-mt323.dll
 0001:000074a4       ?wheelEvent@QWidget@@MAEXPAVQWheelEvent@@@Z 100084a4 f   qt-mt323:qt-mt323.dll
 0001:000074aa       ?width@QListViewItem@@UBEHABVQFontMetrics@@PBVQListView@@H@Z 100084aa f   qt-mt323:qt-mt323.dll
 0001:000074b0       ?winEvent@QWidget@@MAE_NPAUtagMSG@@@Z 100084b0 f   qt-mt323:qt-mt323.dll
 0001:000074b6       ?windowActivationChange@QWidget@@MAEX_N@Z 100084b6 f   qt-mt323:qt-mt323.dll
 0001:000074bc       ?write@QGDict@@MBEAAVQDataStream@@AAV2@PAX@Z 100084bc f   qt-mt323:qt-mt323.dll
 0001:000074c2       ?write@QGList@@MBEAAVQDataStream@@AAV2@PAX@Z 100084c2 f   qt-mt323:qt-mt323.dll
 0001:000074c8       ?activateNextCell@QTable@@MAEXXZ 100084c8 f   qt-mt323:qt-mt323.dll
 0001:000074ce       ?addChild@QScrollView@@UAEXPAVQWidget@@HH@Z 100084ce f   qt-mt323:qt-mt323.dll
 0001:000074d4       ?addItem@QBoxLayout@@UAEXPAVQLayoutItem@@@Z 100084d4 f   qt-mt323:qt-mt323.dll
 0001:000074da       ?addSelection@QTable@@UAEHABVQTableSelection@@@Z 100084da f   qt-mt323:qt-mt323.dll
 0001:000074e0       ?addTab@QTabWidget@@UAEXPAVQWidget@@ABVQIconSet@@ABVQString@@@Z 100084e0 f   qt-mt323:qt-mt323.dll
 0001:000074e6       ?addTab@QTabWidget@@UAEXPAVQWidget@@ABVQString@@@Z 100084e6 f   qt-mt323:qt-mt323.dll
 0001:000074ec       ?addTab@QTabWidget@@UAEXPAVQWidget@@PAVQTab@@@Z 100084ec f   qt-mt323:qt-mt323.dll
 0001:000074f2       ?adjustColumn@QTable@@UAEXH@Z 100084f2 f   qt-mt323:qt-mt323.dll
 0001:000074f8       ?adjustRow@QTable@@UAEXH@Z 100084f8 f   qt-mt323:qt-mt323.dll
 0001:000074fe       ?append@QTextEdit@@UAEXABVQString@@@Z 100084fe f   qt-mt323:qt-mt323.dll
 0001:00007504       ?beginEdit@QTable@@MAEPAVQWidget@@HH_N@Z 10008504 f   qt-mt323:qt-mt323.dll
 0001:0000750a       ?cellGeometry@QTable@@UBE?AVQRect@@HH@Z 1000850a f   qt-mt323:qt-mt323.dll
 0001:00007510       ?cellRect@QTable@@UBE?AVQRect@@HH@Z 10008510 f   qt-mt323:qt-mt323.dll
 0001:00007516       ?cellWidget@QTable@@UBEPAVQWidget@@HH@Z 10008516 f   qt-mt323:qt-mt323.dll
 0001:0000751c       ?childEvent@QLayout@@MAEXPAVQChildEvent@@@Z 1000851c f   qt-mt323:qt-mt323.dll
 0001:00007522       ?className@QHBoxLayout@@UBEPBDXZ 10008522 f   qt-mt323:qt-mt323.dll
 0001:00007528       ?className@QLabel@@UBEPBDXZ 10008528 f   qt-mt323:qt-mt323.dll
 0001:0000752e       ?className@QLineEdit@@UBEPBDXZ 1000852e f   qt-mt323:qt-mt323.dll
 0001:00007534       ?className@QTabWidget@@UBEPBDXZ 10008534 f   qt-mt323:qt-mt323.dll
 0001:0000753a       ?className@QTable@@UBEPBDXZ 1000853a f   qt-mt323:qt-mt323.dll
 0001:00007540       ?className@QTextEdit@@UBEPBDXZ 10008540 f   qt-mt323:qt-mt323.dll
 0001:00007546       ?className@QVBoxLayout@@UBEPBDXZ 10008546 f   qt-mt323:qt-mt323.dll
 0001:0000754c       ?clear@QLineEdit@@UAEXXZ   1000854c f   qt-mt323:qt-mt323.dll
 0001:00007552       ?clear@QTextEdit@@UAEXXZ   10008552 f   qt-mt323:qt-mt323.dll
 0001:00007558       ?clearCell@QTable@@UAEXHH@Z 10008558 f   qt-mt323:qt-mt323.dll
 0001:0000755e       ?clearCellWidget@QTable@@UAEXHH@Z 1000855e f   qt-mt323:qt-mt323.dll
 0001:00007564       ?clearParagraphBackground@QTextEdit@@UAEXH@Z 10008564 f   qt-mt323:qt-mt323.dll
 0001:0000756a       ?clearValidator@QLineEdit@@UAEXXZ 1000856a f   qt-mt323:qt-mt323.dll
 0001:00007570       ?columnAt@QTable@@UBEHH@Z  10008570 f   qt-mt323:qt-mt323.dll
 0001:00007576       ?columnClicked@QTable@@MAEXH@Z 10008576 f   qt-mt323:qt-mt323.dll
 0001:0000757c       ?columnIndexChanged@QTable@@MAEXHHH@Z 1000857c f   qt-mt323:qt-mt323.dll
 0001:00007582       ?columnPos@QTable@@UBEHH@Z 10008582 f   qt-mt323:qt-mt323.dll
 0001:00007588       ?columnWidth@QTable@@UBEHH@Z 10008588 f   qt-mt323:qt-mt323.dll
 0001:0000758e       ?columnWidthChanged@QTable@@MAEXH@Z 1000858e f   qt-mt323:qt-mt323.dll
 0001:00007594       ?contentsContextMenuEvent@QTable@@MAEXPAVQContextMenuEvent@@@Z 10008594 f   qt-mt323:qt-mt323.dll
 0001:0000759a       ?contentsContextMenuEvent@QTextEdit@@MAEXPAVQContextMenuEvent@@@Z 1000859a f   qt-mt323:qt-mt323.dll
 0001:000075a0       ?contentsDragEnterEvent@QTable@@MAEXPAVQDragEnterEvent@@@Z 100085a0 f   qt-mt323:qt-mt323.dll
 0001:000075a6       ?contentsDragEnterEvent@QTextEdit@@MAEXPAVQDragEnterEvent@@@Z 100085a6 f   qt-mt323:qt-mt323.dll
 0001:000075ac       ?contentsDragLeaveEvent@QTable@@MAEXPAVQDragLeaveEvent@@@Z 100085ac f   qt-mt323:qt-mt323.dll
 0001:000075b2       ?contentsDragLeaveEvent@QTextEdit@@MAEXPAVQDragLeaveEvent@@@Z 100085b2 f   qt-mt323:qt-mt323.dll
 0001:000075b8       ?contentsDragMoveEvent@QTable@@MAEXPAVQDragMoveEvent@@@Z 100085b8 f   qt-mt323:qt-mt323.dll
 0001:000075be       ?contentsDragMoveEvent@QTextEdit@@MAEXPAVQDragMoveEvent@@@Z 100085be f   qt-mt323:qt-mt323.dll
 0001:000075c4       ?contentsDropEvent@QTable@@MAEXPAVQDropEvent@@@Z 100085c4 f   qt-mt323:qt-mt323.dll
 0001:000075ca       ?contentsDropEvent@QTextEdit@@MAEXPAVQDropEvent@@@Z 100085ca f   qt-mt323:qt-mt323.dll
 0001:000075d0       ?contentsMouseDoubleClickEvent@QTable@@MAEXPAVQMouseEvent@@@Z 100085d0 f   qt-mt323:qt-mt323.dll
 0001:000075d6       ?contentsMouseDoubleClickEvent@QTextEdit@@MAEXPAVQMouseEvent@@@Z 100085d6 f   qt-mt323:qt-mt323.dll
 0001:000075dc       ?contentsMouseMoveEvent@QTable@@MAEXPAVQMouseEvent@@@Z 100085dc f   qt-mt323:qt-mt323.dll
 0001:000075e2       ?contentsMouseMoveEvent@QTextEdit@@MAEXPAVQMouseEvent@@@Z 100085e2 f   qt-mt323:qt-mt323.dll
 0001:000075e8       ?contentsMousePressEvent@QTable@@MAEXPAVQMouseEvent@@@Z 100085e8 f   qt-mt323:qt-mt323.dll
 0001:000075ee       ?contentsMousePressEvent@QTextEdit@@MAEXPAVQMouseEvent@@@Z 100085ee f   qt-mt323:qt-mt323.dll
 0001:000075f4       ?contentsMouseReleaseEvent@QTable@@MAEXPAVQMouseEvent@@@Z 100085f4 f   qt-mt323:qt-mt323.dll
 0001:000075fa       ?contentsMouseReleaseEvent@QTextEdit@@MAEXPAVQMouseEvent@@@Z 100085fa f   qt-mt323:qt-mt323.dll
 0001:00007600       ?contentsWheelEvent@QScrollView@@MAEXPAVQWheelEvent@@@Z 10008600 f   qt-mt323:qt-mt323.dll
 0001:00007606       ?contentsWheelEvent@QTextEdit@@MAEXPAVQWheelEvent@@@Z 10008606 f   qt-mt323:qt-mt323.dll
 0001:0000760c       ?contextMenuEvent@QLineEdit@@MAEXPAVQContextMenuEvent@@@Z 1000860c f   qt-mt323:qt-mt323.dll
 0001:00007612       ?contextMenuEvent@QScrollView@@MAEXPAVQContextMenuEvent@@@Z 10008612 f   qt-mt323:qt-mt323.dll
 0001:00007618       ?copy@QLineEdit@@UBEXXZ    10008618 f   qt-mt323:qt-mt323.dll
 0001:0000761e       ?copy@QTextEdit@@UAEXXZ    1000861e f   qt-mt323:qt-mt323.dll
 0001:00007624       ?createEditor@QTable@@MBEPAVQWidget@@HH_N@Z 10008624 f   qt-mt323:qt-mt323.dll
 0001:0000762a       ?createPopupMenu@QLineEdit@@MAEPAVQPopupMenu@@XZ 1000862a f   qt-mt323:qt-mt323.dll
 0001:00007630       ?createPopupMenu@QTextEdit@@MAEPAVQPopupMenu@@ABVQPoint@@@Z 10008630 f   qt-mt323:qt-mt323.dll
 0001:00007636       ?createPopupMenu@QTextEdit@@MAEPAVQPopupMenu@@XZ 10008636 f   qt-mt323:qt-mt323.dll
 0001:0000763c       ?currentSelection@QTable@@UBEHXZ 1000863c f   qt-mt323:qt-mt323.dll
 0001:00007642       ?cut@QLineEdit@@UAEXXZ     10008642 f   qt-mt323:qt-mt323.dll
 0001:00007648       ?cut@QTextEdit@@UAEXXZ     10008648 f   qt-mt323:qt-mt323.dll
 0001:0000764e       ?del@QTextEdit@@UAEXXZ     1000864e f   qt-mt323:qt-mt323.dll
 0001:00007654       ?deselect@QLineEdit@@UAEXXZ 10008654 f   qt-mt323:qt-mt323.dll
 0001:0000765a       ?doChangeInterval@QTextEdit@@MAEXXZ 1000865a f   qt-mt323:qt-mt323.dll
 0001:00007660       ?doKeyboardAction@QTextEdit@@UAEXW4KeyboardAction@1@@Z 10008660 f   qt-mt323:qt-mt323.dll
 0001:00007666       ?dragEnterEvent@QLineEdit@@MAEXPAVQDragEnterEvent@@@Z 10008666 f   qt-mt323:qt-mt323.dll
 0001:0000766c       ?dragLeaveEvent@QLineEdit@@MAEXPAVQDragLeaveEvent@@@Z 1000866c f   qt-mt323:qt-mt323.dll
 0001:00007672       ?dragMoveEvent@QLineEdit@@MAEXPAVQDragMoveEvent@@@Z 10008672 f   qt-mt323:qt-mt323.dll
 0001:00007678       ?dragObject@QTable@@MAEPAVQDragObject@@XZ 10008678 f   qt-mt323:qt-mt323.dll
 0001:0000767e       ?drawContents@QLabel@@MAEXPAVQPainter@@@Z 1000867e f   qt-mt323:qt-mt323.dll
 0001:00007684       ?drawContents@QLineEdit@@MAEXPAVQPainter@@@Z 10008684 f   qt-mt323:qt-mt323.dll
 0001:0000768a       ?drawContents@QTable@@EAEXPAVQPainter@@@Z 1000868a f   qt-mt323:qt-mt323.dll
 0001:00007690       ?drawContents@QTable@@MAEXPAVQPainter@@HHHH@Z 10008690 f   qt-mt323:qt-mt323.dll
 0001:00007696       ?drawContents@QTextEdit@@EAEXPAVQPainter@@@Z 10008696 f   qt-mt323:qt-mt323.dll
 0001:0000769c       ?drawContents@QTextEdit@@MAEXPAVQPainter@@HHHH@Z 1000869c f   qt-mt323:qt-mt323.dll
 0001:000076a2       ?drawContentsOffset@QScrollView@@MAEXPAVQPainter@@HHHHHH@Z 100086a2 f   qt-mt323:qt-mt323.dll
 0001:000076a8       ?dropEvent@QLineEdit@@MAEXPAVQDropEvent@@@Z 100086a8 f   qt-mt323:qt-mt323.dll
 0001:000076ae       ?editCell@QTable@@UAEXHH_N@Z 100086ae f   qt-mt323:qt-mt323.dll
 0001:000076b4       ?emitHighlighted@QTextEdit@@EAEXABVQString@@@Z 100086b4 f   qt-mt323:qt-mt323.dll
 0001:000076ba       ?emitLinkClicked@QTextEdit@@EAEXABVQString@@@Z 100086ba f   qt-mt323:qt-mt323.dll
 0001:000076c0       ?endEdit@QTable@@MAEXHH_N0@Z 100086c0 f   qt-mt323:qt-mt323.dll
 0001:000076c6       ?ensureCursorVisible@QTextEdit@@UAEXXZ 100086c6 f   qt-mt323:qt-mt323.dll
 0001:000076cc       ?event@QLineEdit@@MAE_NPAVQEvent@@@Z 100086cc f   qt-mt323:qt-mt323.dll
 0001:000076d2       ?event@QTextEdit@@MAE_NPAVQEvent@@@Z 100086d2 f   qt-mt323:qt-mt323.dll
 0001:000076d8       ?eventFilter@QLayout@@MAE_NPAVQObject@@PAVQEvent@@@Z 100086d8 f   qt-mt323:qt-mt323.dll
 0001:000076de       ?eventFilter@QTabWidget@@MAE_NPAVQObject@@PAVQEvent@@@Z 100086de f   qt-mt323:qt-mt323.dll
 0001:000076e4       ?eventFilter@QTable@@UAE_NPAVQObject@@PAVQEvent@@@Z 100086e4 f   qt-mt323:qt-mt323.dll
 0001:000076ea       ?eventFilter@QTextEdit@@UAE_NPAVQObject@@PAVQEvent@@@Z 100086ea f   qt-mt323:qt-mt323.dll
 0001:000076f0       ?expanding@QBoxLayout@@UBE?AW4ExpandData@QSizePolicy@@XZ 100086f0 f   qt-mt323:qt-mt323.dll
 0001:000076f6       ?expanding@QSpacerItem@@UBE?AW4ExpandData@QSizePolicy@@XZ 100086f6 f   qt-mt323:qt-mt323.dll
 0001:000076fc       ?find@QTextEdit@@UAE_NABVQString@@_N11PAH2@Z 100086fc f   qt-mt323:qt-mt323.dll
 0001:00007702       ?focusInEvent@QLineEdit@@MAEXPAVQFocusEvent@@@Z 10008702 f   qt-mt323:qt-mt323.dll
 0001:00007708       ?focusInEvent@QTable@@MAEXPAVQFocusEvent@@@Z 10008708 f   qt-mt323:qt-mt323.dll
 0001:0000770e       ?focusNextPrevChild@QScrollView@@MAE_N_N@Z 1000870e f   qt-mt323:qt-mt323.dll
 0001:00007714       ?focusNextPrevChild@QTextEdit@@MAE_N_N@Z 10008714 f   qt-mt323:qt-mt323.dll
 0001:0000771a       ?focusOutEvent@QLineEdit@@MAEXPAVQFocusEvent@@@Z 1000871a f   qt-mt323:qt-mt323.dll
 0001:00007720       ?focusOutEvent@QTable@@MAEXPAVQFocusEvent@@@Z 10008720 f   qt-mt323:qt-mt323.dll
 0001:00007726       ?fontChange@QLabel@@MAEXABVQFont@@@Z 10008726 f   qt-mt323:qt-mt323.dll
 0001:0000772c       ?fontChange@QScrollView@@MAEXABVQFont@@@Z 1000872c f   qt-mt323:qt-mt323.dll
 0001:00007732       ?frameChanged@QScrollView@@MAEXXZ 10008732 f   qt-mt323:qt-mt323.dll
 0001:00007738       ?geometry@QLayout@@UBE?AVQRect@@XZ 10008738 f   qt-mt323:qt-mt323.dll
 0001:0000773e       ?geometry@QSpacerItem@@UBE?AVQRect@@XZ 1000873e f   qt-mt323:qt-mt323.dll
 0001:00007744       ?getFormat@QTextEdit@@UAE_NHHPAVQFont@@PAVQColor@@PAW4VerticalAlignment@1@@Z 10008744 f   qt-mt323:qt-mt323.dll
 0001:0000774a       ?getParagraphFormat@QTextEdit@@UAE_NHPAVQFont@@PAVQColor@@PAW4VerticalAlignment@1@PAHPAW4DisplayMode@QStyleSheetItem@@PAW4ListStyle@6@3@Z 1000874a f   qt-mt323:qt-mt323.dll
 0001:00007750       ?hasHeightForWidth@QBoxLayout@@UBE_NXZ 10008750 f   qt-mt323:qt-mt323.dll
 0001:00007756       ?hasHeightForWidth@QLayoutItem@@UBE_NXZ 10008756 f   qt-mt323:qt-mt323.dll
 0001:0000775c       ?heightForWidth@QBoxLayout@@UBEHH@Z 1000875c f   qt-mt323:qt-mt323.dll
 0001:00007762       ?heightForWidth@QLabel@@UBEHH@Z 10008762 f   qt-mt323:qt-mt323.dll
 0001:00007768       ?heightForWidth@QLayoutItem@@UBEHH@Z 10008768 f   qt-mt323:qt-mt323.dll
 0001:0000776e       ?heightForWidth@QTextEdit@@UBEHH@Z 1000876e f   qt-mt323:qt-mt323.dll
 0001:00007774       ?hideColumn@QTable@@UAEXH@Z 10008774 f   qt-mt323:qt-mt323.dll
 0001:0000777a       ?hideRow@QTable@@UAEXH@Z   1000877a f   qt-mt323:qt-mt323.dll
 0001:00007780       ?imComposeEvent@QLineEdit@@MAEXPAVQIMEvent@@@Z 10008780 f   qt-mt323:qt-mt323.dll
 0001:00007786       ?imComposeEvent@QTextEdit@@MAEXPAVQIMEvent@@@Z 10008786 f   qt-mt323:qt-mt323.dll
 0001:0000778c       ?imEndEvent@QLineEdit@@MAEXPAVQIMEvent@@@Z 1000878c f   qt-mt323:qt-mt323.dll
 0001:00007792       ?imEndEvent@QTextEdit@@MAEXPAVQIMEvent@@@Z 10008792 f   qt-mt323:qt-mt323.dll
 0001:00007798       ?imStartEvent@QLineEdit@@MAEXPAVQIMEvent@@@Z 10008798 f   qt-mt323:qt-mt323.dll
 0001:0000779e       ?imStartEvent@QTextEdit@@MAEXPAVQIMEvent@@@Z 1000879e f   qt-mt323:qt-mt323.dll
 0001:000077a4       ?indent@QTextEdit@@UAEXXZ  100087a4 f   qt-mt323:qt-mt323.dll
 0001:000077aa       ?insert@QLineEdit@@UAEXABVQString@@@Z 100087aa f   qt-mt323:qt-mt323.dll
 0001:000077b0       ?insert@QTextEdit@@UAEXABVQString@@_N11@Z 100087b0 f   qt-mt323:qt-mt323.dll
 0001:000077b6       ?insertAt@QTextEdit@@UAEXABVQString@@HH@Z 100087b6 f   qt-mt323:qt-mt323.dll
 0001:000077bc       ?insertColumns@QTable@@UAEXHH@Z 100087bc f   qt-mt323:qt-mt323.dll
 0001:000077c2       ?insertParagraph@QTextEdit@@UAEXABVQString@@H@Z 100087c2 f   qt-mt323:qt-mt323.dll
 0001:000077c8       ?insertRows@QTable@@UAEXHH@Z 100087c8 f   qt-mt323:qt-mt323.dll
 0001:000077ce       ?insertTab@QTabWidget@@UAEXPAVQWidget@@ABVQIconSet@@ABVQString@@H@Z 100087ce f   qt-mt323:qt-mt323.dll
 0001:000077d4       ?insertTab@QTabWidget@@UAEXPAVQWidget@@ABVQString@@H@Z 100087d4 f   qt-mt323:qt-mt323.dll
 0001:000077da       ?insertTab@QTabWidget@@UAEXPAVQWidget@@PAVQTab@@H@Z 100087da f   qt-mt323:qt-mt323.dll
 0001:000077e0       ?insertWidget@QTable@@MAEXHHPAVQWidget@@@Z 100087e0 f   qt-mt323:qt-mt323.dll
 0001:000077e6       ?invalidate@QBoxLayout@@UAEXXZ 100087e6 f   qt-mt323:qt-mt323.dll
 0001:000077ec       ?invalidate@QLayoutItem@@UAEXXZ 100087ec f   qt-mt323:qt-mt323.dll
 0001:000077f2       ?isEmpty@QLayout@@UBE_NXZ  100087f2 f   qt-mt323:qt-mt323.dll
 0001:000077f8       ?isEmpty@QSpacerItem@@UBE_NXZ 100087f8 f   qt-mt323:qt-mt323.dll
 0001:000077fe       ?item@QTable@@UBEPAVQTableItem@@HH@Z 100087fe f   qt-mt323:qt-mt323.dll
 0001:00007804       ?iterator@QBoxLayout@@UAE?AVQLayoutIterator@@XZ 10008804 f   qt-mt323:qt-mt323.dll
 0001:0000780a       ?iterator@QLayoutItem@@UAE?AVQLayoutIterator@@XZ 1000880a f   qt-mt323:qt-mt323.dll
 0001:00007810       ?keyPressEvent@QLineEdit@@MAEXPAVQKeyEvent@@@Z 10008810 f   qt-mt323:qt-mt323.dll
 0001:00007816       ?keyPressEvent@QTable@@MAEXPAVQKeyEvent@@@Z 10008816 f   qt-mt323:qt-mt323.dll
 0001:0000781c       ?keyPressEvent@QTextEdit@@MAEXPAVQKeyEvent@@@Z 1000881c f   qt-mt323:qt-mt323.dll
 0001:00007822       ?layout@QLayout@@UAEPAV1@XZ 10008822 f   qt-mt323:qt-mt323.dll
 0001:00007828       ?layout@QLayoutItem@@UAEPAVQLayout@@XZ 10008828 f   qt-mt323:qt-mt323.dll
 0001:0000782e       ?linksEnabled@QTextEdit@@EBE_NXZ 1000882e f   qt-mt323:qt-mt323.dll
 0001:00007834       ?maximumSize@QBoxLayout@@UBE?AVQSize@@XZ 10008834 f   qt-mt323:qt-mt323.dll
 0001:0000783a       ?maximumSize@QSpacerItem@@UBE?AVQSize@@XZ 1000883a f   qt-mt323:qt-mt323.dll
 0001:00007840       ?metaObject@QHBoxLayout@@UBEPAVQMetaObject@@XZ 10008840 f   qt-mt323:qt-mt323.dll
 0001:00007846       ?metaObject@QLabel@@UBEPAVQMetaObject@@XZ 10008846 f   qt-mt323:qt-mt323.dll
 0001:0000784c       ?metaObject@QLineEdit@@UBEPAVQMetaObject@@XZ 1000884c f   qt-mt323:qt-mt323.dll
 0001:00007852       ?metaObject@QTabWidget@@UBEPAVQMetaObject@@XZ 10008852 f   qt-mt323:qt-mt323.dll
 0001:00007858       ?metaObject@QTable@@UBEPAVQMetaObject@@XZ 10008858 f   qt-mt323:qt-mt323.dll
 0001:0000785e       ?metaObject@QTextEdit@@UBEPAVQMetaObject@@XZ 1000885e f   qt-mt323:qt-mt323.dll
 0001:00007864       ?metaObject@QVBoxLayout@@UBEPAVQMetaObject@@XZ 10008864 f   qt-mt323:qt-mt323.dll
 0001:0000786a       ?minimumSize@QBoxLayout@@UBE?AVQSize@@XZ 1000886a f   qt-mt323:qt-mt323.dll
 0001:00007870       ?minimumSize@QSpacerItem@@UBE?AVQSize@@XZ 10008870 f   qt-mt323:qt-mt323.dll
 0001:00007876       ?minimumSizeHint@QLabel@@UBE?AVQSize@@XZ 10008876 f   qt-mt323:qt-mt323.dll
 0001:0000787c       ?minimumSizeHint@QLineEdit@@UBE?AVQSize@@XZ 1000887c f   qt-mt323:qt-mt323.dll
 0001:00007882       ?minimumSizeHint@QScrollView@@UBE?AVQSize@@XZ 10008882 f   qt-mt323:qt-mt323.dll
 0001:00007888       ?minimumSizeHint@QTabWidget@@UBE?AVQSize@@XZ 10008888 f   qt-mt323:qt-mt323.dll
 0001:0000788e       ?mouseDoubleClickEvent@QLineEdit@@MAEXPAVQMouseEvent@@@Z 1000888e f   qt-mt323:qt-mt323.dll
 0001:00007894       ?mouseDoubleClickEvent@QScrollView@@MAEXPAVQMouseEvent@@@Z 10008894 f   qt-mt323:qt-mt323.dll
 0001:0000789a       ?mouseMoveEvent@QLineEdit@@MAEXPAVQMouseEvent@@@Z 1000889a f   qt-mt323:qt-mt323.dll
 0001:000078a0       ?mouseMoveEvent@QScrollView@@MAEXPAVQMouseEvent@@@Z 100088a0 f   qt-mt323:qt-mt323.dll
 0001:000078a6       ?mousePressEvent@QLineEdit@@MAEXPAVQMouseEvent@@@Z 100088a6 f   qt-mt323:qt-mt323.dll
 0001:000078ac       ?mousePressEvent@QScrollView@@MAEXPAVQMouseEvent@@@Z 100088ac f   qt-mt323:qt-mt323.dll
 0001:000078b2       ?mouseReleaseEvent@QLineEdit@@MAEXPAVQMouseEvent@@@Z 100088b2 f   qt-mt323:qt-mt323.dll
 0001:000078b8       ?mouseReleaseEvent@QScrollView@@MAEXPAVQMouseEvent@@@Z 100088b8 f   qt-mt323:qt-mt323.dll
 0001:000078be       ?moveChild@QScrollView@@UAEXPAVQWidget@@HH@Z 100088be f   qt-mt323:qt-mt323.dll
 0001:000078c4       ?moveCursor@QTextEdit@@UAEXW4CursorAction@1@_N@Z 100088c4 f   qt-mt323:qt-mt323.dll
 0001:000078ca       ?numCols@QTable@@UBEHXZ    100088ca f   qt-mt323:qt-mt323.dll
 0001:000078d0       ?numRows@QTable@@UBEHXZ    100088d0 f   qt-mt323:qt-mt323.dll
 0001:000078d6       ?paintCell@QTable@@UAEXPAVQPainter@@HHABVQRect@@_N@Z 100088d6 f   qt-mt323:qt-mt323.dll
 0001:000078dc       ?paintCell@QTable@@UAEXPAVQPainter@@HHABVQRect@@_NABVQColorGroup@@@Z 100088dc f   qt-mt323:qt-mt323.dll
 0001:000078e2       ?paintEmptyArea@QTable@@MAEXPAVQPainter@@HHHH@Z 100088e2 f   qt-mt323:qt-mt323.dll
 0001:000078e8       ?paintEvent@QTable@@MAEXPAVQPaintEvent@@@Z 100088e8 f   qt-mt323:qt-mt323.dll
 0001:000078ee       ?paintFocus@QTable@@UAEXPAVQPainter@@ABVQRect@@@Z 100088ee f   qt-mt323:qt-mt323.dll
 0001:000078f4       ?paste@QLineEdit@@UAEXXZ   100088f4 f   qt-mt323:qt-mt323.dll
 0001:000078fa       ?paste@QTextEdit@@UAEXXZ   100088fa f   qt-mt323:qt-mt323.dll
 0001:00007900       ?pasteSubType@QTextEdit@@UAEXABVQCString@@@Z 10008900 f   qt-mt323:qt-mt323.dll
 0001:00007906       ?pixmap@QTable@@UBE?AVQPixmap@@HH@Z 10008906 f   qt-mt323:qt-mt323.dll
 0001:0000790c       ?placeCursor@QTextEdit@@UAEXABVQPoint@@PAVQTextCursor@@@Z 1000890c f   qt-mt323:qt-mt323.dll
 0001:00007912       ?polish@QTextEdit@@UAEXXZ  10008912 f   qt-mt323:qt-mt323.dll
 0001:00007918       ?qt_cast@QHBoxLayout@@UAEPAXPBD@Z 10008918 f   qt-mt323:qt-mt323.dll
 0001:0000791e       ?qt_cast@QLabel@@UAEPAXPBD@Z 1000891e f   qt-mt323:qt-mt323.dll
 0001:00007924       ?qt_cast@QLineEdit@@UAEPAXPBD@Z 10008924 f   qt-mt323:qt-mt323.dll
 0001:0000792a       ?qt_cast@QTabWidget@@UAEPAXPBD@Z 1000892a f   qt-mt323:qt-mt323.dll
 0001:00007930       ?qt_cast@QTable@@UAEPAXPBD@Z 10008930 f   qt-mt323:qt-mt323.dll
 0001:00007936       ?qt_cast@QTextEdit@@UAEPAXPBD@Z 10008936 f   qt-mt323:qt-mt323.dll
 0001:0000793c       ?qt_cast@QVBoxLayout@@UAEPAXPBD@Z 1000893c f   qt-mt323:qt-mt323.dll
 0001:00007942       ?qt_emit@QHBoxLayout@@UAE_NHPAUQUObject@@@Z 10008942 f   qt-mt323:qt-mt323.dll
 0001:00007948       ?qt_emit@QLabel@@UAE_NHPAUQUObject@@@Z 10008948 f   qt-mt323:qt-mt323.dll
 0001:0000794e       ?qt_emit@QLineEdit@@UAE_NHPAUQUObject@@@Z 1000894e f   qt-mt323:qt-mt323.dll
 0001:00007954       ?qt_emit@QTabWidget@@UAE_NHPAUQUObject@@@Z 10008954 f   qt-mt323:qt-mt323.dll
 0001:0000795a       ?qt_emit@QTable@@UAE_NHPAUQUObject@@@Z 1000895a f   qt-mt323:qt-mt323.dll
 0001:00007960       ?qt_emit@QTextEdit@@UAE_NHPAUQUObject@@@Z 10008960 f   qt-mt323:qt-mt323.dll
 0001:00007966       ?qt_emit@QVBoxLayout@@UAE_NHPAUQUObject@@@Z 10008966 f   qt-mt323:qt-mt323.dll
 0001:0000796c       ?qt_invoke@QHBoxLayout@@UAE_NHPAUQUObject@@@Z 1000896c f   qt-mt323:qt-mt323.dll
 0001:00007972       ?qt_invoke@QLabel@@UAE_NHPAUQUObject@@@Z 10008972 f   qt-mt323:qt-mt323.dll
 0001:00007978       ?qt_invoke@QLineEdit@@UAE_NHPAUQUObject@@@Z 10008978 f   qt-mt323:qt-mt323.dll
 0001:0000797e       ?qt_invoke@QTabWidget@@UAE_NHPAUQUObject@@@Z 1000897e f   qt-mt323:qt-mt323.dll
 0001:00007984       ?qt_invoke@QTable@@UAE_NHPAUQUObject@@@Z 10008984 f   qt-mt323:qt-mt323.dll
 0001:0000798a       ?qt_invoke@QTextEdit@@UAE_NHPAUQUObject@@@Z 1000898a f   qt-mt323:qt-mt323.dll
 0001:00007990       ?qt_invoke@QVBoxLayout@@UAE_NHPAUQUObject@@@Z 10008990 f   qt-mt323:qt-mt323.dll
 0001:00007996       ?qt_property@QHBoxLayout@@UAE_NHHPAVQVariant@@@Z 10008996 f   qt-mt323:qt-mt323.dll
 0001:0000799c       ?qt_property@QLabel@@UAE_NHHPAVQVariant@@@Z 1000899c f   qt-mt323:qt-mt323.dll
 0001:000079a2       ?qt_property@QLineEdit@@UAE_NHHPAVQVariant@@@Z 100089a2 f   qt-mt323:qt-mt323.dll
 0001:000079a8       ?qt_property@QTabWidget@@UAE_NHHPAVQVariant@@@Z 100089a8 f   qt-mt323:qt-mt323.dll
 0001:000079ae       ?qt_property@QTable@@UAE_NHHPAVQVariant@@@Z 100089ae f   qt-mt323:qt-mt323.dll
 0001:000079b4       ?qt_property@QTextEdit@@UAE_NHHPAVQVariant@@@Z 100089b4 f   qt-mt323:qt-mt323.dll
 0001:000079ba       ?qt_property@QVBoxLayout@@UAE_NHHPAVQVariant@@@Z 100089ba f   qt-mt323:qt-mt323.dll
 0001:000079c0       ?redo@QLineEdit@@UAEXXZ    100089c0 f   qt-mt323:qt-mt323.dll
 0001:000079c6       ?redo@QTextEdit@@UAEXXZ    100089c6 f   qt-mt323:qt-mt323.dll
 0001:000079cc       ?removeChild@QScrollView@@UAEXPAVQObject@@@Z 100089cc f   qt-mt323:qt-mt323.dll
 0001:000079d2       ?removeColumn@QTable@@UAEXH@Z 100089d2 f   qt-mt323:qt-mt323.dll
 0001:000079d8       ?removeColumns@QTable@@UAEXABV?$QMemArray@H@@@Z 100089d8 f   qt-mt323:qt-mt323.dll
 0001:000079de       ?removePage@QTabWidget@@UAEXPAVQWidget@@@Z 100089de f   qt-mt323:qt-mt323.dll
 0001:000079e4       ?removeParagraph@QTextEdit@@UAEXH@Z 100089e4 f   qt-mt323:qt-mt323.dll
 0001:000079ea       ?removeRow@QTable@@UAEXH@Z 100089ea f   qt-mt323:qt-mt323.dll
 0001:000079f0       ?removeRows@QTable@@UAEXABV?$QMemArray@H@@@Z 100089f0 f   qt-mt323:qt-mt323.dll
 0001:000079f6       ?removeSelectedText@QTextEdit@@UAEXH@Z 100089f6 f   qt-mt323:qt-mt323.dll
 0001:000079fc       ?removeSelection@QTable@@UAEXABVQTableSelection@@@Z 100089fc f   qt-mt323:qt-mt323.dll
 0001:00007a02       ?removeSelection@QTable@@UAEXH@Z 10008a02 f   qt-mt323:qt-mt323.dll
 0001:00007a08       ?removeSelection@QTextEdit@@UAEXH@Z 10008a08 f   qt-mt323:qt-mt323.dll
 0001:00007a0e       ?resetFormat@QTextEdit@@UAEXXZ 10008a0e f   qt-mt323:qt-mt323.dll
 0001:00007a14       ?resize@QScrollView@@UAEXHH@Z 10008a14 f   qt-mt323:qt-mt323.dll
 0001:00007a1a       ?resizeContents@QScrollView@@UAEXHH@Z 10008a1a f   qt-mt323:qt-mt323.dll
 0001:00007a20       ?resizeData@QTable@@MAEXH@Z 10008a20 f   qt-mt323:qt-mt323.dll
 0001:00007a26       ?resizeEvent@QLabel@@MAEXPAVQResizeEvent@@@Z 10008a26 f   qt-mt323:qt-mt323.dll
 0001:00007a2c       ?resizeEvent@QLineEdit@@MAEXPAVQResizeEvent@@@Z 10008a2c f   qt-mt323:qt-mt323.dll
 0001:00007a32       ?resizeEvent@QScrollView@@MAEXPAVQResizeEvent@@@Z 10008a32 f   qt-mt323:qt-mt323.dll
 0001:00007a38       ?resizeEvent@QTabWidget@@MAEXPAVQResizeEvent@@@Z 10008a38 f   qt-mt323:qt-mt323.dll
 0001:00007a3e       ?resizeEvent@QTextEdit@@MAEXPAVQResizeEvent@@@Z 10008a3e f   qt-mt323:qt-mt323.dll
 0001:00007a44       ?rowAt@QTable@@UBEHH@Z     10008a44 f   qt-mt323:qt-mt323.dll
 0001:00007a4a       ?rowHeight@QTable@@UBEHH@Z 10008a4a f   qt-mt323:qt-mt323.dll
 0001:00007a50       ?rowHeightChanged@QTable@@MAEXH@Z 10008a50 f   qt-mt323:qt-mt323.dll
 0001:00007a56       ?rowIndexChanged@QTable@@MAEXHHH@Z 10008a56 f   qt-mt323:qt-mt323.dll
 0001:00007a5c       ?rowPos@QTable@@UBEHH@Z    10008a5c f   qt-mt323:qt-mt323.dll
 0001:00007a62       ?scrollToAnchor@QTextEdit@@UAEXABVQString@@@Z 10008a62 f   qt-mt323:qt-mt323.dll
 0001:00007a68       ?scrollToBottom@QTextEdit@@UAEXXZ 10008a68 f   qt-mt323:qt-mt323.dll
 0001:00007a6e       ?selectAll@QLineEdit@@UAEXXZ 10008a6e f   qt-mt323:qt-mt323.dll
 0001:00007a74       ?selectAll@QTextEdit@@UAEX_N@Z 10008a74 f   qt-mt323:qt-mt323.dll
 0001:00007a7a       ?setAlignment@QLabel@@UAEXH@Z 10008a7a f   qt-mt323:qt-mt323.dll
 0001:00007a80       ?setAlignment@QLayoutItem@@UAEXH@Z 10008a80 f   qt-mt323:qt-mt323.dll
 0001:00007a86       ?setAlignment@QLineEdit@@UAEXH@Z 10008a86 f   qt-mt323:qt-mt323.dll
 0001:00007a8c       ?setAlignment@QTextEdit@@UAEXH@Z 10008a8c f   qt-mt323:qt-mt323.dll
 0001:00007a92       ?setAutoAdd@QLayout@@UAEX_N@Z 10008a92 f   qt-mt323:qt-mt323.dll
 0001:00007a98       ?setAutoResize@QLabel@@UAEX_N@Z 10008a98 f   qt-mt323:qt-mt323.dll
 0001:00007a9e       ?setBold@QTextEdit@@UAEX_N@Z 10008a9e f   qt-mt323:qt-mt323.dll
 0001:00007aa4       ?setBuddy@QLabel@@UAEXPAVQWidget@@@Z 10008aa4 f   qt-mt323:qt-mt323.dll
 0001:00007aaa       ?setCellContentFromEditor@QTable@@MAEXHH@Z 10008aaa f   qt-mt323:qt-mt323.dll
 0001:00007ab0       ?setCellWidget@QTable@@UAEXHHPAVQWidget@@@Z 10008ab0 f   qt-mt323:qt-mt323.dll
 0001:00007ab6       ?setColor@QTextEdit@@UAEXABVQColor@@@Z 10008ab6 f   qt-mt323:qt-mt323.dll
 0001:00007abc       ?setColumnMovingEnabled@QTable@@UAEX_N@Z 10008abc f   qt-mt323:qt-mt323.dll
 0001:00007ac2       ?setColumnReadOnly@QTable@@UAEXH_N@Z 10008ac2 f   qt-mt323:qt-mt323.dll
 0001:00007ac8       ?setColumnStretchable@QTable@@UAEXH_N@Z 10008ac8 f   qt-mt323:qt-mt323.dll
 0001:00007ace       ?setColumnWidth@QTable@@UAEXHH@Z 10008ace f   qt-mt323:qt-mt323.dll
 0001:00007ad4       ?setContentsPos@QScrollView@@UAEXHH@Z 10008ad4 f   qt-mt323:qt-mt323.dll
 0001:00007ada       ?setCornerWidget@QScrollView@@UAEXPAVQWidget@@@Z 10008ada f   qt-mt323:qt-mt323.dll
 0001:00007ae0       ?setCurrentCell@QTable@@UAEXHH@Z 10008ae0 f   qt-mt323:qt-mt323.dll
 0001:00007ae6       ?setCurrentFont@QTextEdit@@UAEXABVQFont@@@Z 10008ae6 f   qt-mt323:qt-mt323.dll
 0001:00007aec       ?setCursorPosition@QLineEdit@@UAEXH@Z 10008aec f   qt-mt323:qt-mt323.dll
 0001:00007af2       ?setCursorPosition@QTextEdit@@UAEXHH@Z 10008af2 f   qt-mt323:qt-mt323.dll
 0001:00007af8       ?setDragAutoScroll@QScrollView@@UAEX_N@Z 10008af8 f   qt-mt323:qt-mt323.dll
 0001:00007afe       ?setDragEnabled@QLineEdit@@UAEX_N@Z 10008afe f   qt-mt323:qt-mt323.dll
 0001:00007b04       ?setDragEnabled@QTable@@UAEX_N@Z 10008b04 f   qt-mt323:qt-mt323.dll
 0001:00007b0a       ?setEchoMode@QLineEdit@@UAEXW4EchoMode@1@@Z 10008b0a f   qt-mt323:qt-mt323.dll
 0001:00007b10       ?setEnabled@QTable@@UAEX_N@Z 10008b10 f   qt-mt323:qt-mt323.dll
 0001:00007b16       ?setEnabled@QTextEdit@@UAEX_N@Z 10008b16 f   qt-mt323:qt-mt323.dll
 0001:00007b1c       ?setFamily@QTextEdit@@UAEXABVQString@@@Z 10008b1c f   qt-mt323:qt-mt323.dll
 0001:00007b22       ?setFocusStyle@QTable@@UAEXW4FocusStyle@1@@Z 10008b22 f   qt-mt323:qt-mt323.dll
 0001:00007b28       ?setFont@QLabel@@UAEXABVQFont@@@Z 10008b28 f   qt-mt323:qt-mt323.dll
 0001:00007b2e       ?setFont@QLineEdit@@UAEXABVQFont@@@Z 10008b2e f   qt-mt323:qt-mt323.dll
 0001:00007b34       ?setFont@QTextEdit@@UAEXABVQFont@@@Z 10008b34 f   qt-mt323:qt-mt323.dll
 0001:00007b3a       ?setFormat@QTextEdit@@UAEXPAVQTextFormat@@H@Z 10008b3a f   qt-mt323:qt-mt323.dll
 0001:00007b40       ?setFrame@QLineEdit@@UAEX_N@Z 10008b40 f   qt-mt323:qt-mt323.dll
 0001:00007b46       ?setGeometry@QBoxLayout@@UAEXABVQRect@@@Z 10008b46 f   qt-mt323:qt-mt323.dll
 0001:00007b4c       ?setGeometry@QSpacerItem@@UAEXABVQRect@@@Z 10008b4c f   qt-mt323:qt-mt323.dll
 0001:00007b52       ?setHBarGeometry@QScrollView@@MAEXAAVQScrollBar@@HHHH@Z 10008b52 f   qt-mt323:qt-mt323.dll
 0001:00007b58       ?setHScrollBarMode@QScrollView@@UAEXW4ScrollBarMode@1@@Z 10008b58 f   qt-mt323:qt-mt323.dll
 0001:00007b5e       ?setItalic@QTextEdit@@UAEX_N@Z 10008b5e f   qt-mt323:qt-mt323.dll
 0001:00007b64       ?setItem@QTable@@UAEXHHPAVQTableItem@@@Z 10008b64 f   qt-mt323:qt-mt323.dll
 0001:00007b6a       ?setLeftMargin@QTable@@UAEXH@Z 10008b6a f   qt-mt323:qt-mt323.dll
 0001:00007b70       ?setLinkUnderline@QTextEdit@@UAEX_N@Z 10008b70 f   qt-mt323:qt-mt323.dll
 0001:00007b76       ?setMargin@QLayout@@UAEXH@Z 10008b76 f   qt-mt323:qt-mt323.dll
 0001:00007b7c       ?setMargins@QScrollView@@MAEXHHHH@Z 10008b7c f   qt-mt323:qt-mt323.dll
 0001:00007b82       ?setMaxLength@QLineEdit@@UAEXH@Z 10008b82 f   qt-mt323:qt-mt323.dll
 0001:00007b88       ?setMenuBar@QLayout@@UAEXPAVQMenuBar@@@Z 10008b88 f   qt-mt323:qt-mt323.dll
 0001:00007b8e       ?setMimeSourceFactory@QTextEdit@@UAEXPAVQMimeSourceFactory@@@Z 10008b8e f   qt-mt323:qt-mt323.dll
 0001:00007b94       ?setModified@QTextEdit@@UAEX_N@Z 10008b94 f   qt-mt323:qt-mt323.dll
 0001:00007b9a       ?setMovie@QLabel@@UAEXABVQMovie@@@Z 10008b9a f   qt-mt323:qt-mt323.dll
 0001:00007ba0       ?setNum@QLabel@@UAEXH@Z    10008ba0 f   qt-mt323:qt-mt323.dll
 0001:00007ba6       ?setNum@QLabel@@UAEXN@Z    10008ba6 f   qt-mt323:qt-mt323.dll
 0001:00007bac       ?setNumCols@QTable@@UAEXH@Z 10008bac f   qt-mt323:qt-mt323.dll
 0001:00007bb2       ?setNumRows@QTable@@UAEXH@Z 10008bb2 f   qt-mt323:qt-mt323.dll
 0001:00007bb8       ?setOverwriteMode@QTextEdit@@UAEX_N@Z 10008bb8 f   qt-mt323:qt-mt323.dll
 0001:00007bbe       ?setPalette@QLineEdit@@UAEXABVQPalette@@@Z 10008bbe f   qt-mt323:qt-mt323.dll
 0001:00007bc4       ?setPalette@QTextEdit@@UAEXABVQPalette@@@Z 10008bc4 f   qt-mt323:qt-mt323.dll
 0001:00007bca       ?setPaper@QTextEdit@@UAEXABVQBrush@@@Z 10008bca f   qt-mt323:qt-mt323.dll
 0001:00007bd0       ?setParagType@QTextEdit@@UAEXW4DisplayMode@QStyleSheetItem@@W4ListStyle@3@@Z 10008bd0 f   qt-mt323:qt-mt323.dll
 0001:00007bd6       ?setParagraphBackgroundColor@QTextEdit@@UAEXHABVQColor@@@Z 10008bd6 f   qt-mt323:qt-mt323.dll
 0001:00007bdc       ?setPicture@QLabel@@UAEXABVQPicture@@@Z 10008bdc f   qt-mt323:qt-mt323.dll
 0001:00007be2       ?setPixmap@QLabel@@UAEXABVQPixmap@@@Z 10008be2 f   qt-mt323:qt-mt323.dll
 0001:00007be8       ?setPixmap@QTable@@UAEXHHABVQPixmap@@@Z 10008be8 f   qt-mt323:qt-mt323.dll
 0001:00007bee       ?setPointSize@QTextEdit@@UAEXH@Z 10008bee f   qt-mt323:qt-mt323.dll
 0001:00007bf4       ?setReadOnly@QLineEdit@@UAEX_N@Z 10008bf4 f   qt-mt323:qt-mt323.dll
 0001:00007bfa       ?setReadOnly@QTable@@UAEX_N@Z 10008bfa f   qt-mt323:qt-mt323.dll
 0001:00007c00       ?setReadOnly@QTextEdit@@UAEX_N@Z 10008c00 f   qt-mt323:qt-mt323.dll
 0001:00007c06       ?setResizePolicy@QScrollView@@UAEXW4ResizePolicy@1@@Z 10008c06 f   qt-mt323:qt-mt323.dll
 0001:00007c0c       ?setRowHeight@QTable@@UAEXHH@Z 10008c0c f   qt-mt323:qt-mt323.dll
 0001:00007c12       ?setRowMovingEnabled@QTable@@UAEX_N@Z 10008c12 f   qt-mt323:qt-mt323.dll
 0001:00007c18       ?setRowReadOnly@QTable@@UAEXH_N@Z 10008c18 f   qt-mt323:qt-mt323.dll
 0001:00007c1e       ?setRowStretchable@QTable@@UAEXH_N@Z 10008c1e f   qt-mt323:qt-mt323.dll
 0001:00007c24       ?setSelection@QLineEdit@@UAEXHH@Z 10008c24 f   qt-mt323:qt-mt323.dll
 0001:00007c2a       ?setSelection@QTextEdit@@UAEXHHHHH@Z 10008c2a f   qt-mt323:qt-mt323.dll
 0001:00007c30       ?setSelectionAttributes@QTextEdit@@UAEXHABVQColor@@_N@Z 10008c30 f   qt-mt323:qt-mt323.dll
 0001:00007c36       ?setSelectionMode@QTable@@UAEXW4SelectionMode@1@@Z 10008c36 f   qt-mt323:qt-mt323.dll
 0001:00007c3c       ?setShowGrid@QTable@@UAEX_N@Z 10008c3c f   qt-mt323:qt-mt323.dll
 0001:00007c42       ?setSorting@QTable@@UAEX_N@Z 10008c42 f   qt-mt323:qt-mt323.dll
 0001:00007c48       ?setSpacing@QLayout@@UAEXH@Z 10008c48 f   qt-mt323:qt-mt323.dll
 0001:00007c4e       ?setStyleSheet@QTextEdit@@UAEXPAVQStyleSheet@@@Z 10008c4e f   qt-mt323:qt-mt323.dll
 0001:00007c54       ?setTabStopWidth@QTextEdit@@UAEXH@Z 10008c54 f   qt-mt323:qt-mt323.dll
 0001:00007c5a       ?setText@QLabel@@UAEXABVQString@@@Z 10008c5a f   qt-mt323:qt-mt323.dll
 0001:00007c60       ?setText@QLineEdit@@UAEXABVQString@@@Z 10008c60 f   qt-mt323:qt-mt323.dll
 0001:00007c66       ?setText@QTable@@UAEXHHABVQString@@@Z 10008c66 f   qt-mt323:qt-mt323.dll
 0001:00007c6c       ?setText@QTextEdit@@UAEXABVQString@@0@Z 10008c6c f   qt-mt323:qt-mt323.dll
 0001:00007c72       ?setTextFormat@QTextEdit@@UAEXW4TextFormat@Qt@@@Z 10008c72 f   qt-mt323:qt-mt323.dll
 0001:00007c78       ?setTopMargin@QTable@@UAEXH@Z 10008c78 f   qt-mt323:qt-mt323.dll
 0001:00007c7e       ?setUnderline@QTextEdit@@UAEX_N@Z 10008c7e f   qt-mt323:qt-mt323.dll
 0001:00007c84       ?setUndoDepth@QTextEdit@@UAEXH@Z 10008c84 f   qt-mt323:qt-mt323.dll
 0001:00007c8a       ?setUndoRedoEnabled@QTextEdit@@UAEX_N@Z 10008c8a f   qt-mt323:qt-mt323.dll
 0001:00007c90       ?setVBarGeometry@QScrollView@@MAEXAAVQScrollBar@@HHHH@Z 10008c90 f   qt-mt323:qt-mt323.dll
 0001:00007c96       ?setVScrollBarMode@QScrollView@@UAEXW4ScrollBarMode@1@@Z 10008c96 f   qt-mt323:qt-mt323.dll
 0001:00007c9c       ?setValidator@QLineEdit@@UAEXPBVQValidator@@@Z 10008c9c f   qt-mt323:qt-mt323.dll
 0001:00007ca2       ?setVerticalAlignment@QTextEdit@@UAEXW4VerticalAlignment@1@@Z 10008ca2 f   qt-mt323:qt-mt323.dll
 0001:00007ca8       ?setWordWrap@QTextEdit@@UAEXW4WordWrap@1@@Z 10008ca8 f   qt-mt323:qt-mt323.dll
 0001:00007cae       ?setWrapColumnOrWidth@QTextEdit@@UAEXH@Z 10008cae f   qt-mt323:qt-mt323.dll
 0001:00007cb4       ?setWrapPolicy@QTextEdit@@UAEXW4WrapPolicy@1@@Z 10008cb4 f   qt-mt323:qt-mt323.dll
 0001:00007cba       ?show@QScrollView@@UAEXXZ  10008cba f   qt-mt323:qt-mt323.dll
 0001:00007cc0       ?showColumn@QTable@@UAEXH@Z 10008cc0 f   qt-mt323:qt-mt323.dll
 0001:00007cc6       ?showEvent@QTabWidget@@MAEXPAVQShowEvent@@@Z 10008cc6 f   qt-mt323:qt-mt323.dll
 0001:00007ccc       ?showEvent@QTable@@MAEXPAVQShowEvent@@@Z 10008ccc f   qt-mt323:qt-mt323.dll
 0001:00007cd2       ?showPage@QTabWidget@@UAEXPAVQWidget@@@Z 10008cd2 f   qt-mt323:qt-mt323.dll
 0001:00007cd8       ?showRow@QTable@@UAEXH@Z   10008cd8 f   qt-mt323:qt-mt323.dll
 0001:00007cde       ?sizeHint@QBoxLayout@@UBE?AVQSize@@XZ 10008cde f   qt-mt323:qt-mt323.dll
 0001:00007ce4       ?sizeHint@QLabel@@UBE?AVQSize@@XZ 10008ce4 f   qt-mt323:qt-mt323.dll
 0001:00007cea       ?sizeHint@QLineEdit@@UBE?AVQSize@@XZ 10008cea f   qt-mt323:qt-mt323.dll
 0001:00007cf0       ?sizeHint@QSpacerItem@@UBE?AVQSize@@XZ 10008cf0 f   qt-mt323:qt-mt323.dll
 0001:00007cf6       ?sizeHint@QTabWidget@@UBE?AVQSize@@XZ 10008cf6 f   qt-mt323:qt-mt323.dll
 0001:00007cfc       ?sizeHint@QTable@@UBE?AVQSize@@XZ 10008cfc f   qt-mt323:qt-mt323.dll
 0001:00007d02       ?sizeHint@QTextEdit@@UBE?AVQSize@@XZ 10008d02 f   qt-mt323:qt-mt323.dll
 0001:00007d08       ?sortColumn@QTable@@UAEXH_N0@Z 10008d08 f   qt-mt323:qt-mt323.dll
 0001:00007d0e       ?spacerItem@QLayoutItem@@UAEPAVQSpacerItem@@XZ 10008d0e f   qt-mt323:qt-mt323.dll
 0001:00007d14       ?spacerItem@QSpacerItem@@UAEPAV1@XZ 10008d14 f   qt-mt323:qt-mt323.dll
 0001:00007d1a       ?startDrag@QTable@@MAEXXZ  10008d1a f   qt-mt323:qt-mt323.dll
 0001:00007d20       ?styleChange@QScrollView@@UAEXAAVQStyle@@@Z 10008d20 f   qt-mt323:qt-mt323.dll
 0001:00007d26       ?styleChange@QTabWidget@@MAEXAAVQStyle@@@Z 10008d26 f   qt-mt323:qt-mt323.dll
 0001:00007d2c       ?swapCells@QTable@@UAEXHHHH@Z 10008d2c f   qt-mt323:qt-mt323.dll
 0001:00007d32       ?swapColumns@QTable@@UAEXHH_N@Z 10008d32 f   qt-mt323:qt-mt323.dll
 0001:00007d38       ?swapRows@QTable@@UAEXHH_N@Z 10008d38 f   qt-mt323:qt-mt323.dll
 0001:00007d3e       ?sync@QTextEdit@@UAEXXZ    10008d3e f   qt-mt323:qt-mt323.dll
 0001:00007d44       ?takeItem@QTable@@UAEXPAVQTableItem@@@Z 10008d44 f   qt-mt323:qt-mt323.dll
 0001:00007d4a       ?text@QTable@@UBE?AVQString@@HH@Z 10008d4a f   qt-mt323:qt-mt323.dll
 0001:00007d50       ?undo@QLineEdit@@UAEXXZ    10008d50 f   qt-mt323:qt-mt323.dll
 0001:00007d56       ?undo@QTextEdit@@UAEXXZ    10008d56 f   qt-mt323:qt-mt323.dll
 0001:00007d5c       ?updateMask@QTabWidget@@MAEXXZ 10008d5c f   qt-mt323:qt-mt323.dll
 0001:00007d62       ?viewportContextMenuEvent@QScrollView@@MAEXPAVQContextMenuEvent@@@Z 10008d62 f   qt-mt323:qt-mt323.dll
 0001:00007d68       ?viewportDragEnterEvent@QScrollView@@MAEXPAVQDragEnterEvent@@@Z 10008d68 f   qt-mt323:qt-mt323.dll
 0001:00007d6e       ?viewportDragLeaveEvent@QScrollView@@MAEXPAVQDragLeaveEvent@@@Z 10008d6e f   qt-mt323:qt-mt323.dll
 0001:00007d74       ?viewportDragMoveEvent@QScrollView@@MAEXPAVQDragMoveEvent@@@Z 10008d74 f   qt-mt323:qt-mt323.dll
 0001:00007d7a       ?viewportDropEvent@QScrollView@@MAEXPAVQDropEvent@@@Z 10008d7a f   qt-mt323:qt-mt323.dll
 0001:00007d80       ?viewportMouseDoubleClickEvent@QScrollView@@MAEXPAVQMouseEvent@@@Z 10008d80 f   qt-mt323:qt-mt323.dll
 0001:00007d86       ?viewportMouseMoveEvent@QScrollView@@MAEXPAVQMouseEvent@@@Z 10008d86 f   qt-mt323:qt-mt323.dll
 0001:00007d8c       ?viewportMousePressEvent@QScrollView@@MAEXPAVQMouseEvent@@@Z 10008d8c f   qt-mt323:qt-mt323.dll
 0001:00007d92       ?viewportMouseReleaseEvent@QScrollView@@MAEXPAVQMouseEvent@@@Z 10008d92 f   qt-mt323:qt-mt323.dll
 0001:00007d98       ?viewportPaintEvent@QScrollView@@MAEXPAVQPaintEvent@@@Z 10008d98 f   qt-mt323:qt-mt323.dll
 0001:00007d9e       ?viewportResizeEvent@QTable@@MAEXPAVQResizeEvent@@@Z 10008d9e f   qt-mt323:qt-mt323.dll
 0001:00007da4       ?viewportResizeEvent@QTextEdit@@MAEXPAVQResizeEvent@@@Z 10008da4 f   qt-mt323:qt-mt323.dll
 0001:00007daa       ?viewportWheelEvent@QScrollView@@MAEXPAVQWheelEvent@@@Z 10008daa f   qt-mt323:qt-mt323.dll
 0001:00007db0       ?wheelEvent@QScrollView@@MAEXPAVQWheelEvent@@@Z 10008db0 f   qt-mt323:qt-mt323.dll
 0001:00007db6       ?widget@QLayoutItem@@UAEPAVQWidget@@XZ 10008db6 f   qt-mt323:qt-mt323.dll
 0001:00007dbc       ?windowActivationChange@QLineEdit@@MAEX_N@Z 10008dbc f   qt-mt323:qt-mt323.dll
 0001:00007dc2       ?windowActivationChange@QTable@@MAEX_N@Z 10008dc2 f   qt-mt323:qt-mt323.dll
 0001:00007dc8       ?windowActivationChange@QTextEdit@@MAEX_N@Z 10008dc8 f   qt-mt323:qt-mt323.dll
 0001:00007dce       ?zoomIn@QTextEdit@@UAEXH@Z 10008dce f   qt-mt323:qt-mt323.dll
 0001:00007dd4       ?zoomIn@QTextEdit@@UAEXXZ  10008dd4 f   qt-mt323:qt-mt323.dll
 0001:00007dda       ?zoomOut@QTextEdit@@UAEXH@Z 10008dda f   qt-mt323:qt-mt323.dll
 0001:00007de0       ?zoomOut@QTextEdit@@UAEXXZ 10008de0 f   qt-mt323:qt-mt323.dll
 0001:00007de6       ?zoomTo@QTextEdit@@UAEXH@Z 10008de6 f   qt-mt323:qt-mt323.dll
 0001:00007dec       ?addColumn@QListView@@UAEHABVQIconSet@@ABVQString@@H@Z 10008dec f   qt-mt323:qt-mt323.dll
 0001:00007df2       ?addColumn@QListView@@UAEHABVQString@@H@Z 10008df2 f   qt-mt323:qt-mt323.dll
 0001:00007df8       ?className@QListView@@UBEPBDXZ 10008df8 f   qt-mt323:qt-mt323.dll
 0001:00007dfe       ?clear@QListView@@UAEXXZ   10008dfe f   qt-mt323:qt-mt323.dll
 0001:00007e04       ?clearSelection@QListView@@UAEXXZ 10008e04 f   qt-mt323:qt-mt323.dll
 0001:00007e0a       ?contentsContextMenuEvent@QListView@@MAEXPAVQContextMenuEvent@@@Z 10008e0a f   qt-mt323:qt-mt323.dll
 0001:00007e10       ?contentsDragEnterEvent@QListView@@MAEXPAVQDragEnterEvent@@@Z 10008e10 f   qt-mt323:qt-mt323.dll
 0001:00007e16       ?contentsDragLeaveEvent@QListView@@MAEXPAVQDragLeaveEvent@@@Z 10008e16 f   qt-mt323:qt-mt323.dll
 0001:00007e1c       ?contentsDragMoveEvent@QListView@@MAEXPAVQDragMoveEvent@@@Z 10008e1c f   qt-mt323:qt-mt323.dll
 0001:00007e22       ?contentsDropEvent@QListView@@MAEXPAVQDropEvent@@@Z 10008e22 f   qt-mt323:qt-mt323.dll
 0001:00007e28       ?contentsMouseDoubleClickEvent@QListView@@MAEXPAVQMouseEvent@@@Z 10008e28 f   qt-mt323:qt-mt323.dll
 0001:00007e2e       ?contentsMouseMoveEvent@QListView@@MAEXPAVQMouseEvent@@@Z 10008e2e f   qt-mt323:qt-mt323.dll
 0001:00007e34       ?contentsMousePressEvent@QListView@@MAEXPAVQMouseEvent@@@Z 10008e34 f   qt-mt323:qt-mt323.dll
 0001:00007e3a       ?contentsMouseReleaseEvent@QListView@@MAEXPAVQMouseEvent@@@Z 10008e3a f   qt-mt323:qt-mt323.dll
 0001:00007e40       ?dragObject@QListView@@MAEPAVQDragObject@@XZ 10008e40 f   qt-mt323:qt-mt323.dll
 0001:00007e46       ?drawContents@QScrollView@@EAEXPAVQPainter@@@Z 10008e46 f   qt-mt323:qt-mt323.dll
 0001:00007e4c       ?drawContents@QScrollView@@MAEXPAVQPainter@@HHHH@Z 10008e4c f   qt-mt323:qt-mt323.dll
 0001:00007e52       ?drawContentsOffset@QListView@@MAEXPAVQPainter@@HHHHHH@Z 10008e52 f   qt-mt323:qt-mt323.dll
 0001:00007e58       ?eventFilter@QListView@@UAE_NPAVQObject@@PAVQEvent@@@Z 10008e58 f   qt-mt323:qt-mt323.dll
 0001:00007e5e       ?focusInEvent@QListView@@MAEXPAVQFocusEvent@@@Z 10008e5e f   qt-mt323:qt-mt323.dll
 0001:00007e64       ?focusOutEvent@QListView@@MAEXPAVQFocusEvent@@@Z 10008e64 f   qt-mt323:qt-mt323.dll
 0001:00007e6a       ?insertItem@QListView@@UAEXPAVQListViewItem@@@Z 10008e6a f   qt-mt323:qt-mt323.dll
 0001:00007e70       ?invertSelection@QListView@@UAEXXZ 10008e70 f   qt-mt323:qt-mt323.dll
 0001:00007e76       ?keyPressEvent@QListView@@MAEXPAVQKeyEvent@@@Z 10008e76 f   qt-mt323:qt-mt323.dll
 0001:00007e7c       ?metaObject@QListView@@UBEPAVQMetaObject@@XZ 10008e7c f   qt-mt323:qt-mt323.dll
 0001:00007e82       ?minimumSizeHint@QListView@@UBE?AVQSize@@XZ 10008e82 f   qt-mt323:qt-mt323.dll
 0001:00007e88       ?paintEmptyArea@QListView@@MAEXPAVQPainter@@ABVQRect@@@Z 10008e88 f   qt-mt323:qt-mt323.dll
 0001:00007e8e       ?qt_cast@QListView@@UAEPAXPBD@Z 10008e8e f   qt-mt323:qt-mt323.dll
 0001:00007e94       ?qt_emit@QListView@@UAE_NHPAUQUObject@@@Z 10008e94 f   qt-mt323:qt-mt323.dll
 0001:00007e9a       ?qt_invoke@QListView@@UAE_NHPAUQUObject@@@Z 10008e9a f   qt-mt323:qt-mt323.dll
 0001:00007ea0       ?qt_property@QListView@@UAE_NHHPAVQVariant@@@Z 10008ea0 f   qt-mt323:qt-mt323.dll
 0001:00007ea6       ?removeColumn@QListView@@UAEXH@Z 10008ea6 f   qt-mt323:qt-mt323.dll
 0001:00007eac       ?removeItem@QListView@@UAEXPAVQListViewItem@@@Z 10008eac f   qt-mt323:qt-mt323.dll
 0001:00007eb2       ?resizeEvent@QListView@@MAEXPAVQResizeEvent@@@Z 10008eb2 f   qt-mt323:qt-mt323.dll
 0001:00007eb8       ?selectAll@QListView@@UAEX_N@Z 10008eb8 f   qt-mt323:qt-mt323.dll
 0001:00007ebe       ?setAllColumnsShowFocus@QListView@@UAEX_N@Z 10008ebe f   qt-mt323:qt-mt323.dll
 0001:00007ec4       ?setColumnAlignment@QListView@@UAEXHH@Z 10008ec4 f   qt-mt323:qt-mt323.dll
 0001:00007eca       ?setColumnText@QListView@@UAEXHABVQIconSet@@ABVQString@@@Z 10008eca f   qt-mt323:qt-mt323.dll
 0001:00007ed0       ?setColumnText@QListView@@UAEXHABVQString@@@Z 10008ed0 f   qt-mt323:qt-mt323.dll
 0001:00007ed6       ?setColumnWidth@QListView@@UAEXHH@Z 10008ed6 f   qt-mt323:qt-mt323.dll
 0001:00007edc       ?setColumnWidthMode@QListView@@UAEXHW4WidthMode@1@@Z 10008edc f   qt-mt323:qt-mt323.dll
 0001:00007ee2       ?setContentsPos@QListView@@UAEXHH@Z 10008ee2 f   qt-mt323:qt-mt323.dll
 0001:00007ee8       ?setCurrentItem@QListView@@UAEXPAVQListViewItem@@@Z 10008ee8 f   qt-mt323:qt-mt323.dll
 0001:00007eee       ?setDefaultRenameAction@QListView@@UAEXW4RenameAction@1@@Z 10008eee f   qt-mt323:qt-mt323.dll
 0001:00007ef4       ?setEnabled@QScrollView@@UAEX_N@Z 10008ef4 f   qt-mt323:qt-mt323.dll
 0001:00007efa       ?setFont@QListView@@UAEXABVQFont@@@Z 10008efa f   qt-mt323:qt-mt323.dll
 0001:00007f00       ?setItemMargin@QListView@@UAEXH@Z 10008f00 f   qt-mt323:qt-mt323.dll
 0001:00007f06       ?setMultiSelection@QListView@@UAEX_N@Z 10008f06 f   qt-mt323:qt-mt323.dll
 0001:00007f0c       ?setOpen@QListView@@UAEXPAVQListViewItem@@_N@Z 10008f0c f   qt-mt323:qt-mt323.dll
 0001:00007f12       ?setPalette@QListView@@UAEXABVQPalette@@@Z 10008f12 f   qt-mt323:qt-mt323.dll
 0001:00007f18       ?setResizeMode@QListView@@UAEXW4ResizeMode@1@@Z 10008f18 f   qt-mt323:qt-mt323.dll
 0001:00007f1e       ?setRootIsDecorated@QListView@@UAEX_N@Z 10008f1e f   qt-mt323:qt-mt323.dll
 0001:00007f24       ?setSelected@QListView@@UAEXPAVQListViewItem@@_N@Z 10008f24 f   qt-mt323:qt-mt323.dll
 0001:00007f2a       ?setShowSortIndicator@QListView@@UAEX_N@Z 10008f2a f   qt-mt323:qt-mt323.dll
 0001:00007f30       ?setShowToolTips@QListView@@UAEX_N@Z 10008f30 f   qt-mt323:qt-mt323.dll
 0001:00007f36       ?setSorting@QListView@@UAEXH_N@Z 10008f36 f   qt-mt323:qt-mt323.dll
 0001:00007f3c       ?setTreeStepSize@QListView@@UAEXH@Z 10008f3c f   qt-mt323:qt-mt323.dll
 0001:00007f42       ?show@QListView@@UAEXXZ    10008f42 f   qt-mt323:qt-mt323.dll
 0001:00007f48       ?showEvent@QListView@@MAEXPAVQShowEvent@@@Z 10008f48 f   qt-mt323:qt-mt323.dll
 0001:00007f4e       ?sizeHint@QListView@@UBE?AVQSize@@XZ 10008f4e f   qt-mt323:qt-mt323.dll
 0001:00007f54       ?sort@QListView@@UAEXXZ    10008f54 f   qt-mt323:qt-mt323.dll
 0001:00007f5a       ?startDrag@QListView@@MAEXXZ 10008f5a f   qt-mt323:qt-mt323.dll
 0001:00007f60       ?styleChange@QListView@@MAEXAAVQStyle@@@Z 10008f60 f   qt-mt323:qt-mt323.dll
 0001:00007f66       ?takeItem@QListView@@UAEXPAVQListViewItem@@@Z 10008f66 f   qt-mt323:qt-mt323.dll
 0001:00007f6c       ?viewportResizeEvent@QListView@@MAEXPAVQResizeEvent@@@Z 10008f6c f   qt-mt323:qt-mt323.dll
 0001:00007f72       ?windowActivationChange@QListView@@MAEX_N@Z 10008f72 f   qt-mt323:qt-mt323.dll
 0001:00007f78       ??2@YAPAXI@Z               10008f78 f   MSVCRT:MSVCR120.dll
 0001:00007f7e       ??3@YAXPAX@Z               10008f7e f   MSVCRT:MSVCR120.dll
 0001:00007f84       @__security_check_cookie@4 10008f84 f   MSVCRT:secchk.obj
 0001:00007f93       __EH_epilog3               10008f93 f   MSVCRT:ehprolg3.obj
 0001:00007fa7       __EH_epilog3_GS            10008fa7 f   MSVCRT:ehprolg3.obj
 0001:00007fb6       __EH_prolog3               10008fb6 f   MSVCRT:ehprolg3.obj
 0001:00007fe9       __EH_prolog3_GS            10008fe9 f   MSVCRT:ehprolg3.obj
 0001:00008020       ___CxxFrameHandler3        10009020 f   MSVCRT:MSVCR120.dll
 0001:00008026       ??_Etype_info@@UAEPAXI@Z   10009026 f i MSVCRT:ti_inst.obj
 0001:00008070       __purecall                 10009070 f   MSVCRT:MSVCR120.dll
 0001:00008076       ??_L@YGXPAXIHP6EX0@Z1@Z    10009076 f   MSVCRT:ehvecctr.obj
 0001:000080d8       ??_M@YGXPAXIHP6EX0@Z@Z     100090d8 f   MSVCRT:ehvecdtr.obj
 0001:00008147       ?__ArrayUnwind@@YGXPAXIHP6EX0@Z@Z 10009147 f   MSVCRT:ehvecdtr.obj
 0001:000081a5       ___atonexitinit            100091a5 f   MSVCRT:atonexit.obj
 0001:000081e1       __onexit                   100091e1 f   MSVCRT:atonexit.obj
 0001:0000828a       _atexit                    1000928a f   MSVCRT:atonexit.obj
 0001:000082eb       __CRT_INIT@12              100092eb f   MSVCRT:crtdll.obj
 0001:000084e2       __DllMainCRTStartup@12     100094e2 f   MSVCRT:crtdll.obj
 0001:00008638       ___raise_securityfailure   10009638 f   MSVCRT:gs_report.obj
 0001:00008675       ___report_gsfailure        10009675 f   MSVCRT:gs_report.obj
 0001:00008770       ??1type_info@@UAE@XZ       10009770 f   MSVCRT:MSVCR120.dll
 0001:00008780       __SEH_prolog4              10009780 f   MSVCRT:sehprolg4.obj
 0001:000087c5       __SEH_epilog4              100097c5 f   MSVCRT:sehprolg4.obj
 0001:000087d9       __except_handler4          100097d9 f   MSVCRT:chandler4gs.obj
 0001:000087fc       ?terminate@@YAXXZ          100097fc f   MSVCRT:MSVCR120.dll
 0001:00008802       __lock                     10009802 f   MSVCRT:MSVCR120.dll
 0001:00008808       __unlock                   10009808 f   MSVCRT:MSVCR120.dll
 0001:0000880e       ___dllonexit               1000980e f   MSVCRT:MSVCR120.dll
 0001:00008814       ___CppXcptFilter           10009814 f   MSVCRT:MSVCR120.dll
 0001:0000881a       __amsg_exit                1000981a f   MSVCRT:MSVCR120.dll
 0001:00008820       __FindPESection            10009820 f   MSVCRT:pesect.obj
 0001:00008870       __IsNonwritableInCurrentImage 10009870 f   MSVCRT:pesect.obj
 0001:00008930       __ValidateImageBase        10009930 f   MSVCRT:pesect.obj
 0001:00008961       ___security_init_cookie    10009961 f   MSVCRT:gs_support.obj
 0001:000089fd       _DllMain@12                100099fd f   MSVCRT:dllmain.obj
 0001:00008a1f       __RTC_Initialize           10009a1f f   MSVCRT:initsect.obj
 0001:00008a3f       __RTC_Terminate            10009a3f f   MSVCRT:initsect.obj
 0001:00008a60       __initterm                 10009a60 f   MSVCRT:MSVCR120.dll
 0001:00008a66       __initterm_e               10009a66 f   MSVCRT:MSVCR120.dll
 0001:00008a6c       ___clean_type_info_names   10009a6c f   MSVCRT:tncleanup.obj
 0001:00008a78       __crt_debugger_hook        10009a78 f   MSVCRT:MSVCR120.dll
 0001:00008a7e       ___crtUnhandledException   10009a7e f   MSVCRT:MSVCR120.dll
 0001:00008a84       ___crtTerminateProcess     10009a84 f   MSVCRT:MSVCR120.dll
 0001:00008a8a       __except_handler4_common   10009a8a f   MSVCRT:MSVCR120.dll
 0001:00008a90       ___clean_type_info_names_internal 10009a90 f   MSVCRT:MSVCR120.dll
 0001:00008a96       _IsProcessorFeaturePresent@4 10009a96 f   kernel32:KERNEL32.dll
 0002:00000000       __imp__DisableThreadLibraryCalls@4 1000b000     kernel32:KERNEL32.dll
 0002:00000004       __imp__GetSystemTimeAsFileTime@4 1000b004     kernel32:KERNEL32.dll
 0002:00000008       __imp__GetCurrentThreadId@0 1000b008     kernel32:KERNEL32.dll
 0002:0000000c       __imp__GetCurrentProcessId@0 1000b00c     kernel32:KERNEL32.dll
 0002:00000010       __imp__QueryPerformanceCounter@4 1000b010     kernel32:KERNEL32.dll
 0002:00000014       __imp__IsProcessorFeaturePresent@4 1000b014     kernel32:KERNEL32.dll
 0002:00000018       __imp__IsDebuggerPresent@0 1000b018     kernel32:KERNEL32.dll
 0002:0000001c       __imp__DecodePointer@4     1000b01c     kernel32:KERNEL32.dll
 0002:00000020       __imp__EncodePointer@4     1000b020     kernel32:KERNEL32.dll
 0002:00000024       __imp__GetPrivateProfileStringA@24 1000b024     kernel32:KERNEL32.dll
 0002:00000028       \177KERNEL32_NULL_THUNK_DATA 1000b028     kernel32:KERNEL32.dll
 0002:0000002c       __imp___except_handler4_common 1000b02c     MSVCRT:MSVCR120.dll
 0002:00000030       __imp____crtTerminateProcess 1000b030     MSVCRT:MSVCR120.dll
 0002:00000034       __imp____crtUnhandledException 1000b034     MSVCRT:MSVCR120.dll
 0002:00000038       __imp___crt_debugger_hook  1000b038     MSVCRT:MSVCR120.dll
 0002:0000003c       __imp___initterm_e         1000b03c     MSVCRT:MSVCR120.dll
 0002:00000040       __imp___initterm           1000b040     MSVCRT:MSVCR120.dll
 0002:00000044       __imp____clean_type_info_names_internal 1000b044     MSVCRT:MSVCR120.dll
 0002:00000048       __imp__free                1000b048     MSVCRT:MSVCR120.dll
 0002:0000004c       __imp___amsg_exit          1000b04c     MSVCRT:MSVCR120.dll
 0002:00000050       __imp____CppXcptFilter     1000b050     MSVCRT:MSVCR120.dll
 0002:00000054       __imp___onexit             1000b054     MSVCRT:MSVCR120.dll
 0002:00000058       __imp____dllonexit         1000b058     MSVCRT:MSVCR120.dll
 0002:0000005c       __imp___calloc_crt         1000b05c     MSVCRT:MSVCR120.dll
 0002:00000060       __imp___unlock             1000b060     MSVCRT:MSVCR120.dll
 0002:00000064       __imp___lock               1000b064     MSVCRT:MSVCR120.dll
 0002:00000068       __imp_?terminate@@YAXXZ    1000b068     MSVCRT:MSVCR120.dll
 0002:0000006c       __imp_??1type_info@@UAE@XZ 1000b06c     MSVCRT:MSVCR120.dll
 0002:00000070       __imp___purecall           1000b070     MSVCRT:MSVCR120.dll
 0002:00000074       __imp__strchr              1000b074     MSVCRT:MSVCR120.dll
 0002:00000078       __imp____CxxFrameHandler3  1000b078     MSVCRT:MSVCR120.dll
 0002:0000007c       __imp__atoi                1000b07c     MSVCRT:MSVCR120.dll
 0002:00000080       __imp_??3@YAXPAX@Z         1000b080     MSVCRT:MSVCR120.dll
 0002:00000084       __imp_??2@YAPAXI@Z         1000b084     MSVCRT:MSVCR120.dll
 0002:00000088       __imp___malloc_crt         1000b088     MSVCRT:MSVCR120.dll
 0002:0000008c       \177MSVCR120_NULL_THUNK_DATA 1000b08c     MSVCRT:MSVCR120.dll
 0002:00000090       __imp_?fnConfig_icons@@YAPAPBDPBD@Z 1000b090     config_icons:config_icons.dll
 0002:00000094       \177config_icons_NULL_THUNK_DATA 1000b094     config_icons:config_icons.dll
 0002:00000098       __imp_??0QListViewItem@@QAE@PAVQListView@@VQString@@1111111@Z 1000b098     qt-mt323:qt-mt323.dll
 0002:0000009c       __imp_??1QListViewItem@@UAE@XZ 1000b09c     qt-mt323:qt-mt323.dll
 0002:000000a0       __imp_?findItem@QListView@@QBEPAVQListViewItem@@ABVQString@@HI@Z 1000b0a0     qt-mt323:qt-mt323.dll
 0002:000000a4       __imp_??0QAction@@QAE@ABVQString@@ABVQIconSet@@0VQKeySequence@@PAVQObject@@PBD_N@Z 1000b0a4     qt-mt323:qt-mt323.dll
 0002:000000a8       __imp_??1QAction@@UAE@XZ   1000b0a8     qt-mt323:qt-mt323.dll
 0002:000000ac       __imp_??0QDockWindow@@QAE@PAVQWidget@@PBDI@Z 1000b0ac     qt-mt323:qt-mt323.dll
 0002:000000b0       __imp_??1QDockWindow@@UAE@XZ 1000b0b0     qt-mt323:qt-mt323.dll
 0002:000000b4       __imp_??1?$QPtrList@VQDockWindow@@@@UAE@XZ 1000b0b4     qt-mt323:qt-mt323.dll
 0002:000000b8       __imp_??0QToolBar@@QAE@PAVQMainWindow@@PBD@Z 1000b0b8     qt-mt323:qt-mt323.dll
 0002:000000bc       __imp_??1QToolBar@@UAE@XZ  1000b0bc     qt-mt323:qt-mt323.dll
 0002:000000c0       __imp_??9QDateTime@@QBE_NABV0@@Z 1000b0c0     qt-mt323:qt-mt323.dll
 0002:000000c4       __imp_??0QFileInfo@@QAE@ABVQString@@@Z 1000b0c4     qt-mt323:qt-mt323.dll
 0002:000000c8       __imp_??1QFileInfo@@QAE@XZ 1000b0c8     qt-mt323:qt-mt323.dll
 0002:000000cc       __imp_?lastModified@QFileInfo@@QBE?AVQDateTime@@XZ 1000b0cc     qt-mt323:qt-mt323.dll
 0002:000000d0       __imp_??0QGuardedPtrPrivate@@QAE@PAVQObject@@@Z 1000b0d0     qt-mt323:qt-mt323.dll
 0002:000000d4       __imp_??1QGuardedPtrPrivate@@UAE@XZ 1000b0d4     qt-mt323:qt-mt323.dll
 0002:000000d8       __imp_?reconnect@QGuardedPtrPrivate@@QAEXPAVQObject@@@Z 1000b0d8     qt-mt323:qt-mt323.dll
 0002:000000dc       __imp_??0QPopupMenu@@QAE@PAVQWidget@@PBD@Z 1000b0dc     qt-mt323:qt-mt323.dll
 0002:000000e0       __imp_??1QPopupMenu@@UAE@XZ 1000b0e0     qt-mt323:qt-mt323.dll
 0002:000000e4       __imp_?look_string@QGDict@@QAEPAXABVQString@@PAXH@Z 1000b0e4     qt-mt323:qt-mt323.dll
 0002:000000e8       __imp_??0QGDict@@IAE@IW4KeyType@0@_N1@Z 1000b0e8     qt-mt323:qt-mt323.dll
 0002:000000ec       __imp_??1QGDict@@MAE@XZ    1000b0ec     qt-mt323:qt-mt323.dll
 0002:000000f0       __imp_?clear@QGDict@@MAEXXZ 1000b0f0     qt-mt323:qt-mt323.dll
 0002:000000f4       __imp_?acceptDrop@QListViewItem@@UBE_NPBVQMimeSource@@@Z 1000b0f4     qt-mt323:qt-mt323.dll
 0002:000000f8       __imp_?activate@QListViewItem@@MAEXXZ 1000b0f8     qt-mt323:qt-mt323.dll
 0002:000000fc       __imp_?activateItemAt@QPopupMenu@@UAEXH@Z 1000b0fc     qt-mt323:qt-mt323.dll
 0002:00000100       __imp_?addTo@QAction@@UAE_NPAVQWidget@@@Z 1000b100     qt-mt323:qt-mt323.dll
 0002:00000104       __imp_?addedTo@QAction@@MAEXHPAVQPopupMenu@@@Z 1000b104     qt-mt323:qt-mt323.dll
 0002:00000108       __imp_?addedTo@QAction@@MAEXPAVQWidget@@0@Z 1000b108     qt-mt323:qt-mt323.dll
 0002:0000010c       __imp_?adjustSize@QWidget@@UAEXXZ 1000b10c     qt-mt323:qt-mt323.dll
 0002:00000110       __imp_?cancelRename@QListViewItem@@MAEXH@Z 1000b110     qt-mt323:qt-mt323.dll
 0002:00000114       __imp_?checkConnectArgs@QObject@@MAE_NPBDPBV1@0@Z 1000b114     qt-mt323:qt-mt323.dll
 0002:00000118       __imp_?childEvent@QObject@@MAEXPAVQChildEvent@@@Z 1000b118     qt-mt323:qt-mt323.dll
 0002:0000011c       __imp_?className@QAction@@UBEPBDXZ 1000b11c     qt-mt323:qt-mt323.dll
 0002:00000120       __imp_?className@QDockWindow@@UBEPBDXZ 1000b120     qt-mt323:qt-mt323.dll
 0002:00000124       __imp_?className@QGuardedPtrPrivate@@UBEPBDXZ 1000b124     qt-mt323:qt-mt323.dll
 0002:00000128       __imp_?className@QPopupMenu@@UBEPBDXZ 1000b128     qt-mt323:qt-mt323.dll
 0002:0000012c       __imp_?className@QToolBar@@UBEPBDXZ 1000b12c     qt-mt323:qt-mt323.dll
 0002:00000130       __imp_?className@QWidget@@UBEPBDXZ 1000b130     qt-mt323:qt-mt323.dll
 0002:00000134       __imp_?clear@?$QPtrList@VQDockWindow@@@@UAEXXZ 1000b134     qt-mt323:qt-mt323.dll
 0002:00000138       __imp_?clear@QToolBar@@UAEXXZ 1000b138     qt-mt323:qt-mt323.dll
 0002:0000013c       __imp_?close@QWidget@@UAE_N_N@Z 1000b13c     qt-mt323:qt-mt323.dll
 0002:00000140       __imp_?closeEvent@QPopupMenu@@MAEXPAVQCloseEvent@@@Z 1000b140     qt-mt323:qt-mt323.dll
 0002:00000144       __imp_?cmd@QPaintDevice@@MAE_NHPAVQPainter@@PATQPDevCmdParam@@@Z 1000b144     qt-mt323:qt-mt323.dll
 0002:00000148       __imp_?compare@QListViewItem@@UBEHPAV1@H_N@Z 1000b148     qt-mt323:qt-mt323.dll
 0002:0000014c       __imp_?compareItems@QGList@@MAEHPAX0@Z 1000b14c     qt-mt323:qt-mt323.dll
 0002:00000150       __imp_?connectNotify@QObject@@MAEXPBD@Z 1000b150     qt-mt323:qt-mt323.dll
 0002:00000154       __imp_?contextMenuEvent@QDockWindow@@MAEXPAVQContextMenuEvent@@@Z 1000b154     qt-mt323:qt-mt323.dll
 0002:00000158       __imp_?contextMenuEvent@QWidget@@MAEXPAVQContextMenuEvent@@@Z 1000b158     qt-mt323:qt-mt323.dll
 0002:0000015c       __imp_?count@?$QPtrList@VQDockWindow@@@@UBEIXZ 1000b15c     qt-mt323:qt-mt323.dll
 0002:00000160       __imp_?create@QWidget@@MAEXPAUHWND__@@_N1@Z 1000b160     qt-mt323:qt-mt323.dll
 0002:00000164       __imp_?customEvent@QObject@@MAEXPAVQCustomEvent@@@Z 1000b164     qt-mt323:qt-mt323.dll
 0002:00000168       __imp_?customWhatsThis@QPopupMenu@@UBE_NXZ 1000b168     qt-mt323:qt-mt323.dll
 0002:0000016c       __imp_?customWhatsThis@QWidget@@UBE_NXZ 1000b16c     qt-mt323:qt-mt323.dll
 0002:00000170       __imp_?deleteItem@?$QPtrList@VQDockWindow@@@@EAEXPAX@Z 1000b170     qt-mt323:qt-mt323.dll
 0002:00000174       __imp_?destroy@QWidget@@MAEX_N0@Z 1000b174     qt-mt323:qt-mt323.dll
 0002:00000178       __imp_?disconnectNotify@QObject@@MAEXPBD@Z 1000b178     qt-mt323:qt-mt323.dll
 0002:0000017c       __imp_?dock@QDockWindow@@UAEXXZ 1000b17c     qt-mt323:qt-mt323.dll
 0002:00000180       __imp_?dragEnterEvent@QWidget@@MAEXPAVQDragEnterEvent@@@Z 1000b180     qt-mt323:qt-mt323.dll
 0002:00000184       __imp_?dragEntered@QListViewItem@@MAEXXZ 1000b184     qt-mt323:qt-mt323.dll
 0002:00000188       __imp_?dragLeaveEvent@QWidget@@MAEXPAVQDragLeaveEvent@@@Z 1000b188     qt-mt323:qt-mt323.dll
 0002:0000018c       __imp_?dragLeft@QListViewItem@@MAEXXZ 1000b18c     qt-mt323:qt-mt323.dll
 0002:00000190       __imp_?dragMoveEvent@QWidget@@MAEXPAVQDragMoveEvent@@@Z 1000b190     qt-mt323:qt-mt323.dll
 0002:00000194       __imp_?drawContents@QDockWindow@@MAEXPAVQPainter@@@Z 1000b194     qt-mt323:qt-mt323.dll
 0002:00000198       __imp_?drawContents@QPopupMenu@@MAEXPAVQPainter@@@Z 1000b198     qt-mt323:qt-mt323.dll
 0002:0000019c       __imp_?drawFrame@QDockWindow@@MAEXPAVQPainter@@@Z 1000b19c     qt-mt323:qt-mt323.dll
 0002:000001a0       __imp_?drawFrame@QFrame@@MAEXPAVQPainter@@@Z 1000b1a0     qt-mt323:qt-mt323.dll
 0002:000001a4       __imp_?dropEvent@QWidget@@MAEXPAVQDropEvent@@@Z 1000b1a4     qt-mt323:qt-mt323.dll
 0002:000001a8       __imp_?dropped@QListViewItem@@MAEXPAVQDropEvent@@@Z 1000b1a8     qt-mt323:qt-mt323.dll
 0002:000001ac       __imp_?enabledChange@QPopupMenu@@MAEX_N@Z 1000b1ac     qt-mt323:qt-mt323.dll
 0002:000001b0       __imp_?enabledChange@QWidget@@MAEX_N@Z 1000b1b0     qt-mt323:qt-mt323.dll
 0002:000001b4       __imp_?enforceSortOrder@QListViewItem@@MBEXXZ 1000b1b4     qt-mt323:qt-mt323.dll
 0002:000001b8       __imp_?enterEvent@QWidget@@MAEXPAVQEvent@@@Z 1000b1b8     qt-mt323:qt-mt323.dll
 0002:000001bc       __imp_?event@QDockWindow@@MAE_NPAVQEvent@@@Z 1000b1bc     qt-mt323:qt-mt323.dll
 0002:000001c0       __imp_?event@QObject@@UAE_NPAVQEvent@@@Z 1000b1c0     qt-mt323:qt-mt323.dll
 0002:000001c4       __imp_?event@QToolBar@@UAE_NPAVQEvent@@@Z 1000b1c4     qt-mt323:qt-mt323.dll
 0002:000001c8       __imp_?event@QWidget@@MAE_NPAVQEvent@@@Z 1000b1c8     qt-mt323:qt-mt323.dll
 0002:000001cc       __imp_?eventFilter@QDockWindow@@UAE_NPAVQObject@@PAVQEvent@@@Z 1000b1cc     qt-mt323:qt-mt323.dll
 0002:000001d0       __imp_?eventFilter@QObject@@UAE_NPAV1@PAVQEvent@@@Z 1000b1d0     qt-mt323:qt-mt323.dll
 0002:000001d4       __imp_?focusInEvent@QPopupMenu@@MAEXPAVQFocusEvent@@@Z 1000b1d4     qt-mt323:qt-mt323.dll
 0002:000001d8       __imp_?focusInEvent@QWidget@@MAEXPAVQFocusEvent@@@Z 1000b1d8     qt-mt323:qt-mt323.dll
 0002:000001dc       __imp_?focusNextPrevChild@QPopupMenu@@MAE_N_N@Z 1000b1dc     qt-mt323:qt-mt323.dll
 0002:000001e0       __imp_?focusNextPrevChild@QWidget@@MAE_N_N@Z 1000b1e0     qt-mt323:qt-mt323.dll
 0002:000001e4       __imp_?focusOutEvent@QPopupMenu@@MAEXPAVQFocusEvent@@@Z 1000b1e4     qt-mt323:qt-mt323.dll
 0002:000001e8       __imp_?focusOutEvent@QWidget@@MAEXPAVQFocusEvent@@@Z 1000b1e8     qt-mt323:qt-mt323.dll
 0002:000001ec       __imp_?fontChange@QWidget@@MAEXABVQFont@@@Z 1000b1ec     qt-mt323:qt-mt323.dll
 0002:000001f0       __imp_?fontInf@QPaintDevice@@MBEHPAVQFont@@H@Z 1000b1f0     qt-mt323:qt-mt323.dll
 0002:000001f4       __imp_?fontMet@QPaintDevice@@MBEHPAVQFont@@HPBDH@Z 1000b1f4     qt-mt323:qt-mt323.dll
 0002:000001f8       __imp_?frameChanged@QFrame@@MAEXXZ 1000b1f8     qt-mt323:qt-mt323.dll
 0002:000001fc       __imp_?frameChanged@QPopupMenu@@EAEXXZ 1000b1fc     qt-mt323:qt-mt323.dll
 0002:00000200       __imp_?handle@QPaintDevice@@UBEPAUHDC__@@XZ 1000b200     qt-mt323:qt-mt323.dll
 0002:00000204       __imp_?heightForWidth@QWidget@@UBEHH@Z 1000b204     qt-mt323:qt-mt323.dll
 0002:00000208       __imp_?hide@QPopupMenu@@UAEXXZ 1000b208     qt-mt323:qt-mt323.dll
 0002:0000020c       __imp_?hide@QToolBar@@UAEXXZ 1000b20c     qt-mt323:qt-mt323.dll
 0002:00000210       __imp_?hide@QWidget@@UAEXXZ 1000b210     qt-mt323:qt-mt323.dll
 0002:00000214       __imp_?hideEvent@QDockWindow@@MAEXPAVQHideEvent@@@Z 1000b214     qt-mt323:qt-mt323.dll
 0002:00000218       __imp_?hideEvent@QWidget@@MAEXPAVQHideEvent@@@Z 1000b218     qt-mt323:qt-mt323.dll
 0002:0000021c       __imp_?imComposeEvent@QWidget@@MAEXPAVQIMEvent@@@Z 1000b21c     qt-mt323:qt-mt323.dll
 0002:00000220       __imp_?imEndEvent@QWidget@@MAEXPAVQIMEvent@@@Z 1000b220     qt-mt323:qt-mt323.dll
 0002:00000224       __imp_?imStartEvent@QWidget@@MAEXPAVQIMEvent@@@Z 1000b224     qt-mt323:qt-mt323.dll
 0002:00000228       __imp_?insertChild@QObject@@UAEXPAV1@@Z 1000b228     qt-mt323:qt-mt323.dll
 0002:0000022c       __imp_?insertItem@QListViewItem@@UAEXPAV1@@Z 1000b22c     qt-mt323:qt-mt323.dll
 0002:00000230       __imp_?invalidateHeight@QListViewItem@@UAEXXZ 1000b230     qt-mt323:qt-mt323.dll
 0002:00000234       __imp_?key@QListViewItem@@UBE?AVQString@@H_N@Z 1000b234     qt-mt323:qt-mt323.dll
 0002:00000238       __imp_?keyPressEvent@QPopupMenu@@MAEXPAVQKeyEvent@@@Z 1000b238     qt-mt323:qt-mt323.dll
 0002:0000023c       __imp_?keyPressEvent@QWidget@@MAEXPAVQKeyEvent@@@Z 1000b23c     qt-mt323:qt-mt323.dll
 0002:00000240       __imp_?keyReleaseEvent@QWidget@@MAEXPAVQKeyEvent@@@Z 1000b240     qt-mt323:qt-mt323.dll
 0002:00000244       __imp_?leaveEvent@QPopupMenu@@MAEXPAVQEvent@@@Z 1000b244     qt-mt323:qt-mt323.dll
 0002:00000248       __imp_?leaveEvent@QWidget@@MAEXPAVQEvent@@@Z 1000b248     qt-mt323:qt-mt323.dll
 0002:0000024c       __imp_?menuContentsChanged@QPopupMenu@@EAEXXZ 1000b24c     qt-mt323:qt-mt323.dll
 0002:00000250       __imp_?menuDelPopup@QPopupMenu@@EAEXPAV1@@Z 1000b250     qt-mt323:qt-mt323.dll
 0002:00000254       __imp_?menuInsPopup@QPopupMenu@@EAEXPAV1@@Z 1000b254     qt-mt323:qt-mt323.dll
 0002:00000258       __imp_?menuStateChanged@QPopupMenu@@EAEXXZ 1000b258     qt-mt323:qt-mt323.dll
 0002:0000025c       __imp_?metaObject@QAction@@UBEPAVQMetaObject@@XZ 1000b25c     qt-mt323:qt-mt323.dll
 0002:00000260       __imp_?metaObject@QDockWindow@@UBEPAVQMetaObject@@XZ 1000b260     qt-mt323:qt-mt323.dll
 0002:00000264       __imp_?metaObject@QGuardedPtrPrivate@@UBEPAVQMetaObject@@XZ 1000b264     qt-mt323:qt-mt323.dll
 0002:00000268       __imp_?metaObject@QPopupMenu@@UBEPAVQMetaObject@@XZ 1000b268     qt-mt323:qt-mt323.dll
 0002:0000026c       __imp_?metaObject@QToolBar@@UBEPAVQMetaObject@@XZ 1000b26c     qt-mt323:qt-mt323.dll
 0002:00000270       __imp_?metaObject@QWidget@@UBEPAVQMetaObject@@XZ 1000b270     qt-mt323:qt-mt323.dll
 0002:00000274       __imp_?metric@QWidget@@MBEHH@Z 1000b274     qt-mt323:qt-mt323.dll
 0002:00000278       __imp_?minimumSizeHint@QDockWindow@@UBE?AVQSize@@XZ 1000b278     qt-mt323:qt-mt323.dll
 0002:0000027c       __imp_?minimumSizeHint@QToolBar@@UBE?AVQSize@@XZ 1000b27c     qt-mt323:qt-mt323.dll
 0002:00000280       __imp_?minimumSizeHint@QWidget@@UBE?AVQSize@@XZ 1000b280     qt-mt323:qt-mt323.dll
 0002:00000284       __imp_?mouseDoubleClickEvent@QWidget@@MAEXPAVQMouseEvent@@@Z 1000b284     qt-mt323:qt-mt323.dll
 0002:00000288       __imp_?mouseMoveEvent@QPopupMenu@@MAEXPAVQMouseEvent@@@Z 1000b288     qt-mt323:qt-mt323.dll
 0002:0000028c       __imp_?mouseMoveEvent@QWidget@@MAEXPAVQMouseEvent@@@Z 1000b28c     qt-mt323:qt-mt323.dll
 0002:00000290       __imp_?mousePressEvent@QPopupMenu@@MAEXPAVQMouseEvent@@@Z 1000b290     qt-mt323:qt-mt323.dll
 0002:00000294       __imp_?mousePressEvent@QWidget@@MAEXPAVQMouseEvent@@@Z 1000b294     qt-mt323:qt-mt323.dll
 0002:00000298       __imp_?mouseReleaseEvent@QPopupMenu@@MAEXPAVQMouseEvent@@@Z 1000b298     qt-mt323:qt-mt323.dll
 0002:0000029c       __imp_?mouseReleaseEvent@QWidget@@MAEXPAVQMouseEvent@@@Z 1000b29c     qt-mt323:qt-mt323.dll
 0002:000002a0       __imp_?move@QWidget@@UAEXHH@Z 1000b2a0     qt-mt323:qt-mt323.dll
 0002:000002a4       __imp_?moveEvent@QWidget@@MAEXPAVQMoveEvent@@@Z 1000b2a4     qt-mt323:qt-mt323.dll
 0002:000002a8       __imp_?newItem@QPtrCollection@@MAEPAXPAX@Z 1000b2a8     qt-mt323:qt-mt323.dll
 0002:000002ac       __imp_?okRename@QListViewItem@@MAEXH@Z 1000b2ac     qt-mt323:qt-mt323.dll
 0002:000002b0       __imp_?paintBranches@QListViewItem@@UAEXPAVQPainter@@ABVQColorGroup@@HHH@Z 1000b2b0     qt-mt323:qt-mt323.dll
 0002:000002b4       __imp_?paintCell@QListViewItem@@UAEXPAVQPainter@@ABVQColorGroup@@HHH@Z 1000b2b4     qt-mt323:qt-mt323.dll
 0002:000002b8       __imp_?paintEvent@QFrame@@MAEXPAVQPaintEvent@@@Z 1000b2b8     qt-mt323:qt-mt323.dll
 0002:000002bc       __imp_?paintEvent@QPopupMenu@@MAEXPAVQPaintEvent@@@Z 1000b2bc     qt-mt323:qt-mt323.dll
 0002:000002c0       __imp_?paintEvent@QWidget@@MAEXPAVQPaintEvent@@@Z 1000b2c0     qt-mt323:qt-mt323.dll
 0002:000002c4       __imp_?paintFocus@QListViewItem@@UAEXPAVQPainter@@ABVQColorGroup@@ABVQRect@@@Z 1000b2c4     qt-mt323:qt-mt323.dll
 0002:000002c8       __imp_?paletteChange@QWidget@@MAEXABVQPalette@@@Z 1000b2c8     qt-mt323:qt-mt323.dll
 0002:000002cc       __imp_?pixmap@QListViewItem@@UBEPBVQPixmap@@H@Z 1000b2cc     qt-mt323:qt-mt323.dll
 0002:000002d0       __imp_?polish@QWidget@@UAEXXZ 1000b2d0     qt-mt323:qt-mt323.dll
 0002:000002d4       __imp_?property@QObject@@UBE?AVQVariant@@PBD@Z 1000b2d4     qt-mt323:qt-mt323.dll
 0002:000002d8       __imp_?qt_cast@QAction@@UAEPAXPBD@Z 1000b2d8     qt-mt323:qt-mt323.dll
 0002:000002dc       __imp_?qt_cast@QDockWindow@@UAEPAXPBD@Z 1000b2dc     qt-mt323:qt-mt323.dll
 0002:000002e0       __imp_?qt_cast@QGuardedPtrPrivate@@UAEPAXPBD@Z 1000b2e0     qt-mt323:qt-mt323.dll
 0002:000002e4       __imp_?qt_cast@QPopupMenu@@UAEPAXPBD@Z 1000b2e4     qt-mt323:qt-mt323.dll
 0002:000002e8       __imp_?qt_cast@QToolBar@@UAEPAXPBD@Z 1000b2e8     qt-mt323:qt-mt323.dll
 0002:000002ec       __imp_?qt_cast@QWidget@@UAEPAXPBD@Z 1000b2ec     qt-mt323:qt-mt323.dll
 0002:000002f0       __imp_?qt_emit@QAction@@UAE_NHPAUQUObject@@@Z 1000b2f0     qt-mt323:qt-mt323.dll
 0002:000002f4       __imp_?qt_emit@QDockWindow@@UAE_NHPAUQUObject@@@Z 1000b2f4     qt-mt323:qt-mt323.dll
 0002:000002f8       __imp_?qt_emit@QGuardedPtrPrivate@@UAE_NHPAUQUObject@@@Z 1000b2f8     qt-mt323:qt-mt323.dll
 0002:000002fc       __imp_?qt_emit@QPopupMenu@@UAE_NHPAUQUObject@@@Z 1000b2fc     qt-mt323:qt-mt323.dll
 0002:00000300       __imp_?qt_emit@QToolBar@@UAE_NHPAUQUObject@@@Z 1000b300     qt-mt323:qt-mt323.dll
 0002:00000304       __imp_?qt_emit@QWidget@@UAE_NHPAUQUObject@@@Z 1000b304     qt-mt323:qt-mt323.dll
 0002:00000308       __imp_?qt_invoke@QAction@@UAE_NHPAUQUObject@@@Z 1000b308     qt-mt323:qt-mt323.dll
 0002:0000030c       __imp_?qt_invoke@QDockWindow@@UAE_NHPAUQUObject@@@Z 1000b30c     qt-mt323:qt-mt323.dll
 0002:00000310       __imp_?qt_invoke@QGuardedPtrPrivate@@UAE_NHPAUQUObject@@@Z 1000b310     qt-mt323:qt-mt323.dll
 0002:00000314       __imp_?qt_invoke@QPopupMenu@@UAE_NHPAUQUObject@@@Z 1000b314     qt-mt323:qt-mt323.dll
 0002:00000318       __imp_?qt_invoke@QToolBar@@UAE_NHPAUQUObject@@@Z 1000b318     qt-mt323:qt-mt323.dll
 0002:0000031c       __imp_?qt_invoke@QWidget@@UAE_NHPAUQUObject@@@Z 1000b31c     qt-mt323:qt-mt323.dll
 0002:00000320       __imp_?qt_property@QAction@@UAE_NHHPAVQVariant@@@Z 1000b320     qt-mt323:qt-mt323.dll
 0002:00000324       __imp_?qt_property@QDockWindow@@UAE_NHHPAVQVariant@@@Z 1000b324     qt-mt323:qt-mt323.dll
 0002:00000328       __imp_?qt_property@QGuardedPtrPrivate@@UAE_NHHPAVQVariant@@@Z 1000b328     qt-mt323:qt-mt323.dll
 0002:0000032c       __imp_?qt_property@QPopupMenu@@UAE_NHHPAVQVariant@@@Z 1000b32c     qt-mt323:qt-mt323.dll
 0002:00000330       __imp_?qt_property@QToolBar@@UAE_NHHPAVQVariant@@@Z 1000b330     qt-mt323:qt-mt323.dll
 0002:00000334       __imp_?qt_property@QWidget@@UAE_NHHPAVQVariant@@@Z 1000b334     qt-mt323:qt-mt323.dll
 0002:00000338       __imp_?read@QGDict@@MAEAAVQDataStream@@AAV2@AAPAX@Z 1000b338     qt-mt323:qt-mt323.dll
 0002:0000033c       __imp_?read@QGList@@MAEAAVQDataStream@@AAV2@AAPAX@Z 1000b33c     qt-mt323:qt-mt323.dll
 0002:00000340       __imp_?removeChild@QObject@@UAEXPAV1@@Z 1000b340     qt-mt323:qt-mt323.dll
 0002:00000344       __imp_?removeFrom@QAction@@UAE_NPAVQWidget@@@Z 1000b344     qt-mt323:qt-mt323.dll
 0002:00000348       __imp_?removeItem@QListViewItem@@UAEXPAV1@@Z 1000b348     qt-mt323:qt-mt323.dll
 0002:0000034c       __imp_?reparent@QWidget@@UAEXPAV1@IABVQPoint@@_N@Z 1000b34c     qt-mt323:qt-mt323.dll
 0002:00000350       __imp_?resize@QWidget@@UAEXHH@Z 1000b350     qt-mt323:qt-mt323.dll
 0002:00000354       __imp_?resizeEvent@QDockWindow@@MAEXPAVQResizeEvent@@@Z 1000b354     qt-mt323:qt-mt323.dll
 0002:00000358       __imp_?resizeEvent@QFrame@@MAEXPAVQResizeEvent@@@Z 1000b358     qt-mt323:qt-mt323.dll
 0002:0000035c       __imp_?resizeEvent@QToolBar@@MAEXPAVQResizeEvent@@@Z 1000b35c     qt-mt323:qt-mt323.dll
 0002:00000360       __imp_?resizeEvent@QWidget@@MAEXPAVQResizeEvent@@@Z 1000b360     qt-mt323:qt-mt323.dll
 0002:00000364       __imp_?resolution@QPaintDevice@@UBEHXZ 1000b364     qt-mt323:qt-mt323.dll
 0002:00000368       __imp_?rtti@QListViewItem@@UBEHXZ 1000b368     qt-mt323:qt-mt323.dll
 0002:0000036c       __imp_?setAccel@QAction@@UAEXABVQKeySequence@@@Z 1000b36c     qt-mt323:qt-mt323.dll
 0002:00000370       __imp_?setAcceptDrops@QWidget@@UAEX_N@Z 1000b370     qt-mt323:qt-mt323.dll
 0002:00000374       __imp_?setActiveItem@QPopupMenu@@UAEXH@Z 1000b374     qt-mt323:qt-mt323.dll
 0002:00000378       __imp_?setActiveWindow@QWidget@@UAEXXZ 1000b378     qt-mt323:qt-mt323.dll
 0002:0000037c       __imp_?setAutoMask@QWidget@@UAEX_N@Z 1000b37c     qt-mt323:qt-mt323.dll
 0002:00000380       __imp_?setBackgroundColor@QWidget@@UAEXABVQColor@@@Z 1000b380     qt-mt323:qt-mt323.dll
 0002:00000384       __imp_?setBackgroundMode@QWidget@@UAEXW4BackgroundMode@Qt@@@Z 1000b384     qt-mt323:qt-mt323.dll
 0002:00000388       __imp_?setBackgroundOrigin@QWidget@@UAEXW4BackgroundOrigin@1@@Z 1000b388     qt-mt323:qt-mt323.dll
 0002:0000038c       __imp_?setBackgroundPixmap@QWidget@@UAEXABVQPixmap@@@Z 1000b38c     qt-mt323:qt-mt323.dll
 0002:00000390       __imp_?setCaption@QDockWindow@@UAEXABVQString@@@Z 1000b390     qt-mt323:qt-mt323.dll
 0002:00000394       __imp_?setCaption@QWidget@@UAEXABVQString@@@Z 1000b394     qt-mt323:qt-mt323.dll
 0002:00000398       __imp_?setCheckable@QPopupMenu@@UAEX_N@Z 1000b398     qt-mt323:qt-mt323.dll
 0002:0000039c       __imp_?setCloseMode@QDockWindow@@UAEXH@Z 1000b39c     qt-mt323:qt-mt323.dll
 0002:000003a0       __imp_?setCursor@QWidget@@UAEXABVQCursor@@@Z 1000b3a0     qt-mt323:qt-mt323.dll
 0002:000003a4       __imp_?setDragEnabled@QListViewItem@@UAEX_N@Z 1000b3a4     qt-mt323:qt-mt323.dll
 0002:000003a8       __imp_?setDropEnabled@QListViewItem@@UAEX_N@Z 1000b3a8     qt-mt323:qt-mt323.dll
 0002:000003ac       __imp_?setEnabled@QAction@@UAEX_N@Z 1000b3ac     qt-mt323:qt-mt323.dll
 0002:000003b0       __imp_?setEnabled@QListViewItem@@UAEX_N@Z 1000b3b0     qt-mt323:qt-mt323.dll
 0002:000003b4       __imp_?setEnabled@QWidget@@UAEX_N@Z 1000b3b4     qt-mt323:qt-mt323.dll
 0002:000003b8       __imp_?setEraseColor@QWidget@@UAEXABVQColor@@@Z 1000b3b8     qt-mt323:qt-mt323.dll
 0002:000003bc       __imp_?setErasePixmap@QWidget@@UAEXABVQPixmap@@@Z 1000b3bc     qt-mt323:qt-mt323.dll
 0002:000003c0       __imp_?setExpandable@QListViewItem@@UAEX_N@Z 1000b3c0     qt-mt323:qt-mt323.dll
 0002:000003c4       __imp_?setFirstItemActive@QPopupMenu@@EAEXXZ 1000b3c4     qt-mt323:qt-mt323.dll
 0002:000003c8       __imp_?setFixedExtentHeight@QDockWindow@@UAEXH@Z 1000b3c8     qt-mt323:qt-mt323.dll
 0002:000003cc       __imp_?setFixedExtentWidth@QDockWindow@@UAEXH@Z 1000b3cc     qt-mt323:qt-mt323.dll
 0002:000003d0       __imp_?setFocus@QWidget@@UAEXXZ 1000b3d0     qt-mt323:qt-mt323.dll
 0002:000003d4       __imp_?setFocusPolicy@QWidget@@UAEXW4FocusPolicy@1@@Z 1000b3d4     qt-mt323:qt-mt323.dll
 0002:000003d8       __imp_?setFocusProxy@QWidget@@UAEXPAV1@@Z 1000b3d8     qt-mt323:qt-mt323.dll
 0002:000003dc       __imp_?setFont@QPopupMenu@@UAEXABVQFont@@@Z 1000b3dc     qt-mt323:qt-mt323.dll
 0002:000003e0       __imp_?setFont@QWidget@@UAEXABVQFont@@@Z 1000b3e0     qt-mt323:qt-mt323.dll
 0002:000003e4       __imp_?setFrameRect@QFrame@@UAEXABVQRect@@@Z 1000b3e4     qt-mt323:qt-mt323.dll
 0002:000003e8       __imp_?setFrameStyle@QFrame@@UAEXH@Z 1000b3e8     qt-mt323:qt-mt323.dll
 0002:000003ec       __imp_?setGeometry@QWidget@@UAEXABVQRect@@@Z 1000b3ec     qt-mt323:qt-mt323.dll
 0002:000003f0       __imp_?setGeometry@QWidget@@UAEXHHHH@Z 1000b3f0     qt-mt323:qt-mt323.dll
 0002:000003f4       __imp_?setHeight@QListViewItem@@MAEXH@Z 1000b3f4     qt-mt323:qt-mt323.dll
 0002:000003f8       __imp_?setHorizontallyStretchable@QDockWindow@@UAEX_N@Z 1000b3f8     qt-mt323:qt-mt323.dll
 0002:000003fc       __imp_?setIcon@QWidget@@UAEXABVQPixmap@@@Z 1000b3fc     qt-mt323:qt-mt323.dll
 0002:00000400       __imp_?setIconSet@QAction@@UAEXABVQIconSet@@@Z 1000b400     qt-mt323:qt-mt323.dll
 0002:00000404       __imp_?setIconText@QWidget@@UAEXABVQString@@@Z 1000b404     qt-mt323:qt-mt323.dll
 0002:00000408       __imp_?setId@QMenuData@@UAEXHH@Z 1000b408     qt-mt323:qt-mt323.dll
 0002:0000040c       __imp_?setKeyCompression@QWidget@@MAEX_N@Z 1000b40c     qt-mt323:qt-mt323.dll
 0002:00000410       __imp_?setLabel@QToolBar@@UAEXABVQString@@@Z 1000b410     qt-mt323:qt-mt323.dll
 0002:00000414       __imp_?setLineWidth@QFrame@@UAEXH@Z 1000b414     qt-mt323:qt-mt323.dll
 0002:00000418       __imp_?setMargin@QFrame@@UAEXH@Z 1000b418     qt-mt323:qt-mt323.dll
 0002:0000041c       __imp_?setMask@QWidget@@UAEXABVQBitmap@@@Z 1000b41c     qt-mt323:qt-mt323.dll
 0002:00000420       __imp_?setMask@QWidget@@UAEXABVQRegion@@@Z 1000b420     qt-mt323:qt-mt323.dll
 0002:00000424       __imp_?setMaximumSize@QWidget@@UAEXHH@Z 1000b424     qt-mt323:qt-mt323.dll
 0002:00000428       __imp_?setMenuText@QAction@@UAEXABVQString@@@Z 1000b428     qt-mt323:qt-mt323.dll
 0002:0000042c       __imp_?setMicroFocusHint@QWidget@@MAEXHHHH_NPAVQFont@@@Z 1000b42c     qt-mt323:qt-mt323.dll
 0002:00000430       __imp_?setMidLineWidth@QFrame@@UAEXH@Z 1000b430     qt-mt323:qt-mt323.dll
 0002:00000434       __imp_?setMinimumSize@QToolBar@@UAEXHH@Z 1000b434     qt-mt323:qt-mt323.dll
 0002:00000438       __imp_?setMinimumSize@QWidget@@UAEXHH@Z 1000b438     qt-mt323:qt-mt323.dll
 0002:0000043c       __imp_?setMouseTracking@QWidget@@UAEX_N@Z 1000b43c     qt-mt323:qt-mt323.dll
 0002:00000440       __imp_?setMovingEnabled@QDockWindow@@UAEX_N@Z 1000b440     qt-mt323:qt-mt323.dll
 0002:00000444       __imp_?setMultiLinesEnabled@QListViewItem@@UAEX_N@Z 1000b444     qt-mt323:qt-mt323.dll
 0002:00000448       __imp_?setName@QObject@@UAEXPBD@Z 1000b448     qt-mt323:qt-mt323.dll
 0002:0000044c       __imp_?setNewLine@QDockWindow@@UAEX_N@Z 1000b44c     qt-mt323:qt-mt323.dll
 0002:00000450       __imp_?setOffset@QDockWindow@@UAEXH@Z 1000b450     qt-mt323:qt-mt323.dll
 0002:00000454       __imp_?setOn@QAction@@UAEX_N@Z 1000b454     qt-mt323:qt-mt323.dll
 0002:00000458       __imp_?setOpaqueMoving@QDockWindow@@UAEX_N@Z 1000b458     qt-mt323:qt-mt323.dll
 0002:0000045c       __imp_?setOpen@QListViewItem@@UAEX_N@Z 1000b45c     qt-mt323:qt-mt323.dll
 0002:00000460       __imp_?setOrientation@QDockWindow@@UAEXW4Orientation@Qt@@@Z 1000b460     qt-mt323:qt-mt323.dll
 0002:00000464       __imp_?setOrientation@QToolBar@@UAEXW4Orientation@Qt@@@Z 1000b464     qt-mt323:qt-mt323.dll
 0002:00000468       __imp_?setPalette@QWidget@@UAEXABVQPalette@@@Z 1000b468     qt-mt323:qt-mt323.dll
 0002:0000046c       __imp_?setPaletteBackgroundColor@QWidget@@UAEXABVQColor@@@Z 1000b46c     qt-mt323:qt-mt323.dll
 0002:00000470       __imp_?setPaletteBackgroundPixmap@QWidget@@UAEXABVQPixmap@@@Z 1000b470     qt-mt323:qt-mt323.dll
 0002:00000474       __imp_?setPixmap@QListViewItem@@UAEXHABVQPixmap@@@Z 1000b474     qt-mt323:qt-mt323.dll
 0002:00000478       __imp_?setProperty@QObject@@UAE_NPBDABVQVariant@@@Z 1000b478     qt-mt323:qt-mt323.dll
 0002:0000047c       __imp_?setRenameEnabled@QListViewItem@@UAEXH_N@Z 1000b47c     qt-mt323:qt-mt323.dll
 0002:00000480       __imp_?setResizeEnabled@QDockWindow@@UAEX_N@Z 1000b480     qt-mt323:qt-mt323.dll
 0002:00000484       __imp_?setResolution@QPaintDevice@@UAEXH@Z 1000b484     qt-mt323:qt-mt323.dll
 0002:00000488       __imp_?setSelectable@QListViewItem@@UAEX_N@Z 1000b488     qt-mt323:qt-mt323.dll
 0002:0000048c       __imp_?setSelected@QListViewItem@@UAEX_N@Z 1000b48c     qt-mt323:qt-mt323.dll
 0002:00000490       __imp_?setSizeIncrement@QWidget@@UAEXHH@Z 1000b490     qt-mt323:qt-mt323.dll
 0002:00000494       __imp_?setSizePolicy@QWidget@@UAEXVQSizePolicy@@@Z 1000b494     qt-mt323:qt-mt323.dll
 0002:00000498       __imp_?setStatusTip@QAction@@UAEXABVQString@@@Z 1000b498     qt-mt323:qt-mt323.dll
 0002:0000049c       __imp_?setStretchableWidget@QToolBar@@UAEXPAVQWidget@@@Z 1000b49c     qt-mt323:qt-mt323.dll
 0002:000004a0       __imp_?setText@QAction@@UAEXABVQString@@@Z 1000b4a0     qt-mt323:qt-mt323.dll
 0002:000004a4       __imp_?setText@QListViewItem@@UAEXHABVQString@@@Z 1000b4a4     qt-mt323:qt-mt323.dll
 0002:000004a8       __imp_?setToggleAction@QAction@@UAEX_N@Z 1000b4a8     qt-mt323:qt-mt323.dll
 0002:000004ac       __imp_?setToolTip@QAction@@UAEXABVQString@@@Z 1000b4ac     qt-mt323:qt-mt323.dll
 0002:000004b0       __imp_?setUpdatesEnabled@QWidget@@UAEX_N@Z 1000b4b0     qt-mt323:qt-mt323.dll
 0002:000004b4       __imp_?setVerticallyStretchable@QDockWindow@@UAEX_N@Z 1000b4b4     qt-mt323:qt-mt323.dll
 0002:000004b8       __imp_?setWFlags@QWidget@@MAEXI@Z 1000b4b8     qt-mt323:qt-mt323.dll
 0002:000004bc       __imp_?setWState@QWidget@@MAEXI@Z 1000b4bc     qt-mt323:qt-mt323.dll
 0002:000004c0       __imp_?setWhatsThis@QAction@@UAEXABVQString@@@Z 1000b4c0     qt-mt323:qt-mt323.dll
 0002:000004c4       __imp_?setWidget@QDockWindow@@UAEXPAVQWidget@@@Z 1000b4c4     qt-mt323:qt-mt323.dll
 0002:000004c8       __imp_?setup@QListViewItem@@UAEXXZ 1000b4c8     qt-mt323:qt-mt323.dll
 0002:000004cc       __imp_?show@QPopupMenu@@UAEXXZ 1000b4cc     qt-mt323:qt-mt323.dll
 0002:000004d0       __imp_?show@QToolBar@@UAEXXZ 1000b4d0     qt-mt323:qt-mt323.dll
 0002:000004d4       __imp_?show@QWidget@@UAEXXZ 1000b4d4     qt-mt323:qt-mt323.dll
 0002:000004d8       __imp_?showEvent@QDockWindow@@MAEXPAVQShowEvent@@@Z 1000b4d8     qt-mt323:qt-mt323.dll
 0002:000004dc       __imp_?showEvent@QWidget@@MAEXPAVQShowEvent@@@Z 1000b4dc     qt-mt323:qt-mt323.dll
 0002:000004e0       __imp_?showMaximized@QWidget@@UAEXXZ 1000b4e0     qt-mt323:qt-mt323.dll
 0002:000004e4       __imp_?showMinimized@QWidget@@UAEXXZ 1000b4e4     qt-mt323:qt-mt323.dll
 0002:000004e8       __imp_?showNormal@QWidget@@UAEXXZ 1000b4e8     qt-mt323:qt-mt323.dll
 0002:000004ec       __imp_?sizeHint@QDockWindow@@UBE?AVQSize@@XZ 1000b4ec     qt-mt323:qt-mt323.dll
 0002:000004f0       __imp_?sizeHint@QPopupMenu@@UBE?AVQSize@@XZ 1000b4f0     qt-mt323:qt-mt323.dll
 0002:000004f4       __imp_?sizeHint@QWidget@@UBE?AVQSize@@XZ 1000b4f4     qt-mt323:qt-mt323.dll
 0002:000004f8       __imp_?sizePolicy@QWidget@@UBE?AVQSizePolicy@@XZ 1000b4f8     qt-mt323:qt-mt323.dll
 0002:000004fc       __imp_?sort@QListViewItem@@UAEXXZ 1000b4fc     qt-mt323:qt-mt323.dll
 0002:00000500       __imp_?sortChildItems@QListViewItem@@UAEXH_N@Z 1000b500     qt-mt323:qt-mt323.dll
 0002:00000504       __imp_?startRename@QListViewItem@@UAEXH@Z 1000b504     qt-mt323:qt-mt323.dll
 0002:00000508       __imp_?styleChange@QFrame@@MAEXAAVQStyle@@@Z 1000b508     qt-mt323:qt-mt323.dll
 0002:0000050c       __imp_?styleChange@QPopupMenu@@MAEXAAVQStyle@@@Z 1000b50c     qt-mt323:qt-mt323.dll
 0002:00000510       __imp_?styleChange@QToolBar@@MAEXAAVQStyle@@@Z 1000b510     qt-mt323:qt-mt323.dll
 0002:00000514       __imp_?styleChange@QWidget@@MAEXAAVQStyle@@@Z 1000b514     qt-mt323:qt-mt323.dll
 0002:00000518       __imp_?tabletEvent@QWidget@@MAEXPAVQTabletEvent@@@Z 1000b518     qt-mt323:qt-mt323.dll
 0002:0000051c       __imp_?takeItem@QListViewItem@@UAEXPAV1@@Z 1000b51c     qt-mt323:qt-mt323.dll
 0002:00000520       __imp_?text@QListViewItem@@UBE?AVQString@@H@Z 1000b520     qt-mt323:qt-mt323.dll
 0002:00000524       __imp_?timerEvent@QObject@@MAEXPAVQTimerEvent@@@Z 1000b524     qt-mt323:qt-mt323.dll
 0002:00000528       __imp_?timerEvent@QPopupMenu@@MAEXPAVQTimerEvent@@@Z 1000b528     qt-mt323:qt-mt323.dll
 0002:0000052c       __imp_?undock@QDockWindow@@UAEXPAVQWidget@@@Z 1000b52c     qt-mt323:qt-mt323.dll
 0002:00000530       __imp_?undock@QDockWindow@@UAEXXZ 1000b530     qt-mt323:qt-mt323.dll
 0002:00000534       __imp_?unsetCursor@QWidget@@UAEXXZ 1000b534     qt-mt323:qt-mt323.dll
 0002:00000538       __imp_?updateItem@QPopupMenu@@UAEXH@Z 1000b538     qt-mt323:qt-mt323.dll
 0002:0000053c       __imp_?updateMask@QWidget@@MAEXXZ 1000b53c     qt-mt323:qt-mt323.dll
 0002:00000540       __imp_?wheelEvent@QWidget@@MAEXPAVQWheelEvent@@@Z 1000b540     qt-mt323:qt-mt323.dll
 0002:00000544       __imp_?width@QListViewItem@@UBEHABVQFontMetrics@@PBVQListView@@H@Z 1000b544     qt-mt323:qt-mt323.dll
 0002:00000548       __imp_?winEvent@QWidget@@MAE_NPAUtagMSG@@@Z 1000b548     qt-mt323:qt-mt323.dll
 0002:0000054c       __imp_?windowActivationChange@QWidget@@MAEX_N@Z 1000b54c     qt-mt323:qt-mt323.dll
 0002:00000550       __imp_?write@QGDict@@MBEAAVQDataStream@@AAV2@PAX@Z 1000b550     qt-mt323:qt-mt323.dll
 0002:00000554       __imp_?write@QGList@@MBEAAVQDataStream@@AAV2@PAX@Z 1000b554     qt-mt323:qt-mt323.dll
 0002:00000558       __imp_?null@QString@@2V1@A 1000b558     qt-mt323:qt-mt323.dll
 0002:0000055c       __imp_??_7?$QPtrList@VQDockWindow@@@@6B@ 1000b55c     qt-mt323:qt-mt323.dll
 0002:00000560       __imp_?arg@QString@@QBE?AV1@HHH@Z 1000b560     qt-mt323:qt-mt323.dll
 0002:00000564       __imp_??0QTextStream@@QAE@PAVQIODevice@@@Z 1000b564     qt-mt323:qt-mt323.dll
 0002:00000568       __imp_??1QTextStream@@UAE@XZ 1000b568     qt-mt323:qt-mt323.dll
 0002:0000056c       __imp_?read@QTextStream@@QAE?AVQString@@XZ 1000b56c     qt-mt323:qt-mt323.dll
 0002:00000570       __imp_??A?$QValueList@VQString@@@@QAEAAVQString@@I@Z 1000b570     qt-mt323:qt-mt323.dll
 0002:00000574       __imp_??0?$QMap@VQString@@V1@@@QAE@XZ 1000b574     qt-mt323:qt-mt323.dll
 0002:00000578       __imp_??1?$QMap@VQString@@V1@@@QAE@XZ 1000b578     qt-mt323:qt-mt323.dll
 0002:0000057c       __imp_?begin@?$QMap@VQString@@V1@@@QAE?AV?$QMapIterator@VQString@@V1@@@XZ 1000b57c     qt-mt323:qt-mt323.dll
 0002:00000580       __imp_?end@?$QMap@VQString@@V1@@@QAE?AV?$QMapIterator@VQString@@V1@@@XZ 1000b580     qt-mt323:qt-mt323.dll
 0002:00000584       __imp_??A?$QMap@VQString@@V1@@@QAEAAVQString@@ABV1@@Z 1000b584     qt-mt323:qt-mt323.dll
 0002:00000588       __imp_?inherits@QObject@@QBE_NPBD@Z 1000b588     qt-mt323:qt-mt323.dll
 0002:0000058c       __imp_?blockSignals@QObject@@QAEX_N@Z 1000b58c     qt-mt323:qt-mt323.dll
 0002:00000590       __imp_?sender@QObject@@IAEPBV1@XZ 1000b590     qt-mt323:qt-mt323.dll
 0002:00000594       __imp_?split@QStringList@@SA?AV1@ABVQString@@0_N@Z 1000b594     qt-mt323:qt-mt323.dll
 0002:00000598       __imp_??1QStringList@@QAE@XZ 1000b598     qt-mt323:qt-mt323.dll
 0002:0000059c       __imp_?updateContents@QScrollView@@QAEXXZ 1000b59c     qt-mt323:qt-mt323.dll
 0002:000005a0       __imp_?look_int@QGDict@@QAEPAXJPAXH@Z 1000b5a0     qt-mt323:qt-mt323.dll
 0002:000005a4       __imp_?setText@QTextEdit@@QAEXABVQString@@@Z 1000b5a4     qt-mt323:qt-mt323.dll
 0002:000005a8       __imp_??0QFile@@QAE@ABVQString@@@Z 1000b5a8     qt-mt323:qt-mt323.dll
 0002:000005ac       __imp_??1QFile@@UAE@XZ     1000b5ac     qt-mt323:qt-mt323.dll
 0002:000005b0       __imp_?open@QFile@@UAE_NH@Z 1000b5b0     qt-mt323:qt-mt323.dll
 0002:000005b4       __imp_?readLine@QFile@@UAEJPADK@Z 1000b5b4     qt-mt323:qt-mt323.dll
 0002:000005b8       __imp_?horizontalHeader@QTable@@QBEPAVQHeader@@XZ 1000b5b8     qt-mt323:qt-mt323.dll
 0002:000005bc       __imp_?setTabLabel@QTabWidget@@QAEXPAVQWidget@@ABVQString@@@Z 1000b5bc     qt-mt323:qt-mt323.dll
 0002:000005c0       __imp_?page@QTabWidget@@QBEPAVQWidget@@H@Z 1000b5c0     qt-mt323:qt-mt323.dll
 0002:000005c4       __imp_?setCurrentPage@QTabWidget@@QAEXH@Z 1000b5c4     qt-mt323:qt-mt323.dll
 0002:000005c8       __imp_??6?$QValueList@VQString@@@@QAEAAV0@ABVQString@@@Z 1000b5c8     qt-mt323:qt-mt323.dll
 0002:000005cc       __imp_??0QStringList@@QAE@XZ 1000b5cc     qt-mt323:qt-mt323.dll
 0002:000005d0       __imp_?resize@QWidget@@QAEXABVQSize@@@Z 1000b5d0     qt-mt323:qt-mt323.dll
 0002:000005d4       __imp_?setFrameShape@QFrame@@QAEXW4Shape@1@@Z 1000b5d4     qt-mt323:qt-mt323.dll
 0002:000005d8       __imp_?setFrameShadow@QFrame@@QAEXW4Shadow@1@@Z 1000b5d8     qt-mt323:qt-mt323.dll
 0002:000005dc       __imp_??0QLabel@@QAE@PAVQWidget@@PBDI@Z 1000b5dc     qt-mt323:qt-mt323.dll
 0002:000005e0       __imp_??1QLabel@@UAE@XZ    1000b5e0     qt-mt323:qt-mt323.dll
 0002:000005e4       __imp_??0QTabWidget@@QAE@PAVQWidget@@PBDI@Z 1000b5e4     qt-mt323:qt-mt323.dll
 0002:000005e8       __imp_??1QTabWidget@@UAE@XZ 1000b5e8     qt-mt323:qt-mt323.dll
 0002:000005ec       __imp_?changeTab@QTabWidget@@QAEXPAVQWidget@@ABVQString@@@Z 1000b5ec     qt-mt323:qt-mt323.dll
 0002:000005f0       __imp_??0QLineEdit@@QAE@PAVQWidget@@PBD@Z 1000b5f0     qt-mt323:qt-mt323.dll
 0002:000005f4       __imp_??1QLineEdit@@UAE@XZ 1000b5f4     qt-mt323:qt-mt323.dll
 0002:000005f8       __imp_??0QTextEdit@@QAE@PAVQWidget@@PBD@Z 1000b5f8     qt-mt323:qt-mt323.dll
 0002:000005fc       __imp_??1QTextEdit@@UAE@XZ 1000b5fc     qt-mt323:qt-mt323.dll
 0002:00000600       __imp_??0QTable@@QAE@PAVQWidget@@PBD@Z 1000b600     qt-mt323:qt-mt323.dll
 0002:00000604       __imp_??1QTable@@UAE@XZ    1000b604     qt-mt323:qt-mt323.dll
 0002:00000608       __imp_??1QLayoutItem@@UAE@XZ 1000b608     qt-mt323:qt-mt323.dll
 0002:0000060c       __imp_??0QSpacerItem@@QAE@HHW4SizeType@QSizePolicy@@0@Z 1000b60c     qt-mt323:qt-mt323.dll
 0002:00000610       __imp_?addWidget@QBoxLayout@@QAEXPAVQWidget@@HH@Z 1000b610     qt-mt323:qt-mt323.dll
 0002:00000614       __imp_?addLayout@QBoxLayout@@QAEXPAVQLayout@@H@Z 1000b614     qt-mt323:qt-mt323.dll
 0002:00000618       __imp_??0QHBoxLayout@@QAE@PAVQWidget@@HHPBD@Z 1000b618     qt-mt323:qt-mt323.dll
 0002:0000061c       __imp_??1QHBoxLayout@@UAE@XZ 1000b61c     qt-mt323:qt-mt323.dll
 0002:00000620       __imp_??0QVBoxLayout@@QAE@PAVQWidget@@HHPBD@Z 1000b620     qt-mt323:qt-mt323.dll
 0002:00000624       __imp_??1QVBoxLayout@@UAE@XZ 1000b624     qt-mt323:qt-mt323.dll
 0002:00000628       __imp_?activateNextCell@QTable@@MAEXXZ 1000b628     qt-mt323:qt-mt323.dll
 0002:0000062c       __imp_?addChild@QScrollView@@UAEXPAVQWidget@@HH@Z 1000b62c     qt-mt323:qt-mt323.dll
 0002:00000630       __imp_?addItem@QBoxLayout@@UAEXPAVQLayoutItem@@@Z 1000b630     qt-mt323:qt-mt323.dll
 0002:00000634       __imp_?addSelection@QTable@@UAEHABVQTableSelection@@@Z 1000b634     qt-mt323:qt-mt323.dll
 0002:00000638       __imp_?addTab@QTabWidget@@UAEXPAVQWidget@@ABVQIconSet@@ABVQString@@@Z 1000b638     qt-mt323:qt-mt323.dll
 0002:0000063c       __imp_?addTab@QTabWidget@@UAEXPAVQWidget@@ABVQString@@@Z 1000b63c     qt-mt323:qt-mt323.dll
 0002:00000640       __imp_?addTab@QTabWidget@@UAEXPAVQWidget@@PAVQTab@@@Z 1000b640     qt-mt323:qt-mt323.dll
 0002:00000644       __imp_?adjustColumn@QTable@@UAEXH@Z 1000b644     qt-mt323:qt-mt323.dll
 0002:00000648       __imp_?adjustRow@QTable@@UAEXH@Z 1000b648     qt-mt323:qt-mt323.dll
 0002:0000064c       __imp_?append@QTextEdit@@UAEXABVQString@@@Z 1000b64c     qt-mt323:qt-mt323.dll
 0002:00000650       __imp_?beginEdit@QTable@@MAEPAVQWidget@@HH_N@Z 1000b650     qt-mt323:qt-mt323.dll
 0002:00000654       __imp_?cellGeometry@QTable@@UBE?AVQRect@@HH@Z 1000b654     qt-mt323:qt-mt323.dll
 0002:00000658       __imp_?cellRect@QTable@@UBE?AVQRect@@HH@Z 1000b658     qt-mt323:qt-mt323.dll
 0002:0000065c       __imp_?cellWidget@QTable@@UBEPAVQWidget@@HH@Z 1000b65c     qt-mt323:qt-mt323.dll
 0002:00000660       __imp_?childEvent@QLayout@@MAEXPAVQChildEvent@@@Z 1000b660     qt-mt323:qt-mt323.dll
 0002:00000664       __imp_?className@QHBoxLayout@@UBEPBDXZ 1000b664     qt-mt323:qt-mt323.dll
 0002:00000668       __imp_?className@QLabel@@UBEPBDXZ 1000b668     qt-mt323:qt-mt323.dll
 0002:0000066c       __imp_?className@QLineEdit@@UBEPBDXZ 1000b66c     qt-mt323:qt-mt323.dll
 0002:00000670       __imp_?className@QTabWidget@@UBEPBDXZ 1000b670     qt-mt323:qt-mt323.dll
 0002:00000674       __imp_?className@QTable@@UBEPBDXZ 1000b674     qt-mt323:qt-mt323.dll
 0002:00000678       __imp_?className@QTextEdit@@UBEPBDXZ 1000b678     qt-mt323:qt-mt323.dll
 0002:0000067c       __imp_?className@QVBoxLayout@@UBEPBDXZ 1000b67c     qt-mt323:qt-mt323.dll
 0002:00000680       __imp_?clear@QLineEdit@@UAEXXZ 1000b680     qt-mt323:qt-mt323.dll
 0002:00000684       __imp_?clear@QTextEdit@@UAEXXZ 1000b684     qt-mt323:qt-mt323.dll
 0002:00000688       __imp_?clearCell@QTable@@UAEXHH@Z 1000b688     qt-mt323:qt-mt323.dll
 0002:0000068c       __imp_?clearCellWidget@QTable@@UAEXHH@Z 1000b68c     qt-mt323:qt-mt323.dll
 0002:00000690       __imp_?clearParagraphBackground@QTextEdit@@UAEXH@Z 1000b690     qt-mt323:qt-mt323.dll
 0002:00000694       __imp_?clearValidator@QLineEdit@@UAEXXZ 1000b694     qt-mt323:qt-mt323.dll
 0002:00000698       __imp_?columnAt@QTable@@UBEHH@Z 1000b698     qt-mt323:qt-mt323.dll
 0002:0000069c       __imp_?columnClicked@QTable@@MAEXH@Z 1000b69c     qt-mt323:qt-mt323.dll
 0002:000006a0       __imp_?columnIndexChanged@QTable@@MAEXHHH@Z 1000b6a0     qt-mt323:qt-mt323.dll
 0002:000006a4       __imp_?columnPos@QTable@@UBEHH@Z 1000b6a4     qt-mt323:qt-mt323.dll
 0002:000006a8       __imp_?columnWidth@QTable@@UBEHH@Z 1000b6a8     qt-mt323:qt-mt323.dll
 0002:000006ac       __imp_?columnWidthChanged@QTable@@MAEXH@Z 1000b6ac     qt-mt323:qt-mt323.dll
 0002:000006b0       __imp_?contentsContextMenuEvent@QTable@@MAEXPAVQContextMenuEvent@@@Z 1000b6b0     qt-mt323:qt-mt323.dll
 0002:000006b4       __imp_?contentsContextMenuEvent@QTextEdit@@MAEXPAVQContextMenuEvent@@@Z 1000b6b4     qt-mt323:qt-mt323.dll
 0002:000006b8       __imp_?contentsDragEnterEvent@QTable@@MAEXPAVQDragEnterEvent@@@Z 1000b6b8     qt-mt323:qt-mt323.dll
 0002:000006bc       __imp_?contentsDragEnterEvent@QTextEdit@@MAEXPAVQDragEnterEvent@@@Z 1000b6bc     qt-mt323:qt-mt323.dll
 0002:000006c0       __imp_?contentsDragLeaveEvent@QTable@@MAEXPAVQDragLeaveEvent@@@Z 1000b6c0     qt-mt323:qt-mt323.dll
 0002:000006c4       __imp_?contentsDragLeaveEvent@QTextEdit@@MAEXPAVQDragLeaveEvent@@@Z 1000b6c4     qt-mt323:qt-mt323.dll
 0002:000006c8       __imp_?contentsDragMoveEvent@QTable@@MAEXPAVQDragMoveEvent@@@Z 1000b6c8     qt-mt323:qt-mt323.dll
 0002:000006cc       __imp_?contentsDragMoveEvent@QTextEdit@@MAEXPAVQDragMoveEvent@@@Z 1000b6cc     qt-mt323:qt-mt323.dll
 0002:000006d0       __imp_?contentsDropEvent@QTable@@MAEXPAVQDropEvent@@@Z 1000b6d0     qt-mt323:qt-mt323.dll
 0002:000006d4       __imp_?contentsDropEvent@QTextEdit@@MAEXPAVQDropEvent@@@Z 1000b6d4     qt-mt323:qt-mt323.dll
 0002:000006d8       __imp_?contentsMouseDoubleClickEvent@QTable@@MAEXPAVQMouseEvent@@@Z 1000b6d8     qt-mt323:qt-mt323.dll
 0002:000006dc       __imp_?contentsMouseDoubleClickEvent@QTextEdit@@MAEXPAVQMouseEvent@@@Z 1000b6dc     qt-mt323:qt-mt323.dll
 0002:000006e0       __imp_?contentsMouseMoveEvent@QTable@@MAEXPAVQMouseEvent@@@Z 1000b6e0     qt-mt323:qt-mt323.dll
 0002:000006e4       __imp_?contentsMouseMoveEvent@QTextEdit@@MAEXPAVQMouseEvent@@@Z 1000b6e4     qt-mt323:qt-mt323.dll
 0002:000006e8       __imp_?contentsMousePressEvent@QTable@@MAEXPAVQMouseEvent@@@Z 1000b6e8     qt-mt323:qt-mt323.dll
 0002:000006ec       __imp_?contentsMousePressEvent@QTextEdit@@MAEXPAVQMouseEvent@@@Z 1000b6ec     qt-mt323:qt-mt323.dll
 0002:000006f0       __imp_?contentsMouseReleaseEvent@QTable@@MAEXPAVQMouseEvent@@@Z 1000b6f0     qt-mt323:qt-mt323.dll
 0002:000006f4       __imp_?contentsMouseReleaseEvent@QTextEdit@@MAEXPAVQMouseEvent@@@Z 1000b6f4     qt-mt323:qt-mt323.dll
 0002:000006f8       __imp_?contentsWheelEvent@QScrollView@@MAEXPAVQWheelEvent@@@Z 1000b6f8     qt-mt323:qt-mt323.dll
 0002:000006fc       __imp_?contentsWheelEvent@QTextEdit@@MAEXPAVQWheelEvent@@@Z 1000b6fc     qt-mt323:qt-mt323.dll
 0002:00000700       __imp_?contextMenuEvent@QLineEdit@@MAEXPAVQContextMenuEvent@@@Z 1000b700     qt-mt323:qt-mt323.dll
 0002:00000704       __imp_?contextMenuEvent@QScrollView@@MAEXPAVQContextMenuEvent@@@Z 1000b704     qt-mt323:qt-mt323.dll
 0002:00000708       __imp_?copy@QLineEdit@@UBEXXZ 1000b708     qt-mt323:qt-mt323.dll
 0002:0000070c       __imp_?copy@QTextEdit@@UAEXXZ 1000b70c     qt-mt323:qt-mt323.dll
 0002:00000710       __imp_?createEditor@QTable@@MBEPAVQWidget@@HH_N@Z 1000b710     qt-mt323:qt-mt323.dll
 0002:00000714       __imp_?createPopupMenu@QLineEdit@@MAEPAVQPopupMenu@@XZ 1000b714     qt-mt323:qt-mt323.dll
 0002:00000718       __imp_??1QRegExp@@QAE@XZ   1000b718     qt-mt323:qt-mt323.dll
 0002:0000071c       __imp_?createPopupMenu@QTextEdit@@MAEPAVQPopupMenu@@XZ 1000b71c     qt-mt323:qt-mt323.dll
 0002:00000720       __imp_?currentSelection@QTable@@UBEHXZ 1000b720     qt-mt323:qt-mt323.dll
 0002:00000724       __imp_?cut@QLineEdit@@UAEXXZ 1000b724     qt-mt323:qt-mt323.dll
 0002:00000728       __imp_?cut@QTextEdit@@UAEXXZ 1000b728     qt-mt323:qt-mt323.dll
 0002:0000072c       __imp_?del@QTextEdit@@UAEXXZ 1000b72c     qt-mt323:qt-mt323.dll
 0002:00000730       __imp_?deselect@QLineEdit@@UAEXXZ 1000b730     qt-mt323:qt-mt323.dll
 0002:00000734       __imp_?doChangeInterval@QTextEdit@@MAEXXZ 1000b734     qt-mt323:qt-mt323.dll
 0002:00000738       __imp_?doKeyboardAction@QTextEdit@@UAEXW4KeyboardAction@1@@Z 1000b738     qt-mt323:qt-mt323.dll
 0002:0000073c       __imp_?dragEnterEvent@QLineEdit@@MAEXPAVQDragEnterEvent@@@Z 1000b73c     qt-mt323:qt-mt323.dll
 0002:00000740       __imp_?dragLeaveEvent@QLineEdit@@MAEXPAVQDragLeaveEvent@@@Z 1000b740     qt-mt323:qt-mt323.dll
 0002:00000744       __imp_?dragMoveEvent@QLineEdit@@MAEXPAVQDragMoveEvent@@@Z 1000b744     qt-mt323:qt-mt323.dll
 0002:00000748       __imp_?dragObject@QTable@@MAEPAVQDragObject@@XZ 1000b748     qt-mt323:qt-mt323.dll
 0002:0000074c       __imp_?drawContents@QLabel@@MAEXPAVQPainter@@@Z 1000b74c     qt-mt323:qt-mt323.dll
 0002:00000750       __imp_?drawContents@QLineEdit@@MAEXPAVQPainter@@@Z 1000b750     qt-mt323:qt-mt323.dll
 0002:00000754       __imp_?drawContents@QTable@@EAEXPAVQPainter@@@Z 1000b754     qt-mt323:qt-mt323.dll
 0002:00000758       __imp_?drawContents@QTable@@MAEXPAVQPainter@@HHHH@Z 1000b758     qt-mt323:qt-mt323.dll
 0002:0000075c       __imp_?drawContents@QTextEdit@@EAEXPAVQPainter@@@Z 1000b75c     qt-mt323:qt-mt323.dll
 0002:00000760       __imp_?drawContents@QTextEdit@@MAEXPAVQPainter@@HHHH@Z 1000b760     qt-mt323:qt-mt323.dll
 0002:00000764       __imp_?drawContentsOffset@QScrollView@@MAEXPAVQPainter@@HHHHHH@Z 1000b764     qt-mt323:qt-mt323.dll
 0002:00000768       __imp_?dropEvent@QLineEdit@@MAEXPAVQDropEvent@@@Z 1000b768     qt-mt323:qt-mt323.dll
 0002:0000076c       __imp_?editCell@QTable@@UAEXHH_N@Z 1000b76c     qt-mt323:qt-mt323.dll
 0002:00000770       __imp_?emitHighlighted@QTextEdit@@EAEXABVQString@@@Z 1000b770     qt-mt323:qt-mt323.dll
 0002:00000774       __imp_?emitLinkClicked@QTextEdit@@EAEXABVQString@@@Z 1000b774     qt-mt323:qt-mt323.dll
 0002:00000778       __imp_?endEdit@QTable@@MAEXHH_N0@Z 1000b778     qt-mt323:qt-mt323.dll
 0002:0000077c       __imp_?ensureCursorVisible@QTextEdit@@UAEXXZ 1000b77c     qt-mt323:qt-mt323.dll
 0002:00000780       __imp_?event@QLineEdit@@MAE_NPAVQEvent@@@Z 1000b780     qt-mt323:qt-mt323.dll
 0002:00000784       __imp_?event@QTextEdit@@MAE_NPAVQEvent@@@Z 1000b784     qt-mt323:qt-mt323.dll
 0002:00000788       __imp_?eventFilter@QLayout@@MAE_NPAVQObject@@PAVQEvent@@@Z 1000b788     qt-mt323:qt-mt323.dll
 0002:0000078c       __imp_?eventFilter@QTabWidget@@MAE_NPAVQObject@@PAVQEvent@@@Z 1000b78c     qt-mt323:qt-mt323.dll
 0002:00000790       __imp_?eventFilter@QTable@@UAE_NPAVQObject@@PAVQEvent@@@Z 1000b790     qt-mt323:qt-mt323.dll
 0002:00000794       __imp_?eventFilter@QTextEdit@@UAE_NPAVQObject@@PAVQEvent@@@Z 1000b794     qt-mt323:qt-mt323.dll
 0002:00000798       __imp_?expanding@QBoxLayout@@UBE?AW4ExpandData@QSizePolicy@@XZ 1000b798     qt-mt323:qt-mt323.dll
 0002:0000079c       __imp_?expanding@QSpacerItem@@UBE?AW4ExpandData@QSizePolicy@@XZ 1000b79c     qt-mt323:qt-mt323.dll
 0002:000007a0       __imp_?find@QTextEdit@@UAE_NABVQString@@_N11PAH2@Z 1000b7a0     qt-mt323:qt-mt323.dll
 0002:000007a4       __imp_?focusInEvent@QLineEdit@@MAEXPAVQFocusEvent@@@Z 1000b7a4     qt-mt323:qt-mt323.dll
 0002:000007a8       __imp_?focusInEvent@QTable@@MAEXPAVQFocusEvent@@@Z 1000b7a8     qt-mt323:qt-mt323.dll
 0002:000007ac       __imp_?focusNextPrevChild@QScrollView@@MAE_N_N@Z 1000b7ac     qt-mt323:qt-mt323.dll
 0002:000007b0       __imp_?focusNextPrevChild@QTextEdit@@MAE_N_N@Z 1000b7b0     qt-mt323:qt-mt323.dll
 0002:000007b4       __imp_?focusOutEvent@QLineEdit@@MAEXPAVQFocusEvent@@@Z 1000b7b4     qt-mt323:qt-mt323.dll
 0002:000007b8       __imp_?focusOutEvent@QTable@@MAEXPAVQFocusEvent@@@Z 1000b7b8     qt-mt323:qt-mt323.dll
 0002:000007bc       __imp_?fontChange@QLabel@@MAEXABVQFont@@@Z 1000b7bc     qt-mt323:qt-mt323.dll
 0002:000007c0       __imp_?fontChange@QScrollView@@MAEXABVQFont@@@Z 1000b7c0     qt-mt323:qt-mt323.dll
 0002:000007c4       __imp_?frameChanged@QScrollView@@MAEXXZ 1000b7c4     qt-mt323:qt-mt323.dll
 0002:000007c8       __imp_?geometry@QLayout@@UBE?AVQRect@@XZ 1000b7c8     qt-mt323:qt-mt323.dll
 0002:000007cc       __imp_?geometry@QSpacerItem@@UBE?AVQRect@@XZ 1000b7cc     qt-mt323:qt-mt323.dll
 0002:000007d0       __imp_?getFormat@QTextEdit@@UAE_NHHPAVQFont@@PAVQColor@@PAW4VerticalAlignment@1@@Z 1000b7d0     qt-mt323:qt-mt323.dll
 0002:000007d4       __imp_?getParagraphFormat@QTextEdit@@UAE_NHPAVQFont@@PAVQColor@@PAW4VerticalAlignment@1@PAHPAW4DisplayMode@QStyleSheetItem@@PAW4ListStyle@6@3@Z 1000b7d4     qt-mt323:qt-mt323.dll
 0002:000007d8       __imp_?hasHeightForWidth@QBoxLayout@@UBE_NXZ 1000b7d8     qt-mt323:qt-mt323.dll
 0002:000007dc       __imp_?hasHeightForWidth@QLayoutItem@@UBE_NXZ 1000b7dc     qt-mt323:qt-mt323.dll
 0002:000007e0       __imp_?heightForWidth@QBoxLayout@@UBEHH@Z 1000b7e0     qt-mt323:qt-mt323.dll
 0002:000007e4       __imp_?heightForWidth@QLabel@@UBEHH@Z 1000b7e4     qt-mt323:qt-mt323.dll
 0002:000007e8       __imp_?heightForWidth@QLayoutItem@@UBEHH@Z 1000b7e8     qt-mt323:qt-mt323.dll
 0002:000007ec       __imp_?heightForWidth@QTextEdit@@UBEHH@Z 1000b7ec     qt-mt323:qt-mt323.dll
 0002:000007f0       __imp_?hideColumn@QTable@@UAEXH@Z 1000b7f0     qt-mt323:qt-mt323.dll
 0002:000007f4       __imp_?hideRow@QTable@@UAEXH@Z 1000b7f4     qt-mt323:qt-mt323.dll
 0002:000007f8       __imp_?imComposeEvent@QLineEdit@@MAEXPAVQIMEvent@@@Z 1000b7f8     qt-mt323:qt-mt323.dll
 0002:000007fc       __imp_?imComposeEvent@QTextEdit@@MAEXPAVQIMEvent@@@Z 1000b7fc     qt-mt323:qt-mt323.dll
 0002:00000800       __imp_?imEndEvent@QLineEdit@@MAEXPAVQIMEvent@@@Z 1000b800     qt-mt323:qt-mt323.dll
 0002:00000804       __imp_?imEndEvent@QTextEdit@@MAEXPAVQIMEvent@@@Z 1000b804     qt-mt323:qt-mt323.dll
 0002:00000808       __imp_?imStartEvent@QLineEdit@@MAEXPAVQIMEvent@@@Z 1000b808     qt-mt323:qt-mt323.dll
 0002:0000080c       __imp_?imStartEvent@QTextEdit@@MAEXPAVQIMEvent@@@Z 1000b80c     qt-mt323:qt-mt323.dll
 0002:00000810       __imp_?indent@QTextEdit@@UAEXXZ 1000b810     qt-mt323:qt-mt323.dll
 0002:00000814       __imp_?insert@QLineEdit@@UAEXABVQString@@@Z 1000b814     qt-mt323:qt-mt323.dll
 0002:00000818       __imp_?insert@QTextEdit@@UAEXABVQString@@_N11@Z 1000b818     qt-mt323:qt-mt323.dll
 0002:0000081c       __imp_?insertAt@QTextEdit@@UAEXABVQString@@HH@Z 1000b81c     qt-mt323:qt-mt323.dll
 0002:00000820       __imp_?insertColumns@QTable@@UAEXHH@Z 1000b820     qt-mt323:qt-mt323.dll
 0002:00000824       __imp_?insertParagraph@QTextEdit@@UAEXABVQString@@H@Z 1000b824     qt-mt323:qt-mt323.dll
 0002:00000828       __imp_?insertRows@QTable@@UAEXHH@Z 1000b828     qt-mt323:qt-mt323.dll
 0002:0000082c       __imp_?insertTab@QTabWidget@@UAEXPAVQWidget@@ABVQIconSet@@ABVQString@@H@Z 1000b82c     qt-mt323:qt-mt323.dll
 0002:00000830       __imp_?insertTab@QTabWidget@@UAEXPAVQWidget@@ABVQString@@H@Z 1000b830     qt-mt323:qt-mt323.dll
 0002:00000834       __imp_?insertTab@QTabWidget@@UAEXPAVQWidget@@PAVQTab@@H@Z 1000b834     qt-mt323:qt-mt323.dll
 0002:00000838       __imp_?insertWidget@QTable@@MAEXHHPAVQWidget@@@Z 1000b838     qt-mt323:qt-mt323.dll
 0002:0000083c       __imp_?invalidate@QBoxLayout@@UAEXXZ 1000b83c     qt-mt323:qt-mt323.dll
 0002:00000840       __imp_?invalidate@QLayoutItem@@UAEXXZ 1000b840     qt-mt323:qt-mt323.dll
 0002:00000844       __imp_?isEmpty@QLayout@@UBE_NXZ 1000b844     qt-mt323:qt-mt323.dll
 0002:00000848       __imp_?isEmpty@QSpacerItem@@UBE_NXZ 1000b848     qt-mt323:qt-mt323.dll
 0002:0000084c       __imp_?item@QTable@@UBEPAVQTableItem@@HH@Z 1000b84c     qt-mt323:qt-mt323.dll
 0002:00000850       __imp_?iterator@QBoxLayout@@UAE?AVQLayoutIterator@@XZ 1000b850     qt-mt323:qt-mt323.dll
 0002:00000854       __imp_?iterator@QLayoutItem@@UAE?AVQLayoutIterator@@XZ 1000b854     qt-mt323:qt-mt323.dll
 0002:00000858       __imp_?keyPressEvent@QLineEdit@@MAEXPAVQKeyEvent@@@Z 1000b858     qt-mt323:qt-mt323.dll
 0002:0000085c       __imp_?keyPressEvent@QTable@@MAEXPAVQKeyEvent@@@Z 1000b85c     qt-mt323:qt-mt323.dll
 0002:00000860       __imp_?keyPressEvent@QTextEdit@@MAEXPAVQKeyEvent@@@Z 1000b860     qt-mt323:qt-mt323.dll
 0002:00000864       __imp_?layout@QLayout@@UAEPAV1@XZ 1000b864     qt-mt323:qt-mt323.dll
 0002:00000868       __imp_?layout@QLayoutItem@@UAEPAVQLayout@@XZ 1000b868     qt-mt323:qt-mt323.dll
 0002:0000086c       __imp_?linksEnabled@QTextEdit@@EBE_NXZ 1000b86c     qt-mt323:qt-mt323.dll
 0002:00000870       __imp_?maximumSize@QBoxLayout@@UBE?AVQSize@@XZ 1000b870     qt-mt323:qt-mt323.dll
 0002:00000874       __imp_?maximumSize@QSpacerItem@@UBE?AVQSize@@XZ 1000b874     qt-mt323:qt-mt323.dll
 0002:00000878       __imp_?metaObject@QHBoxLayout@@UBEPAVQMetaObject@@XZ 1000b878     qt-mt323:qt-mt323.dll
 0002:0000087c       __imp_?metaObject@QLabel@@UBEPAVQMetaObject@@XZ 1000b87c     qt-mt323:qt-mt323.dll
 0002:00000880       __imp_?metaObject@QLineEdit@@UBEPAVQMetaObject@@XZ 1000b880     qt-mt323:qt-mt323.dll
 0002:00000884       __imp_?metaObject@QTabWidget@@UBEPAVQMetaObject@@XZ 1000b884     qt-mt323:qt-mt323.dll
 0002:00000888       __imp_?metaObject@QTable@@UBEPAVQMetaObject@@XZ 1000b888     qt-mt323:qt-mt323.dll
 0002:0000088c       __imp_?metaObject@QTextEdit@@UBEPAVQMetaObject@@XZ 1000b88c     qt-mt323:qt-mt323.dll
 0002:00000890       __imp_?metaObject@QVBoxLayout@@UBEPAVQMetaObject@@XZ 1000b890     qt-mt323:qt-mt323.dll
 0002:00000894       __imp_?minimumSize@QBoxLayout@@UBE?AVQSize@@XZ 1000b894     qt-mt323:qt-mt323.dll
 0002:00000898       __imp_?minimumSize@QSpacerItem@@UBE?AVQSize@@XZ 1000b898     qt-mt323:qt-mt323.dll
 0002:0000089c       __imp_?minimumSizeHint@QLabel@@UBE?AVQSize@@XZ 1000b89c     qt-mt323:qt-mt323.dll
 0002:000008a0       __imp_?minimumSizeHint@QLineEdit@@UBE?AVQSize@@XZ 1000b8a0     qt-mt323:qt-mt323.dll
 0002:000008a4       __imp_?minimumSizeHint@QScrollView@@UBE?AVQSize@@XZ 1000b8a4     qt-mt323:qt-mt323.dll
 0002:000008a8       __imp_?minimumSizeHint@QTabWidget@@UBE?AVQSize@@XZ 1000b8a8     qt-mt323:qt-mt323.dll
 0002:000008ac       __imp_?mouseDoubleClickEvent@QLineEdit@@MAEXPAVQMouseEvent@@@Z 1000b8ac     qt-mt323:qt-mt323.dll
 0002:000008b0       __imp_?mouseDoubleClickEvent@QScrollView@@MAEXPAVQMouseEvent@@@Z 1000b8b0     qt-mt323:qt-mt323.dll
 0002:000008b4       __imp_?mouseMoveEvent@QLineEdit@@MAEXPAVQMouseEvent@@@Z 1000b8b4     qt-mt323:qt-mt323.dll
 0002:000008b8       __imp_?mouseMoveEvent@QScrollView@@MAEXPAVQMouseEvent@@@Z 1000b8b8     qt-mt323:qt-mt323.dll
 0002:000008bc       __imp_?mousePressEvent@QLineEdit@@MAEXPAVQMouseEvent@@@Z 1000b8bc     qt-mt323:qt-mt323.dll
 0002:000008c0       __imp_?mousePressEvent@QScrollView@@MAEXPAVQMouseEvent@@@Z 1000b8c0     qt-mt323:qt-mt323.dll
 0002:000008c4       __imp_?mouseReleaseEvent@QLineEdit@@MAEXPAVQMouseEvent@@@Z 1000b8c4     qt-mt323:qt-mt323.dll
 0002:000008c8       __imp_?mouseReleaseEvent@QScrollView@@MAEXPAVQMouseEvent@@@Z 1000b8c8     qt-mt323:qt-mt323.dll
 0002:000008cc       __imp_?moveChild@QScrollView@@UAEXPAVQWidget@@HH@Z 1000b8cc     qt-mt323:qt-mt323.dll
 0002:000008d0       __imp_?moveCursor@QTextEdit@@UAEXW4CursorAction@1@_N@Z 1000b8d0     qt-mt323:qt-mt323.dll
 0002:000008d4       __imp_?numCols@QTable@@UBEHXZ 1000b8d4     qt-mt323:qt-mt323.dll
 0002:000008d8       __imp_?numRows@QTable@@UBEHXZ 1000b8d8     qt-mt323:qt-mt323.dll
 0002:000008dc       __imp_?paintCell@QTable@@UAEXPAVQPainter@@HHABVQRect@@_N@Z 1000b8dc     qt-mt323:qt-mt323.dll
 0002:000008e0       __imp_?paintCell@QTable@@UAEXPAVQPainter@@HHABVQRect@@_NABVQColorGroup@@@Z 1000b8e0     qt-mt323:qt-mt323.dll
 0002:000008e4       __imp_?paintEmptyArea@QTable@@MAEXPAVQPainter@@HHHH@Z 1000b8e4     qt-mt323:qt-mt323.dll
 0002:000008e8       __imp_?paintEvent@QTable@@MAEXPAVQPaintEvent@@@Z 1000b8e8     qt-mt323:qt-mt323.dll
 0002:000008ec       __imp_?paintFocus@QTable@@UAEXPAVQPainter@@ABVQRect@@@Z 1000b8ec     qt-mt323:qt-mt323.dll
 0002:000008f0       __imp_?paste@QLineEdit@@UAEXXZ 1000b8f0     qt-mt323:qt-mt323.dll
 0002:000008f4       __imp_?paste@QTextEdit@@UAEXXZ 1000b8f4     qt-mt323:qt-mt323.dll
 0002:000008f8       __imp_?pasteSubType@QTextEdit@@UAEXABVQCString@@@Z 1000b8f8     qt-mt323:qt-mt323.dll
 0002:000008fc       __imp_?pixmap@QTable@@UBE?AVQPixmap@@HH@Z 1000b8fc     qt-mt323:qt-mt323.dll
 0002:00000900       __imp_?placeCursor@QTextEdit@@UAEXABVQPoint@@PAVQTextCursor@@@Z 1000b900     qt-mt323:qt-mt323.dll
 0002:00000904       __imp_?polish@QTextEdit@@UAEXXZ 1000b904     qt-mt323:qt-mt323.dll
 0002:00000908       __imp_?qt_cast@QHBoxLayout@@UAEPAXPBD@Z 1000b908     qt-mt323:qt-mt323.dll
 0002:0000090c       __imp_?qt_cast@QLabel@@UAEPAXPBD@Z 1000b90c     qt-mt323:qt-mt323.dll
 0002:00000910       __imp_?qt_cast@QLineEdit@@UAEPAXPBD@Z 1000b910     qt-mt323:qt-mt323.dll
 0002:00000914       __imp_?qt_cast@QTabWidget@@UAEPAXPBD@Z 1000b914     qt-mt323:qt-mt323.dll
 0002:00000918       __imp_?qt_cast@QTable@@UAEPAXPBD@Z 1000b918     qt-mt323:qt-mt323.dll
 0002:0000091c       __imp_?qt_cast@QTextEdit@@UAEPAXPBD@Z 1000b91c     qt-mt323:qt-mt323.dll
 0002:00000920       __imp_?qt_cast@QVBoxLayout@@UAEPAXPBD@Z 1000b920     qt-mt323:qt-mt323.dll
 0002:00000924       __imp_?qt_emit@QHBoxLayout@@UAE_NHPAUQUObject@@@Z 1000b924     qt-mt323:qt-mt323.dll
 0002:00000928       __imp_?qt_emit@QLabel@@UAE_NHPAUQUObject@@@Z 1000b928     qt-mt323:qt-mt323.dll
 0002:0000092c       __imp_?qt_emit@QLineEdit@@UAE_NHPAUQUObject@@@Z 1000b92c     qt-mt323:qt-mt323.dll
 0002:00000930       __imp_?qt_emit@QTabWidget@@UAE_NHPAUQUObject@@@Z 1000b930     qt-mt323:qt-mt323.dll
 0002:00000934       __imp_?qt_emit@QTable@@UAE_NHPAUQUObject@@@Z 1000b934     qt-mt323:qt-mt323.dll
 0002:00000938       __imp_?qt_emit@QTextEdit@@UAE_NHPAUQUObject@@@Z 1000b938     qt-mt323:qt-mt323.dll
 0002:0000093c       __imp_?qt_emit@QVBoxLayout@@UAE_NHPAUQUObject@@@Z 1000b93c     qt-mt323:qt-mt323.dll
 0002:00000940       __imp_?qt_invoke@QHBoxLayout@@UAE_NHPAUQUObject@@@Z 1000b940     qt-mt323:qt-mt323.dll
 0002:00000944       __imp_?qt_invoke@QLabel@@UAE_NHPAUQUObject@@@Z 1000b944     qt-mt323:qt-mt323.dll
 0002:00000948       __imp_?qt_invoke@QLineEdit@@UAE_NHPAUQUObject@@@Z 1000b948     qt-mt323:qt-mt323.dll
 0002:0000094c       __imp_?qt_invoke@QTabWidget@@UAE_NHPAUQUObject@@@Z 1000b94c     qt-mt323:qt-mt323.dll
 0002:00000950       __imp_?qt_invoke@QTable@@UAE_NHPAUQUObject@@@Z 1000b950     qt-mt323:qt-mt323.dll
 0002:00000954       __imp_?qt_invoke@QTextEdit@@UAE_NHPAUQUObject@@@Z 1000b954     qt-mt323:qt-mt323.dll
 0002:00000958       __imp_?qt_invoke@QVBoxLayout@@UAE_NHPAUQUObject@@@Z 1000b958     qt-mt323:qt-mt323.dll
 0002:0000095c       __imp_?qt_property@QHBoxLayout@@UAE_NHHPAVQVariant@@@Z 1000b95c     qt-mt323:qt-mt323.dll
 0002:00000960       __imp_?qt_property@QLabel@@UAE_NHHPAVQVariant@@@Z 1000b960     qt-mt323:qt-mt323.dll
 0002:00000964       __imp_?qt_property@QLineEdit@@UAE_NHHPAVQVariant@@@Z 1000b964     qt-mt323:qt-mt323.dll
 0002:00000968       __imp_?qt_property@QTabWidget@@UAE_NHHPAVQVariant@@@Z 1000b968     qt-mt323:qt-mt323.dll
 0002:0000096c       __imp_?qt_property@QTable@@UAE_NHHPAVQVariant@@@Z 1000b96c     qt-mt323:qt-mt323.dll
 0002:00000970       __imp_?qt_property@QTextEdit@@UAE_NHHPAVQVariant@@@Z 1000b970     qt-mt323:qt-mt323.dll
 0002:00000974       __imp_?qt_property@QVBoxLayout@@UAE_NHHPAVQVariant@@@Z 1000b974     qt-mt323:qt-mt323.dll
 0002:00000978       __imp_?redo@QLineEdit@@UAEXXZ 1000b978     qt-mt323:qt-mt323.dll
 0002:0000097c       __imp_?redo@QTextEdit@@UAEXXZ 1000b97c     qt-mt323:qt-mt323.dll
 0002:00000980       __imp_?removeChild@QScrollView@@UAEXPAVQObject@@@Z 1000b980     qt-mt323:qt-mt323.dll
 0002:00000984       __imp_?removeColumn@QTable@@UAEXH@Z 1000b984     qt-mt323:qt-mt323.dll
 0002:00000988       __imp_?removeColumns@QTable@@UAEXABV?$QMemArray@H@@@Z 1000b988     qt-mt323:qt-mt323.dll
 0002:0000098c       __imp_?removePage@QTabWidget@@UAEXPAVQWidget@@@Z 1000b98c     qt-mt323:qt-mt323.dll
 0002:00000990       __imp_?removeParagraph@QTextEdit@@UAEXH@Z 1000b990     qt-mt323:qt-mt323.dll
 0002:00000994       __imp_?removeRow@QTable@@UAEXH@Z 1000b994     qt-mt323:qt-mt323.dll
 0002:00000998       __imp_?removeRows@QTable@@UAEXABV?$QMemArray@H@@@Z 1000b998     qt-mt323:qt-mt323.dll
 0002:0000099c       __imp_?removeSelectedText@QTextEdit@@UAEXH@Z 1000b99c     qt-mt323:qt-mt323.dll
 0002:000009a0       __imp_?removeSelection@QTable@@UAEXABVQTableSelection@@@Z 1000b9a0     qt-mt323:qt-mt323.dll
 0002:000009a4       __imp_?removeSelection@QTable@@UAEXH@Z 1000b9a4     qt-mt323:qt-mt323.dll
 0002:000009a8       __imp_?removeSelection@QTextEdit@@UAEXH@Z 1000b9a8     qt-mt323:qt-mt323.dll
 0002:000009ac       __imp_?resetFormat@QTextEdit@@UAEXXZ 1000b9ac     qt-mt323:qt-mt323.dll
 0002:000009b0       __imp_?resize@QScrollView@@UAEXHH@Z 1000b9b0     qt-mt323:qt-mt323.dll
 0002:000009b4       __imp_?resizeContents@QScrollView@@UAEXHH@Z 1000b9b4     qt-mt323:qt-mt323.dll
 0002:000009b8       __imp_?resizeData@QTable@@MAEXH@Z 1000b9b8     qt-mt323:qt-mt323.dll
 0002:000009bc       __imp_?resizeEvent@QLabel@@MAEXPAVQResizeEvent@@@Z 1000b9bc     qt-mt323:qt-mt323.dll
 0002:000009c0       __imp_?resizeEvent@QLineEdit@@MAEXPAVQResizeEvent@@@Z 1000b9c0     qt-mt323:qt-mt323.dll
 0002:000009c4       __imp_?resizeEvent@QScrollView@@MAEXPAVQResizeEvent@@@Z 1000b9c4     qt-mt323:qt-mt323.dll
 0002:000009c8       __imp_?resizeEvent@QTabWidget@@MAEXPAVQResizeEvent@@@Z 1000b9c8     qt-mt323:qt-mt323.dll
 0002:000009cc       __imp_?resizeEvent@QTextEdit@@MAEXPAVQResizeEvent@@@Z 1000b9cc     qt-mt323:qt-mt323.dll
 0002:000009d0       __imp_?rowAt@QTable@@UBEHH@Z 1000b9d0     qt-mt323:qt-mt323.dll
 0002:000009d4       __imp_?rowHeight@QTable@@UBEHH@Z 1000b9d4     qt-mt323:qt-mt323.dll
 0002:000009d8       __imp_?rowHeightChanged@QTable@@MAEXH@Z 1000b9d8     qt-mt323:qt-mt323.dll
 0002:000009dc       __imp_?rowIndexChanged@QTable@@MAEXHHH@Z 1000b9dc     qt-mt323:qt-mt323.dll
 0002:000009e0       __imp_?rowPos@QTable@@UBEHH@Z 1000b9e0     qt-mt323:qt-mt323.dll
 0002:000009e4       __imp_?scrollToAnchor@QTextEdit@@UAEXABVQString@@@Z 1000b9e4     qt-mt323:qt-mt323.dll
 0002:000009e8       __imp_?scrollToBottom@QTextEdit@@UAEXXZ 1000b9e8     qt-mt323:qt-mt323.dll
 0002:000009ec       __imp_?selectAll@QLineEdit@@UAEXXZ 1000b9ec     qt-mt323:qt-mt323.dll
 0002:000009f0       __imp_?selectAll@QTextEdit@@UAEX_N@Z 1000b9f0     qt-mt323:qt-mt323.dll
 0002:000009f4       __imp_?setAlignment@QLabel@@UAEXH@Z 1000b9f4     qt-mt323:qt-mt323.dll
 0002:000009f8       __imp_?setAlignment@QLayoutItem@@UAEXH@Z 1000b9f8     qt-mt323:qt-mt323.dll
 0002:000009fc       __imp_?setAlignment@QLineEdit@@UAEXH@Z 1000b9fc     qt-mt323:qt-mt323.dll
 0002:00000a00       __imp_?setAlignment@QTextEdit@@UAEXH@Z 1000ba00     qt-mt323:qt-mt323.dll
 0002:00000a04       __imp_?setAutoAdd@QLayout@@UAEX_N@Z 1000ba04     qt-mt323:qt-mt323.dll
 0002:00000a08       __imp_?setAutoResize@QLabel@@UAEX_N@Z 1000ba08     qt-mt323:qt-mt323.dll
 0002:00000a0c       __imp_?setBold@QTextEdit@@UAEX_N@Z 1000ba0c     qt-mt323:qt-mt323.dll
 0002:00000a10       __imp_?setBuddy@QLabel@@UAEXPAVQWidget@@@Z 1000ba10     qt-mt323:qt-mt323.dll
 0002:00000a14       __imp_?setCellContentFromEditor@QTable@@MAEXHH@Z 1000ba14     qt-mt323:qt-mt323.dll
 0002:00000a18       __imp_?setCellWidget@QTable@@UAEXHHPAVQWidget@@@Z 1000ba18     qt-mt323:qt-mt323.dll
 0002:00000a1c       __imp_?setColor@QTextEdit@@UAEXABVQColor@@@Z 1000ba1c     qt-mt323:qt-mt323.dll
 0002:00000a20       __imp_?setColumnMovingEnabled@QTable@@UAEX_N@Z 1000ba20     qt-mt323:qt-mt323.dll
 0002:00000a24       __imp_?setColumnReadOnly@QTable@@UAEXH_N@Z 1000ba24     qt-mt323:qt-mt323.dll
 0002:00000a28       __imp_?setColumnStretchable@QTable@@UAEXH_N@Z 1000ba28     qt-mt323:qt-mt323.dll
 0002:00000a2c       __imp_?setColumnWidth@QTable@@UAEXHH@Z 1000ba2c     qt-mt323:qt-mt323.dll
 0002:00000a30       __imp_?setContentsPos@QScrollView@@UAEXHH@Z 1000ba30     qt-mt323:qt-mt323.dll
 0002:00000a34       __imp_?setCornerWidget@QScrollView@@UAEXPAVQWidget@@@Z 1000ba34     qt-mt323:qt-mt323.dll
 0002:00000a38       __imp_?setCurrentCell@QTable@@UAEXHH@Z 1000ba38     qt-mt323:qt-mt323.dll
 0002:00000a3c       __imp_?setCurrentFont@QTextEdit@@UAEXABVQFont@@@Z 1000ba3c     qt-mt323:qt-mt323.dll
 0002:00000a40       __imp_?setCursorPosition@QLineEdit@@UAEXH@Z 1000ba40     qt-mt323:qt-mt323.dll
 0002:00000a44       __imp_?setCursorPosition@QTextEdit@@UAEXHH@Z 1000ba44     qt-mt323:qt-mt323.dll
 0002:00000a48       __imp_?setDragAutoScroll@QScrollView@@UAEX_N@Z 1000ba48     qt-mt323:qt-mt323.dll
 0002:00000a4c       __imp_?setDragEnabled@QLineEdit@@UAEX_N@Z 1000ba4c     qt-mt323:qt-mt323.dll
 0002:00000a50       __imp_?setDragEnabled@QTable@@UAEX_N@Z 1000ba50     qt-mt323:qt-mt323.dll
 0002:00000a54       __imp_?setEchoMode@QLineEdit@@UAEXW4EchoMode@1@@Z 1000ba54     qt-mt323:qt-mt323.dll
 0002:00000a58       __imp_?setEnabled@QTable@@UAEX_N@Z 1000ba58     qt-mt323:qt-mt323.dll
 0002:00000a5c       __imp_?setEnabled@QTextEdit@@UAEX_N@Z 1000ba5c     qt-mt323:qt-mt323.dll
 0002:00000a60       __imp_?setFamily@QTextEdit@@UAEXABVQString@@@Z 1000ba60     qt-mt323:qt-mt323.dll
 0002:00000a64       __imp_?setFocusStyle@QTable@@UAEXW4FocusStyle@1@@Z 1000ba64     qt-mt323:qt-mt323.dll
 0002:00000a68       __imp_?setFont@QLabel@@UAEXABVQFont@@@Z 1000ba68     qt-mt323:qt-mt323.dll
 0002:00000a6c       __imp_?setFont@QLineEdit@@UAEXABVQFont@@@Z 1000ba6c     qt-mt323:qt-mt323.dll
 0002:00000a70       __imp_?setFont@QTextEdit@@UAEXABVQFont@@@Z 1000ba70     qt-mt323:qt-mt323.dll
 0002:00000a74       __imp_?setFormat@QTextEdit@@UAEXPAVQTextFormat@@H@Z 1000ba74     qt-mt323:qt-mt323.dll
 0002:00000a78       __imp_?setFrame@QLineEdit@@UAEX_N@Z 1000ba78     qt-mt323:qt-mt323.dll
 0002:00000a7c       __imp_?setGeometry@QBoxLayout@@UAEXABVQRect@@@Z 1000ba7c     qt-mt323:qt-mt323.dll
 0002:00000a80       __imp_?setGeometry@QSpacerItem@@UAEXABVQRect@@@Z 1000ba80     qt-mt323:qt-mt323.dll
 0002:00000a84       __imp_?setHBarGeometry@QScrollView@@MAEXAAVQScrollBar@@HHHH@Z 1000ba84     qt-mt323:qt-mt323.dll
 0002:00000a88       __imp_?setHScrollBarMode@QScrollView@@UAEXW4ScrollBarMode@1@@Z 1000ba88     qt-mt323:qt-mt323.dll
 0002:00000a8c       __imp_?setItalic@QTextEdit@@UAEX_N@Z 1000ba8c     qt-mt323:qt-mt323.dll
 0002:00000a90       __imp_?setItem@QTable@@UAEXHHPAVQTableItem@@@Z 1000ba90     qt-mt323:qt-mt323.dll
 0002:00000a94       __imp_?setLeftMargin@QTable@@UAEXH@Z 1000ba94     qt-mt323:qt-mt323.dll
 0002:00000a98       __imp_?setLinkUnderline@QTextEdit@@UAEX_N@Z 1000ba98     qt-mt323:qt-mt323.dll
 0002:00000a9c       __imp_?setMargin@QLayout@@UAEXH@Z 1000ba9c     qt-mt323:qt-mt323.dll
 0002:00000aa0       __imp_?setMargins@QScrollView@@MAEXHHHH@Z 1000baa0     qt-mt323:qt-mt323.dll
 0002:00000aa4       __imp_?setMaxLength@QLineEdit@@UAEXH@Z 1000baa4     qt-mt323:qt-mt323.dll
 0002:00000aa8       __imp_?setMenuBar@QLayout@@UAEXPAVQMenuBar@@@Z 1000baa8     qt-mt323:qt-mt323.dll
 0002:00000aac       __imp_?setMimeSourceFactory@QTextEdit@@UAEXPAVQMimeSourceFactory@@@Z 1000baac     qt-mt323:qt-mt323.dll
 0002:00000ab0       __imp_?setModified@QTextEdit@@UAEX_N@Z 1000bab0     qt-mt323:qt-mt323.dll
 0002:00000ab4       __imp_?setMovie@QLabel@@UAEXABVQMovie@@@Z 1000bab4     qt-mt323:qt-mt323.dll
 0002:00000ab8       __imp_?setNum@QLabel@@UAEXH@Z 1000bab8     qt-mt323:qt-mt323.dll
 0002:00000abc       __imp_?setNum@QLabel@@UAEXN@Z 1000babc     qt-mt323:qt-mt323.dll
 0002:00000ac0       __imp_?setNumCols@QTable@@UAEXH@Z 1000bac0     qt-mt323:qt-mt323.dll
 0002:00000ac4       __imp_?setNumRows@QTable@@UAEXH@Z 1000bac4     qt-mt323:qt-mt323.dll
 0002:00000ac8       __imp_?setOverwriteMode@QTextEdit@@UAEX_N@Z 1000bac8     qt-mt323:qt-mt323.dll
 0002:00000acc       __imp_?setPalette@QLineEdit@@UAEXABVQPalette@@@Z 1000bacc     qt-mt323:qt-mt323.dll
 0002:00000ad0       __imp_?setPalette@QTextEdit@@UAEXABVQPalette@@@Z 1000bad0     qt-mt323:qt-mt323.dll
 0002:00000ad4       __imp_?setPaper@QTextEdit@@UAEXABVQBrush@@@Z 1000bad4     qt-mt323:qt-mt323.dll
 0002:00000ad8       __imp_?setParagType@QTextEdit@@UAEXW4DisplayMode@QStyleSheetItem@@W4ListStyle@3@@Z 1000bad8     qt-mt323:qt-mt323.dll
 0002:00000adc       __imp_?setParagraphBackgroundColor@QTextEdit@@UAEXHABVQColor@@@Z 1000badc     qt-mt323:qt-mt323.dll
 0002:00000ae0       __imp_?setPicture@QLabel@@UAEXABVQPicture@@@Z 1000bae0     qt-mt323:qt-mt323.dll
 0002:00000ae4       __imp_?setPixmap@QLabel@@UAEXABVQPixmap@@@Z 1000bae4     qt-mt323:qt-mt323.dll
 0002:00000ae8       __imp_?setPixmap@QTable@@UAEXHHABVQPixmap@@@Z 1000bae8     qt-mt323:qt-mt323.dll
 0002:00000aec       __imp_?setPointSize@QTextEdit@@UAEXH@Z 1000baec     qt-mt323:qt-mt323.dll
 0002:00000af0       __imp_?setReadOnly@QLineEdit@@UAEX_N@Z 1000baf0     qt-mt323:qt-mt323.dll
 0002:00000af4       __imp_?setReadOnly@QTable@@UAEX_N@Z 1000baf4     qt-mt323:qt-mt323.dll
 0002:00000af8       __imp_?setReadOnly@QTextEdit@@UAEX_N@Z 1000baf8     qt-mt323:qt-mt323.dll
 0002:00000afc       __imp_?setResizePolicy@QScrollView@@UAEXW4ResizePolicy@1@@Z 1000bafc     qt-mt323:qt-mt323.dll
 0002:00000b00       __imp_?setRowHeight@QTable@@UAEXHH@Z 1000bb00     qt-mt323:qt-mt323.dll
 0002:00000b04       __imp_?setRowMovingEnabled@QTable@@UAEX_N@Z 1000bb04     qt-mt323:qt-mt323.dll
 0002:00000b08       __imp_?setRowReadOnly@QTable@@UAEXH_N@Z 1000bb08     qt-mt323:qt-mt323.dll
 0002:00000b0c       __imp_?setRowStretchable@QTable@@UAEXH_N@Z 1000bb0c     qt-mt323:qt-mt323.dll
 0002:00000b10       __imp_?setSelection@QLineEdit@@UAEXHH@Z 1000bb10     qt-mt323:qt-mt323.dll
 0002:00000b14       __imp_?setSelection@QTextEdit@@UAEXHHHHH@Z 1000bb14     qt-mt323:qt-mt323.dll
 0002:00000b18       __imp_?setSelectionAttributes@QTextEdit@@UAEXHABVQColor@@_N@Z 1000bb18     qt-mt323:qt-mt323.dll
 0002:00000b1c       __imp_?setSelectionMode@QTable@@UAEXW4SelectionMode@1@@Z 1000bb1c     qt-mt323:qt-mt323.dll
 0002:00000b20       __imp_?setShowGrid@QTable@@UAEX_N@Z 1000bb20     qt-mt323:qt-mt323.dll
 0002:00000b24       __imp_?setSorting@QTable@@UAEX_N@Z 1000bb24     qt-mt323:qt-mt323.dll
 0002:00000b28       __imp_?setSpacing@QLayout@@UAEXH@Z 1000bb28     qt-mt323:qt-mt323.dll
 0002:00000b2c       __imp_?setStyleSheet@QTextEdit@@UAEXPAVQStyleSheet@@@Z 1000bb2c     qt-mt323:qt-mt323.dll
 0002:00000b30       __imp_?setTabStopWidth@QTextEdit@@UAEXH@Z 1000bb30     qt-mt323:qt-mt323.dll
 0002:00000b34       __imp_?setText@QLabel@@UAEXABVQString@@@Z 1000bb34     qt-mt323:qt-mt323.dll
 0002:00000b38       __imp_?setText@QLineEdit@@UAEXABVQString@@@Z 1000bb38     qt-mt323:qt-mt323.dll
 0002:00000b3c       __imp_?setText@QTable@@UAEXHHABVQString@@@Z 1000bb3c     qt-mt323:qt-mt323.dll
 0002:00000b40       __imp_?setText@QTextEdit@@UAEXABVQString@@0@Z 1000bb40     qt-mt323:qt-mt323.dll
 0002:00000b44       __imp_?setTextFormat@QTextEdit@@UAEXW4TextFormat@Qt@@@Z 1000bb44     qt-mt323:qt-mt323.dll
 0002:00000b48       __imp_?setTopMargin@QTable@@UAEXH@Z 1000bb48     qt-mt323:qt-mt323.dll
 0002:00000b4c       __imp_?setUnderline@QTextEdit@@UAEX_N@Z 1000bb4c     qt-mt323:qt-mt323.dll
 0002:00000b50       __imp_?setUndoDepth@QTextEdit@@UAEXH@Z 1000bb50     qt-mt323:qt-mt323.dll
 0002:00000b54       __imp_?setUndoRedoEnabled@QTextEdit@@UAEX_N@Z 1000bb54     qt-mt323:qt-mt323.dll
 0002:00000b58       __imp_?setVBarGeometry@QScrollView@@MAEXAAVQScrollBar@@HHHH@Z 1000bb58     qt-mt323:qt-mt323.dll
 0002:00000b5c       __imp_?setVScrollBarMode@QScrollView@@UAEXW4ScrollBarMode@1@@Z 1000bb5c     qt-mt323:qt-mt323.dll
 0002:00000b60       __imp_?setValidator@QLineEdit@@UAEXPBVQValidator@@@Z 1000bb60     qt-mt323:qt-mt323.dll
 0002:00000b64       __imp_?setVerticalAlignment@QTextEdit@@UAEXW4VerticalAlignment@1@@Z 1000bb64     qt-mt323:qt-mt323.dll
 0002:00000b68       __imp_?setWordWrap@QTextEdit@@UAEXW4WordWrap@1@@Z 1000bb68     qt-mt323:qt-mt323.dll
 0002:00000b6c       __imp_?setWrapColumnOrWidth@QTextEdit@@UAEXH@Z 1000bb6c     qt-mt323:qt-mt323.dll
 0002:00000b70       __imp_?setWrapPolicy@QTextEdit@@UAEXW4WrapPolicy@1@@Z 1000bb70     qt-mt323:qt-mt323.dll
 0002:00000b74       __imp_?show@QScrollView@@UAEXXZ 1000bb74     qt-mt323:qt-mt323.dll
 0002:00000b78       __imp_?showColumn@QTable@@UAEXH@Z 1000bb78     qt-mt323:qt-mt323.dll
 0002:00000b7c       __imp_?showEvent@QTabWidget@@MAEXPAVQShowEvent@@@Z 1000bb7c     qt-mt323:qt-mt323.dll
 0002:00000b80       __imp_?showEvent@QTable@@MAEXPAVQShowEvent@@@Z 1000bb80     qt-mt323:qt-mt323.dll
 0002:00000b84       __imp_?showPage@QTabWidget@@UAEXPAVQWidget@@@Z 1000bb84     qt-mt323:qt-mt323.dll
 0002:00000b88       __imp_?showRow@QTable@@UAEXH@Z 1000bb88     qt-mt323:qt-mt323.dll
 0002:00000b8c       __imp_?sizeHint@QBoxLayout@@UBE?AVQSize@@XZ 1000bb8c     qt-mt323:qt-mt323.dll
 0002:00000b90       __imp_?sizeHint@QLabel@@UBE?AVQSize@@XZ 1000bb90     qt-mt323:qt-mt323.dll
 0002:00000b94       __imp_?sizeHint@QLineEdit@@UBE?AVQSize@@XZ 1000bb94     qt-mt323:qt-mt323.dll
 0002:00000b98       __imp_?sizeHint@QSpacerItem@@UBE?AVQSize@@XZ 1000bb98     qt-mt323:qt-mt323.dll
 0002:00000b9c       __imp_?sizeHint@QTabWidget@@UBE?AVQSize@@XZ 1000bb9c     qt-mt323:qt-mt323.dll
 0002:00000ba0       __imp_?sizeHint@QTable@@UBE?AVQSize@@XZ 1000bba0     qt-mt323:qt-mt323.dll
 0002:00000ba4       __imp_?sizeHint@QTextEdit@@UBE?AVQSize@@XZ 1000bba4     qt-mt323:qt-mt323.dll
 0002:00000ba8       __imp_?sortColumn@QTable@@UAEXH_N0@Z 1000bba8     qt-mt323:qt-mt323.dll
 0002:00000bac       __imp_?spacerItem@QLayoutItem@@UAEPAVQSpacerItem@@XZ 1000bbac     qt-mt323:qt-mt323.dll
 0002:00000bb0       __imp_?spacerItem@QSpacerItem@@UAEPAV1@XZ 1000bbb0     qt-mt323:qt-mt323.dll
 0002:00000bb4       __imp_?startDrag@QTable@@MAEXXZ 1000bbb4     qt-mt323:qt-mt323.dll
 0002:00000bb8       __imp_?styleChange@QScrollView@@UAEXAAVQStyle@@@Z 1000bbb8     qt-mt323:qt-mt323.dll
 0002:00000bbc       __imp_?styleChange@QTabWidget@@MAEXAAVQStyle@@@Z 1000bbbc     qt-mt323:qt-mt323.dll
 0002:00000bc0       __imp_?swapCells@QTable@@UAEXHHHH@Z 1000bbc0     qt-mt323:qt-mt323.dll
 0002:00000bc4       __imp_?swapColumns@QTable@@UAEXHH_N@Z 1000bbc4     qt-mt323:qt-mt323.dll
 0002:00000bc8       __imp_?swapRows@QTable@@UAEXHH_N@Z 1000bbc8     qt-mt323:qt-mt323.dll
 0002:00000bcc       __imp_?sync@QTextEdit@@UAEXXZ 1000bbcc     qt-mt323:qt-mt323.dll
 0002:00000bd0       __imp_?takeItem@QTable@@UAEXPAVQTableItem@@@Z 1000bbd0     qt-mt323:qt-mt323.dll
 0002:00000bd4       __imp_?text@QTable@@UBE?AVQString@@HH@Z 1000bbd4     qt-mt323:qt-mt323.dll
 0002:00000bd8       __imp_?undo@QLineEdit@@UAEXXZ 1000bbd8     qt-mt323:qt-mt323.dll
 0002:00000bdc       __imp_?undo@QTextEdit@@UAEXXZ 1000bbdc     qt-mt323:qt-mt323.dll
 0002:00000be0       __imp_?updateMask@QTabWidget@@MAEXXZ 1000bbe0     qt-mt323:qt-mt323.dll
 0002:00000be4       __imp_?viewportContextMenuEvent@QScrollView@@MAEXPAVQContextMenuEvent@@@Z 1000bbe4     qt-mt323:qt-mt323.dll
 0002:00000be8       __imp_?viewportDragEnterEvent@QScrollView@@MAEXPAVQDragEnterEvent@@@Z 1000bbe8     qt-mt323:qt-mt323.dll
 0002:00000bec       __imp_?viewportDragLeaveEvent@QScrollView@@MAEXPAVQDragLeaveEvent@@@Z 1000bbec     qt-mt323:qt-mt323.dll
 0002:00000bf0       __imp_?viewportDragMoveEvent@QScrollView@@MAEXPAVQDragMoveEvent@@@Z 1000bbf0     qt-mt323:qt-mt323.dll
 0002:00000bf4       __imp_?viewportDropEvent@QScrollView@@MAEXPAVQDropEvent@@@Z 1000bbf4     qt-mt323:qt-mt323.dll
 0002:00000bf8       __imp_?viewportMouseDoubleClickEvent@QScrollView@@MAEXPAVQMouseEvent@@@Z 1000bbf8     qt-mt323:qt-mt323.dll
 0002:00000bfc       __imp_?viewportMouseMoveEvent@QScrollView@@MAEXPAVQMouseEvent@@@Z 1000bbfc     qt-mt323:qt-mt323.dll
 0002:00000c00       __imp_?viewportMousePressEvent@QScrollView@@MAEXPAVQMouseEvent@@@Z 1000bc00     qt-mt323:qt-mt323.dll
 0002:00000c04       __imp_?viewportMouseReleaseEvent@QScrollView@@MAEXPAVQMouseEvent@@@Z 1000bc04     qt-mt323:qt-mt323.dll
 0002:00000c08       __imp_?viewportPaintEvent@QScrollView@@MAEXPAVQPaintEvent@@@Z 1000bc08     qt-mt323:qt-mt323.dll
 0002:00000c0c       __imp_?viewportResizeEvent@QTable@@MAEXPAVQResizeEvent@@@Z 1000bc0c     qt-mt323:qt-mt323.dll
 0002:00000c10       __imp_?viewportResizeEvent@QTextEdit@@MAEXPAVQResizeEvent@@@Z 1000bc10     qt-mt323:qt-mt323.dll
 0002:00000c14       __imp_?viewportWheelEvent@QScrollView@@MAEXPAVQWheelEvent@@@Z 1000bc14     qt-mt323:qt-mt323.dll
 0002:00000c18       __imp_?wheelEvent@QScrollView@@MAEXPAVQWheelEvent@@@Z 1000bc18     qt-mt323:qt-mt323.dll
 0002:00000c1c       __imp_?widget@QLayoutItem@@UAEPAVQWidget@@XZ 1000bc1c     qt-mt323:qt-mt323.dll
 0002:00000c20       __imp_?windowActivationChange@QLineEdit@@MAEX_N@Z 1000bc20     qt-mt323:qt-mt323.dll
 0002:00000c24       __imp_?windowActivationChange@QTable@@MAEX_N@Z 1000bc24     qt-mt323:qt-mt323.dll
 0002:00000c28       __imp_?windowActivationChange@QTextEdit@@MAEX_N@Z 1000bc28     qt-mt323:qt-mt323.dll
 0002:00000c2c       __imp_?zoomIn@QTextEdit@@UAEXH@Z 1000bc2c     qt-mt323:qt-mt323.dll
 0002:00000c30       __imp_?zoomIn@QTextEdit@@UAEXXZ 1000bc30     qt-mt323:qt-mt323.dll
 0002:00000c34       __imp_?zoomOut@QTextEdit@@UAEXH@Z 1000bc34     qt-mt323:qt-mt323.dll
 0002:00000c38       __imp_?zoomOut@QTextEdit@@UAEXXZ 1000bc38     qt-mt323:qt-mt323.dll
 0002:00000c3c       __imp_?zoomTo@QTextEdit@@UAEXH@Z 1000bc3c     qt-mt323:qt-mt323.dll
 0002:00000c40       __imp_?qstrcmp@@YAHPBD0@Z  1000bc40     qt-mt323:qt-mt323.dll
 0002:00000c44       __imp_?fromLatin1@QString@@SA?AV1@PBDH@Z 1000bc44     qt-mt323:qt-mt323.dll
 0002:00000c48       __imp_?receivers@QObject@@IBEPAVQConnectionList@@H@Z 1000bc48     qt-mt323:qt-mt323.dll
 0002:00000c4c       __imp_?activate_signal@QObject@@IAEXPAVQConnectionList@@PAUQUObject@@@Z 1000bc4c     qt-mt323:qt-mt323.dll
 0002:00000c50       __imp_?staticMetaObject@QWidget@@SAPAVQMetaObject@@XZ 1000bc50     qt-mt323:qt-mt323.dll
 0002:00000c54       __imp_?new_metaobject@QMetaObject@@SAPAV1@PBDPAV1@QBUQMetaData@@H2HQBVQMetaProperty@@HQBUQMetaEnum@@HQBUQClassInfo@@H@Z 1000bc54     qt-mt323:qt-mt323.dll
 0002:00000c58       __imp_??0QMetaObjectCleanUp@@QAE@PBDP6APAVQMetaObject@@XZ@Z 1000bc58     qt-mt323:qt-mt323.dll
 0002:00000c5c       __imp_??1QMetaObjectCleanUp@@QAE@XZ 1000bc5c     qt-mt323:qt-mt323.dll
 0002:00000c60       __imp_?setMetaObject@QMetaObjectCleanUp@@QAEXAAPAVQMetaObject@@@Z 1000bc60     qt-mt323:qt-mt323.dll
 0002:00000c64       __imp_?translate@QApplication@@QBE?AVQString@@PBD00W4Encoding@1@@Z 1000bc64     qt-mt323:qt-mt323.dll
 0002:00000c68       __imp_??0QUObject@@QAE@XZ  1000bc68     qt-mt323:qt-mt323.dll
 0002:00000c6c       __imp_??1QUObject@@QAE@XZ  1000bc6c     qt-mt323:qt-mt323.dll
 0002:00000c70       __imp_?set@QUType_QString@@QAEXPAUQUObject@@ABVQString@@@Z 1000bc70     qt-mt323:qt-mt323.dll
 0002:00000c74       __imp_?qApp@@3PAVQApplication@@A 1000bc74     qt-mt323:qt-mt323.dll
 0002:00000c78       __imp_?static_QUType_QString@@3UQUType_QString@@A 1000bc78     qt-mt323:qt-mt323.dll
 0002:00000c7c       __imp_?static_QUType_int@@3UQUType_int@@A 1000bc7c     qt-mt323:qt-mt323.dll
 0002:00000c80       __imp_?activate_signal@QObject@@IAEXHVQString@@@Z 1000bc80     qt-mt323:qt-mt323.dll
 0002:00000c84       __imp_?static_QUType_ptr@@3UQUType_ptr@@A 1000bc84     qt-mt323:qt-mt323.dll
 0002:00000c88       __imp_??0QListView@@QAE@PAVQWidget@@PBDI@Z 1000bc88     qt-mt323:qt-mt323.dll
 0002:00000c8c       __imp_??1QListView@@UAE@XZ 1000bc8c     qt-mt323:qt-mt323.dll
 0002:00000c90       __imp_?header@QListView@@QBEPAVQHeader@@XZ 1000bc90     qt-mt323:qt-mt323.dll
 0002:00000c94       __imp_?addColumn@QListView@@UAEHABVQIconSet@@ABVQString@@H@Z 1000bc94     qt-mt323:qt-mt323.dll
 0002:00000c98       __imp_?addColumn@QListView@@UAEHABVQString@@H@Z 1000bc98     qt-mt323:qt-mt323.dll
 0002:00000c9c       __imp_?className@QListView@@UBEPBDXZ 1000bc9c     qt-mt323:qt-mt323.dll
 0002:00000ca0       __imp_?clear@QListView@@UAEXXZ 1000bca0     qt-mt323:qt-mt323.dll
 0002:00000ca4       __imp_?clearSelection@QListView@@UAEXXZ 1000bca4     qt-mt323:qt-mt323.dll
 0002:00000ca8       __imp_?contentsContextMenuEvent@QListView@@MAEXPAVQContextMenuEvent@@@Z 1000bca8     qt-mt323:qt-mt323.dll
 0002:00000cac       __imp_?contentsDragEnterEvent@QListView@@MAEXPAVQDragEnterEvent@@@Z 1000bcac     qt-mt323:qt-mt323.dll
 0002:00000cb0       __imp_?contentsDragLeaveEvent@QListView@@MAEXPAVQDragLeaveEvent@@@Z 1000bcb0     qt-mt323:qt-mt323.dll
 0002:00000cb4       __imp_?contentsDragMoveEvent@QListView@@MAEXPAVQDragMoveEvent@@@Z 1000bcb4     qt-mt323:qt-mt323.dll
 0002:00000cb8       __imp_?contentsDropEvent@QListView@@MAEXPAVQDropEvent@@@Z 1000bcb8     qt-mt323:qt-mt323.dll
 0002:00000cbc       __imp_?contentsMouseDoubleClickEvent@QListView@@MAEXPAVQMouseEvent@@@Z 1000bcbc     qt-mt323:qt-mt323.dll
 0002:00000cc0       __imp_?contentsMouseMoveEvent@QListView@@MAEXPAVQMouseEvent@@@Z 1000bcc0     qt-mt323:qt-mt323.dll
 0002:00000cc4       __imp_?contentsMousePressEvent@QListView@@MAEXPAVQMouseEvent@@@Z 1000bcc4     qt-mt323:qt-mt323.dll
 0002:00000cc8       __imp_?contentsMouseReleaseEvent@QListView@@MAEXPAVQMouseEvent@@@Z 1000bcc8     qt-mt323:qt-mt323.dll
 0002:00000ccc       __imp_?dragObject@QListView@@MAEPAVQDragObject@@XZ 1000bccc     qt-mt323:qt-mt323.dll
 0002:00000cd0       __imp_?drawContents@QScrollView@@EAEXPAVQPainter@@@Z 1000bcd0     qt-mt323:qt-mt323.dll
 0002:00000cd4       __imp_?drawContents@QScrollView@@MAEXPAVQPainter@@HHHH@Z 1000bcd4     qt-mt323:qt-mt323.dll
 0002:00000cd8       __imp_?drawContentsOffset@QListView@@MAEXPAVQPainter@@HHHHHH@Z 1000bcd8     qt-mt323:qt-mt323.dll
 0002:00000cdc       __imp_?eventFilter@QListView@@UAE_NPAVQObject@@PAVQEvent@@@Z 1000bcdc     qt-mt323:qt-mt323.dll
 0002:00000ce0       __imp_?focusInEvent@QListView@@MAEXPAVQFocusEvent@@@Z 1000bce0     qt-mt323:qt-mt323.dll
 0002:00000ce4       __imp_?focusOutEvent@QListView@@MAEXPAVQFocusEvent@@@Z 1000bce4     qt-mt323:qt-mt323.dll
 0002:00000ce8       __imp_?insertItem@QListView@@UAEXPAVQListViewItem@@@Z 1000bce8     qt-mt323:qt-mt323.dll
 0002:00000cec       __imp_?invertSelection@QListView@@UAEXXZ 1000bcec     qt-mt323:qt-mt323.dll
 0002:00000cf0       __imp_?keyPressEvent@QListView@@MAEXPAVQKeyEvent@@@Z 1000bcf0     qt-mt323:qt-mt323.dll
 0002:00000cf4       __imp_?metaObject@QListView@@UBEPAVQMetaObject@@XZ 1000bcf4     qt-mt323:qt-mt323.dll
 0002:00000cf8       __imp_?minimumSizeHint@QListView@@UBE?AVQSize@@XZ 1000bcf8     qt-mt323:qt-mt323.dll
 0002:00000cfc       __imp_?paintEmptyArea@QListView@@MAEXPAVQPainter@@ABVQRect@@@Z 1000bcfc     qt-mt323:qt-mt323.dll
 0002:00000d00       __imp_?qt_cast@QListView@@UAEPAXPBD@Z 1000bd00     qt-mt323:qt-mt323.dll
 0002:00000d04       __imp_?qt_emit@QListView@@UAE_NHPAUQUObject@@@Z 1000bd04     qt-mt323:qt-mt323.dll
 0002:00000d08       __imp_?qt_invoke@QListView@@UAE_NHPAUQUObject@@@Z 1000bd08     qt-mt323:qt-mt323.dll
 0002:00000d0c       __imp_?qt_property@QListView@@UAE_NHHPAVQVariant@@@Z 1000bd0c     qt-mt323:qt-mt323.dll
 0002:00000d10       __imp_?removeColumn@QListView@@UAEXH@Z 1000bd10     qt-mt323:qt-mt323.dll
 0002:00000d14       __imp_?removeItem@QListView@@UAEXPAVQListViewItem@@@Z 1000bd14     qt-mt323:qt-mt323.dll
 0002:00000d18       __imp_?resizeEvent@QListView@@MAEXPAVQResizeEvent@@@Z 1000bd18     qt-mt323:qt-mt323.dll
 0002:00000d1c       __imp_?selectAll@QListView@@UAEX_N@Z 1000bd1c     qt-mt323:qt-mt323.dll
 0002:00000d20       __imp_?setAllColumnsShowFocus@QListView@@UAEX_N@Z 1000bd20     qt-mt323:qt-mt323.dll
 0002:00000d24       __imp_?setColumnAlignment@QListView@@UAEXHH@Z 1000bd24     qt-mt323:qt-mt323.dll
 0002:00000d28       __imp_?setColumnText@QListView@@UAEXHABVQIconSet@@ABVQString@@@Z 1000bd28     qt-mt323:qt-mt323.dll
 0002:00000d2c       __imp_?setColumnText@QListView@@UAEXHABVQString@@@Z 1000bd2c     qt-mt323:qt-mt323.dll
 0002:00000d30       __imp_?setColumnWidth@QListView@@UAEXHH@Z 1000bd30     qt-mt323:qt-mt323.dll
 0002:00000d34       __imp_?setColumnWidthMode@QListView@@UAEXHW4WidthMode@1@@Z 1000bd34     qt-mt323:qt-mt323.dll
 0002:00000d38       __imp_?setContentsPos@QListView@@UAEXHH@Z 1000bd38     qt-mt323:qt-mt323.dll
 0002:00000d3c       __imp_?setCurrentItem@QListView@@UAEXPAVQListViewItem@@@Z 1000bd3c     qt-mt323:qt-mt323.dll
 0002:00000d40       __imp_?setDefaultRenameAction@QListView@@UAEXW4RenameAction@1@@Z 1000bd40     qt-mt323:qt-mt323.dll
 0002:00000d44       __imp_?setEnabled@QScrollView@@UAEX_N@Z 1000bd44     qt-mt323:qt-mt323.dll
 0002:00000d48       __imp_?setFont@QListView@@UAEXABVQFont@@@Z 1000bd48     qt-mt323:qt-mt323.dll
 0002:00000d4c       __imp_?setItemMargin@QListView@@UAEXH@Z 1000bd4c     qt-mt323:qt-mt323.dll
 0002:00000d50       __imp_?setMultiSelection@QListView@@UAEX_N@Z 1000bd50     qt-mt323:qt-mt323.dll
 0002:00000d54       __imp_?setOpen@QListView@@UAEXPAVQListViewItem@@_N@Z 1000bd54     qt-mt323:qt-mt323.dll
 0002:00000d58       __imp_?setPalette@QListView@@UAEXABVQPalette@@@Z 1000bd58     qt-mt323:qt-mt323.dll
 0002:00000d5c       __imp_?setResizeMode@QListView@@UAEXW4ResizeMode@1@@Z 1000bd5c     qt-mt323:qt-mt323.dll
 0002:00000d60       __imp_?setRootIsDecorated@QListView@@UAEX_N@Z 1000bd60     qt-mt323:qt-mt323.dll
 0002:00000d64       __imp_?setSelected@QListView@@UAEXPAVQListViewItem@@_N@Z 1000bd64     qt-mt323:qt-mt323.dll
 0002:00000d68       __imp_?setShowSortIndicator@QListView@@UAEX_N@Z 1000bd68     qt-mt323:qt-mt323.dll
 0002:00000d6c       __imp_?setShowToolTips@QListView@@UAEX_N@Z 1000bd6c     qt-mt323:qt-mt323.dll
 0002:00000d70       __imp_?setSorting@QListView@@UAEXH_N@Z 1000bd70     qt-mt323:qt-mt323.dll
 0002:00000d74       __imp_?setTreeStepSize@QListView@@UAEXH@Z 1000bd74     qt-mt323:qt-mt323.dll
 0002:00000d78       __imp_?show@QListView@@UAEXXZ 1000bd78     qt-mt323:qt-mt323.dll
 0002:00000d7c       __imp_?showEvent@QListView@@MAEXPAVQShowEvent@@@Z 1000bd7c     qt-mt323:qt-mt323.dll
 0002:00000d80       __imp_?sizeHint@QListView@@UBE?AVQSize@@XZ 1000bd80     qt-mt323:qt-mt323.dll
 0002:00000d84       __imp_?sort@QListView@@UAEXXZ 1000bd84     qt-mt323:qt-mt323.dll
 0002:00000d88       __imp_?startDrag@QListView@@MAEXXZ 1000bd88     qt-mt323:qt-mt323.dll
 0002:00000d8c       __imp_?styleChange@QListView@@MAEXAAVQStyle@@@Z 1000bd8c     qt-mt323:qt-mt323.dll
 0002:00000d90       __imp_?takeItem@QListView@@UAEXPAVQListViewItem@@@Z 1000bd90     qt-mt323:qt-mt323.dll
 0002:00000d94       __imp_?viewportResizeEvent@QListView@@MAEXPAVQResizeEvent@@@Z 1000bd94     qt-mt323:qt-mt323.dll
 0002:00000d98       __imp_?windowActivationChange@QListView@@MAEX_N@Z 1000bd98     qt-mt323:qt-mt323.dll
 0002:00000d9c       __imp_??0QRegExp@@QAE@ABVQString@@_N1@Z 1000bd9c     qt-mt323:qt-mt323.dll
 0002:00000da0       __imp_??1QIconSet@@UAE@XZ  1000bda0     qt-mt323:qt-mt323.dll
 0002:00000da4       __imp_??0QIconSet@@QAE@ABVQPixmap@@W4Size@0@@Z 1000bda4     qt-mt323:qt-mt323.dll
 0002:00000da8       __imp_??1QPixmap@@UAE@XZ   1000bda8     qt-mt323:qt-mt323.dll
 0002:00000dac       __imp_??0QPixmap@@QAE@QAPBD@Z 1000bdac     qt-mt323:qt-mt323.dll
 0002:00000db0       __imp_??0QKeySequence@@QAE@H@Z 1000bdb0     qt-mt323:qt-mt323.dll
 0002:00000db4       __imp_?information@QMessageBox@@SAHPAVQWidget@@ABVQString@@1111HH@Z 1000bdb4     qt-mt323:qt-mt323.dll
 0002:00000db8       __imp_?closeEvent@QWidget@@MAEXPAVQCloseEvent@@@Z 1000bdb8     qt-mt323:qt-mt323.dll
 0002:00000dbc       __imp_?rect@QWidget@@QBE?AVQRect@@XZ 1000bdbc     qt-mt323:qt-mt323.dll
 0002:00000dc0       __imp_?setName@QWidget@@UAEXPBD@Z 1000bdc0     qt-mt323:qt-mt323.dll
 0002:00000dc4       __imp_??1QWidget@@UAE@XZ   1000bdc4     qt-mt323:qt-mt323.dll
 0002:00000dc8       __imp_??0QWidget@@QAE@PAV0@PBDI@Z 1000bdc8     qt-mt323:qt-mt323.dll
 0002:00000dcc       __imp_?connect@QObject@@SA_NPBV1@PBD01@Z 1000bdcc     qt-mt323:qt-mt323.dll
 0002:00000dd0       __imp_?clear@QGList@@MAEXXZ 1000bdd0     qt-mt323:qt-mt323.dll
 0002:00000dd4       __imp_?append@QGList@@IAEXPAX@Z 1000bdd4     qt-mt323:qt-mt323.dll
 0002:00000dd8       __imp_??1QGList@@MAE@XZ    1000bdd8     qt-mt323:qt-mt323.dll
 0002:00000ddc       __imp_??0QGList@@IAE@XZ    1000bddc     qt-mt323:qt-mt323.dll
 0002:00000de0       __imp_??H@YA?BVQString@@PBDABV0@@Z 1000bde0     qt-mt323:qt-mt323.dll
 0002:00000de4       __imp_??H@YA?BVQString@@ABV0@PBD@Z 1000bde4     qt-mt323:qt-mt323.dll
 0002:00000de8       __imp_??H@YA?BVQString@@ABV0@0@Z 1000bde8     qt-mt323:qt-mt323.dll
 0002:00000dec       __imp_??8@YA_NABVQString@@PBD@Z 1000bdec     qt-mt323:qt-mt323.dll
 0002:00000df0       __imp_?ascii@QString@@QBEPBDXZ 1000bdf0     qt-mt323:qt-mt323.dll
 0002:00000df4       __imp_?remove@QString@@QAEAAV1@II@Z 1000bdf4     qt-mt323:qt-mt323.dll
 0002:00000df8       __imp_?lower@QString@@QBE?AV1@XZ 1000bdf8     qt-mt323:qt-mt323.dll
 0002:00000dfc       __imp_?left@QString@@QBE?AV1@I@Z 1000bdfc     qt-mt323:qt-mt323.dll
 0002:00000e00       __imp_?find@QString@@QBEHABVQRegExp@@H@Z 1000be00     qt-mt323:qt-mt323.dll
 0002:00000e04       __imp_?sprintf@QString@@QAAAAV1@PBDZZ 1000be04     qt-mt323:qt-mt323.dll
 0002:00000e08       __imp_?arg@QString@@QBE?AV1@ABV1@H@Z 1000be08     qt-mt323:qt-mt323.dll
 0002:00000e0c       __imp_??4QString@@QAEAAV0@ABV0@@Z 1000be0c     qt-mt323:qt-mt323.dll
 0002:00000e10       __imp_??1QString@@QAE@XZ   1000be10     qt-mt323:qt-mt323.dll
 0002:00000e14       __imp_??0QString@@QAE@PBD@Z 1000be14     qt-mt323:qt-mt323.dll
 0002:00000e18       __imp_??0QString@@QAE@ABV0@@Z 1000be18     qt-mt323:qt-mt323.dll
 0002:00000e1c       __imp_??0QString@@QAE@XZ   1000be1c     qt-mt323:qt-mt323.dll
 0002:00000e20       __imp_?qDebug@@YAXPBDZZ    1000be20     qt-mt323:qt-mt323.dll
 0002:00000e24       __imp_?createPopupMenu@QTextEdit@@MAEPAVQPopupMenu@@ABVQPoint@@@Z 1000be24     qt-mt323:qt-mt323.dll
 0002:00000e28       \177qt-mt323_NULL_THUNK_DATA 1000be28     qt-mt323:qt-mt323.dll
 0002:00000e2c       ___xc_a                    1000be2c     MSVCRT:cinitexe.obj
 0002:00000e44       ___xc_z                    1000be44     MSVCRT:cinitexe.obj
 0002:00000e48       ___xi_a                    1000be48     MSVCRT:cinitexe.obj
 0002:00000e54       ___xi_z                    1000be54     MSVCRT:cinitexe.obj
 0002:00000e58       ??_C@_02GIPFHKNO@OK?$AA@   1000be58     databaseEdit.obj
 0002:00000e64       ??_SQListViewItem@@6B@     1000be64     databaseEdit.obj
 0002:00000f04       ??_SQAction@@6B@           1000bf04     databaseEdit.obj
 0002:00000f94       ??_SQDockWindow@@6BQObject@@@ 1000bf94     databaseEdit.obj
 0002:000011a4       ??_SQDockWindow@@6BQPaintDevice@@@ 1000c1a4     databaseEdit.obj
 0002:000011cc       ??_SQToolBar@@6BQObject@@@ 1000c1cc     databaseEdit.obj
 0002:000013e8       ??_SQToolBar@@6BQPaintDevice@@@ 1000c3e8     databaseEdit.obj
 0002:0000140c       ??_SQGuardedPtrPrivate@@6B@ 1000c40c     databaseEdit.obj
 0002:00001460       ??_7QDockWindowList@@6B@   1000c460     databaseEdit.obj
 0002:00001484       ??_SQPopupMenu@@6BQObject@@@ 1000c484     databaseEdit.obj
 0002:00001664       ??_SQPopupMenu@@6BQPaintDevice@@@ 1000c664     databaseEdit.obj
 0002:00001688       ??_SQPopupMenu@@6B@        1000c688     databaseEdit.obj
 0002:000016ac       ??_7?$QPtrList@VQPopupMenu@@@@6B@ 1000c6ac     databaseEdit.obj
 0002:000016d0       ??_7QPopupMenuList@@6B@    1000c6d0     databaseEdit.obj
 0002:000016f0       ??_C@_04OOEBCMBF@FAIL?$AA@ 1000c6f0     databaseEdit.obj
 0002:000016f8       ??_C@_08OBALAKLA@READONLY?$AA@ 1000c6f8     databaseEdit.obj
 0002:00001704       ??_C@_04KANDKFIK@DONE?$AA@ 1000c704     databaseEdit.obj
 0002:0000170c       ??_C@_07NFANNNEC@UNKNOWN?$AA@ 1000c70c     databaseEdit.obj
 0002:00001718       ??_7config_plugin_base@@6BQObject@@@ 1000c718     databaseEdit.obj
 0002:000018f0       ??_7config_plugin_base@@6BQPaintDevice@@@ 1000c8f0     databaseEdit.obj
 0002:00001910       ??_C@_0EB@GNDACMDJ@?$CC?5?9?5the?5author?5should?5have?5defin@ 1000c910     databaseEdit.obj
 0002:00001954       ??_C@_0CH@BDPDPLDP@This?5is?5the?5default?5?$CCAbout?$CC?5text@ 1000c954     databaseEdit.obj
 0002:00001980       ??_7?$QDict@VQAction@@@@6B@ 1000c980     databaseEdit.obj
 0002:000019a0       ??_7databaseEdit@@6BQObject@@@ 1000c9a0     databaseEdit.obj
 0002:00001b78       ??_7databaseEdit@@6BQPaintDevice@@@ 1000cb78     databaseEdit.obj
 0002:00001b98       ??_C@_0P@BGOPOEEL@databaseEdit?3?5?$AA@ 1000cb98     databaseEdit.obj
 0002:00001ba8       ??_C@_0BN@CEGLABJP@2command?$CI?5QString?0?5QString?5?$CJ?$AA@ 1000cba8     databaseEdit.obj
 0002:00001bc8       ??_C@_0BO@DCHMNGHO@?1Template?5Plugin?5Tools?5Window?$AA@ 1000cbc8     databaseEdit.obj
 0002:00001be8       ??_C@_0N@CDOLEPFK@Tools?5Window?$AA@ 1000cbe8     databaseEdit.obj
 0002:00001bf8       ??_C@_0CA@EDGOBGJD@1fileSelected?$CI?5const?5QString?5?$CG?$CJ?$AA@ 1000cbf8     databaseEdit.obj
 0002:00001c18       ??_C@_0CB@HJMFLJJJ@2fileSelected?$CI?5const?5QString?5?$CG?5?$CJ@ 1000cc18     databaseEdit.obj
 0002:00001c3c       ??_C@_0BI@DJGPDCG@Template?5Plugin?5Toolbar?$AA@ 1000cc3c     databaseEdit.obj
 0002:00001c54       ??_C@_05LHMKEDEH@?$CGEdit?$AA@ 1000cc54     databaseEdit.obj
 0002:00001c5c       ??_C@_03CLCAEGCJ@new?$AA@  1000cc5c     databaseEdit.obj
 0002:00001c60       ??_C@_04CCPFBLLC@?$CGNew?$AA@ 1000cc60     databaseEdit.obj
 0002:00001c68       ??_C@_07EJAINBEK@filenew?$AA@ 1000cc68     databaseEdit.obj
 0002:00001c70       ??_C@_0BA@NPMEGAC@New?5Application?$AA@ 1000cc70     databaseEdit.obj
 0002:00001c80       ??_C@_04PHHEBHMK@?4ini?$AA@ 1000cc80     databaseEdit.obj
 0002:00001c88       ??_C@_06BNCCALCL@unlock?$AA@ 1000cc88     databaseEdit.obj
 0002:00001c90       ??_C@_04GHHNNAGO@?4db0?$AA@ 1000cc90     databaseEdit.obj
 0002:00001c98       ??_C@_04HOGGOBCP@?4db1?$AA@ 1000cc98     databaseEdit.obj
 0002:00001ca0       ??_C@_04FFELLCOM@?4db2?$AA@ 1000cca0     databaseEdit.obj
 0002:00001ca8       ??_C@_04EMFAIDKN@?4db3?$AA@ 1000cca8     databaseEdit.obj
 0002:00001cb0       ??_C@_04DBBBFGK@?4db4?$AA@ 1000ccb0     databaseEdit.obj
 0002:00001cb8       ??_C@_04BKAKCECL@?4db5?$AA@ 1000ccb8     databaseEdit.obj
 0002:00001cc0       ??_C@_04DBCHHHOI@?4db6?$AA@ 1000ccc0     databaseEdit.obj
 0002:00001cc8       ??_C@_04CIDMEGKJ@?4db7?$AA@ 1000ccc8     databaseEdit.obj
 0002:00001cd0       ??_C@_04KPKEFKGG@?4db8?$AA@ 1000ccd0     databaseEdit.obj
 0002:00001cd8       ??_C@_04LGLPGLCH@?4db9?$AA@ 1000ccd8     databaseEdit.obj
 0002:00001ce0       ??_C@_0N@EKBAGMEL@?5?9?5filename?$DN?$AA@ 1000cce0     databaseEdit.obj
 0002:00001cf0       ??_C@_09JLEOPMAJ@?5?9?5error?$DN?$AA@ 1000ccf0     databaseEdit.obj
 0002:00001cfc       ??_C@_09LBCHCBIC@?5?9?5value?$DN?$AA@ 1000ccfc     databaseEdit.obj
 0002:00001d08       ??_C@_0P@ELNNACEA@?5?9?5textStatus?$DN?$AA@ 1000cd08     databaseEdit.obj
 0002:00001d18       ??_C@_0L@LEAPMKGP@Reply?3?5op?$DN?$AA@ 1000cd18     databaseEdit.obj
 0002:00001d24       ??_C@_08HNIAHLMM@download?$AA@ 1000cd24     databaseEdit.obj
 0002:00001d30       ??_C@_0O@IOBCFEKL@config?1system?$AA@ 1000cd30     databaseEdit.obj
 0002:00001d40       ??_C@_0CD@BLKHMJDB@?$FOconfig?1system?1dev_?$FL0?99?$FN?$HL3?03?$HN?4in@ 1000cd40     databaseEdit.obj
 0002:00001d64       ??_C@_01KICIPPFI@?2?$AA@   1000cd64     databaseEdit.obj
 0002:00001d66       ??_C@_00CNPNBAHC@?$AA@     1000cd66     databaseEdit.obj
 0002:00001d68       ??_C@_04FABLJDN@Name?$AA@  1000cd68     databaseEdit.obj
 0002:00001d70       ??_C@_06OIEJKIHP@Device?$AA@ 1000cd70     databaseEdit.obj
 0002:00001d78       ??_C@_07LGMPALJ@?5value?$DN?$AA@ 1000cd78     databaseEdit.obj
 0002:00001d80       ??_C@_0M@NAHGLGJG@m_filename?$DN?$AA@ 1000cd80     databaseEdit.obj
 0002:00001d8c       ??_C@_03NLCNLML@?$FO?$CF1?$AA@ 1000cd8c     databaseEdit.obj
 0002:00001d90       ??_C@_04HCDDPBNL@TRUE?$AA@ 1000cd90     databaseEdit.obj
 0002:00001d98       ??_C@_01KMDKNFGN@?1?$AA@   1000cd98     databaseEdit.obj
 0002:00001d9c       ??_C@_05IKKOLOBP@?4ini$?$AA@ 1000cd9c     databaseEdit.obj
 0002:00001da4       ??_C@_05FLIFNACJ@?4db0$?$AA@ 1000cda4     databaseEdit.obj
 0002:00001dac       ??_C@_05FKEHLKBO@?4db1$?$AA@ 1000cdac     databaseEdit.obj
 0002:00001db4       ??_C@_05FIABAEEH@?4db2$?$AA@ 1000cdb4     databaseEdit.obj
 0002:00001dbc       ??_C@_05FJMDGOHA@?4db3$?$AA@ 1000cdbc     databaseEdit.obj
 0002:00001dc4       ??_C@_05FMIMHIPF@?4db4$?$AA@ 1000cdc4     databaseEdit.obj
 0002:00001dcc       ??_C@_05FNEOBCMC@?4db5$?$AA@ 1000cdcc     databaseEdit.obj
 0002:00001dd4       ??_C@_05FPAIKMJL@?4db6$?$AA@ 1000cdd4     databaseEdit.obj
 0002:00001ddc       ??_C@_05FOMKMGKM@?4db7$?$AA@ 1000cddc     databaseEdit.obj
 0002:00001de4       ??_C@_05FFJGIBJB@?4db8$?$AA@ 1000cde4     databaseEdit.obj
 0002:00001dec       ??_C@_05FEFEOLKG@?4db9$?$AA@ 1000cdec     databaseEdit.obj
 0002:00001df4       ??_C@_04MKMCLCOO@lock?$AA@ 1000cdf4     databaseEdit.obj
 0002:00001dfc       ??_C@_06KAOCKAGB@upload?$AA@ 1000cdfc     databaseEdit.obj
 0002:00001e04       ??_C@_09NKPGGJLP@?4db?$FL0?99?$FN$?$AA@ 1000ce04     databaseEdit.obj
 0002:00001e10       ??_C@_0BC@OLADGOOO@There?5is?5no?5file?5?$AA@ 1000ce10     databaseEdit.obj
 0002:00001e24       ??_C@_0M@EBFEGAAI@Information?$AA@ 1000ce24     databaseEdit.obj
 0002:00001e30       ??_C@_03DAPAKLGM@dir?$AA@  1000ce30     databaseEdit.obj
 0002:00001e34       ??_C@_0BE@FHCPCNPG@got?5dir?5listing?5of?5?$AA@ 1000ce34     databaseEdit.obj
 0002:00001e48       ??_C@_0CO@GKAEALGF@Being?5asked?5to?5navigate?5to?5?$CF1?5wi@ 1000ce48     databaseEdit.obj
 0002:00001e78       ??_C@_0BA@GNHMHBBC@syncDirDownload?$AA@ 1000ce78     databaseEdit.obj
 0002:00001e88       ??_C@_0N@EHHLDFOB@checkoutFile?$AA@ 1000ce88     databaseEdit.obj
 0002:00001e98       ??_C@_0L@CIKGEHEG@uploadFile?$AA@ 1000ce98     databaseEdit.obj
 0002:00001ea8       ??_C@_0EM@BEMJAICD@?$DMh3?$DODevice?5Database?5Editor?5Confi@ 1000cea8     databaseEdit.obj
 0002:00001ef4       ??_C@_08EHFONDEF@13?324?301?$AA@ 1000cef4     databaseEdit.obj
 0002:00001f00       ??_C@_0M@JEDEHNP@Sep?523?52021?$AA@ 1000cf00     databaseEdit.obj
 0002:00001f0c       ??_C@_0BH@OIGCMNOE@config?1system?1dev_?$CF03d?$AA@ 1000cf0c     databaseEdit.obj
 0002:00001f24       ??_C@_0BF@LFIMMLAF@trying?5to?5get?5file?3?5?$AA@ 1000cf24     databaseEdit.obj
 0002:00001f40       ??_7?$QIntDict@VQTable@@@@6B@ 1000cf40     databaseEditdlgimpl.obj
 0002:00001f60       ??_7databaseEditDlg@@6BQObject@@@ 1000cf60     databaseEditdlgimpl.obj
 0002:00002118       ??_7databaseEditDlg@@6BQPaintDevice@@@ 1000d118     databaseEditdlgimpl.obj
 0002:00002138       ??_C@_0BD@PHPDBBBM@1sortColumn?$CI?5int?5?$CJ?$AA@ 1000d138     databaseEditdlgimpl.obj
 0002:0000214c       ??_C@_0BA@HHAILMBL@2clicked?$CI?5int?5?$CJ?$AA@ 1000d14c     databaseEditdlgimpl.obj
 0002:0000215c       ??_C@_05CFEJGMAI@dirty?$AA@ 1000d15c     databaseEditdlgimpl.obj
 0002:00002164       ??_C@_05OEOKGKGJ@?$DM?1h1?$DO?$AA@ 1000d164     databaseEditdlgimpl.obj
 0002:0000216c       ??_C@_0BO@JBGALGII@?$DMh1?$DODevice?5Database?5Editor?5?9?5?$AA@ 1000d16c     databaseEditdlgimpl.obj
 0002:0000218c       ??_C@_07DGJCLIHL@?$CF1?4db?$CF2?$AA@ 1000d18c     databaseEditdlgimpl.obj
 0002:00002194       ??_C@_0BB@IMNFBOLL@?$FO?2?$FLDatabase_?$CF1?2?$FN?$AA@ 1000d194     databaseEditdlgimpl.obj
 0002:000021a8       ??_C@_01NEMOKFLO@?$DN?$AA@ 1000d1a8     databaseEditdlgimpl.obj
 0002:000021ac       ??_C@_04DMJLGFFO@db?$CF1?$AA@ 1000d1ac     databaseEditdlgimpl.obj
 0002:000021b4       ??_C@_06BMBEEELA@QTable?$AA@ 1000d1b4     databaseEditdlgimpl.obj
 0002:000021bc       ??_C@_09OFODDICG@14?514?52?51?$AA@ 1000d1bc     plugindesc.obj
 0002:000021c8       ??_C@_0M@KEPPNGJB@?$CD?5c?5?$CD000000?$AA@ 1000d1c8     plugindesc.obj
 0002:000021d4       ??_C@_08IMFNEMJ@?4?5c?5none?$AA@ 1000d1d4     plugindesc.obj
 0002:000021e0       ??_C@_0P@HFKAALMG@?4?4?4?4?4?4?4?4?4?4?4?4?4?4?$AA@ 1000d1e0     plugindesc.obj
 0002:000021f0       ??_C@_0P@HBCKOD@?4?$CD?4?4?$CD?4?$CD?$CD?$CD?4?$CD?$CD?$CD?4?$AA@ 1000d1f0     plugindesc.obj
 0002:00002200       ??_C@_0P@CMBAAIKO@?4?$CD?$CD?4?$CD?4?$CD?4?$CD?4?4?$CD?4?4?$AA@ 1000d200     plugindesc.obj
 0002:00002210       ??_C@_0P@PFJDGJDO@?4?$CD?4?$CD?$CD?4?$CD?4?$CD?4?4?$CD?4?4?$AA@ 1000d210     plugindesc.obj
 0002:00002220       ??_C@_0P@PADJHNAB@?4?$CD?4?4?$CD?4?$CD?$CD?$CD?4?4?$CD?4?4?$AA@ 1000d220     plugindesc.obj
 0002:00002230       ??_C@_0P@MPFEALAD@?4?$CD?4?4?4?$CD?4?$CD?$CD?4?$CD?$CD?$CD?4?$AA@ 1000d230     plugindesc.obj
 0002:00002240       ??_C@_0P@JAHHOLLD@?4?4?$CD?4?$CD?4?4?$CD?4?4?4?$CD?4?4?$AA@ 1000d240     plugindesc.obj
 0002:00002250       ??_C@_0P@ODLHKGOE@?4?4?4?$CD?4?4?4?$CD?$CD?4?4?$CD?4?4?$AA@ 1000d250     plugindesc.obj
 0002:00002260       ??_C@_0P@ICGAMHCE@?4?4?4?$CD?4?4?4?$CD?4?4?4?$CD?4?4?$AA@ 1000d260     plugindesc.obj
 0002:00002274       ??_7config_plugin_desc_base@@6B@ 1000d274     plugindesc.obj
 0002:00002288       ??_7plugindesc@@6B@        1000d288     plugindesc.obj
 0002:00002298       ??_C@_0CD@CBPIMHKA@Home?1System?1Device?5Database?5Edit@ 1000d298     plugindesc.obj
 0002:000022c0       ??_7toolWindow@@6BQObject@@@ 1000d2c0     toolwindowimpl.obj
 0002:00002478       ??_7toolWindow@@6BQPaintDevice@@@ 1000d478     toolwindowimpl.obj
 0002:00002498       ??_C@_0CF@OPOOCIJN@1selectionChanged?$CI?5QListViewItem@ 1000d498     toolwindowimpl.obj
 0002:000024c0       ??_C@_0CF@LFIPBHPN@2selectionChanged?$CI?5QListViewItem@ 1000d4c0     toolwindowimpl.obj
 0002:000024ec       ??_SQWidget@@6BQObject@@@  1000d4ec     databaseEditdlg.obj
 0002:000026a0       ??_SQWidget@@6BQPaintDevice@@@ 1000d6a0     databaseEditdlg.obj
 0002:000026c4       ??_7databaseEditDlgBase@@6BQObject@@@ 1000d6c4     databaseEditdlg.obj
 0002:0000287c       ??_7databaseEditDlgBase@@6BQPaintDevice@@@ 1000d87c     databaseEditdlg.obj
 0002:000028a4       ??_SQLabel@@6BQObject@@@   1000d8a4     databaseEditdlg.obj
 0002:00002a9c       ??_SQLabel@@6BQPaintDevice@@@ 1000da9c     databaseEditdlg.obj
 0002:00002ac4       ??_SQTabWidget@@6BQObject@@@ 1000dac4     databaseEditdlg.obj
 0002:00002c98       ??_SQTabWidget@@6BQPaintDevice@@@ 1000dc98     databaseEditdlg.obj
 0002:00002cbc       ??_SQLineEdit@@6BQObject@@@ 1000dcbc     databaseEditdlg.obj
 0002:00002ee4       ??_SQLineEdit@@6BQPaintDevice@@@ 1000dee4     databaseEditdlg.obj
 0002:00002f0c       ??_SQTextEdit@@6BQObject@@@ 1000df0c     databaseEditdlg.obj
 0002:00003288       ??_SQTextEdit@@6BQPaintDevice@@@ 1000e288     databaseEditdlg.obj
 0002:000032ac       ??_SQTable@@6BQObject@@@   1000e2ac     databaseEditdlg.obj
 0002:0000364c       ??_SQTable@@6BQPaintDevice@@@ 1000e64c     databaseEditdlg.obj
 0002:00003674       ??_SQSpacerItem@@6B@       1000e674     databaseEditdlg.obj
 0002:000036bc       ??_SQHBoxLayout@@6BQObject@@@ 1000e6bc     databaseEditdlg.obj
 0002:00003724       ??_SQHBoxLayout@@6BQLayoutItem@@@ 1000e724     databaseEditdlg.obj
 0002:0000376c       ??_SQVBoxLayout@@6BQObject@@@ 1000e76c     databaseEditdlg.obj
 0002:000037d4       ??_SQVBoxLayout@@6BQLayoutItem@@@ 1000e7d4     databaseEditdlg.obj
 0002:00003814       ??_C@_0BE@IAMOMJE@databaseEditDlgBase?$AA@ 1000e814     databaseEditdlg.obj
 0002:00003828       ??_C@_0BK@OBPLCANL@databaseEditDlgBaseLayout?$AA@ 1000e828     databaseEditdlg.obj
 0002:00003844       ??_C@_05PHLGJONK@title?$AA@ 1000e844     databaseEditdlg.obj
 0002:0000384c       ??_C@_02DDDIAJFA@tw?$AA@   1000e84c     databaseEditdlg.obj
 0002:00003850       ??_C@_07MNNHCJEA@TabPage?$AA@ 1000e850     databaseEditdlg.obj
 0002:00003858       ??_C@_0O@CPJAHDHK@TabPageLayout?$AA@ 1000e858     databaseEditdlg.obj
 0002:00003868       ??_C@_07MOFDPJDG@layout1?$AA@ 1000e868     databaseEditdlg.obj
 0002:00003870       ??_C@_0L@KGLFILOJ@textLabel1?$AA@ 1000e870     databaseEditdlg.obj
 0002:0000387c       ??_C@_09NLCNKAKG@lineEdit1?$AA@ 1000e87c     databaseEditdlg.obj
 0002:00003888       ??_C@_0N@HPEGIJEE@textLabel1_2?$AA@ 1000e888     databaseEditdlg.obj
 0002:00003898       ??_C@_0M@KEBLFOFG@lineEdit1_2?$AA@ 1000e898     databaseEditdlg.obj
 0002:000038a4       ??_C@_09HCBNDNHI@textEdit1?$AA@ 1000e8a4     databaseEditdlg.obj
 0002:000038b0       ??_C@_03CEDILPBK@tab?$AA@  1000e8b0     databaseEditdlg.obj
 0002:000038b4       ??_C@_09PEOMDABK@tabLayout?$AA@ 1000e8b4     databaseEditdlg.obj
 0002:000038c0       ??_C@_07OFHOKKPF@layout2?$AA@ 1000e8c0     databaseEditdlg.obj
 0002:000038c8       ??_C@_0N@GGFNLIAF@textLabel1_3?$AA@ 1000e8c8     databaseEditdlg.obj
 0002:000038d8       ??_C@_0M@LNAAGPBH@lineEdit1_3?$AA@ 1000e8d8     databaseEditdlg.obj
 0002:000038e4       ??_C@_03POOKGJAK@db0?$AA@  1000e8e4     databaseEditdlg.obj
 0002:000038e8       ??_C@_05FNNGFGLF@Index?$AA@ 1000e8e8     databaseEditdlg.obj
 0002:000038f0       ??_C@_04DICKPMGH@Data?$AA@ 1000e8f0     databaseEditdlg.obj
 0002:000038f8       ??_C@_05GBGDENAC@tab_2?$AA@ 1000e8f8     databaseEditdlg.obj
 0002:00003900       ??_C@_0M@BMGEADGH@tabLayout_2?$AA@ 1000e900     databaseEditdlg.obj
 0002:0000390c       ??_C@_03OHPBFIEL@db1?$AA@  1000e90c     databaseEditdlg.obj
 0002:00003910       ??_C@_09DIFLCHEC@TabPage_2?$AA@ 1000e910     databaseEditdlg.obj
 0002:0000391c       ??_C@_0BA@JGEMKDJG@TabPageLayout_2?$AA@ 1000e91c     databaseEditdlg.obj
 0002:0000392c       ??_C@_03MMNMALII@db2?$AA@  1000e92c     databaseEditdlg.obj
 0002:00003930       ??_C@_09CBEABGAD@TabPage_3?$AA@ 1000e930     databaseEditdlg.obj
 0002:0000393c       ??_C@_0BA@IPFHJCNH@TabPageLayout_3?$AA@ 1000e93c     databaseEditdlg.obj
 0002:0000394c       ??_C@_03NFMHDKMJ@db3?$AA@  1000e94c     databaseEditdlg.obj
 0002:00003950       ??_C@_09GOABIAME@TabPage_4?$AA@ 1000e950     databaseEditdlg.obj
 0002:0000395c       ??_C@_0BA@MABGAEBA@TabPageLayout_4?$AA@ 1000e95c     databaseEditdlg.obj
 0002:0000396c       ??_C@_03JKIGKMAO@db4?$AA@  1000e96c     databaseEditdlg.obj
 0002:00003970       ??_C@_09HHBKLBIF@TabPage_5?$AA@ 1000e970     databaseEditdlg.obj
 0002:0000397c       ??_C@_0BA@NJANDFFB@TabPageLayout_5?$AA@ 1000e97c     databaseEditdlg.obj
 0002:0000398c       ??_C@_03IDJNJNEP@db5?$AA@  1000e98c     databaseEditdlg.obj
 0002:00003990       ??_C@_09FMDHOCEG@TabPage_6?$AA@ 1000e990     databaseEditdlg.obj
 0002:0000399c       ??_C@_0BA@PCCAGGJC@TabPageLayout_6?$AA@ 1000e99c     databaseEditdlg.obj
 0002:000039ac       ??_C@_03KILAMOIM@db6?$AA@  1000e9ac     databaseEditdlg.obj
 0002:000039b0       ??_C@_09EFCMNDAH@TabPage_7?$AA@ 1000e9b0     databaseEditdlg.obj
 0002:000039bc       ??_C@_0BA@OLDLFHND@TabPageLayout_7?$AA@ 1000e9bc     databaseEditdlg.obj
 0002:000039cc       ??_C@_03LBKLPPMN@db7?$AA@  1000e9cc     databaseEditdlg.obj
 0002:000039d0       ??_C@_09MCLEMPMI@TabPage_8?$AA@ 1000e9d0     databaseEditdlg.obj
 0002:000039dc       ??_C@_0BA@GMKDELBM@TabPageLayout_8?$AA@ 1000e9dc     databaseEditdlg.obj
 0002:000039ec       ??_C@_03DGDDODAC@db8?$AA@  1000e9ec     databaseEditdlg.obj
 0002:000039f0       ??_C@_09NLKPPOIJ@TabPage_9?$AA@ 1000e9f0     databaseEditdlg.obj
 0002:000039fc       ??_C@_0BA@HFLIHKFN@TabPageLayout_9?$AA@ 1000e9fc     databaseEditdlg.obj
 0002:00003a0c       ??_C@_03CPCINCED@db9?$AA@  1000ea0c     databaseEditdlg.obj
 0002:00003a10       ??_C@_0BA@DJMECJJH@databaseEditDlg?$AA@ 1000ea10     databaseEditdlg.obj
 0002:00003a20       ??_C@_0FA@PDKJICKK@?$DMh1?$DO?$DMfont?5color?$DN?$CC?$CDff0000?$CC?$DONON?5WO@ 1000ea20     databaseEditdlg.obj
 0002:00003a70       ??_C@_0P@ONIBKGMN@DatabaseSize_0?$AA@ 1000ea70     databaseEditdlg.obj
 0002:00003a80       ??_C@_0P@PEJKJHIM@DatabaseSize_1?$AA@ 1000ea80     databaseEditdlg.obj
 0002:00003a90       ??_C@_03GDBIGDNC@INI?$AA@  1000ea90     databaseEditdlg.obj
 0002:00003a94       ??_C@_03GGJFIANE@DB0?$AA@  1000ea94     databaseEditdlg.obj
 0002:00003a98       ??_C@_04FLKDCHIP@DB?51?$AA@ 1000ea98     databaseEditdlg.obj
 0002:00003aa0       ??_C@_03FEKDOCFG@DB2?$AA@  1000eaa0     databaseEditdlg.obj
 0002:00003aa4       ??_C@_03ENLINDBH@DB3?$AA@  1000eaa4     databaseEditdlg.obj
 0002:00003aa8       ??_C@_03CPJEFNA@DB4?$AA@   1000eaa8     databaseEditdlg.obj
 0002:00003aac       ??_C@_03BLOCHEJB@DB5?$AA@  1000eaac     databaseEditdlg.obj
 0002:00003ab0       ??_C@_03DAMPCHFC@DB6?$AA@  1000eab0     databaseEditdlg.obj
 0002:00003ab4       ??_C@_03CJNEBGBD@DB7?$AA@  1000eab4     databaseEditdlg.obj
 0002:00003ab8       ??_C@_03KOEMAKNM@DB8?$AA@  1000eab8     databaseEditdlg.obj
 0002:00003abc       ??_C@_03LHFHDLJN@DB9?$AA@  1000eabc     databaseEditdlg.obj
 0002:00003ac0       ??_C@_0N@DOIHMBIF@databaseEdit?$AA@ 1000eac0     moc_databaseEdit.obj
 0002:00003ad0       ??_C@_08BABJIOEM@filename?$AA@ 1000ead0     moc_databaseEdit.obj
 0002:00003ae8       ??_C@_0N@DENPNHIG@fileSelected?$AA@ 1000eae8     moc_databaseEdit.obj
 0002:00003b04       ??_C@_0BN@NHBBIGHD@fileSelected?$CIconst?5QString?$CG?$CJ?$AA@ 1000eb04     moc_databaseEdit.obj
 0002:00003b30       ??_C@_07KMMNMMFF@command?$AA@ 1000eb30     moc_databaseEdit.obj
 0002:00003b44       ??_C@_0BJ@FEFNJDLM@command?$CIQString?0QString?$CJ?$AA@ 1000eb44     moc_databaseEdit.obj
 0002:00003b6c       ??_C@_0P@DMEOIADN@languageChange?$AA@ 1000eb6c     moc_databaseEditdlg.obj
 0002:00003b88       ??_C@_0BB@PFEIHPGD@languageChange?$CI?$CJ?$AA@ 1000eb88     moc_databaseEditdlg.obj
 0002:00003ba8       ??_C@_0M@NJKJFEFJ@textChanged?$AA@ 1000eba8     moc_databaseEditdlgimpl.obj
 0002:00003bb4       ??_C@_03HNOLNALI@col?$AA@  1000ebb4     moc_databaseEditdlgimpl.obj
 0002:00003bc4       ??_C@_0L@BCAIFHPG@sortColumn?$AA@ 1000ebc4     moc_databaseEditdlgimpl.obj
 0002:00003be8       ??_C@_0O@HFGHCCOK@textChanged?$CI?$CJ?$AA@ 1000ebe8     moc_databaseEditdlgimpl.obj
 0002:00003bf8       ??_C@_0BA@FENDPOLN@sortColumn?$CIint?$CJ?$AA@ 1000ebf8     moc_databaseEditdlgimpl.obj
 0002:00003c20       ??_C@_0P@ECKEJGFB@toolWindowBase?$AA@ 1000ec20     moc_toolwindow.obj
 0002:00003c48       ??_C@_0L@IGMLIIOB@toolWindow?$AA@ 1000ec48     moc_toolwindowimpl.obj
 0002:00003c54       ??_C@_0O@LAFKAPIP@QListViewItem?$AA@ 1000ec54     moc_toolwindowimpl.obj
 0002:00003c70       ??_C@_0BB@FFKPNNIH@selectionChanged?$AA@ 1000ec70     moc_toolwindowimpl.obj
 0002:00003c90       ??_C@_0CB@BHPNGIPG@selectionChanged?$CIQListViewItem?$CK?$CJ@ 1000ec90     moc_toolwindowimpl.obj
 0002:00003cd0       ??_7toolWindowBase@@6BQObject@@@ 1000ecd0     toolwindow.obj
 0002:00003e88       ??_7toolWindowBase@@6BQPaintDevice@@@ 1000ee88     toolwindow.obj
 0002:00003eac       ??_SQListView@@6BQObject@@@ 1000eeac     toolwindow.obj
 0002:00004190       ??_SQListView@@6BQPaintDevice@@@ 1000f190     toolwindow.obj
 0002:000041b0       ??_C@_0BF@OGGOGOEO@toolWindowBaseLayout?$AA@ 1000f1b0     toolwindow.obj
 0002:000041c8       ??_C@_0L@NNPJCPDK@tabWidget2?$AA@ 1000f1c8     toolwindow.obj
 0002:000041d4       ??_C@_09MIHIKGED@listView1?$AA@ 1000f1d4     toolwindow.obj
 0002:000041e0       ??_C@_06IONACMBM@Number?$AA@ 1000f1e0     toolwindow.obj
 0002:000041e8       ??_C@_0M@OHKMKKDH@Description?$AA@ 1000f1e8     toolwindow.obj
 0002:000041f4       ??_C@_0P@GOBLAFMA@Database?5Files?$AA@ 1000f1f4     toolwindow.obj
 0002:00004208       ??_7type_info@@6B@         1000f208     MSVCRT:ti_inst.obj
 0002:0000420c       __pRawDllMain              1000f20c     MSVCRT:crtdll.obj
 0002:0000420c       __pDefaultRawDllMain       1000f20c     MSVCRT:crtdll.obj
 0002:00004218       __load_config_used         1000f218     MSVCRT:loadcfg.obj
 0002:00004260       ??_R3QShared@@8            1000f260     databaseEdit.obj
 0002:00004270       ??_R2QShared@@8            1000f270     databaseEdit.obj
 0002:00004278       ??_R1A@?0A@EA@QShared@@8   1000f278     databaseEdit.obj
 0002:00004294       ??_R1A@?0A@EA@QGList@@8    1000f294     databaseEdit.obj
 0002:000042b0       ??_R3QGList@@8             1000f2b0     databaseEdit.obj
 0002:000042c0       ??_R2QGList@@8             1000f2c0     databaseEdit.obj
 0002:000042cc       ??_R1A@?0A@EA@QPtrCollection@@8 1000f2cc     databaseEdit.obj
 0002:000042e8       ??_R3QPtrCollection@@8     1000f2e8     databaseEdit.obj
 0002:000042f8       ??_R2QPtrCollection@@8     1000f2f8     databaseEdit.obj
 0002:00004300       ??_R4QToolBar@@6BQObject@@@ 1000f300     databaseEdit.obj
 0002:00004314       ??_R3QToolBar@@8           1000f314     databaseEdit.obj
 0002:00004324       ??_R2QToolBar@@8           1000f324     databaseEdit.obj
 0002:00004344       ??_R1A@?0A@EA@QToolBar@@8  1000f344     databaseEdit.obj
 0002:00004360       ??_R1A@?0A@EA@QDockWindow@@8 1000f360     databaseEdit.obj
 0002:0000437c       ??_R3QDockWindow@@8        1000f37c     databaseEdit.obj
 0002:0000438c       ??_R2QDockWindow@@8        1000f38c     databaseEdit.obj
 0002:000043a8       ??_R1A@?0A@EA@QFrame@@8    1000f3a8     databaseEdit.obj
 0002:000043c4       ??_R3QFrame@@8             1000f3c4     databaseEdit.obj
 0002:000043d4       ??_R2QFrame@@8             1000f3d4     databaseEdit.obj
 0002:000043ec       ??_R1A@?0A@EA@QWidget@@8   1000f3ec     databaseEdit.obj
 0002:00004408       ??_R3QWidget@@8            1000f408     databaseEdit.obj
 0002:00004418       ??_R2QWidget@@8            1000f418     databaseEdit.obj
 0002:0000442c       ??_R1A@?0A@EA@QObject@@8   1000f42c     databaseEdit.obj
 0002:00004448       ??_R3QObject@@8            1000f448     databaseEdit.obj
 0002:00004458       ??_R2QObject@@8            1000f458     databaseEdit.obj
 0002:00004464       ??_R13?0A@EA@Qt@@8         1000f464     databaseEdit.obj
 0002:00004480       ??_R3Qt@@8                 1000f480     databaseEdit.obj
 0002:00004490       ??_R2Qt@@8                 1000f490     databaseEdit.obj
 0002:00004498       ??_R1A@?0A@EA@Qt@@8        1000f498     databaseEdit.obj
 0002:000044b4       ??_R1CI@?0A@EA@QPaintDevice@@8 1000f4b4     databaseEdit.obj
 0002:000044d0       ??_R3QPaintDevice@@8       1000f4d0     databaseEdit.obj
 0002:000044e0       ??_R2QPaintDevice@@8       1000f4e0     databaseEdit.obj
 0002:000044e8       ??_R1A@?0A@EA@QPaintDevice@@8 1000f4e8     databaseEdit.obj
 0002:00004504       ??_R4QToolBar@@6BQPaintDevice@@@ 1000f504     databaseEdit.obj
 0002:00004518       ??_R4QPopupMenu@@6BQObject@@@ 1000f518     databaseEdit.obj
 0002:0000452c       ??_R3QPopupMenu@@8         1000f52c     databaseEdit.obj
 0002:0000453c       ??_R2QPopupMenu@@8         1000f53c     databaseEdit.obj
 0002:0000455c       ??_R1A@?0A@EA@QPopupMenu@@8 1000f55c     databaseEdit.obj
 0002:00004578       ??_R1IM@?0A@EA@QMenuData@@8 1000f578     databaseEdit.obj
 0002:00004594       ??_R3QMenuData@@8          1000f594     databaseEdit.obj
 0002:000045a4       ??_R2QMenuData@@8          1000f5a4     databaseEdit.obj
 0002:000045ac       ??_R1A@?0A@EA@QMenuData@@8 1000f5ac     databaseEdit.obj
 0002:000045c8       ??_R4QPopupMenu@@6BQPaintDevice@@@ 1000f5c8     databaseEdit.obj
 0002:000045dc       ??_R4QPopupMenu@@6B@       1000f5dc     databaseEdit.obj
 0002:000045f0       ??_R4QDockWindow@@6BQObject@@@ 1000f5f0     databaseEdit.obj
 0002:00004604       ??_R4QDockWindow@@6BQPaintDevice@@@ 1000f604     databaseEdit.obj
 0002:00004618       ??_R4QListViewItem@@6B@    1000f618     databaseEdit.obj
 0002:0000462c       ??_R3QListViewItem@@8      1000f62c     databaseEdit.obj
 0002:0000463c       ??_R2QListViewItem@@8      1000f63c     databaseEdit.obj
 0002:00004648       ??_R1A@?0A@EA@QListViewItem@@8 1000f648     databaseEdit.obj
 0002:00004664       ??_R4QAction@@6B@          1000f664     databaseEdit.obj
 0002:00004678       ??_R3QAction@@8            1000f678     databaseEdit.obj
 0002:00004688       ??_R2QAction@@8            1000f688     databaseEdit.obj
 0002:00004698       ??_R1A@?0A@EA@QAction@@8   1000f698     databaseEdit.obj
 0002:000046b4       ??_R4QGuardedPtrPrivate@@6B@ 1000f6b4     databaseEdit.obj
 0002:000046c8       ??_R3QGuardedPtrPrivate@@8 1000f6c8     databaseEdit.obj
 0002:000046d8       ??_R2QGuardedPtrPrivate@@8 1000f6d8     databaseEdit.obj
 0002:000046ec       ??_R1A@?0A@EA@QGuardedPtrPrivate@@8 1000f6ec     databaseEdit.obj
 0002:00004708       ??_R1CI@?0A@EA@QShared@@8  1000f708     databaseEdit.obj
 0002:00004724       ??_R4QDockWindowList@@6B@  1000f724     databaseEdit.obj
 0002:00004738       ??_R3QDockWindowList@@8    1000f738     databaseEdit.obj
 0002:00004748       ??_R2QDockWindowList@@8    1000f748     databaseEdit.obj
 0002:0000475c       ??_R1A@?0A@EA@QDockWindowList@@8 1000f75c     databaseEdit.obj
 0002:00004778       ??_R1A@?0A@EA@?$QPtrList@VQDockWindow@@@@8 1000f778     databaseEdit.obj
 0002:00004794       ??_R3?$QPtrList@VQDockWindow@@@@8 1000f794     databaseEdit.obj
 0002:000047a4       ??_R2?$QPtrList@VQDockWindow@@@@8 1000f7a4     databaseEdit.obj
 0002:000047b4       ??_R4QPopupMenuList@@6B@   1000f7b4     databaseEdit.obj
 0002:000047c8       ??_R3QPopupMenuList@@8     1000f7c8     databaseEdit.obj
 0002:000047d8       ??_R2QPopupMenuList@@8     1000f7d8     databaseEdit.obj
 0002:000047ec       ??_R1A@?0A@EA@QPopupMenuList@@8 1000f7ec     databaseEdit.obj
 0002:00004808       ??_R1A@?0A@EA@?$QPtrList@VQPopupMenu@@@@8 1000f808     databaseEdit.obj
 0002:00004824       ??_R3?$QPtrList@VQPopupMenu@@@@8 1000f824     databaseEdit.obj
 0002:00004834       ??_R2?$QPtrList@VQPopupMenu@@@@8 1000f834     databaseEdit.obj
 0002:00004844       ??_R4?$QPtrList@VQPopupMenu@@@@6B@ 1000f844     databaseEdit.obj
 0002:00004858       ??_R4config_plugin_base@@6BQObject@@@ 1000f858     databaseEdit.obj
 0002:0000486c       ??_R3config_plugin_base@@8 1000f86c     databaseEdit.obj
 0002:0000487c       ??_R2config_plugin_base@@8 1000f87c     databaseEdit.obj
 0002:00004894       ??_R1A@?0A@EA@config_plugin_base@@8 1000f894     databaseEdit.obj
 0002:000048b0       ??_R4config_plugin_base@@6BQPaintDevice@@@ 1000f8b0     databaseEdit.obj
 0002:000048c4       ??_R1A@?0A@EA@QGDict@@8    1000f8c4     databaseEdit.obj
 0002:000048e0       ??_R3QGDict@@8             1000f8e0     databaseEdit.obj
 0002:000048f0       ??_R2QGDict@@8             1000f8f0     databaseEdit.obj
 0002:000048fc       ??_R4databaseEdit@@6BQObject@@@ 1000f8fc     databaseEdit.obj
 0002:00004910       ??_R3databaseEdit@@8       1000f910     databaseEdit.obj
 0002:00004920       ??_R2databaseEdit@@8       1000f920     databaseEdit.obj
 0002:0000493c       ??_R1A@?0A@EA@databaseEdit@@8 1000f93c     databaseEdit.obj
 0002:00004958       ??_R4databaseEdit@@6BQPaintDevice@@@ 1000f958     databaseEdit.obj
 0002:0000496c       ??_R4?$QDict@VQAction@@@@6B@ 1000f96c     databaseEdit.obj
 0002:00004980       ??_R3?$QDict@VQAction@@@@8 1000f980     databaseEdit.obj
 0002:00004990       ??_R2?$QDict@VQAction@@@@8 1000f990     databaseEdit.obj
 0002:000049a0       ??_R1A@?0A@EA@?$QDict@VQAction@@@@8 1000f9a0     databaseEdit.obj
 0002:000049bc       ??_R4databaseEditDlg@@6BQObject@@@ 1000f9bc     databaseEditdlgimpl.obj
 0002:000049d0       ??_R3databaseEditDlg@@8    1000f9d0     databaseEditdlgimpl.obj
 0002:000049e0       ??_R2databaseEditDlg@@8    1000f9e0     databaseEditdlgimpl.obj
 0002:000049fc       ??_R1A@?0A@EA@databaseEditDlg@@8 1000f9fc     databaseEditdlgimpl.obj
 0002:00004a18       ??_R1A@?0A@EA@databaseEditDlgBase@@8 1000fa18     databaseEditdlgimpl.obj
 0002:00004a34       ??_R3databaseEditDlgBase@@8 1000fa34     databaseEditdlgimpl.obj
 0002:00004a44       ??_R2databaseEditDlgBase@@8 1000fa44     databaseEditdlgimpl.obj
 0002:00004a5c       ??_R4databaseEditDlg@@6BQPaintDevice@@@ 1000fa5c     databaseEditdlgimpl.obj
 0002:00004a70       ??_R4?$QIntDict@VQTable@@@@6B@ 1000fa70     databaseEditdlgimpl.obj
 0002:00004a84       ??_R3?$QIntDict@VQTable@@@@8 1000fa84     databaseEditdlgimpl.obj
 0002:00004a94       ??_R2?$QIntDict@VQTable@@@@8 1000fa94     databaseEditdlgimpl.obj
 0002:00004aa4       ??_R1A@?0A@EA@?$QIntDict@VQTable@@@@8 1000faa4     databaseEditdlgimpl.obj
 0002:00004ac0       ??_R4config_plugin_desc_base@@6B@ 1000fac0     plugindesc.obj
 0002:00004ad4       ??_R3config_plugin_desc_base@@8 1000fad4     plugindesc.obj
 0002:00004ae4       ??_R2config_plugin_desc_base@@8 1000fae4     plugindesc.obj
 0002:00004aec       ??_R1A@?0A@EA@config_plugin_desc_base@@8 1000faec     plugindesc.obj
 0002:00004b08       ??_R4plugindesc@@6B@       1000fb08     plugindesc.obj
 0002:00004b1c       ??_R3plugindesc@@8         1000fb1c     plugindesc.obj
 0002:00004b2c       ??_R2plugindesc@@8         1000fb2c     plugindesc.obj
 0002:00004b38       ??_R1A@?0A@EA@plugindesc@@8 1000fb38     plugindesc.obj
 0002:00004b54       ??_R4toolWindow@@6BQObject@@@ 1000fb54     toolwindowimpl.obj
 0002:00004b68       ??_R3toolWindow@@8         1000fb68     toolwindowimpl.obj
 0002:00004b78       ??_R2toolWindow@@8         1000fb78     toolwindowimpl.obj
 0002:00004b94       ??_R1A@?0A@EA@toolWindow@@8 1000fb94     toolwindowimpl.obj
 0002:00004bb0       ??_R1A@?0A@EA@toolWindowBase@@8 1000fbb0     toolwindowimpl.obj
 0002:00004bcc       ??_R3toolWindowBase@@8     1000fbcc     toolwindowimpl.obj
 0002:00004bdc       ??_R2toolWindowBase@@8     1000fbdc     toolwindowimpl.obj
 0002:00004bf4       ??_R4toolWindow@@6BQPaintDevice@@@ 1000fbf4     toolwindowimpl.obj
 0002:00004c08       ??_R4QWidget@@6BQObject@@@ 1000fc08     databaseEditdlg.obj
 0002:00004c1c       ??_R4QWidget@@6BQPaintDevice@@@ 1000fc1c     databaseEditdlg.obj
 0002:00004c30       ??_R4QVBoxLayout@@6BQObject@@@ 1000fc30     databaseEditdlg.obj
 0002:00004c44       ??_R3QVBoxLayout@@8        1000fc44     databaseEditdlg.obj
 0002:00004c54       ??_R2QVBoxLayout@@8        1000fc54     databaseEditdlg.obj
 0002:00004c70       ??_R1A@?0A@EA@QVBoxLayout@@8 1000fc70     databaseEditdlg.obj
 0002:00004c8c       ??_R1A@?0A@EA@QBoxLayout@@8 1000fc8c     databaseEditdlg.obj
 0002:00004ca8       ??_R3QBoxLayout@@8         1000fca8     databaseEditdlg.obj
 0002:00004cb8       ??_R2QBoxLayout@@8         1000fcb8     databaseEditdlg.obj
 0002:00004cd0       ??_R1A@?0A@EA@QLayout@@8   1000fcd0     databaseEditdlg.obj
 0002:00004cec       ??_R3QLayout@@8            1000fcec     databaseEditdlg.obj
 0002:00004cfc       ??_R2QLayout@@8            1000fcfc     databaseEditdlg.obj
 0002:00004d10       ??_R1CI@?0A@EA@QLayoutItem@@8 1000fd10     databaseEditdlg.obj
 0002:00004d2c       ??_R3QLayoutItem@@8        1000fd2c     databaseEditdlg.obj
 0002:00004d3c       ??_R2QLayoutItem@@8        1000fd3c     databaseEditdlg.obj
 0002:00004d44       ??_R1A@?0A@EA@QLayoutItem@@8 1000fd44     databaseEditdlg.obj
 0002:00004d60       ??_R4QVBoxLayout@@6BQLayoutItem@@@ 1000fd60     databaseEditdlg.obj
 0002:00004d74       ??_R4QHBoxLayout@@6BQObject@@@ 1000fd74     databaseEditdlg.obj
 0002:00004d88       ??_R3QHBoxLayout@@8        1000fd88     databaseEditdlg.obj
 0002:00004d98       ??_R2QHBoxLayout@@8        1000fd98     databaseEditdlg.obj
 0002:00004db4       ??_R1A@?0A@EA@QHBoxLayout@@8 1000fdb4     databaseEditdlg.obj
 0002:00004dd0       ??_R4QHBoxLayout@@6BQLayoutItem@@@ 1000fdd0     databaseEditdlg.obj
 0002:00004de4       ??_R4QLabel@@6BQObject@@@  1000fde4     databaseEditdlg.obj
 0002:00004df8       ??_R3QLabel@@8             1000fdf8     databaseEditdlg.obj
 0002:00004e08       ??_R2QLabel@@8             1000fe08     databaseEditdlg.obj
 0002:00004e24       ??_R1A@?0A@EA@QLabel@@8    1000fe24     databaseEditdlg.obj
 0002:00004e40       ??_R4QLabel@@6BQPaintDevice@@@ 1000fe40     databaseEditdlg.obj
 0002:00004e54       ??_R4QTabWidget@@6BQObject@@@ 1000fe54     databaseEditdlg.obj
 0002:00004e68       ??_R3QTabWidget@@8         1000fe68     databaseEditdlg.obj
 0002:00004e78       ??_R2QTabWidget@@8         1000fe78     databaseEditdlg.obj
 0002:00004e90       ??_R1A@?0A@EA@QTabWidget@@8 1000fe90     databaseEditdlg.obj
 0002:00004eac       ??_R4QTabWidget@@6BQPaintDevice@@@ 1000feac     databaseEditdlg.obj
 0002:00004ec0       ??_R4QLineEdit@@6BQObject@@@ 1000fec0     databaseEditdlg.obj
 0002:00004ed4       ??_R3QLineEdit@@8          1000fed4     databaseEditdlg.obj
 0002:00004ee4       ??_R2QLineEdit@@8          1000fee4     databaseEditdlg.obj
 0002:00004f00       ??_R1A@?0A@EA@QLineEdit@@8 1000ff00     databaseEditdlg.obj
 0002:00004f1c       ??_R4QLineEdit@@6BQPaintDevice@@@ 1000ff1c     databaseEditdlg.obj
 0002:00004f30       ??_R4QTextEdit@@6BQObject@@@ 1000ff30     databaseEditdlg.obj
 0002:00004f44       ??_R3QTextEdit@@8          1000ff44     databaseEditdlg.obj
 0002:00004f54       ??_R2QTextEdit@@8          1000ff54     databaseEditdlg.obj
 0002:00004f74       ??_R1A@?0A@EA@QTextEdit@@8 1000ff74     databaseEditdlg.obj
 0002:00004f90       ??_R1A@?0A@EA@QScrollView@@8 1000ff90     databaseEditdlg.obj
 0002:00004fac       ??_R3QScrollView@@8        1000ffac     databaseEditdlg.obj
 0002:00004fbc       ??_R2QScrollView@@8        1000ffbc     databaseEditdlg.obj
 0002:00004fd8       ??_R4QTextEdit@@6BQPaintDevice@@@ 1000ffd8     databaseEditdlg.obj
 0002:00004fec       ??_R4QTable@@6BQObject@@@  1000ffec     databaseEditdlg.obj
 0002:00005000       ??_R3QTable@@8             10010000     databaseEditdlg.obj
 0002:00005010       ??_R2QTable@@8             10010010     databaseEditdlg.obj
 0002:00005030       ??_R1A@?0A@EA@QTable@@8    10010030     databaseEditdlg.obj
 0002:0000504c       ??_R4QTable@@6BQPaintDevice@@@ 1001004c     databaseEditdlg.obj
 0002:00005060       ??_R4databaseEditDlgBase@@6BQObject@@@ 10010060     databaseEditdlg.obj
 0002:00005074       ??_R4databaseEditDlgBase@@6BQPaintDevice@@@ 10010074     databaseEditdlg.obj
 0002:00005088       ??_R4QSpacerItem@@6B@      10010088     databaseEditdlg.obj
 0002:0000509c       ??_R3QSpacerItem@@8        1001009c     databaseEditdlg.obj
 0002:000050ac       ??_R2QSpacerItem@@8        100100ac     databaseEditdlg.obj
 0002:000050b8       ??_R1A@?0A@EA@QSpacerItem@@8 100100b8     databaseEditdlg.obj
 0002:000050d4       ??_R4QListView@@6BQObject@@@ 100100d4     toolwindow.obj
 0002:000050e8       ??_R3QListView@@8          100100e8     toolwindow.obj
 0002:000050f8       ??_R2QListView@@8          100100f8     toolwindow.obj
 0002:00005118       ??_R1A@?0A@EA@QListView@@8 10010118     toolwindow.obj
 0002:00005134       ??_R4QListView@@6BQPaintDevice@@@ 10010134     toolwindow.obj
 0002:00005148       ??_R4toolWindowBase@@6BQObject@@@ 10010148     toolwindow.obj
 0002:0000515c       ??_R4toolWindowBase@@6BQPaintDevice@@@ 1001015c     toolwindow.obj
 0002:00005170       ??_R4type_info@@6B@        10010170     MSVCRT:ti_inst.obj
 0002:00005184       ??_R3type_info@@8          10010184     MSVCRT:ti_inst.obj
 0002:00005194       ??_R2type_info@@8          10010194     MSVCRT:ti_inst.obj
 0002:0000519c       ??_R1A@?0A@EA@type_info@@8 1001019c     MSVCRT:ti_inst.obj
 0002:000051b8       ___rtc_iaa                 100101b8     MSVCRT:initsect.obj
 0002:000051bc       ___rtc_izz                 100101bc     MSVCRT:initsect.obj
 0002:000051c0       ___rtc_taa                 100101c0     MSVCRT:initsect.obj
 0002:000051c4       ___rtc_tzz                 100101c4     MSVCRT:initsect.obj
 0002:00006460       __IMPORT_DESCRIPTOR_config_icons 10011460     config_icons:config_icons.dll
 0002:00006474       __IMPORT_DESCRIPTOR_qt-mt323 10011474     qt-mt323:qt-mt323.dll
 0002:00006488       __IMPORT_DESCRIPTOR_KERNEL32 10011488     kernel32:KERNEL32.dll
 0002:0000649c       __IMPORT_DESCRIPTOR_MSVCR120 1001149c     MSVCRT:MSVCR120.dll
 0002:000064b0       __NULL_IMPORT_DESCRIPTOR   100114b0     config_icons:config_icons.dll
 0003:00000064       ___security_cookie         1001c064     MSVCRT:gs_cookie.obj
 0003:00000068       ___security_cookie_complement 1001c068     MSVCRT:gs_cookie.obj
 0003:00000070       ___native_dllmain_reason   1001c070     MSVCRT:natstart.obj
 0003:00000074       ??_R0?AUQShared@@@8        1001c074     databaseEdit.obj
 0003:0000008c       ??_R0?AVQGList@@@8         1001c08c     databaseEdit.obj
 0003:000000a4       ??_R0?AVQPtrCollection@@@8 1001c0a4     databaseEdit.obj
 0003:000000c4       ??_R0?AVQToolBar@@@8       1001c0c4     databaseEdit.obj
 0003:000000dc       ??_R0?AVQDockWindow@@@8    1001c0dc     databaseEdit.obj
 0003:000000f8       ??_R0?AVQFrame@@@8         1001c0f8     databaseEdit.obj
 0003:00000110       ??_R0?AVQWidget@@@8        1001c110     databaseEdit.obj
 0003:00000128       ??_R0?AVQObject@@@8        1001c128     databaseEdit.obj
 0003:00000140       ??_R0?AVQt@@@8             1001c140     databaseEdit.obj
 0003:00000154       ??_R0?AVQPaintDevice@@@8   1001c154     databaseEdit.obj
 0003:00000170       ??_R0?AVQPopupMenu@@@8     1001c170     databaseEdit.obj
 0003:0000018c       ??_R0?AVQMenuData@@@8      1001c18c     databaseEdit.obj
 0003:000001a4       ??_R0?AVQListViewItem@@@8  1001c1a4     databaseEdit.obj
 0003:000001c0       ??_R0?AVQAction@@@8        1001c1c0     databaseEdit.obj
 0003:000001d8       ??_R0?AVQGuardedPtrPrivate@@@8 1001c1d8     databaseEdit.obj
 0003:000001fc       ??_R0?AVQDockWindowList@@@8 1001c1fc     databaseEdit.obj
 0003:0000021c       ??_R0?AV?$QPtrList@VQDockWindow@@@@@8 1001c21c     databaseEdit.obj
 0003:00000244       ??_R0?AVQPopupMenuList@@@8 1001c244     databaseEdit.obj
 0003:00000264       ??_R0?AV?$QPtrList@VQPopupMenu@@@@@8 1001c264     databaseEdit.obj
 0003:0000028c       ??_R0?AVconfig_plugin_base@@@8 1001c28c     databaseEdit.obj
 0003:000002b0       ??_R0?AVQGDict@@@8         1001c2b0     databaseEdit.obj
 0003:000002c8       ??_R0?AVdatabaseEdit@@@8   1001c2c8     databaseEdit.obj
 0003:000002e4       ??_R0?AV?$QDict@VQAction@@@@@8 1001c2e4     databaseEdit.obj
 0003:00000308       ??_R0?AVdatabaseEditDlg@@@8 1001c308     databaseEditdlgimpl.obj
 0003:00000328       ??_R0?AVdatabaseEditDlgBase@@@8 1001c328     databaseEditdlgimpl.obj
 0003:0000034c       ??_R0?AV?$QIntDict@VQTable@@@@@8 1001c34c     databaseEditdlgimpl.obj
 0003:00000370       ??_R0?AVconfig_plugin_desc_base@@@8 1001c370     plugindesc.obj
 0003:00000398       ??_R0?AVplugindesc@@@8     1001c398     plugindesc.obj
 0003:000003b4       ??_R0?AVtoolWindow@@@8     1001c3b4     toolwindowimpl.obj
 0003:000003d0       ??_R0?AVtoolWindowBase@@@8 1001c3d0     toolwindowimpl.obj
 0003:000003f0       ??_R0?AVQVBoxLayout@@@8    1001c3f0     databaseEditdlg.obj
 0003:0000040c       ??_R0?AVQBoxLayout@@@8     1001c40c     databaseEditdlg.obj
 0003:00000428       ??_R0?AVQLayout@@@8        1001c428     databaseEditdlg.obj
 0003:00000440       ??_R0?AVQLayoutItem@@@8    1001c440     databaseEditdlg.obj
 0003:0000045c       ??_R0?AVQHBoxLayout@@@8    1001c45c     databaseEditdlg.obj
 0003:00000478       ??_R0?AVQLabel@@@8         1001c478     databaseEditdlg.obj
 0003:00000490       ??_R0?AVQTabWidget@@@8     1001c490     databaseEditdlg.obj
 0003:000004ac       ??_R0?AVQLineEdit@@@8      1001c4ac     databaseEditdlg.obj
 0003:000004c4       ??_R0?AVQTextEdit@@@8      1001c4c4     databaseEditdlg.obj
 0003:000004dc       ??_R0?AVQScrollView@@@8    1001c4dc     databaseEditdlg.obj
 0003:000004f8       ??_R0?AVQTable@@@8         1001c4f8     databaseEditdlg.obj
 0003:00000510       ??_R0?AVQSpacerItem@@@8    1001c510     databaseEditdlg.obj
 0003:0000052c       ??_R0?AVQListView@@@8      1001c52c     toolwindow.obj
 0003:00000544       ??_R0?AVtype_info@@@8      1001c544     MSVCRT:ti_inst.obj
 0003:00000560       ?metaObj@databaseEdit@@0PAVQMetaObject@@A 1001c560     moc_databaseEdit.obj
 0003:0000058c       ?metaObj@databaseEditDlgBase@@0PAVQMetaObject@@A 1001c58c     moc_databaseEditdlg.obj
 0003:00000594       ?metaObj@databaseEditDlg@@0PAVQMetaObject@@A 1001c594     moc_databaseEditdlgimpl.obj
 0003:000005c0       ?metaObj@toolWindowBase@@0PAVQMetaObject@@A 1001c5c0     moc_toolwindow.obj
 0003:000005c8       ?metaObj@toolWindow@@0PAVQMetaObject@@A 1001c5c8     moc_toolwindowimpl.obj
 0003:00000918       ?__type_info_root_node@@3U__type_info_node@@A 1001c918     MSVCRT:tncleanup.obj
 0003:00000920       ___native_startup_lock     1001c920     <common>
 0003:00000924       ___native_startup_state    1001c924     <common>
 0003:00000928       ___dyn_tls_init_callback   1001c928     <common>
 0003:0000092c       ___onexitend               1001c92c     <common>
 0003:00000930       ___onexitbegin             1001c930     <common>

 entry point at        0001:000084e2

 Static symbols

 0001:00000000       ??__EcleanUp_databaseEdit@@YAXXZ 10001000 f   moc_databaseEdit.obj
 0001:00000021       ??__EcleanUp_databaseEditDlgBase@@YAXXZ 10001021 f   moc_databaseEditdlg.obj
 0001:00000042       ??__EcleanUp_databaseEditDlg@@YAXXZ 10001042 f   moc_databaseEditdlgimpl.obj
 0001:00000063       ??__EcleanUp_toolWindowBase@@YAXXZ 10001063 f   moc_toolwindow.obj
 0001:00000084       ??__EcleanUp_toolWindow@@YAXXZ 10001084 f   moc_toolwindowimpl.obj
 0001:0000829f       _pre_c_init                1000929f f   MSVCRT:crtdll.obj
 0001:00008505       ___DllMainCRTStartup       10009505 f   MSVCRT:crtdll.obj
 0001:00008780       $$000000                   10009780     MSVCRT:sehprolg4.obj
 0001:00008a9c       __unwindfunclet$??0config_plugin_base@@QAE@ABVQString@@00@Z$0 10009a9c f   databaseEdit.obj
 0001:00008aa5       __unwindfunclet$??0config_plugin_base@@QAE@ABVQString@@00@Z$1 10009aa5 f   databaseEdit.obj
 0001:00008ab1       __unwindfunclet$??0config_plugin_base@@QAE@ABVQString@@00@Z$2 10009ab1 f   databaseEdit.obj
 0001:00008abd       __unwindfunclet$??0config_plugin_base@@QAE@ABVQString@@00@Z$3 10009abd f   databaseEdit.obj
 0001:00008ac9       __ehhandler$??0config_plugin_base@@QAE@ABVQString@@00@Z 10009ac9 f   databaseEdit.obj
 0001:00008ae4       __unwindfunclet$??0databaseEdit@@QAE@ABVQString@@00@Z$0 10009ae4 f   databaseEdit.obj
 0001:00008aec       __unwindfunclet$??0databaseEdit@@QAE@ABVQString@@00@Z$1 10009aec f   databaseEdit.obj
 0001:00008af7       __unwindfunclet$??0databaseEdit@@QAE@ABVQString@@00@Z$2 10009af7 f   databaseEdit.obj
 0001:00008b02       __unwindfunclet$??0databaseEdit@@QAE@ABVQString@@00@Z$3 10009b02 f   databaseEdit.obj
 0001:00008b10       __unwindfunclet$??0databaseEdit@@QAE@ABVQString@@00@Z$4 10009b10 f   databaseEdit.obj
 0001:00008b1e       __unwindfunclet$??0databaseEdit@@QAE@ABVQString@@00@Z$5 10009b1e f   databaseEdit.obj
 0001:00008b2d       __unwindfunclet$??0databaseEdit@@QAE@ABVQString@@00@Z$6 10009b2d f   databaseEdit.obj
 0001:00008b37       __unwindfunclet$??0databaseEdit@@QAE@ABVQString@@00@Z$7 10009b37 f   databaseEdit.obj
 0001:00008b41       __unwindfunclet$??0databaseEdit@@QAE@ABVQString@@00@Z$8 10009b41 f   databaseEdit.obj
 0001:00008b5b       __unwindfunclet$??0databaseEdit@@QAE@ABVQString@@00@Z$9 10009b5b f   databaseEdit.obj
 0001:00008b64       __unwindfunclet$??0databaseEdit@@QAE@ABVQString@@00@Z$10 10009b64 f   databaseEdit.obj
 0001:00008b6e       __unwindfunclet$??0databaseEdit@@QAE@ABVQString@@00@Z$11 10009b6e f   databaseEdit.obj
 0001:00008b78       __unwindfunclet$??0databaseEdit@@QAE@ABVQString@@00@Z$12 10009b78 f   databaseEdit.obj
 0001:00008b92       __unwindfunclet$??0databaseEdit@@QAE@ABVQString@@00@Z$13 10009b92 f   databaseEdit.obj
 0001:00008b9c       __unwindfunclet$??0databaseEdit@@QAE@ABVQString@@00@Z$14 10009b9c f   databaseEdit.obj
 0001:00008ba6       __unwindfunclet$??0databaseEdit@@QAE@ABVQString@@00@Z$15 10009ba6 f   databaseEdit.obj
 0001:00008bc0       __unwindfunclet$??0databaseEdit@@QAE@ABVQString@@00@Z$16 10009bc0 f   databaseEdit.obj
 0001:00008bda       __unwindfunclet$??0databaseEdit@@QAE@ABVQString@@00@Z$17 10009bda f   databaseEdit.obj
 0001:00008bf4       __unwindfunclet$??0databaseEdit@@QAE@ABVQString@@00@Z$18 10009bf4 f   databaseEdit.obj
 0001:00008c0e       __unwindfunclet$??0databaseEdit@@QAE@ABVQString@@00@Z$20 10009c0e f   databaseEdit.obj
 0001:00008c17       __unwindfunclet$??0databaseEdit@@QAE@ABVQString@@00@Z$21 10009c17 f   databaseEdit.obj
 0001:00008c20       __unwindfunclet$??0databaseEdit@@QAE@ABVQString@@00@Z$22 10009c20 f   databaseEdit.obj
 0001:00008c29       __ehhandler$??0databaseEdit@@QAE@ABVQString@@00@Z 10009c29 f   databaseEdit.obj
 0001:00008c44       __unwindfunclet$??1?$QDict@VQAction@@@@UAE@XZ$0 10009c44 f   databaseEdit.obj
 0001:00008c44       __unwindfunclet$??1?$QIntDict@VQTable@@@@UAE@XZ$0 10009c44 f   databaseEdit.obj
 0001:00008c4d       __ehhandler$??1?$QDict@VQAction@@@@UAE@XZ 10009c4d f   databaseEdit.obj
 0001:00008c4d       __ehhandler$??1?$QIntDict@VQTable@@@@UAE@XZ 10009c4d f   databaseEdit.obj
 0001:00008c68       __unwindfunclet$??1?$QPtrList@VQPopupMenu@@@@UAE@XZ$0 10009c68 f   databaseEdit.obj
 0001:00008c71       __ehhandler$??1?$QPtrList@VQPopupMenu@@@@UAE@XZ 10009c71 f   databaseEdit.obj
 0001:00008c8c       __unwindfunclet$??1QDockWindowList@@UAE@XZ$0 10009c8c f   databaseEdit.obj
 0001:00008c95       __unwindfunclet$??1QDockWindowList@@UAE@XZ$1 10009c95 f   databaseEdit.obj
 0001:00008c9e       __ehhandler$??1QDockWindowList@@UAE@XZ 10009c9e f   databaseEdit.obj
 0001:00008cb9       __unwindfunclet$??1QPopupMenuList@@UAE@XZ$0 10009cb9 f   databaseEdit.obj
 0001:00008cc1       __ehhandler$??1QPopupMenuList@@UAE@XZ 10009cc1 f   databaseEdit.obj
 0001:00008cdc       __unwindfunclet$??1config_plugin_base@@UAE@XZ$0 10009cdc f   databaseEdit.obj
 0001:00008ce5       __unwindfunclet$??1config_plugin_base@@UAE@XZ$1 10009ce5 f   databaseEdit.obj
 0001:00008cf1       __unwindfunclet$??1config_plugin_base@@UAE@XZ$2 10009cf1 f   databaseEdit.obj
 0001:00008cfd       __ehhandler$??1config_plugin_base@@UAE@XZ 10009cfd f   databaseEdit.obj
 0001:00008d18       __unwindfunclet$??1databaseEdit@@UAE@XZ$0 10009d18 f   databaseEdit.obj
 0001:00008d20       __unwindfunclet$??1databaseEdit@@UAE@XZ$1 10009d20 f   databaseEdit.obj
 0001:00008d2b       __unwindfunclet$??1databaseEdit@@UAE@XZ$2 10009d2b f   databaseEdit.obj
 0001:00008d36       __unwindfunclet$??1databaseEdit@@UAE@XZ$3 10009d36 f   databaseEdit.obj
 0001:00008d44       __unwindfunclet$??1databaseEdit@@UAE@XZ$4 10009d44 f   databaseEdit.obj
 0001:00008d52       __unwindfunclet$??1databaseEdit@@UAE@XZ$5 10009d52 f   databaseEdit.obj
 0001:00008d61       __ehhandler$??1databaseEdit@@UAE@XZ 10009d61 f   databaseEdit.obj
 0001:00008d7c       __unwindfunclet$?about@config_plugin_base@@UAE?AVQString@@XZ$0 10009d7c f   databaseEdit.obj
 0001:00008d85       __unwindfunclet$?about@config_plugin_base@@UAE?AVQString@@XZ$1 10009d85 f   databaseEdit.obj
 0001:00008d9f       __ehhandler$?about@config_plugin_base@@UAE?AVQString@@XZ 10009d9f f   databaseEdit.obj
 0001:00008dba       __unwindfunclet$?about@databaseEdit@@UAE?AVQString@@XZ$0 10009dba f   databaseEdit.obj
 0001:00008dc3       __unwindfunclet$?about@databaseEdit@@UAE?AVQString@@XZ$1 10009dc3 f   databaseEdit.obj
 0001:00008dcc       __unwindfunclet$?about@databaseEdit@@UAE?AVQString@@XZ$2 10009dcc f   databaseEdit.obj
 0001:00008dd5       __unwindfunclet$?about@databaseEdit@@UAE?AVQString@@XZ$3 10009dd5 f   databaseEdit.obj
 0001:00008dde       __unwindfunclet$?about@databaseEdit@@UAE?AVQString@@XZ$4 10009dde f   databaseEdit.obj
 0001:00008df8       __ehhandler$?about@databaseEdit@@UAE?AVQString@@XZ 10009df8 f   databaseEdit.obj
 0001:00008e13       __unwindfunclet$?activate@databaseEdit@@UAEX_N@Z$0 10009e13 f   databaseEdit.obj
 0001:00008e1c       __unwindfunclet$?activate@databaseEdit@@UAEX_N@Z$2 10009e1c f   databaseEdit.obj
 0001:00008e25       __unwindfunclet$?activate@databaseEdit@@UAEX_N@Z$4 10009e25 f   databaseEdit.obj
 0001:00008e2e       __unwindfunclet$?activate@databaseEdit@@UAEX_N@Z$6 10009e2e f   databaseEdit.obj
 0001:00008e37       __unwindfunclet$?activate@databaseEdit@@UAEX_N@Z$8 10009e37 f   databaseEdit.obj
 0001:00008e40       __unwindfunclet$?activate@databaseEdit@@UAEX_N@Z$10 10009e40 f   databaseEdit.obj
 0001:00008e49       __unwindfunclet$?activate@databaseEdit@@UAEX_N@Z$12 10009e49 f   databaseEdit.obj
 0001:00008e52       __unwindfunclet$?activate@databaseEdit@@UAEX_N@Z$14 10009e52 f   databaseEdit.obj
 0001:00008e5b       __unwindfunclet$?activate@databaseEdit@@UAEX_N@Z$16 10009e5b f   databaseEdit.obj
 0001:00008e64       __unwindfunclet$?activate@databaseEdit@@UAEX_N@Z$18 10009e64 f   databaseEdit.obj
 0001:00008e6d       __unwindfunclet$?activate@databaseEdit@@UAEX_N@Z$20 10009e6d f   databaseEdit.obj
 0001:00008e76       __unwindfunclet$?activate@databaseEdit@@UAEX_N@Z$22 10009e76 f   databaseEdit.obj
 0001:00008e7f       __unwindfunclet$?activate@databaseEdit@@UAEX_N@Z$24 10009e7f f   databaseEdit.obj
 0001:00008e88       __unwindfunclet$?activate@databaseEdit@@UAEX_N@Z$25 10009e88 f   databaseEdit.obj
 0001:00008e91       __unwindfunclet$?activate@databaseEdit@@UAEX_N@Z$26 10009e91 f   databaseEdit.obj
 0001:00008e9a       __unwindfunclet$?activate@databaseEdit@@UAEX_N@Z$27 10009e9a f   databaseEdit.obj
 0001:00008ea3       __unwindfunclet$?activate@databaseEdit@@UAEX_N@Z$28 10009ea3 f   databaseEdit.obj
 0001:00008eac       __unwindfunclet$?activate@databaseEdit@@UAEX_N@Z$29 10009eac f   databaseEdit.obj
 0001:00008eb5       __unwindfunclet$?activate@databaseEdit@@UAEX_N@Z$30 10009eb5 f   databaseEdit.obj
 0001:00008ebe       __unwindfunclet$?activate@databaseEdit@@UAEX_N@Z$31 10009ebe f   databaseEdit.obj
 0001:00008ec7       __unwindfunclet$?activate@databaseEdit@@UAEX_N@Z$32 10009ec7 f   databaseEdit.obj
 0001:00008ed0       __unwindfunclet$?activate@databaseEdit@@UAEX_N@Z$33 10009ed0 f   databaseEdit.obj
 0001:00008ed9       __ehhandler$?activate@databaseEdit@@UAEX_N@Z 10009ed9 f   databaseEdit.obj
 0001:00008ef4       __unwindfunclet$?apply@databaseEdit@@UAEXXZ$0 10009ef4 f   databaseEdit.obj
 0001:00008efd       __unwindfunclet$?apply@databaseEdit@@UAEXXZ$1 10009efd f   databaseEdit.obj
 0001:00008f06       __unwindfunclet$?apply@databaseEdit@@UAEXXZ$2 10009f06 f   databaseEdit.obj
 0001:00008f0f       __ehhandler$?apply@databaseEdit@@UAEXXZ 10009f0f f   databaseEdit.obj
 0001:00008f2a       __unwindfunclet$?closeEvent@databaseEdit@@UAEXPAVQCloseEvent@@@Z$0 10009f2a f   databaseEdit.obj
 0001:00008f33       __unwindfunclet$?closeEvent@databaseEdit@@UAEXPAVQCloseEvent@@@Z$2 10009f33 f   databaseEdit.obj
 0001:00008f3c       __unwindfunclet$?closeEvent@databaseEdit@@UAEXPAVQCloseEvent@@@Z$4 10009f3c f   databaseEdit.obj
 0001:00008f45       __unwindfunclet$?closeEvent@databaseEdit@@UAEXPAVQCloseEvent@@@Z$6 10009f45 f   databaseEdit.obj
 0001:00008f4e       __unwindfunclet$?closeEvent@databaseEdit@@UAEXPAVQCloseEvent@@@Z$8 10009f4e f   databaseEdit.obj
 0001:00008f57       __unwindfunclet$?closeEvent@databaseEdit@@UAEXPAVQCloseEvent@@@Z$10 10009f57 f   databaseEdit.obj
 0001:00008f60       __unwindfunclet$?closeEvent@databaseEdit@@UAEXPAVQCloseEvent@@@Z$12 10009f60 f   databaseEdit.obj
 0001:00008f69       __unwindfunclet$?closeEvent@databaseEdit@@UAEXPAVQCloseEvent@@@Z$14 10009f69 f   databaseEdit.obj
 0001:00008f72       __unwindfunclet$?closeEvent@databaseEdit@@UAEXPAVQCloseEvent@@@Z$16 10009f72 f   databaseEdit.obj
 0001:00008f7b       __unwindfunclet$?closeEvent@databaseEdit@@UAEXPAVQCloseEvent@@@Z$18 10009f7b f   databaseEdit.obj
 0001:00008f84       __unwindfunclet$?closeEvent@databaseEdit@@UAEXPAVQCloseEvent@@@Z$20 10009f84 f   databaseEdit.obj
 0001:00008f8d       __ehhandler$?closeEvent@databaseEdit@@UAEXPAVQCloseEvent@@@Z 10009f8d f   databaseEdit.obj
 0001:00008fa8       __unwindfunclet$?db@@YAXABVQString@@@Z$0 10009fa8 f   databaseEdit.obj
 0001:00008fb1       __ehhandler$?db@@YAXABVQString@@@Z 10009fb1 f   databaseEdit.obj
 0001:00008fce       __unwindfunclet$?fileSelected@databaseEdit@@AAEXABVQString@@@Z$0 10009fce f   databaseEdit.obj
 0001:00008fd7       __unwindfunclet$?fileSelected@databaseEdit@@AAEXABVQString@@@Z$2 10009fd7 f   databaseEdit.obj
 0001:00008fe0       __unwindfunclet$?fileSelected@databaseEdit@@AAEXABVQString@@@Z$4 10009fe0 f   databaseEdit.obj
 0001:00008fe9       __unwindfunclet$?fileSelected@databaseEdit@@AAEXABVQString@@@Z$6 10009fe9 f   databaseEdit.obj
 0001:00008ff2       __unwindfunclet$?fileSelected@databaseEdit@@AAEXABVQString@@@Z$8 10009ff2 f   databaseEdit.obj
 0001:00008ffb       __unwindfunclet$?fileSelected@databaseEdit@@AAEXABVQString@@@Z$10 10009ffb f   databaseEdit.obj
 0001:00009004       __unwindfunclet$?fileSelected@databaseEdit@@AAEXABVQString@@@Z$12 1000a004 f   databaseEdit.obj
 0001:0000900d       __unwindfunclet$?fileSelected@databaseEdit@@AAEXABVQString@@@Z$14 1000a00d f   databaseEdit.obj
 0001:00009016       __unwindfunclet$?fileSelected@databaseEdit@@AAEXABVQString@@@Z$16 1000a016 f   databaseEdit.obj
 0001:0000901f       __unwindfunclet$?fileSelected@databaseEdit@@AAEXABVQString@@@Z$18 1000a01f f   databaseEdit.obj
 0001:00009028       __unwindfunclet$?fileSelected@databaseEdit@@AAEXABVQString@@@Z$20 1000a028 f   databaseEdit.obj
 0001:00009031       __unwindfunclet$?fileSelected@databaseEdit@@AAEXABVQString@@@Z$22 1000a031 f   databaseEdit.obj
 0001:0000903a       __ehhandler$?fileSelected@databaseEdit@@AAEXABVQString@@@Z 1000a03a f   databaseEdit.obj
 0001:00009055       __unwindfunclet$?menus@databaseEdit@@UAE?AVQPopupMenuList@@XZ$0 1000a055 f   databaseEdit.obj
 0001:0000906e       __ehhandler$?menus@databaseEdit@@UAE?AVQPopupMenuList@@XZ 1000a06e f   databaseEdit.obj
 0001:00009089       __unwindfunclet$?navigate@databaseEdit@@UAEXABVQString@@0@Z$0 1000a089 f   databaseEdit.obj
 0001:00009092       __unwindfunclet$?navigate@databaseEdit@@UAEXABVQString@@0@Z$1 1000a092 f   databaseEdit.obj
 0001:0000909b       __unwindfunclet$?navigate@databaseEdit@@UAEXABVQString@@0@Z$2 1000a09b f   databaseEdit.obj
 0001:000090a4       __ehhandler$?navigate@databaseEdit@@UAEXABVQString@@0@Z 1000a0a4 f   databaseEdit.obj
 0001:000090bf       __unwindfunclet$?reply@databaseEdit@@UAEXPAVresponse@@@Z$0 1000a0bf f   databaseEdit.obj
 0001:000090cb       __unwindfunclet$?reply@databaseEdit@@UAEXPAVresponse@@@Z$1 1000a0cb f   databaseEdit.obj
 0001:000090d7       __unwindfunclet$?reply@databaseEdit@@UAEXPAVresponse@@@Z$2 1000a0d7 f   databaseEdit.obj
 0001:000090e3       __unwindfunclet$?reply@databaseEdit@@UAEXPAVresponse@@@Z$3 1000a0e3 f   databaseEdit.obj
 0001:000090ef       __unwindfunclet$?reply@databaseEdit@@UAEXPAVresponse@@@Z$4 1000a0ef f   databaseEdit.obj
 0001:000090fb       __unwindfunclet$?reply@databaseEdit@@UAEXPAVresponse@@@Z$5 1000a0fb f   databaseEdit.obj
 0001:00009107       __unwindfunclet$?reply@databaseEdit@@UAEXPAVresponse@@@Z$6 1000a107 f   databaseEdit.obj
 0001:00009113       __unwindfunclet$?reply@databaseEdit@@UAEXPAVresponse@@@Z$7 1000a113 f   databaseEdit.obj
 0001:0000911f       __unwindfunclet$?reply@databaseEdit@@UAEXPAVresponse@@@Z$8 1000a11f f   databaseEdit.obj
 0001:0000912b       __unwindfunclet$?reply@databaseEdit@@UAEXPAVresponse@@@Z$9 1000a12b f   databaseEdit.obj
 0001:00009137       __unwindfunclet$?reply@databaseEdit@@UAEXPAVresponse@@@Z$10 1000a137 f   databaseEdit.obj
 0001:00009143       __unwindfunclet$?reply@databaseEdit@@UAEXPAVresponse@@@Z$11 1000a143 f   databaseEdit.obj
 0001:0000914f       __unwindfunclet$?reply@databaseEdit@@UAEXPAVresponse@@@Z$12 1000a14f f   databaseEdit.obj
 0001:0000915b       __unwindfunclet$?reply@databaseEdit@@UAEXPAVresponse@@@Z$13 1000a15b f   databaseEdit.obj
 0001:00009167       __unwindfunclet$?reply@databaseEdit@@UAEXPAVresponse@@@Z$14 1000a167 f   databaseEdit.obj
 0001:00009173       __unwindfunclet$?reply@databaseEdit@@UAEXPAVresponse@@@Z$15 1000a173 f   databaseEdit.obj
 0001:0000917f       __unwindfunclet$?reply@databaseEdit@@UAEXPAVresponse@@@Z$16 1000a17f f   databaseEdit.obj
 0001:0000918b       __unwindfunclet$?reply@databaseEdit@@UAEXPAVresponse@@@Z$17 1000a18b f   databaseEdit.obj
 0001:00009198       __unwindfunclet$?reply@databaseEdit@@UAEXPAVresponse@@@Z$18 1000a198 f   databaseEdit.obj
 0001:000091a4       __unwindfunclet$?reply@databaseEdit@@UAEXPAVresponse@@@Z$19 1000a1a4 f   databaseEdit.obj
 0001:000091b0       __unwindfunclet$?reply@databaseEdit@@UAEXPAVresponse@@@Z$20 1000a1b0 f   databaseEdit.obj
 0001:000091bc       __unwindfunclet$?reply@databaseEdit@@UAEXPAVresponse@@@Z$21 1000a1bc f   databaseEdit.obj
 0001:000091c8       __unwindfunclet$?reply@databaseEdit@@UAEXPAVresponse@@@Z$22 1000a1c8 f   databaseEdit.obj
 0001:000091d4       __unwindfunclet$?reply@databaseEdit@@UAEXPAVresponse@@@Z$23 1000a1d4 f   databaseEdit.obj
 0001:000091e0       __unwindfunclet$?reply@databaseEdit@@UAEXPAVresponse@@@Z$24 1000a1e0 f   databaseEdit.obj
 0001:000091ec       __unwindfunclet$?reply@databaseEdit@@UAEXPAVresponse@@@Z$26 1000a1ec f   databaseEdit.obj
 0001:000091f8       __unwindfunclet$?reply@databaseEdit@@UAEXPAVresponse@@@Z$27 1000a1f8 f   databaseEdit.obj
 0001:00009204       __unwindfunclet$?reply@databaseEdit@@UAEXPAVresponse@@@Z$28 1000a204 f   databaseEdit.obj
 0001:00009210       __unwindfunclet$?reply@databaseEdit@@UAEXPAVresponse@@@Z$29 1000a210 f   databaseEdit.obj
 0001:00009233       __unwindfunclet$?reply@databaseEdit@@UAEXPAVresponse@@@Z$30 1000a233 f   databaseEdit.obj
 0001:00009256       __unwindfunclet$?reply@databaseEdit@@UAEXPAVresponse@@@Z$31 1000a256 f   databaseEdit.obj
 0001:00009279       __unwindfunclet$?reply@databaseEdit@@UAEXPAVresponse@@@Z$32 1000a279 f   databaseEdit.obj
 0001:00009285       __unwindfunclet$?reply@databaseEdit@@UAEXPAVresponse@@@Z$33 1000a285 f   databaseEdit.obj
 0001:00009291       __unwindfunclet$?reply@databaseEdit@@UAEXPAVresponse@@@Z$34 1000a291 f   databaseEdit.obj
 0001:0000929d       __unwindfunclet$?reply@databaseEdit@@UAEXPAVresponse@@@Z$35 1000a29d f   databaseEdit.obj
 0001:000092a9       __unwindfunclet$?reply@databaseEdit@@UAEXPAVresponse@@@Z$36 1000a2a9 f   databaseEdit.obj
 0001:000092b5       __unwindfunclet$?reply@databaseEdit@@UAEXPAVresponse@@@Z$37 1000a2b5 f   databaseEdit.obj
 0001:000092c1       __unwindfunclet$?reply@databaseEdit@@UAEXPAVresponse@@@Z$38 1000a2c1 f   databaseEdit.obj
 0001:000092cd       __unwindfunclet$?reply@databaseEdit@@UAEXPAVresponse@@@Z$39 1000a2cd f   databaseEdit.obj
 0001:000092d9       __unwindfunclet$?reply@databaseEdit@@UAEXPAVresponse@@@Z$40 1000a2d9 f   databaseEdit.obj
 0001:000092e5       __unwindfunclet$?reply@databaseEdit@@UAEXPAVresponse@@@Z$41 1000a2e5 f   databaseEdit.obj
 0001:000092f1       __unwindfunclet$?reply@databaseEdit@@UAEXPAVresponse@@@Z$42 1000a2f1 f   databaseEdit.obj
 0001:000092fd       __unwindfunclet$?reply@databaseEdit@@UAEXPAVresponse@@@Z$43 1000a2fd f   databaseEdit.obj
 0001:00009309       __unwindfunclet$?reply@databaseEdit@@UAEXPAVresponse@@@Z$44 1000a309 f   databaseEdit.obj
 0001:00009315       __unwindfunclet$?reply@databaseEdit@@UAEXPAVresponse@@@Z$45 1000a315 f   databaseEdit.obj
 0001:00009321       __unwindfunclet$?reply@databaseEdit@@UAEXPAVresponse@@@Z$46 1000a321 f   databaseEdit.obj
 0001:0000932d       __unwindfunclet$?reply@databaseEdit@@UAEXPAVresponse@@@Z$47 1000a32d f   databaseEdit.obj
 0001:00009339       __unwindfunclet$?reply@databaseEdit@@UAEXPAVresponse@@@Z$48 1000a339 f   databaseEdit.obj
 0001:00009345       __unwindfunclet$?reply@databaseEdit@@UAEXPAVresponse@@@Z$49 1000a345 f   databaseEdit.obj
 0001:00009351       __unwindfunclet$?reply@databaseEdit@@UAEXPAVresponse@@@Z$50 1000a351 f   databaseEdit.obj
 0001:0000935d       __unwindfunclet$?reply@databaseEdit@@UAEXPAVresponse@@@Z$51 1000a35d f   databaseEdit.obj
 0001:00009369       __unwindfunclet$?reply@databaseEdit@@UAEXPAVresponse@@@Z$52 1000a369 f   databaseEdit.obj
 0001:00009375       __unwindfunclet$?reply@databaseEdit@@UAEXPAVresponse@@@Z$53 1000a375 f   databaseEdit.obj
 0001:00009381       __unwindfunclet$?reply@databaseEdit@@UAEXPAVresponse@@@Z$54 1000a381 f   databaseEdit.obj
 0001:0000938d       __unwindfunclet$?reply@databaseEdit@@UAEXPAVresponse@@@Z$55 1000a38d f   databaseEdit.obj
 0001:00009399       __unwindfunclet$?reply@databaseEdit@@UAEXPAVresponse@@@Z$56 1000a399 f   databaseEdit.obj
 0001:000093a5       __unwindfunclet$?reply@databaseEdit@@UAEXPAVresponse@@@Z$57 1000a3a5 f   databaseEdit.obj
 0001:000093b1       __unwindfunclet$?reply@databaseEdit@@UAEXPAVresponse@@@Z$58 1000a3b1 f   databaseEdit.obj
 0001:000093bd       __unwindfunclet$?reply@databaseEdit@@UAEXPAVresponse@@@Z$59 1000a3bd f   databaseEdit.obj
 0001:000093c9       __unwindfunclet$?reply@databaseEdit@@UAEXPAVresponse@@@Z$60 1000a3c9 f   databaseEdit.obj
 0001:000093d5       __unwindfunclet$?reply@databaseEdit@@UAEXPAVresponse@@@Z$61 1000a3d5 f   databaseEdit.obj
 0001:000093e1       __unwindfunclet$?reply@databaseEdit@@UAEXPAVresponse@@@Z$62 1000a3e1 f   databaseEdit.obj
 0001:000093ed       __unwindfunclet$?reply@databaseEdit@@UAEXPAVresponse@@@Z$63 1000a3ed f   databaseEdit.obj
 0001:000093f9       __unwindfunclet$?reply@databaseEdit@@UAEXPAVresponse@@@Z$64 1000a3f9 f   databaseEdit.obj
 0001:00009405       __unwindfunclet$?reply@databaseEdit@@UAEXPAVresponse@@@Z$65 1000a405 f   databaseEdit.obj
 0001:00009411       __unwindfunclet$?reply@databaseEdit@@UAEXPAVresponse@@@Z$66 1000a411 f   databaseEdit.obj
 0001:0000941d       __unwindfunclet$?reply@databaseEdit@@UAEXPAVresponse@@@Z$67 1000a41d f   databaseEdit.obj
 0001:00009429       __unwindfunclet$?reply@databaseEdit@@UAEXPAVresponse@@@Z$68 1000a429 f   databaseEdit.obj
 0001:00009435       __unwindfunclet$?reply@databaseEdit@@UAEXPAVresponse@@@Z$69 1000a435 f   databaseEdit.obj
 0001:00009441       __unwindfunclet$?reply@databaseEdit@@UAEXPAVresponse@@@Z$70 1000a441 f   databaseEdit.obj
 0001:0000944d       __unwindfunclet$?reply@databaseEdit@@UAEXPAVresponse@@@Z$71 1000a44d f   databaseEdit.obj
 0001:00009459       __unwindfunclet$?reply@databaseEdit@@UAEXPAVresponse@@@Z$72 1000a459 f   databaseEdit.obj
 0001:00009465       __unwindfunclet$?reply@databaseEdit@@UAEXPAVresponse@@@Z$73 1000a465 f   databaseEdit.obj
 0001:00009471       __unwindfunclet$?reply@databaseEdit@@UAEXPAVresponse@@@Z$74 1000a471 f   databaseEdit.obj
 0001:0000947d       __unwindfunclet$?reply@databaseEdit@@UAEXPAVresponse@@@Z$75 1000a47d f   databaseEdit.obj
 0001:00009489       __unwindfunclet$?reply@databaseEdit@@UAEXPAVresponse@@@Z$76 1000a489 f   databaseEdit.obj
 0001:00009495       __unwindfunclet$?reply@databaseEdit@@UAEXPAVresponse@@@Z$77 1000a495 f   databaseEdit.obj
 0001:000094a1       __unwindfunclet$?reply@databaseEdit@@UAEXPAVresponse@@@Z$78 1000a4a1 f   databaseEdit.obj
 0001:000094ad       __unwindfunclet$?reply@databaseEdit@@UAEXPAVresponse@@@Z$79 1000a4ad f   databaseEdit.obj
 0001:000094b9       __unwindfunclet$?reply@databaseEdit@@UAEXPAVresponse@@@Z$80 1000a4b9 f   databaseEdit.obj
 0001:000094c5       __unwindfunclet$?reply@databaseEdit@@UAEXPAVresponse@@@Z$81 1000a4c5 f   databaseEdit.obj
 0001:000094d1       __unwindfunclet$?reply@databaseEdit@@UAEXPAVresponse@@@Z$82 1000a4d1 f   databaseEdit.obj
 0001:000094dd       __unwindfunclet$?reply@databaseEdit@@UAEXPAVresponse@@@Z$83 1000a4dd f   databaseEdit.obj
 0001:000094e9       __unwindfunclet$?reply@databaseEdit@@UAEXPAVresponse@@@Z$84 1000a4e9 f   databaseEdit.obj
 0001:000094f5       __unwindfunclet$?reply@databaseEdit@@UAEXPAVresponse@@@Z$85 1000a4f5 f   databaseEdit.obj
 0001:00009501       __unwindfunclet$?reply@databaseEdit@@UAEXPAVresponse@@@Z$86 1000a501 f   databaseEdit.obj
 0001:0000950d       __unwindfunclet$?reply@databaseEdit@@UAEXPAVresponse@@@Z$87 1000a50d f   databaseEdit.obj
 0001:00009519       __unwindfunclet$?reply@databaseEdit@@UAEXPAVresponse@@@Z$88 1000a519 f   databaseEdit.obj
 0001:00009525       __unwindfunclet$?reply@databaseEdit@@UAEXPAVresponse@@@Z$89 1000a525 f   databaseEdit.obj
 0001:00009531       __unwindfunclet$?reply@databaseEdit@@UAEXPAVresponse@@@Z$90 1000a531 f   databaseEdit.obj
 0001:0000953d       __unwindfunclet$?reply@databaseEdit@@UAEXPAVresponse@@@Z$91 1000a53d f   databaseEdit.obj
 0001:00009549       __unwindfunclet$?reply@databaseEdit@@UAEXPAVresponse@@@Z$92 1000a549 f   databaseEdit.obj
 0001:00009555       __unwindfunclet$?reply@databaseEdit@@UAEXPAVresponse@@@Z$93 1000a555 f   databaseEdit.obj
 0001:00009561       __unwindfunclet$?reply@databaseEdit@@UAEXPAVresponse@@@Z$94 1000a561 f   databaseEdit.obj
 0001:0000956d       __unwindfunclet$?reply@databaseEdit@@UAEXPAVresponse@@@Z$95 1000a56d f   databaseEdit.obj
 0001:00009579       __unwindfunclet$?reply@databaseEdit@@UAEXPAVresponse@@@Z$96 1000a579 f   databaseEdit.obj
 0001:00009585       __unwindfunclet$?reply@databaseEdit@@UAEXPAVresponse@@@Z$97 1000a585 f   databaseEdit.obj
 0001:00009591       __unwindfunclet$?reply@databaseEdit@@UAEXPAVresponse@@@Z$98 1000a591 f   databaseEdit.obj
 0001:0000959d       __unwindfunclet$?reply@databaseEdit@@UAEXPAVresponse@@@Z$99 1000a59d f   databaseEdit.obj
 0001:000095a9       __unwindfunclet$?reply@databaseEdit@@UAEXPAVresponse@@@Z$100 1000a5a9 f   databaseEdit.obj
 0001:000095b5       __unwindfunclet$?reply@databaseEdit@@UAEXPAVresponse@@@Z$101 1000a5b5 f   databaseEdit.obj
 0001:000095c1       __unwindfunclet$?reply@databaseEdit@@UAEXPAVresponse@@@Z$102 1000a5c1 f   databaseEdit.obj
 0001:000095cd       __unwindfunclet$?reply@databaseEdit@@UAEXPAVresponse@@@Z$103 1000a5cd f   databaseEdit.obj
 0001:000095d9       __unwindfunclet$?reply@databaseEdit@@UAEXPAVresponse@@@Z$104 1000a5d9 f   databaseEdit.obj
 0001:000095e5       __unwindfunclet$?reply@databaseEdit@@UAEXPAVresponse@@@Z$105 1000a5e5 f   databaseEdit.obj
 0001:000095f1       __unwindfunclet$?reply@databaseEdit@@UAEXPAVresponse@@@Z$106 1000a5f1 f   databaseEdit.obj
 0001:000095fd       __unwindfunclet$?reply@databaseEdit@@UAEXPAVresponse@@@Z$107 1000a5fd f   databaseEdit.obj
 0001:00009609       __unwindfunclet$?reply@databaseEdit@@UAEXPAVresponse@@@Z$108 1000a609 f   databaseEdit.obj
 0001:00009615       __ehhandler$?reply@databaseEdit@@UAEXPAVresponse@@@Z 1000a615 f   databaseEdit.obj
 0001:0000963d       __unwindfunclet$?toolbars@databaseEdit@@UAE?AVQDockWindowList@@XZ$0 1000a63d f   databaseEdit.obj
 0001:00009656       __ehhandler$?toolbars@databaseEdit@@UAE?AVQDockWindowList@@XZ 1000a656 f   databaseEdit.obj
 0001:00009671       __unwindfunclet$??0databaseEditDlg@@QAE@ABVQString@@PAVQWidget@@PBDI@Z$0 1000a671 f   databaseEditdlgimpl.obj
 0001:00009679       __unwindfunclet$??0databaseEditDlg@@QAE@ABVQString@@PAVQWidget@@PBDI@Z$1 1000a679 f   databaseEditdlgimpl.obj
 0001:00009688       __unwindfunclet$??0databaseEditDlg@@QAE@ABVQString@@PAVQWidget@@PBDI@Z$2 1000a688 f   databaseEditdlgimpl.obj
 0001:00009697       __unwindfunclet$??0databaseEditDlg@@QAE@ABVQString@@PAVQWidget@@PBDI@Z$3 1000a697 f   databaseEditdlgimpl.obj
 0001:000096a5       __ehhandler$??0databaseEditDlg@@QAE@ABVQString@@PAVQWidget@@PBDI@Z 1000a6a5 f   databaseEditdlgimpl.obj
 0001:000096c0       __unwindfunclet$??1databaseEditDlg@@UAE@XZ$0 1000a6c0 f   databaseEditdlgimpl.obj
 0001:000096c8       __unwindfunclet$??1databaseEditDlg@@UAE@XZ$1 1000a6c8 f   databaseEditdlgimpl.obj
 0001:000096d7       __unwindfunclet$??1databaseEditDlg@@UAE@XZ$2 1000a6d7 f   databaseEditdlgimpl.obj
 0001:000096e6       __ehhandler$??1databaseEditDlg@@UAE@XZ 1000a6e6 f   databaseEditdlgimpl.obj
 0001:00009701       __unwindfunclet$?loadDb@databaseEditDlg@@QAE_NABVQString@@H@Z$0 1000a701 f   databaseEditdlgimpl.obj
 0001:0000970d       __unwindfunclet$?loadDb@databaseEditDlg@@QAE_NABVQString@@H@Z$1 1000a70d f   databaseEditdlgimpl.obj
 0001:00009719       __unwindfunclet$?loadDb@databaseEditDlg@@QAE_NABVQString@@H@Z$2 1000a719 f   databaseEditdlgimpl.obj
 0001:00009725       __unwindfunclet$?loadDb@databaseEditDlg@@QAE_NABVQString@@H@Z$3 1000a725 f   databaseEditdlgimpl.obj
 0001:00009731       __unwindfunclet$?loadDb@databaseEditDlg@@QAE_NABVQString@@H@Z$4 1000a731 f   databaseEditdlgimpl.obj
 0001:0000973d       __unwindfunclet$?loadDb@databaseEditDlg@@QAE_NABVQString@@H@Z$5 1000a73d f   databaseEditdlgimpl.obj
 0001:00009749       __unwindfunclet$?loadDb@databaseEditDlg@@QAE_NABVQString@@H@Z$6 1000a749 f   databaseEditdlgimpl.obj
 0001:00009755       __unwindfunclet$?loadDb@databaseEditDlg@@QAE_NABVQString@@H@Z$7 1000a755 f   databaseEditdlgimpl.obj
 0001:00009761       __unwindfunclet$?loadDb@databaseEditDlg@@QAE_NABVQString@@H@Z$8 1000a761 f   databaseEditdlgimpl.obj
 0001:0000976d       __unwindfunclet$?loadDb@databaseEditDlg@@QAE_NABVQString@@H@Z$9 1000a76d f   databaseEditdlgimpl.obj
 0001:00009779       __unwindfunclet$?loadDb@databaseEditDlg@@QAE_NABVQString@@H@Z$10 1000a779 f   databaseEditdlgimpl.obj
 0001:00009785       __unwindfunclet$?loadDb@databaseEditDlg@@QAE_NABVQString@@H@Z$11 1000a785 f   databaseEditdlgimpl.obj
 0001:00009791       __ehhandler$?loadDb@databaseEditDlg@@QAE_NABVQString@@H@Z 1000a791 f   databaseEditdlgimpl.obj
 0001:000097b9       __unwindfunclet$?loadIni@databaseEditDlg@@QAE_NABVQString@@@Z$0 1000a7b9 f   databaseEditdlgimpl.obj
 0001:000097c5       __unwindfunclet$?loadIni@databaseEditDlg@@QAE_NABVQString@@@Z$1 1000a7c5 f   databaseEditdlgimpl.obj
 0001:000097d1       __unwindfunclet$?loadIni@databaseEditDlg@@QAE_NABVQString@@@Z$2 1000a7d1 f   databaseEditdlgimpl.obj
 0001:000097dd       __unwindfunclet$?loadIni@databaseEditDlg@@QAE_NABVQString@@@Z$3 1000a7dd f   databaseEditdlgimpl.obj
 0001:000097e9       __unwindfunclet$?loadIni@databaseEditDlg@@QAE_NABVQString@@@Z$4 1000a7e9 f   databaseEditdlgimpl.obj
 0001:000097f5       __unwindfunclet$?loadIni@databaseEditDlg@@QAE_NABVQString@@@Z$5 1000a7f5 f   databaseEditdlgimpl.obj
 0001:00009801       __unwindfunclet$?loadIni@databaseEditDlg@@QAE_NABVQString@@@Z$6 1000a801 f   databaseEditdlgimpl.obj
 0001:0000980d       __unwindfunclet$?loadIni@databaseEditDlg@@QAE_NABVQString@@@Z$7 1000a80d f   databaseEditdlgimpl.obj
 0001:00009819       __ehhandler$?loadIni@databaseEditDlg@@QAE_NABVQString@@@Z 1000a819 f   databaseEditdlgimpl.obj
 0001:00009841       __unwindfunclet$?resetDisplays@databaseEditDlg@@QAEXXZ$0 1000a841 f   databaseEditdlgimpl.obj
 0001:0000984a       __unwindfunclet$?resetDisplays@databaseEditDlg@@QAEXXZ$1 1000a84a f   databaseEditdlgimpl.obj
 0001:00009853       __ehhandler$?resetDisplays@databaseEditDlg@@QAEXXZ 1000a853 f   databaseEditdlgimpl.obj
 0001:0000986e       __unwindfunclet$?save@databaseEditDlg@@QAEXABVQString@@@Z$0 1000a86e f   databaseEditdlgimpl.obj
 0001:00009877       __ehhandler$?save@databaseEditDlg@@QAEXABVQString@@@Z 1000a877 f   databaseEditdlgimpl.obj
 0001:00009892       __unwindfunclet$?textChanged@databaseEditDlg@@QAEXXZ$0 1000a892 f   databaseEditdlgimpl.obj
 0001:0000989b       __ehhandler$?textChanged@databaseEditDlg@@QAEXXZ 1000a89b f   databaseEditdlgimpl.obj
 0001:000098b6       __unwindfunclet$?create@plugindesc@@UAEPAVconfig_plugin_base@@ABVQString@@00@Z$0 1000a8b6 f   plugindesc.obj
 0001:000098b6       __unwindfunclet$??4?$QGuardedPtr@VQPopupMenu@@@@QAEAAV0@PAVQPopupMenu@@@Z$0 1000a8b6 f   plugindesc.obj
 0001:000098b6       __unwindfunclet$??0?$QGuardedPtr@VQPopupMenu@@@@QAE@XZ$0 1000a8b6 f   plugindesc.obj
 0001:000098b6       __unwindfunclet$??0?$QGuardedPtr@VQDockWindow@@@@QAE@XZ$0 1000a8b6 f   plugindesc.obj
 0001:000098b6       __unwindfunclet$??4?$QGuardedPtr@VQDockWindow@@@@QAEAAV0@PAVQDockWindow@@@Z$0 1000a8b6 f   plugindesc.obj
 0001:000098c0       __ehhandler$??0?$QGuardedPtr@VQDockWindow@@@@QAE@XZ 1000a8c0 f   plugindesc.obj
 0001:000098c0       __ehhandler$?create@plugindesc@@UAEPAVconfig_plugin_base@@ABVQString@@00@Z 1000a8c0 f   plugindesc.obj
 0001:000098c0       __ehhandler$??4?$QGuardedPtr@VQPopupMenu@@@@QAEAAV0@PAVQPopupMenu@@@Z 1000a8c0 f   plugindesc.obj
 0001:000098c0       __ehhandler$??0?$QGuardedPtr@VQPopupMenu@@@@QAE@XZ 1000a8c0 f   plugindesc.obj
 0001:000098c0       __ehhandler$??4?$QGuardedPtr@VQDockWindow@@@@QAEAAV0@PAVQDockWindow@@@Z 1000a8c0 f   plugindesc.obj
 0001:000098db       __unwindfunclet$?keys@plugindesc@@UAE?AVQStringList@@ABVQString@@0@Z$0 1000a8db f   plugindesc.obj
 0001:000098f5       __unwindfunclet$?keys@plugindesc@@UAE?AVQStringList@@ABVQString@@0@Z$1 1000a8f5 f   plugindesc.obj
 0001:000098fe       __ehhandler$?keys@plugindesc@@UAE?AVQStringList@@ABVQString@@0@Z 1000a8fe f   plugindesc.obj
 0001:00009919       __unwindfunclet$??0toolWindow@@QAE@PAVQWidget@@PBDI@Z$0 1000a919 f   toolwindowimpl.obj
 0001:00009921       __ehhandler$??0toolWindow@@QAE@PAVQWidget@@PBDI@Z 1000a921 f   toolwindowimpl.obj
 0001:0000993c       __unwindfunclet$?selectionChanged@toolWindow@@AAEXPAVQListViewItem@@@Z$0 1000a93c f   toolwindowimpl.obj
 0001:00009945       __ehhandler$?selectionChanged@toolWindow@@AAEXPAVQListViewItem@@@Z 1000a945 f   toolwindowimpl.obj
 0001:00009960       __unwindfunclet$??0databaseEditDlgBase@@QAE@PAVQWidget@@PBDI@Z$0 1000a960 f   databaseEditdlg.obj
 0001:00009969       __unwindfunclet$??0databaseEditDlgBase@@QAE@PAVQWidget@@PBDI@Z$1 1000a969 f   databaseEditdlg.obj
 0001:00009973       __unwindfunclet$??0databaseEditDlgBase@@QAE@PAVQWidget@@PBDI@Z$2 1000a973 f   databaseEditdlg.obj
 0001:0000997d       __unwindfunclet$??0databaseEditDlgBase@@QAE@PAVQWidget@@PBDI@Z$3 1000a97d f   databaseEditdlg.obj
 0001:00009987       __unwindfunclet$??0databaseEditDlgBase@@QAE@PAVQWidget@@PBDI@Z$4 1000a987 f   databaseEditdlg.obj
 0001:00009991       __unwindfunclet$??0databaseEditDlgBase@@QAE@PAVQWidget@@PBDI@Z$5 1000a991 f   databaseEditdlg.obj
 0001:0000999b       __unwindfunclet$??0databaseEditDlgBase@@QAE@PAVQWidget@@PBDI@Z$6 1000a99b f   databaseEditdlg.obj
 0001:000099a5       __unwindfunclet$??0databaseEditDlgBase@@QAE@PAVQWidget@@PBDI@Z$7 1000a9a5 f   databaseEditdlg.obj
 0001:000099af       __unwindfunclet$??0databaseEditDlgBase@@QAE@PAVQWidget@@PBDI@Z$8 1000a9af f   databaseEditdlg.obj
 0001:000099b9       __unwindfunclet$??0databaseEditDlgBase@@QAE@PAVQWidget@@PBDI@Z$9 1000a9b9 f   databaseEditdlg.obj
 0001:000099c3       __unwindfunclet$??0databaseEditDlgBase@@QAE@PAVQWidget@@PBDI@Z$10 1000a9c3 f   databaseEditdlg.obj
 0001:000099cd       __unwindfunclet$??0databaseEditDlgBase@@QAE@PAVQWidget@@PBDI@Z$11 1000a9cd f   databaseEditdlg.obj
 0001:000099d7       __unwindfunclet$??0databaseEditDlgBase@@QAE@PAVQWidget@@PBDI@Z$12 1000a9d7 f   databaseEditdlg.obj
 0001:000099e1       __unwindfunclet$??0databaseEditDlgBase@@QAE@PAVQWidget@@PBDI@Z$13 1000a9e1 f   databaseEditdlg.obj
 0001:000099ea       __unwindfunclet$??0databaseEditDlgBase@@QAE@PAVQWidget@@PBDI@Z$14 1000a9ea f   databaseEditdlg.obj
 0001:000099f4       __unwindfunclet$??0databaseEditDlgBase@@QAE@PAVQWidget@@PBDI@Z$15 1000a9f4 f   databaseEditdlg.obj
 0001:000099fe       __unwindfunclet$??0databaseEditDlgBase@@QAE@PAVQWidget@@PBDI@Z$16 1000a9fe f   databaseEditdlg.obj
 0001:00009a08       __unwindfunclet$??0databaseEditDlgBase@@QAE@PAVQWidget@@PBDI@Z$17 1000aa08 f   databaseEditdlg.obj
 0001:00009a12       __unwindfunclet$??0databaseEditDlgBase@@QAE@PAVQWidget@@PBDI@Z$18 1000aa12 f   databaseEditdlg.obj
 0001:00009a1c       __unwindfunclet$??0databaseEditDlgBase@@QAE@PAVQWidget@@PBDI@Z$19 1000aa1c f   databaseEditdlg.obj
 0001:00009a26       __unwindfunclet$??0databaseEditDlgBase@@QAE@PAVQWidget@@PBDI@Z$20 1000aa26 f   databaseEditdlg.obj
 0001:00009a30       __unwindfunclet$??0databaseEditDlgBase@@QAE@PAVQWidget@@PBDI@Z$21 1000aa30 f   databaseEditdlg.obj
 0001:00009a39       __unwindfunclet$??0databaseEditDlgBase@@QAE@PAVQWidget@@PBDI@Z$22 1000aa39 f   databaseEditdlg.obj
 0001:00009a42       __unwindfunclet$??0databaseEditDlgBase@@QAE@PAVQWidget@@PBDI@Z$23 1000aa42 f   databaseEditdlg.obj
 0001:00009a4b       __unwindfunclet$??0databaseEditDlgBase@@QAE@PAVQWidget@@PBDI@Z$24 1000aa4b f   databaseEditdlg.obj
 0001:00009a55       __unwindfunclet$??0databaseEditDlgBase@@QAE@PAVQWidget@@PBDI@Z$25 1000aa55 f   databaseEditdlg.obj
 0001:00009a5f       __unwindfunclet$??0databaseEditDlgBase@@QAE@PAVQWidget@@PBDI@Z$26 1000aa5f f   databaseEditdlg.obj
 0001:00009a69       __unwindfunclet$??0databaseEditDlgBase@@QAE@PAVQWidget@@PBDI@Z$27 1000aa69 f   databaseEditdlg.obj
 0001:00009a72       __unwindfunclet$??0databaseEditDlgBase@@QAE@PAVQWidget@@PBDI@Z$28 1000aa72 f   databaseEditdlg.obj
 0001:00009a7b       __unwindfunclet$??0databaseEditDlgBase@@QAE@PAVQWidget@@PBDI@Z$29 1000aa7b f   databaseEditdlg.obj
 0001:00009a84       __unwindfunclet$??0databaseEditDlgBase@@QAE@PAVQWidget@@PBDI@Z$30 1000aa84 f   databaseEditdlg.obj
 0001:00009a8e       __unwindfunclet$??0databaseEditDlgBase@@QAE@PAVQWidget@@PBDI@Z$31 1000aa8e f   databaseEditdlg.obj
 0001:00009a98       __unwindfunclet$??0databaseEditDlgBase@@QAE@PAVQWidget@@PBDI@Z$32 1000aa98 f   databaseEditdlg.obj
 0001:00009aa2       __unwindfunclet$??0databaseEditDlgBase@@QAE@PAVQWidget@@PBDI@Z$33 1000aaa2 f   databaseEditdlg.obj
 0001:00009aab       __unwindfunclet$??0databaseEditDlgBase@@QAE@PAVQWidget@@PBDI@Z$34 1000aaab f   databaseEditdlg.obj
 0001:00009ab4       __unwindfunclet$??0databaseEditDlgBase@@QAE@PAVQWidget@@PBDI@Z$35 1000aab4 f   databaseEditdlg.obj
 0001:00009abd       __unwindfunclet$??0databaseEditDlgBase@@QAE@PAVQWidget@@PBDI@Z$36 1000aabd f   databaseEditdlg.obj
 0001:00009ac7       __unwindfunclet$??0databaseEditDlgBase@@QAE@PAVQWidget@@PBDI@Z$37 1000aac7 f   databaseEditdlg.obj
 0001:00009ad1       __unwindfunclet$??0databaseEditDlgBase@@QAE@PAVQWidget@@PBDI@Z$38 1000aad1 f   databaseEditdlg.obj
 0001:00009adb       __unwindfunclet$??0databaseEditDlgBase@@QAE@PAVQWidget@@PBDI@Z$39 1000aadb f   databaseEditdlg.obj
 0001:00009ae4       __unwindfunclet$??0databaseEditDlgBase@@QAE@PAVQWidget@@PBDI@Z$40 1000aae4 f   databaseEditdlg.obj
 0001:00009aed       __unwindfunclet$??0databaseEditDlgBase@@QAE@PAVQWidget@@PBDI@Z$41 1000aaed f   databaseEditdlg.obj
 0001:00009af6       __unwindfunclet$??0databaseEditDlgBase@@QAE@PAVQWidget@@PBDI@Z$42 1000aaf6 f   databaseEditdlg.obj
 0001:00009b00       __unwindfunclet$??0databaseEditDlgBase@@QAE@PAVQWidget@@PBDI@Z$43 1000ab00 f   databaseEditdlg.obj
 0001:00009b0a       __unwindfunclet$??0databaseEditDlgBase@@QAE@PAVQWidget@@PBDI@Z$44 1000ab0a f   databaseEditdlg.obj
 0001:00009b14       __unwindfunclet$??0databaseEditDlgBase@@QAE@PAVQWidget@@PBDI@Z$45 1000ab14 f   databaseEditdlg.obj
 0001:00009b1d       __unwindfunclet$??0databaseEditDlgBase@@QAE@PAVQWidget@@PBDI@Z$46 1000ab1d f   databaseEditdlg.obj
 0001:00009b26       __unwindfunclet$??0databaseEditDlgBase@@QAE@PAVQWidget@@PBDI@Z$47 1000ab26 f   databaseEditdlg.obj
 0001:00009b2f       __unwindfunclet$??0databaseEditDlgBase@@QAE@PAVQWidget@@PBDI@Z$48 1000ab2f f   databaseEditdlg.obj
 0001:00009b39       __unwindfunclet$??0databaseEditDlgBase@@QAE@PAVQWidget@@PBDI@Z$49 1000ab39 f   databaseEditdlg.obj
 0001:00009b43       __unwindfunclet$??0databaseEditDlgBase@@QAE@PAVQWidget@@PBDI@Z$50 1000ab43 f   databaseEditdlg.obj
 0001:00009b4d       __unwindfunclet$??0databaseEditDlgBase@@QAE@PAVQWidget@@PBDI@Z$51 1000ab4d f   databaseEditdlg.obj
 0001:00009b56       __unwindfunclet$??0databaseEditDlgBase@@QAE@PAVQWidget@@PBDI@Z$52 1000ab56 f   databaseEditdlg.obj
 0001:00009b5f       __unwindfunclet$??0databaseEditDlgBase@@QAE@PAVQWidget@@PBDI@Z$53 1000ab5f f   databaseEditdlg.obj
 0001:00009b68       __unwindfunclet$??0databaseEditDlgBase@@QAE@PAVQWidget@@PBDI@Z$54 1000ab68 f   databaseEditdlg.obj
 0001:00009b72       __unwindfunclet$??0databaseEditDlgBase@@QAE@PAVQWidget@@PBDI@Z$55 1000ab72 f   databaseEditdlg.obj
 0001:00009b7c       __unwindfunclet$??0databaseEditDlgBase@@QAE@PAVQWidget@@PBDI@Z$56 1000ab7c f   databaseEditdlg.obj
 0001:00009b86       __unwindfunclet$??0databaseEditDlgBase@@QAE@PAVQWidget@@PBDI@Z$57 1000ab86 f   databaseEditdlg.obj
 0001:00009b8f       __unwindfunclet$??0databaseEditDlgBase@@QAE@PAVQWidget@@PBDI@Z$58 1000ab8f f   databaseEditdlg.obj
 0001:00009b98       __unwindfunclet$??0databaseEditDlgBase@@QAE@PAVQWidget@@PBDI@Z$59 1000ab98 f   databaseEditdlg.obj
 0001:00009ba1       __unwindfunclet$??0databaseEditDlgBase@@QAE@PAVQWidget@@PBDI@Z$60 1000aba1 f   databaseEditdlg.obj
 0001:00009bab       __unwindfunclet$??0databaseEditDlgBase@@QAE@PAVQWidget@@PBDI@Z$61 1000abab f   databaseEditdlg.obj
 0001:00009bb5       __unwindfunclet$??0databaseEditDlgBase@@QAE@PAVQWidget@@PBDI@Z$62 1000abb5 f   databaseEditdlg.obj
 0001:00009bbf       __unwindfunclet$??0databaseEditDlgBase@@QAE@PAVQWidget@@PBDI@Z$63 1000abbf f   databaseEditdlg.obj
 0001:00009bc8       __unwindfunclet$??0databaseEditDlgBase@@QAE@PAVQWidget@@PBDI@Z$64 1000abc8 f   databaseEditdlg.obj
 0001:00009bd1       __unwindfunclet$??0databaseEditDlgBase@@QAE@PAVQWidget@@PBDI@Z$65 1000abd1 f   databaseEditdlg.obj
 0001:00009bda       __unwindfunclet$??0databaseEditDlgBase@@QAE@PAVQWidget@@PBDI@Z$66 1000abda f   databaseEditdlg.obj
 0001:00009be4       __unwindfunclet$??0databaseEditDlgBase@@QAE@PAVQWidget@@PBDI@Z$67 1000abe4 f   databaseEditdlg.obj
 0001:00009bee       __unwindfunclet$??0databaseEditDlgBase@@QAE@PAVQWidget@@PBDI@Z$68 1000abee f   databaseEditdlg.obj
 0001:00009bf8       __unwindfunclet$??0databaseEditDlgBase@@QAE@PAVQWidget@@PBDI@Z$69 1000abf8 f   databaseEditdlg.obj
 0001:00009c01       __unwindfunclet$??0databaseEditDlgBase@@QAE@PAVQWidget@@PBDI@Z$70 1000ac01 f   databaseEditdlg.obj
 0001:00009c0a       __unwindfunclet$??0databaseEditDlgBase@@QAE@PAVQWidget@@PBDI@Z$71 1000ac0a f   databaseEditdlg.obj
 0001:00009c13       __unwindfunclet$??0databaseEditDlgBase@@QAE@PAVQWidget@@PBDI@Z$72 1000ac13 f   databaseEditdlg.obj
 0001:00009c1d       __unwindfunclet$??0databaseEditDlgBase@@QAE@PAVQWidget@@PBDI@Z$73 1000ac1d f   databaseEditdlg.obj
 0001:00009c27       __unwindfunclet$??0databaseEditDlgBase@@QAE@PAVQWidget@@PBDI@Z$74 1000ac27 f   databaseEditdlg.obj
 0001:00009c31       __unwindfunclet$??0databaseEditDlgBase@@QAE@PAVQWidget@@PBDI@Z$75 1000ac31 f   databaseEditdlg.obj
 0001:00009c3a       __unwindfunclet$??0databaseEditDlgBase@@QAE@PAVQWidget@@PBDI@Z$76 1000ac3a f   databaseEditdlg.obj
 0001:00009c43       __unwindfunclet$??0databaseEditDlgBase@@QAE@PAVQWidget@@PBDI@Z$77 1000ac43 f   databaseEditdlg.obj
 0001:00009c4c       __ehhandler$??0databaseEditDlgBase@@QAE@PAVQWidget@@PBDI@Z 1000ac4c f   databaseEditdlg.obj
 0001:00009c67       __unwindfunclet$?languageChange@databaseEditDlgBase@@MAEXXZ$0 1000ac67 f   databaseEditdlg.obj
 0001:00009c70       __unwindfunclet$?languageChange@databaseEditDlgBase@@MAEXXZ$1 1000ac70 f   databaseEditdlg.obj
 0001:00009c79       __unwindfunclet$?languageChange@databaseEditDlgBase@@MAEXXZ$2 1000ac79 f   databaseEditdlg.obj
 0001:00009c82       __unwindfunclet$?languageChange@databaseEditDlgBase@@MAEXXZ$3 1000ac82 f   databaseEditdlg.obj
 0001:00009c8b       __unwindfunclet$?languageChange@databaseEditDlgBase@@MAEXXZ$4 1000ac8b f   databaseEditdlg.obj
 0001:00009c94       __unwindfunclet$?languageChange@databaseEditDlgBase@@MAEXXZ$5 1000ac94 f   databaseEditdlg.obj
 0001:00009c9d       __unwindfunclet$?languageChange@databaseEditDlgBase@@MAEXXZ$6 1000ac9d f   databaseEditdlg.obj
 0001:00009ca6       __unwindfunclet$?languageChange@databaseEditDlgBase@@MAEXXZ$7 1000aca6 f   databaseEditdlg.obj
 0001:00009caf       __unwindfunclet$?languageChange@databaseEditDlgBase@@MAEXXZ$8 1000acaf f   databaseEditdlg.obj
 0001:00009cb8       __unwindfunclet$?languageChange@databaseEditDlgBase@@MAEXXZ$9 1000acb8 f   databaseEditdlg.obj
 0001:00009cc1       __unwindfunclet$?languageChange@databaseEditDlgBase@@MAEXXZ$10 1000acc1 f   databaseEditdlg.obj
 0001:00009cca       __unwindfunclet$?languageChange@databaseEditDlgBase@@MAEXXZ$11 1000acca f   databaseEditdlg.obj
 0001:00009cd3       __unwindfunclet$?languageChange@databaseEditDlgBase@@MAEXXZ$12 1000acd3 f   databaseEditdlg.obj
 0001:00009cdc       __unwindfunclet$?languageChange@databaseEditDlgBase@@MAEXXZ$13 1000acdc f   databaseEditdlg.obj
 0001:00009ce5       __unwindfunclet$?languageChange@databaseEditDlgBase@@MAEXXZ$14 1000ace5 f   databaseEditdlg.obj
 0001:00009cee       __unwindfunclet$?languageChange@databaseEditDlgBase@@MAEXXZ$15 1000acee f   databaseEditdlg.obj
 0001:00009cf7       __unwindfunclet$?languageChange@databaseEditDlgBase@@MAEXXZ$16 1000acf7 f   databaseEditdlg.obj
 0001:00009d00       __unwindfunclet$?languageChange@databaseEditDlgBase@@MAEXXZ$17 1000ad00 f   databaseEditdlg.obj
 0001:00009d09       __unwindfunclet$?languageChange@databaseEditDlgBase@@MAEXXZ$18 1000ad09 f   databaseEditdlg.obj
 0001:00009d12       __unwindfunclet$?languageChange@databaseEditDlgBase@@MAEXXZ$19 1000ad12 f   databaseEditdlg.obj
 0001:00009d1b       __unwindfunclet$?languageChange@databaseEditDlgBase@@MAEXXZ$20 1000ad1b f   databaseEditdlg.obj
 0001:00009d24       __unwindfunclet$?languageChange@databaseEditDlgBase@@MAEXXZ$21 1000ad24 f   databaseEditdlg.obj
 0001:00009d2d       __unwindfunclet$?languageChange@databaseEditDlgBase@@MAEXXZ$22 1000ad2d f   databaseEditdlg.obj
 0001:00009d36       __unwindfunclet$?languageChange@databaseEditDlgBase@@MAEXXZ$23 1000ad36 f   databaseEditdlg.obj
 0001:00009d3f       __unwindfunclet$?languageChange@databaseEditDlgBase@@MAEXXZ$24 1000ad3f f   databaseEditdlg.obj
 0001:00009d48       __unwindfunclet$?languageChange@databaseEditDlgBase@@MAEXXZ$25 1000ad48 f   databaseEditdlg.obj
 0001:00009d51       __unwindfunclet$?languageChange@databaseEditDlgBase@@MAEXXZ$26 1000ad51 f   databaseEditdlg.obj
 0001:00009d5a       __unwindfunclet$?languageChange@databaseEditDlgBase@@MAEXXZ$27 1000ad5a f   databaseEditdlg.obj
 0001:00009d63       __unwindfunclet$?languageChange@databaseEditDlgBase@@MAEXXZ$28 1000ad63 f   databaseEditdlg.obj
 0001:00009d6c       __unwindfunclet$?languageChange@databaseEditDlgBase@@MAEXXZ$29 1000ad6c f   databaseEditdlg.obj
 0001:00009d75       __unwindfunclet$?languageChange@databaseEditDlgBase@@MAEXXZ$30 1000ad75 f   databaseEditdlg.obj
 0001:00009d7e       __unwindfunclet$?languageChange@databaseEditDlgBase@@MAEXXZ$31 1000ad7e f   databaseEditdlg.obj
 0001:00009d87       __unwindfunclet$?languageChange@databaseEditDlgBase@@MAEXXZ$32 1000ad87 f   databaseEditdlg.obj
 0001:00009d90       __unwindfunclet$?languageChange@databaseEditDlgBase@@MAEXXZ$33 1000ad90 f   databaseEditdlg.obj
 0001:00009d99       __unwindfunclet$?languageChange@databaseEditDlgBase@@MAEXXZ$34 1000ad99 f   databaseEditdlg.obj
 0001:00009da2       __unwindfunclet$?languageChange@databaseEditDlgBase@@MAEXXZ$35 1000ada2 f   databaseEditdlg.obj
 0001:00009dab       __ehhandler$?languageChange@databaseEditDlgBase@@MAEXXZ 1000adab f   databaseEditdlg.obj
 0001:00009dc6       __unwindfunclet$?qt_emit@databaseEdit@@UAE_NHPAUQUObject@@@Z$0 1000adc6 f   moc_databaseEdit.obj
 0001:00009dc6       __unwindfunclet$?qt_emit@databaseEditDlg@@UAE_NHPAUQUObject@@@Z$0 1000adc6 f   moc_databaseEdit.obj
 0001:00009dcf       __ehhandler$?qt_emit@databaseEdit@@UAE_NHPAUQUObject@@@Z 1000adcf f   moc_databaseEdit.obj
 0001:00009dcf       __ehhandler$?qt_emit@databaseEditDlg@@UAE_NHPAUQUObject@@@Z 1000adcf f   moc_databaseEdit.obj
 0001:00009dea       __unwindfunclet$?command@databaseEdit@@IAEXVQString@@0@Z$0 1000adea f   moc_databaseEditdlgimpl.obj
 0001:00009dea       __unwindfunclet$?command@databaseEditDlg@@IAEXVQString@@0@Z$0 1000adea f   moc_databaseEditdlgimpl.obj
 0001:00009df3       __unwindfunclet$?command@databaseEdit@@IAEXVQString@@0@Z$1 1000adf3 f   moc_databaseEditdlgimpl.obj
 0001:00009df3       __unwindfunclet$?command@databaseEditDlg@@IAEXVQString@@0@Z$1 1000adf3 f   moc_databaseEditdlgimpl.obj
 0001:00009dfc       __unwindfunclet$?command@databaseEdit@@IAEXVQString@@0@Z$2 1000adfc f   moc_databaseEditdlgimpl.obj
 0001:00009dfc       __unwindfunclet$?command@databaseEditDlg@@IAEXVQString@@0@Z$2 1000adfc f   moc_databaseEditdlgimpl.obj
 0001:00009e10       __ehhandler$?command@databaseEdit@@IAEXVQString@@0@Z 1000ae10 f   moc_databaseEditdlgimpl.obj
 0001:00009e10       __ehhandler$?command@databaseEditDlg@@IAEXVQString@@0@Z 1000ae10 f   moc_databaseEditdlgimpl.obj
 0001:00009e35       __unwindfunclet$?fileSelected@toolWindow@@IAEXABVQString@@@Z$0 1000ae35 f   moc_toolwindowimpl.obj
 0001:00009e3e       __ehhandler$?fileSelected@toolWindow@@IAEXABVQString@@@Z 1000ae3e f   moc_toolwindowimpl.obj
 0001:00009e59       __unwindfunclet$??0toolWindowBase@@QAE@PAVQWidget@@PBDI@Z$0 1000ae59 f   toolwindow.obj
 0001:00009e62       __unwindfunclet$??0toolWindowBase@@QAE@PAVQWidget@@PBDI@Z$1 1000ae62 f   toolwindow.obj
 0001:00009e6c       __unwindfunclet$??0toolWindowBase@@QAE@PAVQWidget@@PBDI@Z$2 1000ae6c f   toolwindow.obj
 0001:00009e76       __unwindfunclet$??0toolWindowBase@@QAE@PAVQWidget@@PBDI@Z$3 1000ae76 f   toolwindow.obj
 0001:00009e80       __unwindfunclet$??0toolWindowBase@@QAE@PAVQWidget@@PBDI@Z$4 1000ae80 f   toolwindow.obj
 0001:00009e8a       __unwindfunclet$??0toolWindowBase@@QAE@PAVQWidget@@PBDI@Z$5 1000ae8a f   toolwindow.obj
 0001:00009e94       __unwindfunclet$??0toolWindowBase@@QAE@PAVQWidget@@PBDI@Z$6 1000ae94 f   toolwindow.obj
 0001:00009e9d       __unwindfunclet$??0toolWindowBase@@QAE@PAVQWidget@@PBDI@Z$7 1000ae9d f   toolwindow.obj
 0001:00009ea6       __unwindfunclet$??0toolWindowBase@@QAE@PAVQWidget@@PBDI@Z$8 1000aea6 f   toolwindow.obj
 0001:00009eaf       __ehhandler$??0toolWindowBase@@QAE@PAVQWidget@@PBDI@Z 1000aeaf f   toolwindow.obj
 0001:00009eca       __unwindfunclet$?languageChange@toolWindowBase@@MAEXXZ$0 1000aeca f   toolwindow.obj
 0001:00009ed3       __unwindfunclet$?languageChange@toolWindowBase@@MAEXXZ$1 1000aed3 f   toolwindow.obj
 0001:00009edc       __unwindfunclet$?languageChange@toolWindowBase@@MAEXXZ$2 1000aedc f   toolwindow.obj
 0001:00009ee5       __unwindfunclet$?languageChange@toolWindowBase@@MAEXXZ$3 1000aee5 f   toolwindow.obj
 0001:00009eee       __ehhandler$?languageChange@toolWindowBase@@MAEXXZ 1000aeee f   toolwindow.obj
 0001:00009f09       ??__FcleanUp_databaseEdit@@YAXXZ 1000af09 f   moc_databaseEdit.obj
 0001:00009f14       ??__FcleanUp_databaseEditDlgBase@@YAXXZ 1000af14 f   moc_databaseEditdlg.obj
 0001:00009f1f       ??__FcleanUp_databaseEditDlg@@YAXXZ 1000af1f f   moc_databaseEditdlgimpl.obj
 0001:00009f2a       ??__FcleanUp_toolWindowBase@@YAXXZ 1000af2a f   moc_toolwindow.obj
 0001:00009f35       ??__FcleanUp_toolWindow@@YAXXZ 1000af35 f   moc_toolwindowimpl.obj
 0002:00000e30       _cleanUp_databaseEdit$initializer$ 1000be30     moc_databaseEdit.obj
 0002:00000e34       _cleanUp_databaseEditDlgBase$initializer$ 1000be34     moc_databaseEditdlg.obj
 0002:00000e38       _cleanUp_databaseEditDlg$initializer$ 1000be38     moc_databaseEditdlgimpl.obj
 0002:00000e3c       _cleanUp_toolWindowBase$initializer$ 1000be3c     moc_toolwindow.obj
 0002:00000e40       _cleanUp_toolWindow$initializer$ 1000be40     moc_toolwindowimpl.obj
 0002:00000e4c       _pcinit                    1000be4c     MSVCRT:crtdll.obj
 0002:00000e50       _pinit                     1000be50     MSVCRT:atonexit.obj
 0002:00003adc       ?slot_0@?3??staticMetaObject@databaseEdit@@SAPAVQMetaObject@@XZ@4UQUMethod@@B 1000eadc     moc_databaseEdit.obj
 0002:00003af8       ?slot_tbl@?3??staticMetaObject@databaseEdit@@SAPAVQMetaObject@@XZ@4QBUQMetaData@@B 1000eaf8     moc_databaseEdit.obj
 0002:00003b24       ?signal_0@?3??staticMetaObject@databaseEdit@@SAPAVQMetaObject@@XZ@4UQUMethod@@B 1000eb24     moc_databaseEdit.obj
 0002:00003b38       ?signal_tbl@?3??staticMetaObject@databaseEdit@@SAPAVQMetaObject@@XZ@4QBUQMetaData@@B 1000eb38     moc_databaseEdit.obj
 0002:00003b60       ?slot_0@?3??staticMetaObject@databaseEditDlgBase@@SAPAVQMetaObject@@XZ@4UQUMethod@@B 1000eb60     moc_databaseEditdlg.obj
 0002:00003b7c       ?slot_tbl@?3??staticMetaObject@databaseEditDlgBase@@SAPAVQMetaObject@@XZ@4QBUQMetaData@@B 1000eb7c     moc_databaseEditdlg.obj
 0002:00003b9c       ?slot_0@?3??staticMetaObject@databaseEditDlg@@SAPAVQMetaObject@@XZ@4UQUMethod@@B 1000eb9c     moc_databaseEditdlgimpl.obj
 0002:00003bb8       ?slot_1@?3??staticMetaObject@databaseEditDlg@@SAPAVQMetaObject@@XZ@4UQUMethod@@B 1000ebb8     moc_databaseEditdlgimpl.obj
 0002:00003bd0       ?slot_tbl@?3??staticMetaObject@databaseEditDlg@@SAPAVQMetaObject@@XZ@4QBUQMetaData@@B 1000ebd0     moc_databaseEditdlgimpl.obj
 0002:00003c08       ?signal_0@?3??staticMetaObject@databaseEditDlg@@SAPAVQMetaObject@@XZ@4UQUMethod@@B 1000ec08     moc_databaseEditdlgimpl.obj
 0002:00003c14       ?signal_tbl@?3??staticMetaObject@databaseEditDlg@@SAPAVQMetaObject@@XZ@4QBUQMetaData@@B 1000ec14     moc_databaseEditdlgimpl.obj
 0002:00003c30       ?slot_0@?3??staticMetaObject@toolWindowBase@@SAPAVQMetaObject@@XZ@4UQUMethod@@B 1000ec30     moc_toolwindow.obj
 0002:00003c3c       ?slot_tbl@?3??staticMetaObject@toolWindowBase@@SAPAVQMetaObject@@XZ@4QBUQMetaData@@B 1000ec3c     moc_toolwindow.obj
 0002:00003c64       ?slot_0@?3??staticMetaObject@toolWindow@@SAPAVQMetaObject@@XZ@4UQUMethod@@B 1000ec64     moc_toolwindowimpl.obj
 0002:00003c84       ?slot_tbl@?3??staticMetaObject@toolWindow@@SAPAVQMetaObject@@XZ@4QBUQMetaData@@B 1000ec84     moc_toolwindowimpl.obj
 0002:00003cb4       ?signal_0@?3??staticMetaObject@toolWindow@@SAPAVQMetaObject@@XZ@4UQUMethod@@B 1000ecb4     moc_toolwindowimpl.obj
 0002:00003cc0       ?signal_tbl@?3??staticMetaObject@toolWindow@@SAPAVQMetaObject@@XZ@4QBUQMetaData@@B 1000ecc0     moc_toolwindowimpl.obj
 0002:00004210       _GS_ExceptionPointers      1000f210     MSVCRT:gs_report.obj
 0002:000051c8       __unwindtable$??1QDockWindowList@@UAE@XZ 100101c8     databaseEdit.obj
 0002:000051d8       __ehfuncinfo$??1QDockWindowList@@UAE@XZ 100101d8     databaseEdit.obj
 0002:000051fc       __unwindtable$??1?$QPtrList@VQPopupMenu@@@@UAE@XZ 100101fc     databaseEdit.obj
 0002:00005204       __ehfuncinfo$??1?$QPtrList@VQPopupMenu@@@@UAE@XZ 10010204     databaseEdit.obj
 0002:00005228       __unwindtable$??1QPopupMenuList@@UAE@XZ 10010228     databaseEdit.obj
 0002:00005230       __ehfuncinfo$??1QPopupMenuList@@UAE@XZ 10010230     databaseEdit.obj
 0002:00005254       __unwindtable$??0config_plugin_base@@QAE@ABVQString@@00@Z 10010254     databaseEdit.obj
 0002:00005274       __ehfuncinfo$??0config_plugin_base@@QAE@ABVQString@@00@Z 10010274     databaseEdit.obj
 0002:00005298       __unwindtable$??1config_plugin_base@@UAE@XZ 10010298     databaseEdit.obj
 0002:000052b0       __ehfuncinfo$??1config_plugin_base@@UAE@XZ 100102b0     databaseEdit.obj
 0002:000052d4       __unwindtable$?about@config_plugin_base@@UAE?AVQString@@XZ 100102d4     databaseEdit.obj
 0002:000052e4       __ehfuncinfo$?about@config_plugin_base@@UAE?AVQString@@XZ 100102e4     databaseEdit.obj
 0002:00005308       __ehfuncinfo$??0databaseEdit@@QAE@ABVQString@@00@Z 10010308     databaseEdit.obj
 0002:0000532c       __unwindtable$??0databaseEdit@@QAE@ABVQString@@00@Z 1001032c     databaseEdit.obj
 0002:0000540c       __ehfuncinfo$??1databaseEdit@@UAE@XZ 1001040c     databaseEdit.obj
 0002:00005430       __unwindtable$??1databaseEdit@@UAE@XZ 10010430     databaseEdit.obj
 0002:00005460       __unwindtable$?toolbars@databaseEdit@@UAE?AVQDockWindowList@@XZ 10010460     databaseEdit.obj
 0002:00005468       __ehfuncinfo$?toolbars@databaseEdit@@UAE?AVQDockWindowList@@XZ 10010468     databaseEdit.obj
 0002:0000548c       __unwindtable$?menus@databaseEdit@@UAE?AVQPopupMenuList@@XZ 1001048c     databaseEdit.obj
 0002:00005494       __ehfuncinfo$?menus@databaseEdit@@UAE?AVQPopupMenuList@@XZ 10010494     databaseEdit.obj
 0002:000054b8       __ehfuncinfo$?reply@databaseEdit@@UAEXPAVresponse@@@Z 100104b8     databaseEdit.obj
 0002:000054dc       __unwindtable$?reply@databaseEdit@@UAEXPAVresponse@@@Z 100104dc     databaseEdit.obj
 0002:0000583c       __unwindtable$?navigate@databaseEdit@@UAEXABVQString@@0@Z 1001083c     databaseEdit.obj
 0002:00005854       __ehfuncinfo$?navigate@databaseEdit@@UAEXABVQString@@0@Z 10010854     databaseEdit.obj
 0002:00005878       __ehfuncinfo$?activate@databaseEdit@@UAEX_N@Z 10010878     databaseEdit.obj
 0002:0000589c       __unwindtable$?activate@databaseEdit@@UAEX_N@Z 1001089c     databaseEdit.obj
 0002:0000594c       __ehfuncinfo$?closeEvent@databaseEdit@@UAEXPAVQCloseEvent@@@Z 1001094c     databaseEdit.obj
 0002:00005970       __unwindtable$?closeEvent@databaseEdit@@UAEXPAVQCloseEvent@@@Z 10010970     databaseEdit.obj
 0002:000059c8       __unwindtable$?apply@databaseEdit@@UAEXXZ 100109c8     databaseEdit.obj
 0002:000059e0       __ehfuncinfo$?apply@databaseEdit@@UAEXXZ 100109e0     databaseEdit.obj
 0002:00005a04       __ehfuncinfo$?about@databaseEdit@@UAE?AVQString@@XZ 10010a04     databaseEdit.obj
 0002:00005a28       __unwindtable$?about@databaseEdit@@UAE?AVQString@@XZ 10010a28     databaseEdit.obj
 0002:00005a50       __unwindtable$??1?$QIntDict@VQTable@@@@UAE@XZ 10010a50     databaseEdit.obj
 0002:00005a50       __unwindtable$??1?$QDict@VQAction@@@@UAE@XZ 10010a50     databaseEdit.obj
 0002:00005a58       __ehfuncinfo$??1?$QIntDict@VQTable@@@@UAE@XZ 10010a58     databaseEdit.obj
 0002:00005a58       __ehfuncinfo$??1?$QDict@VQAction@@@@UAE@XZ 10010a58     databaseEdit.obj
 0002:00005a7c       __ehfuncinfo$?fileSelected@databaseEdit@@AAEXABVQString@@@Z 10010a7c     databaseEdit.obj
 0002:00005aa0       __unwindtable$?fileSelected@databaseEdit@@AAEXABVQString@@@Z 10010aa0     databaseEdit.obj
 0002:00005b00       __unwindtable$?db@@YAXABVQString@@@Z 10010b00     databaseEdit.obj
 0002:00005b08       __ehfuncinfo$?db@@YAXABVQString@@@Z 10010b08     databaseEdit.obj
 0002:00005b2c       __unwindtable$??0databaseEditDlg@@QAE@ABVQString@@PAVQWidget@@PBDI@Z 10010b2c     databaseEditdlgimpl.obj
 0002:00005b4c       __ehfuncinfo$??0databaseEditDlg@@QAE@ABVQString@@PAVQWidget@@PBDI@Z 10010b4c     databaseEditdlgimpl.obj
 0002:00005b70       __unwindtable$??1databaseEditDlg@@UAE@XZ 10010b70     databaseEditdlgimpl.obj
 0002:00005b88       __ehfuncinfo$??1databaseEditDlg@@UAE@XZ 10010b88     databaseEditdlgimpl.obj
 0002:00005bac       __unwindtable$?save@databaseEditDlg@@QAEXABVQString@@@Z 10010bac     databaseEditdlgimpl.obj
 0002:00005bb4       __ehfuncinfo$?save@databaseEditDlg@@QAEXABVQString@@@Z 10010bb4     databaseEditdlgimpl.obj
 0002:00005bd8       __ehfuncinfo$?loadIni@databaseEditDlg@@QAE_NABVQString@@@Z 10010bd8     databaseEditdlgimpl.obj
 0002:00005bfc       __unwindtable$?loadIni@databaseEditDlg@@QAE_NABVQString@@@Z 10010bfc     databaseEditdlgimpl.obj
 0002:00005c44       __ehfuncinfo$?loadDb@databaseEditDlg@@QAE_NABVQString@@H@Z 10010c44     databaseEditdlgimpl.obj
 0002:00005c68       __unwindtable$?loadDb@databaseEditDlg@@QAE_NABVQString@@H@Z 10010c68     databaseEditdlgimpl.obj
 0002:00005cf8       __unwindtable$?resetDisplays@databaseEditDlg@@QAEXXZ 10010cf8     databaseEditdlgimpl.obj
 0002:00005d08       __ehfuncinfo$?resetDisplays@databaseEditDlg@@QAEXXZ 10010d08     databaseEditdlgimpl.obj
 0002:00005d2c       __unwindtable$?textChanged@databaseEditDlg@@QAEXXZ 10010d2c     databaseEditdlgimpl.obj
 0002:00005d34       __ehfuncinfo$?textChanged@databaseEditDlg@@QAEXXZ 10010d34     databaseEditdlgimpl.obj
 0002:00005d58       __unwindtable$?keys@plugindesc@@UAE?AVQStringList@@ABVQString@@0@Z 10010d58     plugindesc.obj
 0002:00005d68       __ehfuncinfo$?keys@plugindesc@@UAE?AVQStringList@@ABVQString@@0@Z 10010d68     plugindesc.obj
 0002:00005d8c       __unwindtable$??4?$QGuardedPtr@VQPopupMenu@@@@QAEAAV0@PAVQPopupMenu@@@Z 10010d8c     plugindesc.obj
 0002:00005d8c       __unwindtable$?create@plugindesc@@UAEPAVconfig_plugin_base@@ABVQString@@00@Z 10010d8c     plugindesc.obj
 0002:00005d8c       __unwindtable$??0?$QGuardedPtr@VQPopupMenu@@@@QAE@XZ 10010d8c     plugindesc.obj
 0002:00005d8c       __unwindtable$??0?$QGuardedPtr@VQDockWindow@@@@QAE@XZ 10010d8c     plugindesc.obj
 0002:00005d8c       __unwindtable$??4?$QGuardedPtr@VQDockWindow@@@@QAEAAV0@PAVQDockWindow@@@Z 10010d8c     plugindesc.obj
 0002:00005d94       __ehfuncinfo$??4?$QGuardedPtr@VQPopupMenu@@@@QAEAAV0@PAVQPopupMenu@@@Z 10010d94     plugindesc.obj
 0002:00005d94       __ehfuncinfo$??4?$QGuardedPtr@VQDockWindow@@@@QAEAAV0@PAVQDockWindow@@@Z 10010d94     plugindesc.obj
 0002:00005d94       __ehfuncinfo$?create@plugindesc@@UAEPAVconfig_plugin_base@@ABVQString@@00@Z 10010d94     plugindesc.obj
 0002:00005d94       __ehfuncinfo$??0?$QGuardedPtr@VQDockWindow@@@@QAE@XZ 10010d94     plugindesc.obj
 0002:00005d94       __ehfuncinfo$??0?$QGuardedPtr@VQPopupMenu@@@@QAE@XZ 10010d94     plugindesc.obj
 0002:00005db8       __unwindtable$??0toolWindow@@QAE@PAVQWidget@@PBDI@Z 10010db8     toolwindowimpl.obj
 0002:00005dc0       __ehfuncinfo$??0toolWindow@@QAE@PAVQWidget@@PBDI@Z 10010dc0     toolwindowimpl.obj
 0002:00005de4       __unwindtable$?selectionChanged@toolWindow@@AAEXPAVQListViewItem@@@Z 10010de4     toolwindowimpl.obj
 0002:00005dec       __ehfuncinfo$?selectionChanged@toolWindow@@AAEXPAVQListViewItem@@@Z 10010dec     toolwindowimpl.obj
 0002:00005e10       __ehfuncinfo$??0databaseEditDlgBase@@QAE@PAVQWidget@@PBDI@Z 10010e10     databaseEditdlg.obj
 0002:00005e34       __unwindtable$??0databaseEditDlgBase@@QAE@PAVQWidget@@PBDI@Z 10010e34     databaseEditdlg.obj
 0002:000060a4       __ehfuncinfo$?languageChange@databaseEditDlgBase@@MAEXXZ 100110a4     databaseEditdlg.obj
 0002:000060c8       __unwindtable$?languageChange@databaseEditDlgBase@@MAEXXZ 100110c8     databaseEditdlg.obj
 0002:000061e8       __unwindtable$?qt_emit@databaseEdit@@UAE_NHPAUQUObject@@@Z 100111e8     moc_databaseEdit.obj
 0002:000061e8       __unwindtable$?qt_emit@databaseEditDlg@@UAE_NHPAUQUObject@@@Z 100111e8     moc_databaseEdit.obj
 0002:000061f0       __ehfuncinfo$?qt_emit@databaseEditDlg@@UAE_NHPAUQUObject@@@Z 100111f0     moc_databaseEdit.obj
 0002:000061f0       __ehfuncinfo$?qt_emit@databaseEdit@@UAE_NHPAUQUObject@@@Z 100111f0     moc_databaseEdit.obj
 0002:00006214       __unwindtable$?command@databaseEditDlg@@IAEXVQString@@0@Z 10011214     moc_databaseEditdlgimpl.obj
 0002:00006214       __unwindtable$?command@databaseEdit@@IAEXVQString@@0@Z 10011214     moc_databaseEditdlgimpl.obj
 0002:0000622c       __ehfuncinfo$?command@databaseEditDlg@@IAEXVQString@@0@Z 1001122c     moc_databaseEditdlgimpl.obj
 0002:0000622c       __ehfuncinfo$?command@databaseEdit@@IAEXVQString@@0@Z 1001122c     moc_databaseEditdlgimpl.obj
 0002:00006250       __unwindtable$?fileSelected@toolWindow@@IAEXABVQString@@@Z 10011250     moc_toolwindowimpl.obj
 0002:00006258       __ehfuncinfo$?fileSelected@toolWindow@@IAEXABVQString@@@Z 10011258     moc_toolwindowimpl.obj
 0002:0000627c       __ehfuncinfo$??0toolWindowBase@@QAE@PAVQWidget@@PBDI@Z 1001127c     toolwindow.obj
 0002:000062a0       __unwindtable$??0toolWindowBase@@QAE@PAVQWidget@@PBDI@Z 100112a0     toolwindow.obj
 0002:000062e8       __unwindtable$?languageChange@toolWindowBase@@MAEXXZ 100112e8     toolwindow.obj
 0002:00006308       __ehfuncinfo$?languageChange@toolWindowBase@@MAEXXZ 10011308     toolwindow.obj
 0002:00006330       __sehtable$??_L@YGXPAXIHP6EX0@Z1@Z 10011330     MSVCRT:ehvecctr.obj
 0002:00006350       __sehtable$??_M@YGXPAXIHP6EX0@Z@Z 10011350     MSVCRT:ehvecdtr.obj
 0002:00006370       __sehtable$?__ArrayUnwind@@YGXPAXIHP6EX0@Z@Z 10011370     MSVCRT:ehvecdtr.obj
 0002:00006390       __sehtable$__onexit        10011390     MSVCRT:atonexit.obj
 0002:000063b0       __sehtable$___DllMainCRTStartup 100113b0     MSVCRT:crtdll.obj
 0002:000063d8       __sehtable$__IsNonwritableInCurrentImage 100113d8     MSVCRT:pesect.obj
 0002:00006400       .edata                     10011400     databaseEdit.exp
 0002:00006428       rgpv                       10011428     databaseEdit.exp
 0002:0000642c       rgszName                   1001142c     databaseEdit.exp
 0002:00006430       rgwOrd                     10011430     databaseEdit.exp
 0002:00006432       szName                     10011432     databaseEdit.exp
 0002:00006443       $N00001                    10011443     databaseEdit.exp
 0002:00007310       .idata$6                   10012310     config_icons:config_icons.dll
 0002:0001043e       .idata$6                   1001b43e     qt-mt323:qt-mt323.dll
 0002:00010468       .idata$6                   1001b468     kernel32:KERNEL32.dll
 0002:000104ca       .idata$6                   1001b4ca     MSVCRT:MSVCR120.dll
 0003:00000000       _databaseEdit_XPM          1001c000     plugindesc.obj
 0003:00000044       ?param_slot_0@?3??staticMetaObject@databaseEdit@@SAPAVQMetaObject@@XZ@4QBUQUParameter@@B 1001c044     moc_databaseEdit.obj
 0003:00000054       ?param_slot_1@?3??staticMetaObject@databaseEditDlg@@SAPAVQMetaObject@@XZ@4QBUQUParameter@@B 1001c054     moc_databaseEditdlgimpl.obj
 0003:00000564       _cleanUp_databaseEdit      1001c564     moc_databaseEdit.obj
 0003:00000568       ?$S1@?3??staticMetaObject@databaseEdit@@SAPAVQMetaObject@@XZ@4IA 1001c568     moc_databaseEdit.obj
 0003:0000056c       ?param_signal_0@?3??staticMetaObject@databaseEdit@@SAPAVQMetaObject@@XZ@4QBUQUParameter@@B 1001c56c     moc_databaseEdit.obj
 0003:00000590       _cleanUp_databaseEditDlgBase 1001c590     moc_databaseEditdlg.obj
 0003:00000598       _cleanUp_databaseEditDlg   1001c598     moc_databaseEditdlgimpl.obj
 0003:0000059c       ?$S1@?3??staticMetaObject@databaseEditDlg@@SAPAVQMetaObject@@XZ@4IA 1001c59c     moc_databaseEditdlgimpl.obj
 0003:000005a0       ?param_signal_0@?3??staticMetaObject@databaseEditDlg@@SAPAVQMetaObject@@XZ@4QBUQUParameter@@B 1001c5a0     moc_databaseEditdlgimpl.obj
 0003:000005c4       _cleanUp_toolWindowBase    1001c5c4     moc_toolwindow.obj
 0003:000005cc       _cleanUp_toolWindow        1001c5cc     moc_toolwindowimpl.obj
 0003:000005d0       ?param_slot_0@?3??staticMetaObject@toolWindow@@SAPAVQMetaObject@@XZ@4QBUQUParameter@@B 1001c5d0     moc_toolwindowimpl.obj
 0003:000005e0       ?$S1@?3??staticMetaObject@toolWindow@@SAPAVQMetaObject@@XZ@4IA 1001c5e0     moc_toolwindowimpl.obj
 0003:000005e4       ?param_signal_0@?3??staticMetaObject@toolWindow@@SAPAVQMetaObject@@XZ@4QBUQUParameter@@B 1001c5e4     moc_toolwindowimpl.obj
 0003:000005f4       ___proc_attached           1001c5f4     MSVCRT:crtdll.obj
 0003:000005f8       _GS_ExceptionRecord        1001c5f8     MSVCRT:gs_report.obj
 0003:00000648       _GS_ContextRecord          1001c648     MSVCRT:gs_report.obj
 0003:00000914       _DebuggerWasPresent        1001c914     MSVCRT:gs_report.obj
 0004:000000a0       $R000000                   1001d0a0     Script1.res
 0004:00000528       $R000488                   1001d528     Script1.res
